 glslcompiler

 Timestamp is 4be8c442 (Tue May 11 11:43:14 2010)

 Preferred load address is 10000000

 Start         Length     Name                   Class
 0001:00000000 00000004H .CRT$XCA                CODE
 0001:00000004 00000004H .CRT$XCZ                CODE
 0001:00000008 00000004H .CRT$XIA                CODE
 0001:0000000c 00000004H .CRT$XIZ                CODE
 0001:00000010 00000004H .CRT$XPA                CODE
 0001:00000014 00000004H .CRT$XPZ                CODE
 0001:00000018 00000004H .CRT$XTA                CODE
 0001:0000001c 00000004H .CRT$XTZ                CODE
 0001:00000020 00014071H .rdata                  CODE
 0001:00014094 00000029H .rdata$debug            CODE
 0001:000140c0 000c54d0H .text                   CODE
 0001:000d9590 00000098H .xdata                  CODE
 0001:000d9628 00000028H .idata$2                CODE
 0001:000d9650 00000014H .idata$3                CODE
 0001:000d9664 0000010cH .idata$4                CODE
 0001:000d9770 0000002aH .idata$6                CODE
 0001:000d97a0 000000fcH .edata                  CODE
 0002:00000000 0000010cH .idata$5                DATA
 0002:0000010c 00000008H .data                   DATA
 0002:00000114 00000010H .bss                    DATA
 0003:00000000 000034a0H .pdata                  DATA

  Address         Publics by Value              Rva+Base       Lib:Object

 0000:00000000       ___safe_se_handler_count   00000000     <absolute>
 0000:00000000       ___safe_se_handler_table   00000000     <absolute>
 0001:00000000       __xc_a                     10001000     corelib0:crt0init.obj
 0001:00000004       __xc_z                     10001004     corelib0:crt0init.obj
 0001:00000008       __xi_a                     10001008     corelib0:crt0init.obj
 0001:0000000c       __xi_z                     1000100c     corelib0:crt0init.obj
 0001:00000010       __xp_a                     10001010     corelib0:crt0init.obj
 0001:00000014       __xp_z                     10001014     corelib0:crt0init.obj
 0001:00000018       __xt_a                     10001018     corelib0:crt0init.obj
 0001:0000001c       __xt_z                     1000101c     corelib0:crt0init.obj
 0001:00000118       ??_C@_0GB@MLDDKHPB@H?3?2WINCE600?2PLATFORM?2SMDKV210?2SR@ 10001118     ic2uf.obj
 0001:0000017c       ??_C@_0CP@GMAGJKDF@More?5than?5?$CFd?5samplers?5are?5used?5i@ 1000117c     ic2uf.obj
 0001:000001ac       ??_C@_0BK@BGNLMMDD@Too?5deeply?5nested?5loops?4?6?$AA@ 100011ac     ic2uf.obj
 0001:000001c8       ??_C@_0BF@CBEJDHFG@Too?5many?5functions?4?6?$AA@ 100011c8     ic2uf.obj
 0001:000001e0       ??_C@_0BO@KPIMGECL@Failed?5to?5allocate?5varyings?4?6?$AA@ 100011e0     ic2uf.obj
 0001:00000200       ??_C@_0M@LAALAFHL@gl_FragData?$AA@ 10001200     ic2uf.obj
 0001:0000020c       ??_C@_0N@OHGIGEGG@gl_FragColor?$AA@ 1000120c     ic2uf.obj
 0001:0000021c       ??_C@_0N@KEMBCBC@gl_FragDepth?$AA@ 1000121c     ic2uf.obj
 0001:0000022c       ??_C@_0P@IILMBLMA@gl_FrontFacing?$AA@ 1000122c     ic2uf.obj
 0001:0000023c       ??_C@_0BE@CDEHDHPO@gl_PMXSwapFrontFace?$AA@ 1000123c     ic2uf.obj
 0001:00000250       ??_C@_0BA@DPBMNHEM@gl_PMXPosAdjust?$AA@ 10001250     ic2uf.obj
 0001:00000260       ??_C@_0N@PNLLEOHM@gl_FragCoord?$AA@ 10001260     ic2uf.obj
 0001:00000270       ??_C@_0CM@BOACPCDO@Shader?5needs?5too?5many?5temporary?5@ 10001270     ic2uf.obj
 0001:0000029c       ??_C@_0CC@OIJICMFO@Shader?5needs?5too?5many?5registers?4@ 1000129c     ic2uf.obj
 0001:000002c0       ??_C@_01GFHCPBMG@C?$AA@    100012c0     glsl2uf.obj
 0001:000002c8       ??_C@_0GG@NCKNFHEE@H?3?2WINCE600?2PLATFORM?2SMDKV210?2SR@ 100012c8     bindingsym.obj
 0001:00000330       ??_C@_06HLGAHHGE@?$FL?$CFlu?$FN?4?$AA@ 10001330     bindingsym.obj
 0001:00000338       ??_C@_01LFCBOECM@?4?$AA@   10001338     bindingsym.obj
 0001:0000033c       ??_C@_0BP@HNBKCAIH@?$EA?9?9?9?9?5ScopeModifer?5?$CF03lu?5?9?9?9?9?$EA?$AA@ 1000133c     glsl_parser:symtab.obj
 0001:0000035c       ??_C@_0BB@NDENLPKD@array?5size?5fixed?$AA@ 1000135c     glsl_core:glsltabs.obj
 0001:00000370       ??_C@_0BF@DPBHHNMA@array?5size?5non?5fixed?$AA@ 10001370     glsl_core:glsltabs.obj
 0001:00000388       ??_C@_09NOOGDAF@non?9array?$AA@ 10001388     glsl_core:glsltabs.obj
 0001:00000394       ??_C@_07PBJKAAPN@l?9value?$AA@ 10001394     glsl_core:glsltabs.obj
 0001:0000039c       ??_C@_0BA@EJBDKCFJ@non?9l?9value?$CIds?$CJ?$AA@ 1000139c     glsl_core:glsltabs.obj
 0001:000003ac       ??_C@_0M@FBLCJFCE@non?9l?9value?$AA@ 100013ac     glsl_core:glsltabs.obj
 0001:000003b8       ??_C@_05DNOIDIPO@inout?$AA@ 100013b8     glsl_core:glsltabs.obj
 0001:000003c0       ??_C@_03KEJHNBPP@out?$AA@  100013c0     glsl_core:glsltabs.obj
 0001:000003c4       ??_C@_02LMMGJAGL@in?$AA@   100013c4     glsl_core:glsltabs.obj
 0001:000003c8       ??_C@_05PBLCOKID@highp?$AA@ 100013c8     glsl_core:glsltabs.obj
 0001:000003d0       ??_C@_07DMCLNPOF@mediump?$AA@ 100013d0     glsl_core:glsltabs.obj
 0001:000003d8       ??_C@_04HINLHCNI@lowp?$AA@ 100013d8     glsl_core:glsltabs.obj
 0001:000003e0       ??_C@_07CIFAGBMG@unknown?$AA@ 100013e0     glsl_core:glsltabs.obj
 0001:000003e8       ??_C@_07EBNAHCGH@varying?$AA@ 100013e8     glsl_core:glsltabs.obj
 0001:000003f0       ??_C@_09HGIEBAJ@attribute?$AA@ 100013f0     glsl_core:glsltabs.obj
 0001:000003fc       ??_C@_07HIAOBKCE@uniform?$AA@ 100013fc     glsl_core:glsltabs.obj
 0001:00000404       ??_C@_05BNCCCJPP@const?$AA@ 10001404     glsl_core:glsltabs.obj
 0001:0000040a       ??_C@_00CNPNBAHC@?$AA@     1000140a     glsl_core:glsltabs.obj
 0001:0000040c       ??_C@_06OBMEHEFN@mat4X4?$AA@ 1000140c     glsl_core:glsltabs.obj
 0001:00000414       ??_C@_06KOIFOCJK@mat4X3?$AA@ 10001414     glsl_core:glsltabs.obj
 0001:0000041c       ??_C@_06LHJONDNL@mat4X2?$AA@ 1000141c     glsl_core:glsltabs.obj
 0001:00000424       ??_C@_06HMBDEMOE@mat3X4?$AA@ 10001424     glsl_core:glsltabs.obj
 0001:0000042c       ??_C@_06DDFCNKCD@mat3X3?$AA@ 1000142c     glsl_core:glsltabs.obj
 0001:00000434       ??_C@_06BCAEKNIC@mat3x2?$AA@ 10001434     glsl_core:glsltabs.obj
 0001:0000043c       ??_C@_06PMOCGNGB@mat2x4?$AA@ 1000143c     glsl_core:glsltabs.obj
 0001:00000444       ??_C@_06LDKDPLKG@mat2x3?$AA@ 10001444     glsl_core:glsltabs.obj
 0001:0000044c       ??_C@_06KKLIMKOH@mat2x2?$AA@ 1000144c     glsl_core:glsltabs.obj
 0001:00000454       ??_C@_05IANAGENN@bvec4?$AA@ 10001454     glsl_core:glsltabs.obj
 0001:0000045c       ??_C@_05MPJBPCBK@bvec3?$AA@ 1000145c     glsl_core:glsltabs.obj
 0001:00000464       ??_C@_05NGIKMDFL@bvec2?$AA@ 10001464     glsl_core:glsltabs.obj
 0001:0000046c       ??_C@_05OKBHJEBO@ivec4?$AA@ 1000146c     glsl_core:glsltabs.obj
 0001:00000474       ??_C@_05KFFGACNJ@ivec3?$AA@ 10001474     glsl_core:glsltabs.obj
 0001:0000047c       ??_C@_05LMENDDJI@ivec2?$AA@ 1000147c     glsl_core:glsltabs.obj
 0001:00000484       ??_C@_04LCAMJMDC@vec4?$AA@ 10001484     glsl_core:glsltabs.obj
 0001:0000048c       ??_C@_04PNENAKPF@vec3?$AA@ 1000148c     glsl_core:glsltabs.obj
 0001:00000494       ??_C@_04OEFGDLLE@vec2?$AA@ 10001494     glsl_core:glsltabs.obj
 0001:0000049c       ??_C@_06PBJBIPGK@struct?$AA@ 1000149c     glsl_core:glsltabs.obj
 0001:000004a4       ??_C@_0O@ELDFBPJC@samplerstream?$AA@ 100014a4     glsl_core:glsltabs.obj
 0001:000004b4       ??_C@_0BA@DPDJLMPL@sampler2dshadow?$AA@ 100014b4     glsl_core:glsltabs.obj
 0001:000004c4       ??_C@_0BA@GLEIADO@sampler1dshadow?$AA@ 100014c4     glsl_core:glsltabs.obj
 0001:000004d4       ??_C@_0M@FLJEMIJK@samplercube?$AA@ 100014d4     glsl_core:glsltabs.obj
 0001:000004e0       ??_C@_09CFPLPDNF@sampler3d?$AA@ 100014e0     glsl_core:glsltabs.obj
 0001:000004ec       ??_C@_09CEDJJJOC@sampler2d?$AA@ 100014ec     glsl_core:glsltabs.obj
 0001:000004f8       ??_C@_09CGHPCHLL@sampler1d?$AA@ 100014f8     glsl_core:glsltabs.obj
 0001:00000504       ??_C@_0BE@KAJFKPKD@4X4?5matrix?5of?5float?$AA@ 10001504     glsl_core:glsltabs.obj
 0001:00000518       ??_C@_0BE@EBLLKFMH@4X3?5matrix?5of?5float?$AA@ 10001518     glsl_core:glsltabs.obj
 0001:0000052c       ??_C@_0BE@KOOJBDCG@4X2?5matrix?5of?5float?$AA@ 1000152c     glsl_core:glsltabs.obj
 0001:00000540       ??_C@_0BE@EBNBAJDA@3X4?5matrix?5of?5float?$AA@ 10001540     glsl_core:glsltabs.obj
 0001:00000554       ??_C@_0BE@KAPPADFE@3X3?5matrix?5of?5float?$AA@ 10001554     glsl_core:glsltabs.obj
 0001:00000568       ??_C@_0BE@EPKNLFLF@3X2?5matrix?5of?5float?$AA@ 10001568     glsl_core:glsltabs.obj
 0001:0000057c       ??_C@_0BE@CELGDCHG@2X4?5matrix?5of?5float?$AA@ 1000157c     glsl_core:glsltabs.obj
 0001:00000590       ??_C@_0BE@MFJIDIBC@2X3?5matrix?5of?5float?$AA@ 10001590     glsl_core:glsltabs.obj
 0001:000005a4       ??_C@_0BE@CKMKIOPD@2X2?5matrix?5of?5float?$AA@ 100015a4     glsl_core:glsltabs.obj
 0001:000005b8       ??_C@_0BL@FGFIOMGE@4?9component?5vector?5of?5bool?$AA@ 100015b8     glsl_core:glsltabs.obj
 0001:000005d4       ??_C@_0BL@IEINKKOC@3?9component?5vector?5of?5bool?$AA@ 100015d4     glsl_core:glsltabs.obj
 0001:000005f0       ??_C@_0BL@OKABLBKD@2?9component?5vector?5of?5bool?$AA@ 100015f0     glsl_core:glsltabs.obj
 0001:0000060c       ??_C@_04DDKJGDCM@bool?$AA@ 1000160c     glsl_core:glsltabs.obj
 0001:00000614       ??_C@_0BK@NANJEMOK@4?9component?5vector?5of?5int?$AA@ 10001614     glsl_core:glsltabs.obj
 0001:00000630       ??_C@_0BK@IBKDHMM@3?9component?5vector?5of?5int?$AA@ 10001630     glsl_core:glsltabs.obj
 0001:0000064c       ??_C@_0BK@OPAHJBFL@2?9component?5vector?5of?5int?$AA@ 1000164c     glsl_core:glsltabs.obj
 0001:00000668       ??_C@_03JBIPMCLC@int?$AA@  10001668     glsl_core:glsltabs.obj
 0001:0000066c       ??_C@_0BM@NFDDOKMK@4?9component?5vector?5of?5float?$AA@ 1000166c     glsl_core:glsltabs.obj
 0001:00000688       ??_C@_0BM@NBDKBJJJ@3?9component?5vector?5of?5float?$AA@ 10001688     glsl_core:glsltabs.obj
 0001:000006a4       ??_C@_0BM@NAIPOEIE@2?9component?5vector?5of?5float?$AA@ 100016a4     glsl_core:glsltabs.obj
 0001:000006c0       ??_C@_05KNFBNCOH@float?$AA@ 100016c0     glsl_core:glsltabs.obj
 0001:000006c8       ??_C@_04GKJNKENE@void?$AA@ 100016c8     glsl_core:glsltabs.obj
 0001:000006d0       ??_C@_07MALOAKCI@invalid?$AA@ 100016d0     glsl_core:glsltabs.obj
 0001:000006d8       GLSLTypeSpecifierNumElementsTable 100016d8     glsl_core:glsltabs.obj
 0001:000006f8       GLSLTypeSpecifierDimensionTable 100016f8     glsl_core:glsltabs.obj
 0001:00000718       GLSLTypeSpecifierSizeTable 10001718     glsl_core:glsltabs.obj
 0001:00000738       GLSLTypeSpecifierIndexedTable 10001738     glsl_core:glsltabs.obj
 0001:00000758       GLSLTypeSpecifierColumnsTable 10001758     glsl_core:glsltabs.obj
 0001:00000778       GLSLTypeSpecifierBaseType  10001778     glsl_core:glsltabs.obj
 0001:000007f8       GLSLTypeSpecifierFullDescTable 100017f8     glsl_core:glsltabs.obj
 0001:00000878       GLSLTypeSpecifierDescTable 10001878     glsl_core:glsltabs.obj
 0001:000008f4       GLSLTypeQualifierFullDescTable 100018f4     glsl_core:glsltabs.obj
 0001:0000090c       GLSLPrecisionQualifierFullDescTable 1000190c     glsl_core:glsltabs.obj
 0001:0000091c       GLSLParameterQualifierFullDescTable 1000191c     glsl_core:glsltabs.obj
 0001:0000092c       GLSLLValueStatusFullDescTable 1000192c     glsl_core:glsltabs.obj
 0001:0000093c       GLSLArrayStatusFullDescTable 1000193c     glsl_core:glsltabs.obj
 0001:00000950       GLSLBuiltInFunctionReducibleToConstTable 10001950     glsl_core:glsltabs.obj
 0001:000009b0       GLSLBuiltInFunctionUseGradientsTable 100019b0     glsl_core:glsltabs.obj
 0001:00000a10       GLSLBuiltInFunctionTextureSampler 10001a10     glsl_core:glsltabs.obj
 0001:00000a6c       GLSLTypeSpecifierNumColumnsCMTable 10001a6c     glsl_core:glsltabs.obj
 0001:00000a8c       GLSLTypeSpecifierNumRowsCMTable 10001a8c     glsl_core:glsltabs.obj
 0001:00000aac       GLSLTypeSpecifierNumColumnsRMTable 10001aac     glsl_core:glsltabs.obj
 0001:00000acc       GLSLTypeSpecifierNumRowsRMTable 10001acc     glsl_core:glsltabs.obj
 0001:00000aec       GLSLTypeSpecifierIsNumberTable 10001aec     glsl_core:glsltabs.obj
 0001:00000b10       asICodeOpTable             10001b10     glsl_core:icgen.obj
 0001:00000d30       asNodeTable                10001d30     glsl_core:icgen.obj
 0001:00000e30       ??_C@_09COACJEOO@tmp?$CFs?$EA?$CFlu?$AA@ 10001e30     glsl_core:icgen.obj
 0001:00000e40       ??_C@_0FO@JFMCBJIJ@H?3?2WINCE600?2PLATFORM?2SMDKV210?2SR@ 10001e40     glsl_core:icgen.obj
 0001:00000ea0       ??_C@_08JBFBCINF@pred?$EA?$CFlu?$AA@ 10001ea0     glsl_core:icgen.obj
 0001:00000eac       ??_C@_08MCFFGLHH@fn_main?$EA?$AA@ 10001eac     glsl_core:icgen.obj
 0001:00000eb8       ??_C@_06PIKJLJJK@cst?$EA?$CFs?$AA@ 10001eb8     glsl_core:common.obj
 0001:00000ec0       ??_C@_0M@DADOMJOJ@cst_p?$CFlu?$EA?$CFs?$AA@ 10001ec0     glsl_core:common.obj
 0001:00000ed0       ??_C@_0FP@IOLFOMBF@H?3?2WINCE600?2PLATFORM?2SMDKV210?2SR@ 10001ed0     glsl_core:common.obj
 0001:00000f30       ??_C@_09IDPEJOHI@cst_rv?$EA?$CFs?$AA@ 10001f30     glsl_core:common.obj
 0001:00000f3c       ??_C@_0CD@LPLBODBK@?8?$CFs?8?5?3?5?8struct?8?5type?5redefinitio@ 10001f3c     glsl_core:common.obj
 0001:00000f60       ??_C@_0O@KLAILGIL@?$CFs?$EAstruct_def?$AA@ 10001f60     glsl_core:common.obj
 0001:00000f70       ??_C@_0DC@LCOJIAGM@?8struct?8?5?3?5duplicate?5field?5name?5@ 10001f70     glsl_core:common.obj
 0001:00000fa4       ??_C@_02DKCKIIND@?$CFs?$AA@ 10001fa4     glsl_core:common.obj
 0001:00000fa8       ??_C@_05DNIIFBMG@?$CFs?5?$CFs?$AA@ 10001fa8     glsl_core:common.obj
 0001:00000fb0       ??_C@_03IKGEINEE@?$CFs?5?$AA@ 10001fb0     glsl_core:common.obj
 0001:00000fb4       ??_C@_09GIMGMFEA@array?5of?5?$AA@ 10001fb4     glsl_core:common.obj
 0001:00000fc0       ??_C@_05LAPONLG@false?$AA@ 10001fc0     glsl_core:common.obj
 0001:00000fc8       ??_C@_04LOAJBDKD@true?$AA@ 10001fc8     glsl_core:common.obj
 0001:00000fd0       ??_C@_03JALODAI@?$CFld?$AA@ 10001fd0     glsl_core:common.obj
 0001:00000fd4       ??_C@_07BMHOFEPE@?$CFld_low?$AA@ 10001fd4     glsl_core:common.obj
 0001:00000fdc       ??_C@_07MILKPHNF@?$CFld_med?$AA@ 10001fdc     glsl_core:common.obj
 0001:00000fe4       ??_C@_08NLCFPDJC@?$CFld_high?$AA@ 10001fe4     glsl_core:common.obj
 0001:00000ff0       ??_C@_02NJPGOMH@?$CFf?$AA@ 10001ff0     glsl_core:common.obj
 0001:00000ff4       ??_C@_06MJPNKJHA@?$CFf_low?$AA@ 10001ff4     glsl_core:common.obj
 0001:00000ffc       ??_C@_06BNDJAKFB@?$CFf_med?$AA@ 10001ffc     glsl_core:common.obj
 0001:00001004       ??_C@_07DBCFDHFG@?$CFf_high?$AA@ 10002004     glsl_core:common.obj
 0001:0000100c       ??_C@_06DJHOIPC@?$CFs?3?5?$CFs?$AA@ 1000200c     glsl_core:error.obj
 0001:00001014       ??_C@_0BA@FOHKMLP@?$CFs?3?5?$CFlu?3?$CFlu?3?5?$CFs?$AA@ 10002014     glsl_core:error.obj
 0001:00001024       ??_C@_08MLFDIMPC@INTERNAL?$AA@ 10002024     glsl_core:error.obj
 0001:00001030       ??_C@_05MBDEGLCK@ERROR?$AA@ 10002030     glsl_core:error.obj
 0001:00001038       ??_C@_07KCOHIFOP@WARNING?$AA@ 10002038     glsl_core:error.obj
 0001:00001040       ??_C@_07NFANNNEC@UNKNOWN?$AA@ 10002040     glsl_core:error.obj
 0001:00001048       ??_C@_01EEMJAFIK@?6?$AA@   10002048     glsl_core:glsl.obj
 0001:0000104c       ??_C@_0BG@COOJENBA@Built?9in?5vertex?5state?$AA@ 1000204c     glsl_core:glsl.obj
 0001:00001064       ??_C@_0BI@FOGLGBPC@Built?9in?5fragment?5state?$AA@ 10002064     glsl_core:glsl.obj
 0001:0000107c       ??_C@_0BB@GOFCBDKF@Compile?5failed?4?6?$AA@ 1000207c     glsl_core:glsl.obj
 0001:00001090       ??_C@_09EHKFFFJM@Success?4?6?$AA@ 10002090     glsl_core:glsl.obj
 0001:0000109c       ??_C@_0CM@HLEOFKBF@?$CFd?5compilation?5errors?4?5No?5code?5g@ 1000209c     glsl_core:glsl.obj
 0001:000010c8       ??_C@_0BL@EDLNLOE@?$CFd?5compilation?5warnings?4?6?6?$AA@ 100020c8     glsl_core:glsl.obj
 0001:000010e4       ??_C@_0BB@KELPLCJN@Fragment?5Program?$AA@ 100020e4     glsl_core:glsl.obj
 0001:000010f8       ??_C@_0P@JDCINLJB@Vertex?5Program?$AA@ 100020f8     glsl_core:glsl.obj
 0001:00001108       ??_C@_0BK@LPFOIAFP@No?5source?5code?5supplied?4?6?$AA@ 10002108     glsl_core:glsl.obj
 0001:00001290       ??_C@_09MPJGCHGP@gl_Vertex?$AA@ 10002290     glsl_core:icbuiltin.obj
 0001:0000129c       ??_C@_0BN@HOKGMOHF@gl_ModelViewProjectionMatrix?$AA@ 1000229c     glsl_core:icbuiltin.obj
 0001:000012c0       ??_C@_0GC@EELMKDJE@H?3?2WINCE600?2PLATFORM?2SMDKV210?2SR@ 100022c0     glsl_core:icbuiltin.obj
 0001:00001328       ??_C@_0GB@DEALPPCI@H?3?2WINCE600?2PLATFORM?2SMDKV210?2SR@ 10002328     glsl_core:icunroll.obj
 0001:00001390       ??_C@_0GD@NEMHJPEB@H?3?2WINCE600?2PLATFORM?2SMDKV210?2SR@ 10002390     glsl_core:astbuiltin.obj
 0001:000013f4       ??_C@_05NHLPFGDD@rv_?$CFs?$AA@ 100023f4     glsl_core:astbuiltin.obj
 0001:000013fc       ??_C@_06CFFBLOIB@noise1?$AA@ 100023fc     glsl_core:astbuiltin.obj
 0001:00001404       ??_C@_06OHMONEC@noise2?$AA@ 10002404     glsl_core:astbuiltin.obj
 0001:0000140c       ??_C@_06BHGHNMAD@noise3?$AA@ 1000240c     glsl_core:astbuiltin.obj
 0001:00001414       ??_C@_06FICGEKME@noise4?$AA@ 10002414     glsl_core:astbuiltin.obj
 0001:0000141c       ??_C@_04EDCIEOIM@dFdx?$AA@ 1000241c     glsl_core:astbuiltin.obj
 0001:00001424       ??_C@_04FKDDHPMN@dFdy?$AA@ 10002424     glsl_core:astbuiltin.obj
 0001:0000142c       ??_C@_01JBBJJEPG@p?$AA@    1000242c     glsl_core:astbuiltin.obj
 0001:00001430       ??_C@_06ECGIDAGM@fwidth?$AA@ 10002430     glsl_core:astbuiltin.obj
 0001:00001438       ??_C@_0BB@FNHAJCEE@textureStreamIMG?$AA@ 10002438     glsl_core:astbuiltin.obj
 0001:0000144c       ??_C@_0BF@PEMADAKB@textureStreamProjIMG?$AA@ 1000244c     glsl_core:astbuiltin.obj
 0001:00001464       ??_C@_0BD@GBJBFDJA@textureCubeGradARB?$AA@ 10002464     glsl_core:astbuiltin.obj
 0001:00001478       ??_C@_0P@JOIAHBNL@textureCubeLod?$AA@ 10002478     glsl_core:astbuiltin.obj
 0001:00001488       ??_C@_0M@BNCBNMFA@textureCube?$AA@ 10002488     glsl_core:astbuiltin.obj
 0001:00001494       ??_C@_0BB@IAJJJIBH@texture2DGradARB?$AA@ 10002494     glsl_core:astbuiltin.obj
 0001:000014a8       ??_C@_04CPEBHHIO@dPdy?$AA@ 100024a8     glsl_core:astbuiltin.obj
 0001:000014b0       ??_C@_04DGFKEGMP@dPdx?$AA@ 100024b0     glsl_core:astbuiltin.obj
 0001:000014b8       ??_C@_01EJNLAFE@P?$AA@     100024b8     glsl_core:astbuiltin.obj
 0001:000014bc       ??_C@_0BF@LHPJKFEA@texture2DProjGradARB?$AA@ 100024bc     glsl_core:astbuiltin.obj
 0001:000014d4       ??_C@_0N@HLKCMMAC@texture2DLod?$AA@ 100024d4     glsl_core:astbuiltin.obj
 0001:000014e4       ??_C@_03ONFBEKOG@lod?$AA@  100024e4     glsl_core:astbuiltin.obj
 0001:000014e8       ??_C@_0BB@GONKFCAO@texture2DProjLod?$AA@ 100024e8     glsl_core:astbuiltin.obj
 0001:000014fc       ??_C@_04NBAGBPGE@bias?$AA@ 100024fc     glsl_core:astbuiltin.obj
 0001:00001504       ??_C@_07JLOPPFCD@radians?$AA@ 10002504     glsl_core:astbuiltin.obj
 0001:0000150c       ??_C@_07MHOHEFBH@degrees?$AA@ 1000250c     glsl_core:astbuiltin.obj
 0001:00001514       ??_C@_03BLEJJJBH@sin?$AA@  10002514     glsl_core:astbuiltin.obj
 0001:00001518       ??_C@_03LALBNOCG@cos?$AA@  10002518     glsl_core:astbuiltin.obj
 0001:0000151c       ??_C@_05FECBCJJD@angle?$AA@ 1000251c     glsl_core:astbuiltin.obj
 0001:00001524       ??_C@_03IIINPABG@tan?$AA@  10002524     glsl_core:astbuiltin.obj
 0001:00001528       ??_C@_04FIHNOPOL@asin?$AA@ 10002528     glsl_core:astbuiltin.obj
 0001:00001530       ??_C@_04PDIFKINK@acos?$AA@ 10002530     glsl_core:astbuiltin.obj
 0001:00001538       ??_C@_08HJJHKHDM@y_over_x?$AA@ 10002538     glsl_core:astbuiltin.obj
 0001:00001544       ??_C@_04MLLJIGOK@atan?$AA@ 10002544     glsl_core:astbuiltin.obj
 0001:0000154c       ??_C@_03JGHBODFD@pow?$AA@  1000254c     glsl_core:astbuiltin.obj
 0001:00001550       ??_C@_03KHJOGHMM@exp?$AA@  10002550     glsl_core:astbuiltin.obj
 0001:00001554       ??_C@_03MGHMBJCF@log?$AA@  10002554     glsl_core:astbuiltin.obj
 0001:00001558       ??_C@_04HPAFEEIN@exp2?$AA@ 10002558     glsl_core:astbuiltin.obj
 0001:00001560       ??_C@_04KGLCPMCP@log2?$AA@ 10002560     glsl_core:astbuiltin.obj
 0001:00001568       ??_C@_04EIAKFFMI@sqrt?$AA@ 10002568     glsl_core:astbuiltin.obj
 0001:00001570       ??_C@_0M@MEMLHMJL@inversesqrt?$AA@ 10002570     glsl_core:astbuiltin.obj
 0001:0000157c       ??_C@_03BCGAIFPO@abs?$AA@  1000257c     glsl_core:astbuiltin.obj
 0001:00001580       ??_C@_04HHGHLBPI@sign?$AA@ 10002580     glsl_core:astbuiltin.obj
 0001:00001588       ??_C@_05PBJFFIGL@floor?$AA@ 10002588     glsl_core:astbuiltin.obj
 0001:00001590       ??_C@_04GFPJNGEK@ceil?$AA@ 10002590     glsl_core:astbuiltin.obj
 0001:00001598       ??_C@_05JBNKFIFJ@fract?$AA@ 10002598     glsl_core:astbuiltin.obj
 0001:000015a0       ??_C@_03FFONCNID@mod?$AA@  100025a0     glsl_core:astbuiltin.obj
 0001:000015a4       ??_C@_03KLIPLJLL@min?$AA@  100025a4     glsl_core:astbuiltin.obj
 0001:000015a8       ??_C@_03LJAEFNNE@max?$AA@  100025a8     glsl_core:astbuiltin.obj
 0001:000015ac       ??_C@_06OMMDKPJH@maxVal?$AA@ 100025ac     glsl_core:astbuiltin.obj
 0001:000015b4       ??_C@_06OPDAEPNI@minVal?$AA@ 100025b4     glsl_core:astbuiltin.obj
 0001:000015bc       ??_C@_05HADFAIAH@clamp?$AA@ 100025bc     glsl_core:astbuiltin.obj
 0001:000015c4       ??_C@_01MCMALHOG@a?$AA@    100025c4     glsl_core:astbuiltin.obj
 0001:000015c8       ??_C@_03LHBHAMGM@mix?$AA@  100025c8     glsl_core:astbuiltin.obj
 0001:000015cc       ??_C@_04IJFJNCMM@edge?$AA@ 100025cc     glsl_core:astbuiltin.obj
 0001:000015d4       ??_C@_04CNBNFAL@step?$AA@  100025d4     glsl_core:astbuiltin.obj
 0001:000015dc       ??_C@_05FEAGNAPL@edge1?$AA@ 100025dc     glsl_core:astbuiltin.obj
 0001:000015e4       ??_C@_05ENBNOBLK@edge0?$AA@ 100025e4     glsl_core:astbuiltin.obj
 0001:000015ec       ??_C@_0L@JKDMKNKF@smoothstep?$AA@ 100025ec     glsl_core:astbuiltin.obj
 0001:000015f8       ??_C@_06IJDLPEM@length?$AA@ 100025f8     glsl_core:astbuiltin.obj
 0001:00001600       ??_C@_02JCBCEJAP@p1?$AA@   10002600     glsl_core:astbuiltin.obj
 0001:00001604       ??_C@_02ILAJHIEO@p0?$AA@   10002604     glsl_core:astbuiltin.obj
 0001:00001608       ??_C@_08LHFODBFO@distance?$AA@ 10002608     glsl_core:astbuiltin.obj
 0001:00001614       ??_C@_03GCCHHAFI@dot?$AA@  10002614     glsl_core:astbuiltin.obj
 0001:00001618       ??_C@_05HCKPILGO@cross?$AA@ 10002618     glsl_core:astbuiltin.obj
 0001:00001620       ??_C@_09MMDNNKKJ@normalize?$AA@ 10002620     glsl_core:astbuiltin.obj
 0001:0000162c       ??_C@_04GCJDEDDH@Nref?$AA@ 1000262c     glsl_core:astbuiltin.obj
 0001:00001634       ??_C@_0M@ENCHEFMG@faceforward?$AA@ 10002634     glsl_core:astbuiltin.obj
 0001:00001640       ??_C@_07CCHDGNII@reflect?$AA@ 10002640     glsl_core:astbuiltin.obj
 0001:00001648       ??_C@_03PNFNLNLI@eta?$AA@  10002648     glsl_core:astbuiltin.obj
 0001:0000164c       ??_C@_01NANMIPIL@N?$AA@    1000264c     glsl_core:astbuiltin.obj
 0001:00001650       ??_C@_01JPJNBJEM@I?$AA@    10002650     glsl_core:astbuiltin.obj
 0001:00001654       ??_C@_07HCMBNDDM@refract?$AA@ 10002654     glsl_core:astbuiltin.obj
 0001:0000165c       ??_C@_0P@CHOCONB@matrixCompMult?$AA@ 1000265c     glsl_core:astbuiltin.obj
 0001:0000166c       ??_C@_08OKPGNDDO@lessThan?$AA@ 1000266c     glsl_core:astbuiltin.obj
 0001:00001678       ??_C@_0O@HILDIDCG@lessThanEqual?$AA@ 10002678     glsl_core:astbuiltin.obj
 0001:00001688       ??_C@_0M@DEGMAMMN@greaterThan?$AA@ 10002688     glsl_core:astbuiltin.obj
 0001:00001694       ??_C@_0BB@OGCPNFND@greaterThanEqual?$AA@ 10002694     glsl_core:astbuiltin.obj
 0001:000016a8       ??_C@_05OAKNMNI@equal?$AA@ 100026a8     glsl_core:astbuiltin.obj
 0001:000016b0       ??_C@_01EANLCPLP@y?$AA@    100026b0     glsl_core:astbuiltin.obj
 0001:000016b4       ??_C@_08NLCAHAPK@notEqual?$AA@ 100026b4     glsl_core:astbuiltin.obj
 0001:000016c0       ??_C@_03OBJFJEBA@any?$AA@  100026c0     glsl_core:astbuiltin.obj
 0001:000016c4       ??_C@_03NFKEKGGK@all?$AA@  100026c4     glsl_core:astbuiltin.obj
 0001:000016c8       ??_C@_01FJMABOPO@x?$AA@    100026c8     glsl_core:astbuiltin.obj
 0001:000016cc       ??_C@_03NJKJADM@not?$AA@   100026cc     glsl_core:astbuiltin.obj
 0001:000016d0       ??_C@_09PFEOJLIO@texture2D?$AA@ 100026d0     glsl_core:astbuiltin.obj
 0001:000016dc       ??_C@_05OOJODGPM@coord?$AA@ 100026dc     glsl_core:astbuiltin.obj
 0001:000016e4       ??_C@_07PKJOFHPL@sampler?$AA@ 100026e4     glsl_core:astbuiltin.obj
 0001:000016ec       ??_C@_0O@HKFBFKON@texture2DProj?$AA@ 100026ec     glsl_core:astbuiltin.obj
 0001:000016fc       ??_C@_0O@MPCJJLAI@gl_PointCoord?$AA@ 100026fc     glsl_core:astbuiltin.obj
 0001:0000170c       ??_C@_04EHDLHMJM@near?$AA@ 1000270c     glsl_core:astbuiltin.obj
 0001:00001714       ??_C@_03JEOKDCFP@far?$AA@  10002714     glsl_core:astbuiltin.obj
 0001:00001718       ??_C@_04GMLMBKFF@diff?$AA@ 10002718     glsl_core:astbuiltin.obj
 0001:00001720       ??_C@_0BI@JFLJOAEC@gl_DepthRangeParameters?$AA@ 10002720     glsl_core:astbuiltin.obj
 0001:00001738       ??_C@_0BE@BHIOMCCI@gl_MaxVertexAttribs?$AA@ 10002738     glsl_core:astbuiltin.obj
 0001:0000174c       ??_C@_0BI@PMNFBNJJ@gl_MaxTextureImageUnits?$AA@ 1000274c     glsl_core:astbuiltin.obj
 0001:00001764       ??_C@_0BC@IEPLMJCD@gl_MaxDrawBuffers?$AA@ 10002764     glsl_core:astbuiltin.obj
 0001:00001778       ??_C@_0BO@EAEBIDML@gl_MaxVertexTextureImageUnits?$AA@ 10002778     glsl_core:astbuiltin.obj
 0001:00001798       ??_C@_0CA@BPGFIHPG@gl_MaxCombinedTextureImageUnits?$AA@ 10002798     glsl_core:astbuiltin.obj
 0001:000017b8       ??_C@_0BL@LGAKKEID@gl_MaxVertexUniformVectors?$AA@ 100027b8     glsl_core:astbuiltin.obj
 0001:000017d4       ??_C@_0BF@LOFKNIAP@gl_MaxVaryingVectors?$AA@ 100027d4     glsl_core:astbuiltin.obj
 0001:000017ec       ??_C@_0BN@DEMFANDN@gl_MaxFragmentUniformVectors?$AA@ 100027ec     glsl_core:astbuiltin.obj
 0001:0000180c       ??_C@_0O@EHLCMLBL@gl_DepthRange?$AA@ 1000280c     glsl_core:astbuiltin.obj
 0001:0000181c       ??_C@_0M@LBFKDGNK@gl_Position?$AA@ 1000281c     glsl_core:astbuiltin.obj
 0001:00001828       ??_C@_0N@IDDEBJCE@gl_PointSize?$AA@ 10002828     glsl_core:astbuiltin.obj
 0001:00001838       ??_C@_0DK@IGEMMMBL@ASTBIResetBuiltInData?3?5Failed?5to@ 10002838     glsl_core:astbuiltin.obj
 0001:00001878       GLSLESSyntaxSymbolTable    10002878     glsl_core:glslesgram.obj
 0001:00002398       GLSLESSyntaxGrammar        10003398     glsl_core:glslesgram.obj
 0001:00003070       guSupportedGLSLVersions    10004070     glsl_core:prepro.obj
 0001:00003074       ??_C@_0CC@KGJBNJBG@?8defined?8?5?3?5expected?5define?5name@ 10004074     glsl_core:prepro.obj
 0001:00003098       ??_C@_0CE@EJBLHJEA@?8defined?8?5?3?5expected?5right?5brack@ 10004098     glsl_core:prepro.obj
 0001:000030bc       ??_C@_0CA@OLMHBAPF@?8?8?5?3?5Too?5few?5args?5in?5Macro?5?5?$CFs?6?$AA@ 100040bc     glsl_core:prepro.obj
 0001:000030dc       ??_C@_0CC@JCKNBEKC@?8?$CFs?8?5?3?5Expected?5comma?5or?5bracket@ 100040dc     glsl_core:prepro.obj
 0001:00003100       ??_C@_0CB@CDHGBJNL@?8?8?5?3?5Too?5many?5args?5in?5Macro?5?5?$CFs?6@ 10004100     glsl_core:prepro.obj
 0001:00003124       ??_C@_0CC@DLHJJILD@?8?8?5?3?5Expected?5macro?5argument?5?5?$CFs@ 10004124     glsl_core:prepro.obj
 0001:00003148       ??_C@_0CB@GKCLFFFI@?8?$CFs?8?5?3?5Expected?5macro?5parameter?6@ 10004148     glsl_core:prepro.obj
 0001:0000316c       ??_C@_07MJAJDDLG@defined?$AA@ 1000416c     glsl_core:prepro.obj
 0001:00003178       ??_C@_0FP@FACNNNCP@H?3?2WINCE600?2PLATFORM?2SMDKV210?2SR@ 10004178     glsl_core:prepro.obj
 0001:000031d8       ??_C@_0BM@DEGLEPEH@Syntax?5error?0?5expected?5?8?$CJ?8?6?$AA@ 100041d8     glsl_core:prepro.obj
 0001:000031f4       ??_C@_0CD@GKAKFNBE@Syntax?5error?5?$CIadding?5node?5failed@ 100041f4     glsl_core:prepro.obj
 0001:00003218       ??_C@_0BO@DLAFAMIF@Syntax?5error?0?5unexpected?5?8?$CJ?8?6?$AA@ 10004218     glsl_core:prepro.obj
 0001:00003238       ??_C@_0BC@IBKDGGAO@Syntax?5error?5?$CI2?$CJ?6?$AA@ 10004238     glsl_core:prepro.obj
 0001:0000324c       ??_C@_0O@JJFGCDGG@Syntax?5error?6?$AA@ 1000424c     glsl_core:prepro.obj
 0001:0000325c       ??_C@_0BC@DJBPABGL@Syntax?5error?5?$CI3?$CJ?6?$AA@ 1000425c     glsl_core:prepro.obj
 0001:00003270       ??_C@_0BA@JNEPDCCE@Child?5was?5?8?$CFs?8?6?$AA@ 10004270     glsl_core:prepro.obj
 0001:00003280       ??_C@_0CD@HCBNCNFN@Max?5number?5of?5nested?5?$CDif?8s?5is?525@ 10004280     glsl_core:prepro.obj
 0001:000032a4       ??_C@_0CF@KPOHIJFF@invalid?5integer?5constant?5express@ 100042a4     glsl_core:prepro.obj
 0001:000032cc       ??_C@_0CC@GKPFBPGO@?8?8?5?3?5syntax?5error?5?$CDelif?5mismatch@ 100042cc     glsl_core:prepro.obj
 0001:000032f0       ??_C@_0CH@MFAFPAKL@?8?8?5?3?5syntax?5error?5?$CDelse?5after?5a?5@ 100042f0     glsl_core:prepro.obj
 0001:00003318       ??_C@_0CC@JDDDANGC@?8?8?5?3?5syntax?5error?5?$CDelse?5mismatch@ 10004318     glsl_core:prepro.obj
 0001:0000333c       ??_C@_0DA@CMGMBEJC@Syntax?5error?0?5?$CDif?$FLn?$FNdef?5expected@ 1000433c     glsl_core:prepro.obj
 0001:0000336c       ??_C@_0CD@CJBMGCMA@?8?8?5?3?5syntax?5error?5?$CDendif?5mismatc@ 1000436c     glsl_core:prepro.obj
 0001:00003390       ??_C@_03OFAPEBGM@?$CFs?6?$AA@ 10004390     glsl_core:prepro.obj
 0001:00003394       ??_C@_0BN@KIPMODCH@?8?8?5?3?5syntax?5error?5?$CI2?$CJ?5?$CDline?6?$AA@ 10004394     glsl_core:prepro.obj
 0001:000033b4       ??_C@_0BN@EDMLFICE@?8?8?5?3?5syntax?5error?5?$CI1?$CJ?5?$CDline?6?$AA@ 100043b4     glsl_core:prepro.obj
 0001:000033d4       ??_C@_0BN@KMAJDDBK@?8?8?5?3?5syntax?5error?5?$CI0?$CJ?5?$CDline?6?$AA@ 100043d4     glsl_core:prepro.obj
 0001:000033f4       ??_C@_0BP@PBODAIDK@?8?8?5?3?5syntax?5error?5?$CDpragma?5?$CI1?$CJ?6?$AA@ 100043f4     glsl_core:prepro.obj
 0001:00003414       ??_C@_0BP@HOIBJPGN@?8?8?5?3?5syntax?5error?5?$CDpragma?5?$CI5?$CJ?6?$AA@ 10004414     glsl_core:prepro.obj
 0001:00003434       ??_C@_03MCADLMAF@off?$AA@  10004434     glsl_core:prepro.obj
 0001:00003438       ??_C@_02LIELOMNJ@on?$AA@   10004438     glsl_core:prepro.obj
 0001:0000343c       ??_C@_0BP@ODFGKHNE@?8?8?5?3?5syntax?5error?5?$CDpragma?5?$CI2?$CJ?6?$AA@ 1000443c     glsl_core:prepro.obj
 0001:0000345c       ??_C@_0BP@FLOKMALB@?8?8?5?3?5syntax?5error?5?$CDpragma?5?$CI3?$CJ?6?$AA@ 1000445c     glsl_core:prepro.obj
 0001:0000347c       ??_C@_0BP@MGDNPIAI@?8?8?5?3?5syntax?5error?5?$CDpragma?5?$CI4?$CJ?6?$AA@ 1000447c     glsl_core:prepro.obj
 0001:0000349c       ??_C@_09LKJAEOAL@invariant?$AA@ 1000449c     glsl_core:prepro.obj
 0001:000034a8       ??_C@_05DENLBJCI@STDGL?$AA@ 100044a8     glsl_core:prepro.obj
 0001:000034b0       ??_C@_05GFCDIDHO@debug?$AA@ 100044b0     glsl_core:prepro.obj
 0001:000034b8       ??_C@_08GHMAOHAP@optimize?$AA@ 100044b8     glsl_core:prepro.obj
 0001:000034c4       ??_C@_0CA@EEONNNLN@?8?$CFs?8?5?3?5Expected?5macro?5argument?6?$AA@ 100044c4     glsl_core:prepro.obj
 0001:000034e4       ??_C@_0CH@BHFFCOAB@Syntax?5error?0?5?8?$CFs?8?5macro?5redefin@ 100044e4     glsl_core:prepro.obj
 0001:00003510       ??_C@_0EK@FBBHFMHJ@Syntax?5error?0?5cannot?5?$CDdefine?5?$CFs?0@ 10004510     glsl_core:prepro.obj
 0001:0000355c       ??_C@_02FKHNAOPL@__?$AA@   1000455c     glsl_core:prepro.obj
 0001:00003560       ??_C@_0EL@LFKEIEFK@Syntax?5error?0?5cannot?5?$CDdefine?5?$CFs?0@ 10004560     glsl_core:prepro.obj
 0001:000035ac       ??_C@_03JMNLHFFI@GL_?$AA@  100045ac     glsl_core:prepro.obj
 0001:000035b0       ??_C@_0CI@IJIPBHKF@Syntax?5error?0?5invalid?5name?5for?5?$CD@ 100045b0     glsl_core:prepro.obj
 0001:000035d8       ??_C@_0DC@OPENOEK@Syntax?5error?0?5no?5parameter?5speci@ 100045d8     glsl_core:prepro.obj
 0001:0000360c       ??_C@_0CJ@LCIHINM@Syntax?5error?0?5?8?$CFs?8?5has?5not?5been?5@ 1000460c     glsl_core:prepro.obj
 0001:00003638       ??_C@_0EJ@BKPGFLAN@Syntax?5error?0?5cannot?5?$CDundef?5?$CFs?0?5@ 10004638     glsl_core:prepro.obj
 0001:00003688       ??_C@_0EK@OCIHNAHI@Syntax?5error?0?5cannot?5?$CDundef?5?$CFs?0?5@ 10004688     glsl_core:prepro.obj
 0001:000036d4       ??_C@_0CH@MLOHABDG@Syntax?5error?0?5invalid?5name?5for?5?$CD@ 100046d4     glsl_core:prepro.obj
 0001:000036fc       ??_C@_0DB@LIINDMKH@Syntax?5error?0?5no?5parameter?5speci@ 100046fc     glsl_core:prepro.obj
 0001:00003730       ??_C@_0CN@OPCCPMJP@Syntax?5error?0?5GLSL?5Version?5?$CFu?5no@ 10004730     glsl_core:prepro.obj
 0001:00003760       ??_C@_0DH@IBPICOMB@Syntax?5error?0?5invalid?5parameter?5@ 10004760     glsl_core:prepro.obj
 0001:00003798       ??_C@_0DD@ENEBBIIF@Syntax?5error?0?5no?5parameter?5speci@ 10004798     glsl_core:prepro.obj
 0001:000037cc       ??_C@_0DP@LOEJHIFO@?$CDversion?5must?5occur?5before?5any?5o@ 100047cc     glsl_core:prepro.obj
 0001:0000380c       ??_C@_0BH@BIPDNBHG@GL_IMG_texture_stream2?$AA@ 1000480c     glsl_core:prepro.obj
 0001:00003824       ??_C@_0BM@PDHDFJJA@GL_OES_standard_derivatives?$AA@ 10004824     glsl_core:prepro.obj
 0001:00003840       ??_C@_0BG@MLPOBCKO@GL_OES_standard_noise?$AA@ 10004840     glsl_core:prepro.obj
 0001:00003858       ??_C@_0BC@HOAGCCFG@GL_OES_texture_3D?$AA@ 10004858     glsl_core:prepro.obj
 0001:0000386c       ??_C@_0CE@OPJBKFOM@?8?8?5?3?5?5extension?5name?5not?5specifi@ 1000486c     glsl_core:prepro.obj
 0001:00003890       ??_C@_0CI@GHIJPKCB@?8?8?5?3?5?5?8?3?8?5missing?5after?5extensio@ 10004890     glsl_core:prepro.obj
 0001:000038b8       ??_C@_0CN@PKNKALFI@?8?8?5?3?5?5behaviour?5for?5extension?5no@ 100048b8     glsl_core:prepro.obj
 0001:000038e8       ??_C@_0CH@PIOIPIG@?8?8?5?3?5?5behaviour?5?8?$CFs?8?5is?5not?5supp@ 100048e8     glsl_core:prepro.obj
 0001:00003910       ??_C@_07DBNODEFN@disable?$AA@ 10004910     glsl_core:prepro.obj
 0001:00003918       ??_C@_04FNLOFOEM@warn?$AA@ 10004918     glsl_core:prepro.obj
 0001:00003920       ??_C@_0EC@FNDPJJJD@?8?8?5?3?5extension?5?8all?8?5cannot?5have@ 10004920     glsl_core:prepro.obj
 0001:00003964       ??_C@_06OFNJOBDK@enable?$AA@ 10004964     glsl_core:prepro.obj
 0001:0000396c       ??_C@_0BM@DLKHKEPF@Extension?5?$CFs?5not?5supported?6?$AA@ 1000496c     glsl_core:prepro.obj
 0001:00003988       ??_C@_07FFLLPPLH@require?$AA@ 10004988     glsl_core:prepro.obj
 0001:00003990       ??_C@_07CPCPJPKL@version?$AA@ 10004990     glsl_core:prepro.obj
 0001:00003998       ??_C@_09ODADEDNA@extension?$AA@ 10004998     glsl_core:prepro.obj
 0001:000039a4       ??_C@_06PGFLMPLC@pragma?$AA@ 100049a4     glsl_core:prepro.obj
 0001:000039ac       ??_C@_04HJPCFDOP@line?$AA@ 100049ac     glsl_core:prepro.obj
 0001:000039b4       ??_C@_05KKCIMGE@error?$AA@ 100049b4     glsl_core:prepro.obj
 0001:000039bc       ??_C@_05PKCPKOLM@undef?$AA@ 100049bc     glsl_core:prepro.obj
 0001:000039c4       ??_C@_06EPMMJFDC@define?$AA@ 100049c4     glsl_core:prepro.obj
 0001:000039cc       ??_C@_05PAODFFED@endif?$AA@ 100049cc     glsl_core:prepro.obj
 0001:000039d4       ??_C@_04GNFOIEOK@elif?$AA@ 100049d4     glsl_core:prepro.obj
 0001:000039dc       ??_C@_06ENONKJGC@ifndef?$AA@ 100049dc     glsl_core:prepro.obj
 0001:000039e4       ??_C@_05LOELCHJN@ifdef?$AA@ 100049e4     glsl_core:prepro.obj
 0001:000039ec       ??_C@_04FHMCPBIP@else?$AA@ 100049ec     glsl_core:prepro.obj
 0001:000039f4       ??_C@_02HEBPBKGD@if?$AA@   100049f4     glsl_core:prepro.obj
 0001:000039f8       ??_C@_0BK@GJEIJPFO@?8?8?5?3?5?5?5Invalid?5directive?6?$AA@ 100049f8     glsl_core:prepro.obj
 0001:00003a14       ??_C@_0BN@FIDJAKIO@?8?8?5?3?5?5?5Invalid?5directive?5?$CFs?6?$AA@ 10004a14     glsl_core:prepro.obj
 0001:00003a34       ??_C@_0P@BBCFBFHE@?$CDdefine?5?$CFs?5?$CFs?6?$AA@ 10004a34     glsl_core:prepro.obj
 0001:00003a44       ??_C@_0DH@OOJOKFBO@Premature?5end?5of?5source?$DL?5preproc@ 10004a44     glsl_core:prepro.obj
 0001:00003a7c       ??_C@_0M@NHEOPBPN@__VERSION__?$AA@ 10004a7c     glsl_core:prepro.obj
 0001:00003a88       ??_C@_08FMJNKKCK@__FILE__?$AA@ 10004a88     glsl_core:prepro.obj
 0001:00003a94       ??_C@_03FKNCMABI@?$CFlu?$AA@ 10004a94     glsl_core:prepro.obj
 0001:00003a98       ??_C@_08ICCNKGAE@__LINE__?$AA@ 10004a98     glsl_core:prepro.obj
 0001:00003aa4       ??_C@_0BD@JNHPGIN@Preprocessor?5state?$AA@ 10004aa4     glsl_core:prepro.obj
 0001:00003ab8       ??_C@_05LFMKIPII@GL_ES?$AA@ 10004ab8     glsl_core:prepro.obj
 0001:00003ac0       ??_C@_0BL@MEHCMLOH@GL_FRAGMENT_PRECISION_HIGH?$AA@ 10004ac0     glsl_core:prepro.obj
 0001:00003adc       ??_C@_01HIHLOKLC@1?$AA@    10004adc     glsl_core:prepro.obj
 0001:00003ae0       ??_C@_0DA@OFOIIK@?$CFsnot?5supported?5in?5this?5language@ 10004ae0     glsl_core:glsltree.obj
 0001:00003b10       ??_C@_01CLKCMJKC@?5?$AA@   10004b10     glsl_core:glsltree.obj
 0001:00003b14       ??_C@_07BGPGDKED@?8?$CFs?8?5?3?5?$AA@ 10004b14     glsl_core:glsltree.obj
 0001:00003b1c       ??_C@_0DF@OHKGDFCN@sampler3D?5requires?5the?5extension@ 10004b1c     glsl_core:glsltree.obj
 0001:00003b54       ??_C@_09EALEHKDP@_?$EAswizzle?$AA@ 10004b54     glsl_core:glsltree.obj
 0001:00003b60       ??_C@_0CH@HBLJCFGF@?8?$CFs?8?5?3?5illegal?5vector?5field?5sele@ 10004b60     glsl_core:glsltree.obj
 0001:00003b88       ??_C@_0GB@KMJPINA@H?3?2WINCE600?2PLATFORM?2SMDKV210?2SR@ 10004b88     glsl_core:glsltree.obj
 0001:00003bec       ??_C@_0BN@PFCALEBB@?8?$CFs?8?5?3?5undeclared?5identifer?6?$AA@ 10004bec     glsl_core:glsltree.obj
 0001:00003c0c       ??_C@_0BC@BMKFIMFD@suffix?5for?5floats?$AA@ 10004c0c     glsl_core:glsltree.obj
 0001:00003c20       ??_C@_0DJ@ECIMHPED@?8void?8?5?3?5cannot?5be?5an?5argument?5t@ 10004c20     glsl_core:glsltree.obj
 0001:00003c5c       ??_C@_0CD@CNJMOGG@?8?$CFs?8?5?3?5illegal?5use?5of?5type?5?8void@ 10004c5c     glsl_core:glsltree.obj
 0001:00003c80       ??_C@_0DI@FBAOMKMA@?8?$CFs?8?5?3?5expected?5formal?5parameter@ 10004c80     glsl_core:glsltree.obj
 0001:00003cb8       ??_C@_0CE@FEHIBDDG@?8?$CFs?8?5?3?5function?5already?5has?5a?5bo@ 10004cb8     glsl_core:glsltree.obj
 0001:00003ce0       ??_C@_0EA@EHOOEHJF@?8?$CFs?8?5?3?5overloaded?5functions?5must@ 10004ce0     glsl_core:glsltree.obj
 0001:00003d20       ??_C@_0EF@IPIFIILD@?8?$CFs?8?5?3?5overloaded?5functions?5must@ 10004d20     glsl_core:glsltree.obj
 0001:00003d68       ??_C@_0DL@BCPLAMHH@?8?$CFs?8?5?3?5overloaded?5function?5must?5@ 10004d68     glsl_core:glsltree.obj
 0001:00003da4       ??_C@_0DM@NFAOPOPI@?8?$CFs?8?5?3?5overloaded?5functions?5must@ 10004da4     glsl_core:glsltree.obj
 0001:00003de0       ??_C@_0CN@ONFDOADB@?8?$CFs?8?5?3?5?5main?5function?5cannot?5ret@ 10004de0     glsl_core:glsltree.obj
 0001:00003e10       ??_C@_0CO@DANJKBKG@?8?$CFs?8?5?3?5function?5cannot?5take?5any?5@ 10004e10     glsl_core:glsltree.obj
 0001:00003e40       ??_C@_04GHJNJNPO@main?$AA@ 10004e40     glsl_core:glsltree.obj
 0001:00003e48       ??_C@_0CO@OEODLIAF@?8?$CFs?8?5?3?5no?5matching?5overloaded?5fu@ 10004e48     glsl_core:glsltree.obj
 0001:00003e78       ??_C@_0DL@GAGGKDE@Invalid?5call?5to?5function?5?$CFs?3?5ext@ 10004e78     glsl_core:glsltree.obj
 0001:00003eb4       ??_C@_0BE@MKEJKJNF@IMG_texture_stream2?$AA@ 10004eb4     glsl_core:glsltree.obj
 0001:00003ec8       ??_C@_0BD@HMADEMII@OES_standard_noise?$AA@ 10004ec8     glsl_core:glsltree.obj
 0001:00003edc       ??_C@_0BJ@BBLIOIPO@OES_standard_derivatives?$AA@ 10004edc     glsl_core:glsltree.obj
 0001:00003ef8       ??_C@_0JK@IAGAKDJC@?8?$CFs?8?5?3?5more?5than?5one?5function?5ma@ 10004ef8     glsl_core:glsltree.obj
 0001:00003f94       ??_C@_0N@LGCNPFJO@struct_?$CFs?$EA?$CFs?$AA@ 10004f94     glsl_core:glsltree.obj
 0001:00003fa4       ??_C@_0CD@FEPDOILB@?8?$CFs?8?5?3?5no?5such?5field?5in?5structur@ 10004fa4     glsl_core:glsltree.obj
 0001:00003fc8       ??_C@_0FA@IMJOPAMG@?8?$CFs?8?5?3?5field?5selection?5requires?5@ 10004fc8     glsl_core:glsltree.obj
 0001:00004018       ??_C@_09HJGOLHNF@precision?$AA@ 10005018     glsl_core:glsltree.obj
 0001:00004024       ??_C@_0CM@GMGAPJE@?8?$CFs?8?5?3?5only?5varyings?5can?5be?5made@ 10005024     glsl_core:glsltree.obj
 0001:00004050       ??_C@_0EB@FPLDGAMG@?8?$CFs?8?5?3?5invariant?5status?5can?5only@ 10005050     glsl_core:glsltree.obj
 0001:00004094       ??_C@_0M@GPJHHEN@prec_mod?$EA?$CFs?$AA@ 10005094     glsl_core:glsltree.obj
 0001:000040a0       ??_C@_0CM@EIKIIPBN@?8?8?5?3?5break?5statement?5only?5allowe@ 100050a0     glsl_core:glsltree.obj
 0001:000040cc       ??_C@_0CP@DNALJDIP@?8?8?5?3?5continue?5statement?5only?5all@ 100050cc     glsl_core:glsltree.obj
 0001:000040fc       ??_C@_0DK@POLMABBI@Function?5call?5depth?5?$DO?51024?5detec@ 100050fc     glsl_core:glsltree.obj
 0001:00004138       ??_C@_0BM@PKEIGAJI@Function?5?8?$CFs?8?5has?5no?5body?4?6?$AA@ 10005138     glsl_core:glsltree.obj
 0001:00004154       ??_C@_0BN@EKNNMDAK@main?$CI?$CJ?5function?5is?5missing?4?6?$AA@ 10005154     glsl_core:glsltree.obj
 0001:00004178       ??_C@_0ED@HBLOLBFI@gl_Position?5must?5be?5written?5by?5a@ 10005178     glsl_core:glsltree.obj
 0001:000041bc       ??_C@_0N@MKOCCMOM@fc_?$CFs_?$CFs?$EA?$CFlu?$AA@ 100051bc     glsl_core:glsltree.obj
 0001:000041cc       ??_C@_0DK@NKMODJLF@?8?$CFs?8?5?3?5cannot?5pass?5array?5of?5unde@ 100051cc     glsl_core:glsltree.obj
 0001:00004208       ??_C@_09LLNDCCMH@bit?5shift?$AA@ 10005208     glsl_core:glsltree.obj
 0001:00004214       ??_C@_0M@EGNPDNBM@bitwise?5AND?$AA@ 10005214     glsl_core:glsltree.obj
 0001:00004220       ??_C@_0M@HGJEPKOJ@bitwise?5XOR?$AA@ 10005220     glsl_core:glsltree.obj
 0001:0000422c       ??_C@_0L@CLNLJAHB@bitwise?5OR?$AA@ 1000522c     glsl_core:glsltree.obj
 0001:00004238       ??_C@_0CL@KIIMFJCA@?8?$CFs?8?5?3?5No?5precision?5defined?5for?5@ 10005238     glsl_core:glsltree.obj
 0001:00004264       ??_C@_0CK@GKAFBAFJ@?8?$CFs?8?5?3?5Precision?5not?5valid?5for?5t@ 10005264     glsl_core:glsltree.obj
 0001:00004290       ??_C@_0CH@NJDKMFMB@array?5size?5must?5be?5a?5positive?5in@ 10005290     glsl_core:glsltree.obj
 0001:000042b8       ??_C@_0CO@BGIDIOLP@?8?$CFs?8?5?3?5array?5size?5must?5be?5a?5posi@ 100052b8     glsl_core:glsltree.obj
 0001:000042e8       ??_C@_0BN@HICHHBBG@array?5size?5must?5be?5declared?6?$AA@ 100052e8     glsl_core:glsltree.obj
 0001:00004308       ??_C@_0BC@OJDELNKH@UnnamedStruct?$EA?$CFlu?$AA@ 10005308     glsl_core:glsltree.obj
 0001:0000431c       ??_C@_0DB@JNIIMJIO@Array?5syntax?5not?5valid?5in?5this?5l@ 1000531c     glsl_core:glsltree.obj
 0001:00004350       ??_C@_0BO@MCHGFDAD@?8?$CFs?8?5?3?5undeclared?5identifier?6?$AA@ 10005350     glsl_core:glsltree.obj
 0001:00004370       ??_C@_0DN@CADEFAIB@?8?$CFs?8?5?3?5variables?5with?5qualifier?5@ 10005370     glsl_core:glsltree.obj
 0001:000043b0       ??_C@_0EB@DOMKMCDB@?8?$CFs?8?5?3?5cannot?5initialise?5arrays?5@ 100053b0     glsl_core:glsltree.obj
 0001:000043f4       ??_C@_0CP@JKBBBOPM@?8?$CFs?8?5?3?5Multi?5dimensional?5arrays?5@ 100053f4     glsl_core:glsltree.obj
 0001:00004428       ??_C@_0EO@FFIINGPK@?8?$CFs?5?$CFs?8?5?3?5cannot?5declare?5arrays?5@ 10005428     glsl_core:glsltree.obj
 0001:00004478       ??_C@_0CK@BBJNPKFJ@?8const?8?5?3?5qualifier?5not?5allowed?5@ 10005478     glsl_core:glsltree.obj
 0001:000044a4       ??_C@_0CM@LBKLBFLP@?8const?8?5?3?5qualifier?5not?5allowed?5@ 100054a4     glsl_core:glsltree.obj
 0001:000044d0       ??_C@_0DJ@OLLPIJJI@?8uniform?8?5?3?5qualifier?5not?5allowe@ 100054d0     glsl_core:glsltree.obj
 0001:00004510       ??_C@_0EL@PLBFHCIL@?5?8?$CFs?8?5?3?5default?5precision?5modifi@ 10005510     glsl_core:glsltree.obj
 0001:0000455c       ??_C@_0DJ@LIMKOKDJ@?5?8?$FL?$FN?8?5?3?5array?5syntax?5not?5valid?5f@ 1000555c     glsl_core:glsltree.obj
 0001:00004598       ??_C@_0CL@KILFBNGK@?8?8?5?3?5function?5does?5not?5return?5a?5@ 10005598     glsl_core:glsltree.obj
 0001:000045c4       ??_C@_0N@GGFFEPLF@returnval_?$CFs?$AA@ 100055c4     glsl_core:icemul.obj
 0001:000045d8       ??_C@_0FP@PPICHKAL@H?3?2WINCE600?2PLATFORM?2SMDKV210?2SR@ 100055d8     glsl_core:icemul.obj
 0001:00004638       ??_C@_0M@JMJDFMPD@pmx_arccos2?$AA@ 10005638     glsl_core:icemul.obj
 0001:00004644       ??_C@_02IIINKMCA@r0?$AA@   10005644     glsl_core:icemul.obj
 0001:00004648       ??_C@_0M@MNOGKEIO@pmx_arcsin2?$AA@ 10005648     glsl_core:icemul.obj
 0001:00004654       ??_C@_0L@GKLBCFHE@pmx_arctan?$AA@ 10005654     glsl_core:icemul.obj
 0001:00004660       ??_C@_0M@LKHCFAHB@pmx_arctan2?$AA@ 10005660     glsl_core:icemul.obj
 0001:0000466c       ??_C@_0BA@LGHEAAEH@pmx_noise1_?$CFluD?$AA@ 1000566c     glsl_core:icemul.obj
 0001:0000467c       ??_C@_0BK@LKJPEAGA@gl_PMXDepthTextureDesc?$CFlu?$AA@ 1000567c     glsl_core:icemul.obj
 0001:00004698       ??_C@_0O@OIPBGHC@acosConstant2?$AA@ 10005698     glsl_core:icemul.obj
 0001:000046a8       ??_C@_0O@CFKCEFLB@acosConstant1?$AA@ 100056a8     glsl_core:icemul.obj
 0001:000046b8       ??_C@_0O@DMLJHEPA@acosConstant0?$AA@ 100056b8     glsl_core:icemul.obj
 0001:000046c8       ??_C@_0O@FCLDNNGD@atanConstant3?$AA@ 100056c8     glsl_core:icemul.obj
 0001:000046d8       ??_C@_0O@ELKIOMCC@atanConstant2?$AA@ 100056d8     glsl_core:icemul.obj
 0001:000046e8       ??_C@_0O@GAIFLPOB@atanConstant1?$AA@ 100056e8     glsl_core:icemul.obj
 0001:000046f8       ??_C@_0O@HJJOIOKA@atanConstant0?$AA@ 100056f8     glsl_core:icemul.obj
 0001:00004708       ??_C@_0P@NGCBMMJA@atan2Constant1?$AA@ 10005708     glsl_core:icemul.obj
 0001:00004718       ??_C@_0P@MPDKPNNB@atan2Constant0?$AA@ 10005718     glsl_core:icemul.obj
 0001:00004728       ??_C@_0P@BJDPKMJH@noiseConstant2?$AA@ 10005728     glsl_core:icemul.obj
 0001:00004738       ??_C@_0P@DCBCPPFE@noiseConstant1?$AA@ 10005738     glsl_core:icemul.obj
 0001:00004748       ??_C@_0P@CLAJMOBF@noiseConstant0?$AA@ 10005748     glsl_core:icemul.obj
 0001:00004758       ??_C@_0BC@KHKLJCIM@gl_PMXPermTexture?$AA@ 10005758     glsl_core:icemul.obj
 0001:0000476c       ??_C@_0BC@DINMMLAH@gl_PMXGradTexture?$AA@ 1000576c     glsl_core:icemul.obj
 0001:00004780       ??_C@_09GHEIANLA@rs_?$CFs?$EA?$CFlu?$AA@ 10005780     glsl_core:semantic.obj
 0001:00004790       ??_C@_0GB@OCJIHKCB@H?3?2WINCE600?2PLATFORM?2SMDKV210?2SR@ 10005790     glsl_core:semantic.obj
 0001:000047f4       ??_C@_0N@LCEEANFM@rs_?$CFs_?$CFs?$EA?$CFlu?$AA@ 100057f4     glsl_core:semantic.obj
 0001:00004804       ??_C@_02GPECMEKF@?$FL?$FN?$AA@ 10005804     glsl_core:semantic.obj
 0001:00004808       ??_C@_06DDGKKJGO@fn_?$CFs?$EA?$AA@ 10005808     glsl_core:semantic.obj
 0001:00004810       ??_C@_0BH@BCBDPBHB@?8?$CFs?8?5is?5not?5constant?4?6?$AA@ 10005810     glsl_core:semantic.obj
 0001:00004828       ??_C@_0IB@GFOIJAH@?8?$CFs?8?5?3?5?5Wrong?5operand?5type?4?5No?5o@ 10005828     glsl_core:semantic.obj
 0001:000048b0       ??_C@_0KM@IIDJDOIG@?8?$CFs?8?5?3?5?5Wrong?5operand?5types?4?5No?5@ 100058b0     glsl_core:semantic.obj
 0001:00004960       ??_C@_0FA@FOGICJBC@?8?$CFs?8?5?3?5?5Wrong?5operand?5types?4?5Arr@ 10005960     glsl_core:semantic.obj
 0001:000049b0       ??_C@_0DN@OGJMDMOH@?8?$CFs?8?5?3?5?5Wrong?5operand?5types?4?5Arr@ 100059b0     glsl_core:semantic.obj
 0001:000049f0       ??_C@_0DM@LACJEOBJ@?8?$CFs?8?5?3?5l?9value?5of?5swizzle?5cannot@ 100059f0     glsl_core:semantic.obj
 0001:00004a2c       ??_C@_0CO@GKOHIBMO@?8?$CFs?8?5?3?5?5l?9value?5required?5?$CIcan?8t?5@ 10005a2c     glsl_core:semantic.obj
 0001:00004a5c       ??_C@_0BK@GDICGMNC@?8?$CFs?8?5?3?5?5l?9value?5required?6?$AA@ 10005a5c     glsl_core:semantic.obj
 0001:00004a78       ??_C@_0FC@CPFEMAHP@?8?$FL?8?5?3?5?5array?5must?5be?5redeclared?5@ 10005a78     glsl_core:semantic.obj
 0001:00004acc       ??_C@_0CJ@FHCFPJKN@?8?$FL?8?5?3?5field?5selection?5out?5of?5ran@ 10005acc     glsl_core:semantic.obj
 0001:00004af8       ??_C@_0DC@LAGKKDPB@Array?5index?5?8?$CFd?8?5out?5of?5bounds?4?5@ 10005af8     glsl_core:semantic.obj
 0001:00004b2c       ??_C@_0CH@HELBFBNP@?8?$CFs?8?5?3?5used?5without?5being?5initia@ 10005b2c     glsl_core:semantic.obj
 0001:00004b54       ??_C@_0CF@KDAONFKO@?8?$CFs?8?5?3?5only?5allowed?5at?5global?5sc@ 10005b54     glsl_core:semantic.obj
 0001:00004b7c       ??_C@_0BO@JPECECG@?8?$CFs?8?5?3?5cannot?5be?5bool?5or?5int?6?$AA@ 10005b7c     glsl_core:semantic.obj
 0001:00004b9c       ??_C@_0CO@NGBAHMIE@?8?$CFs?5?$CFs?8?5?3?5cannot?5declare?5arrays?5@ 10005b9c     glsl_core:semantic.obj
 0001:00004bcc       ??_C@_0CK@JHIFCNNH@?8?$CFs?8?5?3?5?5supported?5in?5vertex?5shad@ 10005bcc     glsl_core:semantic.obj
 0001:00004bf8       ??_C@_0CA@GMKFDLOI@?8gl_?8?5?3?5reserved?5built?9in?5name?6?$AA@ 10005bf8     glsl_core:semantic.obj
 0001:00004c18       ??_C@_03EKEJMIG@gl_?$AA@   10005c18     glsl_core:semantic.obj
 0001:00004c1c       ??_C@_0BF@IPJBEHEB@?8?$CFs?8?5?3?5redefinition?6?$AA@ 10005c1c     glsl_core:semantic.obj
 0001:00004c34       ??_C@_0DG@MPDECNKE@?8?$CFs?8?5?3?5higher?5index?5value?5alread@ 10005c34     glsl_core:semantic.obj
 0001:00004c6c       ??_C@_0DD@GKJIHCLB@?8?$CFs?8?5?3?5redeclaration?5of?5array?5wi@ 10005c6c     glsl_core:semantic.obj
 0001:00004ca0       ??_C@_0CJ@IINGJFMA@?8?$CFs?8?5?3?5redeclaration?5of?5array?5wi@ 10005ca0     glsl_core:semantic.obj
 0001:00004ccc       ??_C@_0CF@HEGOMBE@?8?$CFs?8?5?3?5declaring?5non?9array?5as?5ar@ 10005ccc     glsl_core:semantic.obj
 0001:00004cf8       ??_C@_0HH@CLEFIBKB@Calls?5to?5any?5function?5that?5may?5r@ 10005cf8     glsl_core:semantic.obj
 0001:00004d70       ??_C@_0DL@NFEJNCDD@?8constructor?8?5?3?5not?5enough?5data?5@ 10005d70     glsl_core:semantic.obj
 0001:00004dac       ??_C@_0DB@FADFBNNI@?8constructor?8?5?3?5no?5arguments?5sup@ 10005dac     glsl_core:semantic.obj
 0001:00004de0       ??_C@_0CE@PGLIGOHF@?8constructor?8?5?3?5too?5many?5argumen@ 10005de0     glsl_core:semantic.obj
 0001:00004e08       ??_C@_0FO@GMHJKCLB@?8constructor?8?5?3?5only?5a?5single?5ma@ 10005e08     glsl_core:semantic.obj
 0001:00004e68       ??_C@_0CM@MHBMNBMB@?8constructor?8?5?3?5cannot?5convert?5a@ 10005e68     glsl_core:semantic.obj
 0001:00004e94       ??_C@_0CK@FIECGCOG@?8constructor?8?5?3?5cannot?5convert?5a@ 10005e94     glsl_core:semantic.obj
 0001:00004ec0       ??_C@_0EL@EPHDCKFB@?8?$CFs?8?5?3?5Parameter?5array?5size?5does@ 10005ec0     glsl_core:semantic.obj
 0001:00004f10       ??_C@_0EK@DMJPANOP@?8?$CFs?8?5?3?5Cannot?5convert?5parameter?5@ 10005f10     glsl_core:semantic.obj
 0001:00004f5c       ??_C@_0DG@BMMJAPJE@?8?$CFs?8?5?3?5Cannot?5convert?5parameter?5@ 10005f5c     glsl_core:semantic.obj
 0001:00004f98       ??_C@_0EM@EHJBNNAN@?8Error?8?5?3?5Constant?5value?5cannot?5@ 10005f98     glsl_core:semantic.obj
 0001:00004fe8       ??_C@_0GL@NHELLIMD@?8constructor?8?5?3?5Number?5of?5constr@ 10005fe8     glsl_core:semantic.obj
 0001:00005054       ??_C@_0M@HCIFEBGA@constructor?$AA@ 10006054     glsl_core:semantic.obj
 0001:00005060       ??_C@_0DB@ODIKGIDJ@?8discard?8?5?3?5only?5supported?5in?5fr@ 10006060     glsl_core:semantic.obj
 0001:00005094       ??_C@_0CD@ODLIIFHP@?8?8?5?3?5boolean?5expression?5expected@ 10006094     glsl_core:semantic.obj
 0001:000050b8       ??_C@_0DC@MKNKCLCL@?8return?8?5?3?5function?5return?5has?5w@ 100060b8     glsl_core:semantic.obj
 0001:000050ec       ??_C@_0DC@JGLHIJJP@?8return?8?5?3?5function?5return?5is?5no@ 100060ec     glsl_core:semantic.obj
 0001:00005120       ??_C@_0DA@KIPLKFMI@?8return?8?5?3?5void?5function?5cannot?5@ 10006120     glsl_core:semantic.obj
 0001:00005150       ??_C@_0DC@IABKOPGF@?8return?8?5?3?5non?9void?5function?5mus@ 10006150     glsl_core:semantic.obj
 0001:00005184       ??_C@_0CO@PFBDOOMF@?8assign?8?5?3?5?5cannot?5convert?5from?5@ 10006184     glsl_core:semantic.obj
 0001:000051b4       ??_C@_0DF@OMAKOKIJ@?8const?8?5?3?5?5non?9matching?5types?5fo@ 100061b4     glsl_core:semantic.obj
 0001:000051ec       ??_C@_06IMFOKBKF@assign?$AA@ 100061ec     glsl_core:semantic.obj
 0001:000051f4       ??_C@_0CN@CAADMAMN@?8?$DN?8?5?3?5?5assigning?5non?9constant?5to@ 100061f4     glsl_core:semantic.obj
 0001:00005224       ??_C@_0DC@OPFDDKKG@?8?$CFs?8?5?3?5?5cannot?5initialize?5this?5t@ 10006224     glsl_core:semantic.obj
 0001:00005258       ??_C@_0KJ@EPEAGGHJ@?8?3?8?5?3?5?5wrong?5operand?5types?5?5no?5o@ 10006258     glsl_core:semantic.obj
 0001:00005304       ??_C@_0CC@MKLDGFDA@?8?8?5?3?5boolean?5expression?5expected@ 10006304     glsl_core:semantic.obj
 0001:00005328       ??_C@_0DK@DADEIOGK@?8?8?5?3?5left?5of?5?8?$FL?8?5is?5not?5of?5type?5@ 10006328     glsl_core:semantic.obj
 0001:00005364       ??_C@_0DM@POAJCJK@?8?$CFs?8?5?3?5left?5of?5?8?$FL?8?5is?5not?5of?5typ@ 10006364     glsl_core:semantic.obj
 0001:000053a0       ??_C@_0CE@HCDENGKP@?8?$FL?$FN?8?5?3?5integer?5expression?5requir@ 100063a0     glsl_core:semantic.obj
 0001:000053c4       ??_C@_0CJ@LDAPHGKE@?8?4?8?5?3?5cannot?5apply?5dot?5operator?5@ 100063c4     glsl_core:semantic.obj
 0001:000053f0       ??_C@_0CM@FMCOHPCK@?8?$CFs?8?5?3?5vector?5field?5selection?5ou@ 100063f0     glsl_core:semantic.obj
 0001:00005420       ??_C@_0EH@KMEPABJP@?8?$CFs?8?5?3?5field?5selection?5requires?5@ 10006420     glsl_core:semantic.obj
 0001:00005468       ??_C@_0CN@KPECCIGP@?8?4?8?5?3?5cannot?5apply?5dot?5operator?5@ 10006468     glsl_core:semantic.obj
 0001:00005498       ??_C@_0DD@JAEBPOMH@?8?$CFs?8?5?3?5?4length?$CI?$CJ?5requires?5array?5@ 10006498     glsl_core:semantic.obj
 0001:000054cc       ??_C@_0N@LEEGPDKF@no?9symbol?9id?$AA@ 100064cc     glsl_core:semantic.obj
 0001:00005524       ??_C@_0M@FOBNLFJI@1?44?414?42514?$AA@ 10006524     glsl_binshader:esbinshader.obj
 0001:00005530       ??_C@_07GLJEJNB@EMITCUT?$AA@ 10006530     usc:usc_utils.obj
 0001:00005538       ??_C@_03ODLKKDDL@CUT?$AA@  10006538     usc:usc_utils.obj
 0001:0000553c       ??_C@_04GBCMHBCE@EMIT?$AA@ 1000653c     usc:usc_utils.obj
 0001:00005544       ??_C@_05IALEHOEG@MOVVI?$AA@ 10006544     usc:usc_utils.obj
 0001:0000554c       ??_C@_05BFJLGMF@MOVCP?$AA@ 1000654c     usc:usc_utils.obj
 0001:00005554       ??_C@_06FGGEKBGC@DOT4CP?$AA@ 10006554     usc:usc_utils.obj
 0001:0000555c       ??_C@_04KIMHDDNA@LOGP?$AA@ 1000655c     usc:usc_utils.obj
 0001:00005564       ??_C@_04HBHAILHC@EXPP?$AA@ 10006564     usc:usc_utils.obj
 0001:0000556c       ??_C@_08LKBLKNDD@MOVA_INT?$AA@ 1000656c     usc:usc_utils.obj
 0001:00005578       ??_C@_08GONKFOLN@MOVA_RNE?$AA@ 10006578     usc:usc_utils.obj
 0001:00005584       ??_C@_08INHPMPD@MOVA_TRC?$AA@ 10006584     usc:usc_utils.obj
 0001:00005590       ??_C@_03CAOCJACM@MOV?$AA@  10006590     usc:usc_utils.obj
 0001:00005594       ??_C@_03GEANJIEE@NOP?$AA@  10006594     usc:usc_utils.obj
 0001:00005598       ??_C@_09IHCHNAND@ENDSWITCH?$AA@ 10006598     usc:usc_utils.obj
 0001:000055a4       ??_C@_07MGCPDNLD@DEFAULT?$AA@ 100065a4     usc:usc_utils.obj
 0001:000055ac       ??_C@_04OGNCDOIK@CASE?$AA@ 100065ac     usc:usc_utils.obj
 0001:000055b4       ??_C@_06DKNFLPLN@SWITCH?$AA@ 100065b4     usc:usc_utils.obj
 0001:000055bc       ??_C@_07FMKELLMM@IFNZBIT?$AA@ 100065bc     usc:usc_utils.obj
 0001:000055c4       ??_C@_0O@DACOILJI@CONTINUENZBIT?$AA@ 100065c4     usc:usc_utils.obj
 0001:000055d4       ??_C@_08CEMFIBFD@RETNZBIT?$AA@ 100065d4     usc:usc_utils.obj
 0001:000055e0       ??_C@_09IKPIPGBO@CALLNZBIT?$AA@ 100065e0     usc:usc_utils.obj
 0001:000055ec       ??_C@_0L@EHPDBPCP@BREAKNZBIT?$AA@ 100065ec     usc:usc_utils.obj
 0001:000055f8       ??_C@_0N@NLKMEFNE@GLSLLOOPTAIL?$AA@ 100065f8     usc:usc_utils.obj
 0001:00005608       ??_C@_0N@DNBOGBJP@GLSLCONTINUE?$AA@ 10006608     usc:usc_utils.obj
 0001:00005618       ??_C@_0M@IIPMBMC@GLSLENDLOOP?$AA@ 10006618     usc:usc_utils.obj
 0001:00005624       ??_C@_0P@BNMDBKOA@GLSLSTATICLOOP?$AA@ 10006624     usc:usc_utils.obj
 0001:00005634       ??_C@_08CIJJABIK@GLSLLOOP?$AA@ 10006634     usc:usc_utils.obj
 0001:00005640       ??_C@_05LAJLJJBC@CALLP?$AA@ 10006640     usc:usc_utils.obj
 0001:00005648       ??_C@_06IFIODKDJ@BREAKP?$AA@ 10006648     usc:usc_utils.obj
 0001:00005650       ??_C@_03PGALJLHC@IFP?$AA@  10006650     usc:usc_utils.obj
 0001:00005654       ??_C@_05EILEDKCG@LABEL?$AA@ 10006654     usc:usc_utils.obj
 0001:0000565c       ??_C@_04DLKKMOMO@SETP?$AA@ 1000665c     usc:usc_utils.obj
 0001:00005664       ??_C@_06OEGBHLKL@BREAKC?$AA@ 10006664     usc:usc_utils.obj
 0001:0000566c       ??_C@_05IAGBLAKG@BREAK?$AA@ 1000666c     usc:usc_utils.obj
 0001:00005674       ??_C@_03JHOENKOA@IFC?$AA@  10006674     usc:usc_utils.obj
 0001:00005678       ??_C@_06EBGPDKJM@ENDREP?$AA@ 10006678     usc:usc_utils.obj
 0001:00005680       ??_C@_03HDFFPFLF@REP?$AA@  10006680     usc:usc_utils.obj
 0001:00005684       ??_C@_07OEFEMAML@ENDLOOP?$AA@ 10006684     usc:usc_utils.obj
 0001:0000568c       ??_C@_04KGNEGCGI@LOOP?$AA@ 1000668c     usc:usc_utils.obj
 0001:00005694       ??_C@_03BHDJDALB@RET?$AA@  10006694     usc:usc_utils.obj
 0001:00005698       ??_C@_06KFOFNBHF@CALLNZ?$AA@ 10006698     usc:usc_utils.obj
 0001:000056a0       ??_C@_04CAGKGBIO@CALL?$AA@ 100066a0     usc:usc_utils.obj
 0001:000056a8       ??_C@_05DLHFLCAN@ENDIF?$AA@ 100066a8     usc:usc_utils.obj
 0001:000056b0       ??_C@_04JLPIBDPH@ELSE?$AA@ 100066b0     usc:usc_utils.obj
 0001:000056b8       ??_C@_02NJNGHICB@IF?$AA@   100066b8     usc:usc_utils.obj
 0001:000056bc       ??_C@_07BKIPBFEF@KPNZBIT?$AA@ 100066bc     usc:usc_utils.obj
 0001:000056c4       ??_C@_04CJHNKBPM@KPLE?$AA@ 100066c4     usc:usc_utils.obj
 0001:000056cc       ??_C@_04HKKEICOM@KPLT?$AA@ 100066cc     usc:usc_utils.obj
 0001:000056d4       ??_C@_05CLKBFMGL@LDCLZ?$AA@ 100066d4     usc:usc_utils.obj
 0001:000056dc       ??_C@_03KDLOPOLM@LDC?$AA@  100066dc     usc:usc_utils.obj
 0001:000056e0       ??_C@_03OMPPGIHL@LDD?$AA@  100066e0     usc:usc_utils.obj
 0001:000056e4       ??_C@_07DFIAJNK@LDPIFTC?$AA@ 100066e4     usc:usc_utils.obj
 0001:000056ec       ??_C@_03MCFBLPCO@LDP?$AA@  100066ec     usc:usc_utils.obj
 0001:000056f0       ??_C@_03CECGOCHD@LDL?$AA@  100066f0     usc:usc_utils.obj
 0001:000056f4       ??_C@_03LKKFMPPN@LDB?$AA@  100066f4     usc:usc_utils.obj
 0001:000056f8       ??_C@_02ONCLNIEI@LD?$AA@   100066f8     usc:usc_utils.obj
 0001:000056fc       ??_C@_03CDEJPCIF@XOR?$AA@  100066fc     usc:usc_utils.obj
 0001:00005700       ??_C@_03PBAHGDAB@SHR?$AA@  10006700     usc:usc_utils.obj
 0001:00005704       ??_C@_02PDPFNDMG@OR?$AA@   10006704     usc:usc_utils.obj
 0001:00005708       ??_C@_03GBFNEA@NOT?$AA@    10006708     usc:usc_utils.obj
 0001:0000570c       ??_C@_03BLGELAIE@ASR?$AA@  1000670c     usc:usc_utils.obj
 0001:00005710       ??_C@_03CFEGFMNO@SHL?$AA@  10006710     usc:usc_utils.obj
 0001:00005714       ??_C@_03BDACDFHA@AND?$AA@  10006714     usc:usc_utils.obj
 0001:00005718       ??_C@_04IEDALHLA@SQRT?$AA@ 10006718     usc:usc_utils.obj
 0001:00005720       ??_C@_03FJGHKDBE@DIV?$AA@  10006720     usc:usc_utils.obj
 0001:00005724       ??_C@_07MPADIFOA@MOVCBIT?$AA@ 10006724     usc:usc_utils.obj
 0001:0000572c       ??_C@_06CELPKKED@SETBNE?$AA@ 1000672c     usc:usc_utils.obj
 0001:00005734       ??_C@_06HEOCFNDN@SETBLT?$AA@ 10006734     usc:usc_utils.obj
 0001:0000573c       ??_C@_06CLGOJBMM@SETBGE?$AA@ 1000673c     usc:usc_utils.obj
 0001:00005744       ??_C@_06GEEJCPH@SETBEQ?$AA@ 10006744     usc:usc_utils.obj
 0001:0000574c       ??_C@_03BMCMHJGB@SGN?$AA@  1000674c     usc:usc_utils.obj
 0001:00005750       ??_C@_03PPNIKAKK@SGE?$AA@  10006750     usc:usc_utils.obj
 0001:00005754       ??_C@_03KAFEGMFL@SLT?$AA@  10006754     usc:usc_utils.obj
 0001:00005758       ??_C@_06CPNAGDBH@OGLLIT?$AA@ 10006758     usc:usc_utils.obj
 0001:00005760       ??_C@_03KOOFOJHJ@LIT?$AA@  10006760     usc:usc_utils.obj
 0001:00005764       ??_C@_03HKOAOHDA@DST?$AA@  10006764     usc:usc_utils.obj
 0001:00005768       ??_C@_03MPEOJJHN@DSY?$AA@  10006768     usc:usc_utils.obj
 0001:0000576c       ??_C@_03NGFFKIDM@DSX?$AA@  1000676c     usc:usc_utils.obj
 0001:00005770       ??_C@_04PEPPOICM@M3X2?$AA@ 10006770     usc:usc_utils.obj
 0001:00005778       ??_C@_04ONOENJGN@M3X3?$AA@ 10006778     usc:usc_utils.obj
 0001:00005780       ??_C@_04KCKFEPKK@M3X4?$AA@ 10006780     usc:usc_utils.obj
 0001:00005788       ??_C@_04HADDOBNE@M4X3?$AA@ 10006788     usc:usc_utils.obj
 0001:00005790       ??_C@_04DPHCHHBD@M4X4?$AA@ 10006790     usc:usc_utils.obj
 0001:00005798       ??_C@_07PKBLCBGP@SINCOS2?$AA@ 10006798     usc:usc_utils.obj
 0001:000057a0       ??_C@_06NMMLFNJO@SINCOS?$AA@ 100067a0     usc:usc_utils.obj
 0001:000057a8       ??_C@_03BPJLEIIC@ABS?$AA@  100067a8     usc:usc_utils.obj
 0001:000057ac       ??_C@_03IPJPMEHL@NRM?$AA@  100067ac     usc:usc_utils.obj
 0001:000057b0       ??_C@_03KJLECDHJ@CRS?$AA@  100067b0     usc:usc_utils.obj
 0001:000057b4       ??_C@_03LEPPJAKI@MAX?$AA@  100067b4     usc:usc_utils.obj
 0001:000057b8       ??_C@_03KGHEHEMH@MIN?$AA@  100067b8     usc:usc_utils.obj
 0001:000057bc       ??_C@_03JLIKCOCP@POW?$AA@  100067bc     usc:usc_utils.obj
 0001:000057c0       ??_C@_03NKPKGAOM@LRP?$AA@  100067c0     usc:usc_utils.obj
 0001:000057c4       ??_C@_04KJMDDEDC@CEIL?$AA@ 100067c4     usc:usc_utils.obj
 0001:000057cc       ??_C@_03FBKOMNAB@RND?$AA@  100067cc     usc:usc_utils.obj
 0001:000057d0       ??_C@_03EILFPMEA@RNE?$AA@  100067d0     usc:usc_utils.obj
 0001:000057d4       ??_C@_03COLIFOAO@TRC?$AA@  100067d4     usc:usc_utils.obj
 0001:000057d8       ??_C@_03JBMJGMHA@FLR?$AA@  100067d8     usc:usc_utils.obj
 0001:000057dc       ??_C@_03NEKIMBBK@FRC?$AA@  100067dc     usc:usc_utils.obj
 0001:000057e0       ??_C@_03LJALPNPL@CND?$AA@  100067e0     usc:usc_utils.obj
 0001:000057e4       ??_C@_03JFODJEPH@CMP?$AA@  100067e4     usc:usc_utils.obj
 0001:000057e8       ??_C@_03MLIHNEFJ@LOG?$AA@  100067e8     usc:usc_utils.obj
 0001:000057ec       ??_C@_03KKGFKKLA@EXP?$AA@  100067ec     usc:usc_utils.obj
 0001:000057f0       ??_C@_05LCJGEIPC@RSQRT?$AA@ 100067f0     usc:usc_utils.obj
 0001:000057f8       ??_C@_05NDDJDMFB@RECIP?$AA@ 100067f8     usc:usc_utils.obj
 0001:00005800       ??_C@_04IHEGMLJL@DOT4?$AA@ 10006800     usc:usc_utils.obj
 0001:00005808       ??_C@_04MIAHFNFM@DOT3?$AA@ 10006808     usc:usc_utils.obj
 0001:00005810       ??_C@_07JJJNIFD@DOT2ADD?$AA@ 10006810     usc:usc_utils.obj
 0001:00005818       ??_C@_03FCIIMNPF@MAD?$AA@  10006818     usc:usc_utils.obj
 0001:0000581c       ??_C@_03IBHOEMFB@MUL?$AA@  1000681c     usc:usc_utils.obj
 0001:00005820       ??_C@_03KPDLEBHD@SUB?$AA@  10006820     usc:usc_utils.obj
 0001:00005824       ??_C@_03BOJFLAKG@ADD?$AA@  10006824     usc:usc_utils.obj
 0001:00005828       g_asInputInstDesc          10006828     usc:usc_utils.obj
 0001:00005d78       g_auSetBitCount            10006d78     usc:usc.obj
 0001:00005db8       g_abSingleBitSet           10006db8     usc:usc.obj
 0001:00005df8       g_puSwapRedAndBlueChan     10006df8     usc:usc.obj
 0001:00005e18       g_puSwapRedAndBlueMask     10006e18     usc:usc.obj
 0001:00005e58       g_aiSingleComponent        10006e58     usc:usc.obj
 0001:00005e98       g_puInvertCompOp           10006e98     usc:usc.obj
 0001:00005eb4       g_puNegateCompOp           10006eb4     usc:usc.obj
 0001:00005ed8       ??_C@_0FB@JPGMFLBG@H?3?2WINCE600?2PLATFORM?2SMDKV210?2SR@ 10006ed8     usc:data.obj
 0001:00005f50       ??_C@_0FA@KLHABLIL@H?3?2WINCE600?2PLATFORM?2SMDKV210?2SR@ 10006f50     usc:dce.obj
 0001:00005fa0       ??_C@_0BA@GBOIHAHE@Invalid_Max_Arg?$AA@ 10006fa0     usc:inst.obj
 0001:00005fb0       ??_C@_05DOJLHMDO@IEMIT?$AA@ 10006fb0     usc:inst.obj
 0001:00005fb8       ??_C@_07JACEHJFF@ISUBU16?$AA@ 10006fb8     usc:inst.obj
 0001:00005fc0       ??_C@_04PLJJJCGI@IWOP?$AA@ 10006fc0     usc:inst.obj
 0001:00005fc8       ??_C@_0N@LFLGJNGE@ISMP_USP_NDR?$AA@ 10006fc8     usc:inst.obj
 0001:00005fd8       ??_C@_0N@GMCKLOJH@ISMPGRAD_USP?$AA@ 10006fd8     usc:inst.obj
 0001:00005fe8       ??_C@_0BA@CLBBCJAE@ISMPREPLACE_USP?$AA@ 10006fe8     usc:inst.obj
 0001:00005ff8       ??_C@_0N@BJLPOEIG@ISMPBIAS_USP?$AA@ 10006ff8     usc:inst.obj
 0001:00006008       ??_C@_08LONNMFB@ISMP_USP?$AA@ 10007008     usc:inst.obj
 0001:00006014       ??_C@_09HGMODOHB@ISTARRC10?$AA@ 10007014     usc:inst.obj
 0001:00006020       ??_C@_09BHEKGJMF@ISTARRF16?$AA@ 10007020     usc:inst.obj
 0001:0000602c       ??_C@_09HAKCHIKP@ISTARRF32?$AA@ 1000702c     usc:inst.obj
 0001:00006038       ??_C@_09HJAMICPK@ILDARRC10?$AA@ 10007038     usc:inst.obj
 0001:00006044       ??_C@_09BIIINFEO@ILDARRF16?$AA@ 10007044     usc:inst.obj
 0001:00006050       ??_C@_09HPGAMECE@ILDARRF32?$AA@ 10007050     usc:inst.obj
 0001:0000605c       ??_C@_08GDOOLHHE@IFNRMF16?$AA@ 1000705c     usc:inst.obj
 0001:00006068       ??_C@_05OAPNEMIJ@IFNRM?$AA@ 10007068     usc:inst.obj
 0001:00006070       ??_C@_07CDGDIKMM@IMOVIDX?$AA@ 10007070     usc:inst.obj
 0001:00006078       ??_C@_07OFECAAOA@IFMAD16?$AA@ 10007078     usc:inst.obj
 0001:00006080       ??_C@_07LFJGBJEN@IFMUL16?$AA@ 10007080     usc:inst.obj
 0001:00006088       ??_C@_07FKGAEPOL@IFADD16?$AA@ 10007088     usc:inst.obj
 0001:00006090       ??_C@_07KAGCCBJF@IFMOV16?$AA@ 10007090     usc:inst.obj
 0001:00006098       ??_C@_09PPHBGLKI@IMOVC_I32?$AA@ 10007098     usc:inst.obj
 0001:000060a4       ??_C@_08EABOAKIG@IMOVC_U8?$AA@ 100070a4     usc:inst.obj
 0001:000060b0       ??_C@_09KBHODNCA@IMOVC_C10?$AA@ 100070b0     usc:inst.obj
 0001:000060bc       ??_C@_05LGBLJPKP@IMOVC?$AA@ 100070bc     usc:inst.obj
 0001:000060c4       ??_C@_0M@DHHKFJHD@IU16DOT4OFF?$AA@ 100070c4     usc:inst.obj
 0001:000060d0       ??_C@_0M@IFFKIFGD@IU16DOT3OFF?$AA@ 100070d0     usc:inst.obj
 0001:000060dc       ??_C@_08BEKNCKIA@IU16DOT4?$AA@ 100070dc     usc:inst.obj
 0001:000060e8       ??_C@_08FLOMLMEH@IU16DOT3?$AA@ 100070e8     usc:inst.obj
 0001:000060f4       ??_C@_0L@DOMAIKAF@IU8DOT4OFF?$AA@ 100070f4     usc:inst.obj
 0001:00006100       ??_C@_0L@IMOAFGBF@IU8DOT3OFF?$AA@ 10007100     usc:inst.obj
 0001:0000610c       ??_C@_07ILFAHJPJ@IU8DOT4?$AA@ 1000710c     usc:inst.obj
 0001:00006114       ??_C@_07MEBBOPDO@IU8DOT3?$AA@ 10007114     usc:inst.obj
 0001:0000611c       ??_C@_05BCEHFFAN@IFDPC?$AA@ 1000711c     usc:inst.obj
 0001:00006124       ??_C@_07GALLBODK@IFPSUB8?$AA@ 10007124     usc:inst.obj
 0001:0000612c       ??_C@_07JGLDJGJA@IFPADD8?$AA@ 1000712c     usc:inst.obj
 0001:00006134       ??_C@_05OLPEMHGE@IFPMA?$AA@ 10007134     usc:inst.obj
 0001:0000613c       ??_C@_05DAIMFOJL@ILRP1?$AA@ 1000713c     usc:inst.obj
 0001:00006144       ??_C@_05ECHJLDAI@ISOP3?$AA@ 10007144     usc:inst.obj
 0001:0000614c       ??_C@_05FLGCICEJ@ISOP2?$AA@ 1000714c     usc:inst.obj
 0001:00006154       ??_C@_06EJAKDDF@ISOPWM?$AA@ 10007154     usc:inst.obj
 0001:0000615c       ??_C@_04NGIIIKHN@INOP?$AA@ 1000715c     usc:inst.obj
 0001:00006164       ??_C@_05HEFIDKGH@ISMBO?$AA@ 10007164     usc:inst.obj
 0001:0000616c       ??_C@_06ECCFMIAK@ISETFC?$AA@ 1000716c     usc:inst.obj
 0001:00006174       ??_C@_04EFEJLDND@ISMR?$AA@ 10007174     usc:inst.obj
 0001:0000617c       ??_C@_06HPKHFKK@ISMLSI?$AA@ 1000717c     usc:inst.obj
 0001:00006184       ??_C@_0M@FOBIOFFC@IDRVPADDING?$AA@ 10007184     usc:inst.obj
 0001:00006190       ??_C@_05OIMNNLA@ISAVL?$AA@ 10007190     usc:inst.obj
 0001:00006198       ??_C@_05ICGKJOIJ@ISETL?$AA@ 10007198     usc:inst.obj
 0001:000061a0       ??_C@_05GPCJLNJO@ILAPC?$AA@ 100071a0     usc:inst.obj
 0001:000061a8       ??_C@_06LFIJHEFB@ILABEL?$AA@ 100071a8     usc:inst.obj
 0001:000061b0       ??_C@_05HPNNGMJE@ICALL?$AA@ 100071b0     usc:inst.obj
 0001:000061b8       ??_C@_03MDDEFBCM@IBR?$AA@  100071b8     usc:inst.obj
 0001:000061bc       ??_C@_04MOABNMAD@IRLP?$AA@ 100071bc     usc:inst.obj
 0001:000061c4       ??_C@_03MLOMMCHP@IOR?$AA@  100071c4     usc:inst.obj
 0001:000061c8       ??_C@_04JBMMOALM@IXOR?$AA@ 100071c8     usc:inst.obj
 0001:000061d0       ??_C@_04KBIHCHEJ@IAND?$AA@ 100071d0     usc:inst.obj
 0001:000061d8       ??_C@_04KJOBKCLN@IASR?$AA@ 100071d8     usc:inst.obj
 0001:000061e0       ??_C@_04EDICHBDI@ISHR?$AA@ 100071e0     usc:inst.obj
 0001:000061e8       ??_C@_04JHMDEOOH@ISHL?$AA@ 100071e8     usc:inst.obj
 0001:000061f0       ??_C@_08PHKGJIOA@ISMPGRAD?$AA@ 100071f0     usc:inst.obj
 0001:000061fc       ??_C@_0M@JNGNGGOJ@ISMPREPLACE?$AA@ 100071fc     usc:inst.obj
 0001:00006208       ??_C@_08LNNNEDJI@ISMPBIAS?$AA@ 10007208     usc:inst.obj
 0001:00006214       ??_C@_04HHHPNBFB@ISMP?$AA@ 10007214     usc:inst.obj
 0001:0000621c       ??_C@_08JMCNMCIP@ICOMBC10?$AA@ 1000721c     usc:inst.obj
 0001:00006228       ??_C@_0L@BKKPBEBB@IPCKC10F16?$AA@ 10007228     usc:inst.obj
 0001:00006234       ??_C@_0N@KMJHJNGP@IUNPCKF32F16?$AA@ 10007234     usc:inst.obj
 0001:00006244       ??_C@_0N@MLFADKMC@IUNPCKF32S16?$AA@ 10007244     usc:inst.obj
 0001:00006254       ??_C@_0N@OODLGFBO@IUNPCKF32U16?$AA@ 10007254     usc:inst.obj
 0001:00006264       ??_C@_0M@CPPBGAGA@IUNPCKF32S8?$AA@ 10007264     usc:inst.obj
 0001:00006270       ??_C@_0M@CLHMBMNC@IUNPCKF32U8?$AA@ 10007270     usc:inst.obj
 0001:0000627c       ??_C@_0M@DKMNDKHE@IUNPCKF32O8?$AA@ 1000727c     usc:inst.obj
 0001:00006288       ??_C@_0N@MNBDMKNL@IUNPCKF32C10?$AA@ 10007288     usc:inst.obj
 0001:00006298       ??_C@_0L@KADPNPHM@IPCKF16F32?$AA@ 10007298     usc:inst.obj
 0001:000062a4       ??_C@_0L@MHNHMOBG@IPCKF16F16?$AA@ 100072a4     usc:inst.obj
 0001:000062b0       ??_C@_0N@HDBIDNAJ@IUNPCKF16S16?$AA@ 100072b0     usc:inst.obj
 0001:000062c0       ??_C@_0N@FGHDGCNF@IUNPCKF16U16?$AA@ 100072c0     usc:inst.obj
 0001:000062d0       ??_C@_0M@NKFDKEFH@IUNPCKF16S8?$AA@ 100072d0     usc:inst.obj
 0001:000062dc       ??_C@_0M@NONONIOF@IUNPCKF16U8?$AA@ 100072dc     usc:inst.obj
 0001:000062e8       ??_C@_0M@MPGPPOED@IUNPCKF16O8?$AA@ 100072e8     usc:inst.obj
 0001:000062f4       ??_C@_0N@HFFLMNBA@IUNPCKF16C10?$AA@ 100072f4     usc:inst.obj
 0001:00006304       ??_C@_0L@HNEHAFHL@IPCKC10F32?$AA@ 10007304     usc:inst.obj
 0001:00006310       ??_C@_0L@HLCLEDKF@IPCKC10C10?$AA@ 10007310     usc:inst.obj
 0001:0000631c       ??_C@_09FFKGHMEC@IPCKU8F32?$AA@ 1000731c     usc:inst.obj
 0001:00006328       ??_C@_09DCEOGNCI@IPCKU8F16?$AA@ 10007328     usc:inst.obj
 0001:00006334       ??_C@_0L@INMOFKDI@IUNPCKU8U8?$AA@ 10007334     usc:inst.obj
 0001:00006340       ??_C@_0N@EGNBDIKH@IUNPCKS16F32?$AA@ 10007340     usc:inst.obj
 0001:00006350       ??_C@_0L@PGAJFJCP@IPCKU16F32?$AA@ 10007350     usc:inst.obj
 0001:0000635c       ??_C@_0N@ECOJBMPH@IUNPCKU16F16?$AA@ 1000735c     usc:inst.obj
 0001:0000636c       ??_C@_0N@EFOEIG@IUNPCKU16U16?$AA@ 1000736c     usc:inst.obj
 0001:0000637c       ??_C@_0M@FLJMKINA@IUNPCKU16U8?$AA@ 1000737c     usc:inst.obj
 0001:00006388       ??_C@_0M@IJEIDHHP@IUNPCKS16S8?$AA@ 10007388     usc:inst.obj
 0001:00006394       ??_C@_05KGKBODJH@IIMAE?$AA@ 10007394     usc:inst.obj
 0001:0000639c       ??_C@_06LECJPGPN@IIMA16?$AA@ 1000739c     usc:inst.obj
 0001:000063a4       ??_C@_04OLFEMIFO@IWDF?$AA@ 100073a4     usc:inst.obj
 0001:000063ac       ??_C@_04FLJCOIPC@IIDF?$AA@ 100073ac     usc:inst.obj
 0001:000063b4       ??_C@_05PDIIHMEN@IELDQ?$AA@ 100073b4     usc:inst.obj
 0001:000063bc       ??_C@_05MEDNJKFJ@IELDD?$AA@ 100073bc     usc:inst.obj
 0001:000063c4       ??_C@_05LACDNGLD@ISTLD?$AA@ 100073c4     usc:inst.obj
 0001:000063cc       ??_C@_05CIKIBHP@ILDLD?$AA@ 100073cc     usc:inst.obj
 0001:000063d4       ??_C@_05LIPLEFOA@ISTAD?$AA@ 100073d4     usc:inst.obj
 0001:000063dc       ??_C@_05KFCBCCM@ILDAD?$AA@ 100073dc     usc:inst.obj
 0001:000063e4       ??_C@_05NBMMJHCB@ISTLW?$AA@ 100073e4     usc:inst.obj
 0001:000063ec       ??_C@_05GDGFMAON@ILDLW?$AA@ 100073ec     usc:inst.obj
 0001:000063f4       ??_C@_05NJBEAEHC@ISTAW?$AA@ 100073f4     usc:inst.obj
 0001:000063fc       ??_C@_05GLLNFDLO@ILDAW?$AA@ 100073fc     usc:inst.obj
 0001:00006404       ??_C@_05OGHJHBDF@ISTLB?$AA@ 10007404     usc:inst.obj
 0001:0000640c       ??_C@_05FENACGPJ@ILDLB?$AA@ 1000740c     usc:inst.obj
 0001:00006414       ??_C@_05OOKBOCGG@ISTAB?$AA@ 10007414     usc:inst.obj
 0001:0000641c       ??_C@_05FMAILFKK@ILDAB?$AA@ 1000741c     usc:inst.obj
 0001:00006424       ??_C@_0L@HBCKEBHF@ILOADCONST?$AA@ 10007424     usc:inst.obj
 0001:00006430       ??_C@_09ELIHHLFM@ITESTMASK?$AA@ 10007430     usc:inst.obj
 0001:0000643c       ??_C@_04MDACDIGN@IEFO?$AA@ 1000743c     usc:inst.obj
 0001:00006444       ??_C@_08KHAKLILD@IFSUBFLR?$AA@ 10007444     usc:inst.obj
 0001:00006450       ??_C@_05NLJNBIFK@IFMAX?$AA@ 10007450     usc:inst.obj
 0001:00006458       ??_C@_05MJBGPMDF@IFMIN?$AA@ 10007458     usc:inst.obj
 0001:00006460       ??_C@_05KACMBBIP@IFDSY?$AA@ 10007460     usc:inst.obj
 0001:00006468       ??_C@_05LJDHCAMO@IFDSX?$AA@ 10007468     usc:inst.obj
 0001:00006470       ??_C@_05MFAHCCEC@IFEXP?$AA@ 10007470     usc:inst.obj
 0001:00006478       ??_C@_05KEOFFMKL@IFLOG?$AA@ 10007478     usc:inst.obj
 0001:00006480       ??_C@_05BNIHJDME@IFRSQ?$AA@ 10007480     usc:inst.obj
 0001:00006488       ??_C@_05BILKABPF@IFRCP?$AA@ 10007488     usc:inst.obj
 0001:00006490       ??_C@_05GIIHBPDD@IFDDP?$AA@ 10007490     usc:inst.obj
 0001:00006498       ??_C@_04BPGJENHD@IFDP?$AA@ 10007498     usc:inst.obj
 0001:000064a0       ??_C@_05FPDPMGFM@IFMSA?$AA@ 100074a0     usc:inst.obj
 0001:000064a8       ??_C@_05KADFIDBN@IFADM?$AA@ 100074a8     usc:inst.obj
 0001:000064b0       ??_C@_05DNOKEFAH@IFMAD?$AA@ 100074b0     usc:inst.obj
 0001:000064b8       ??_C@_05OOBMMEKD@IFMUL?$AA@ 100074b8     usc:inst.obj
 0001:000064c0       ??_C@_05MAFJMJIB@IFSUB?$AA@ 100074c0     usc:inst.obj
 0001:000064c8       ??_C@_05HBPHDIFE@IFADD?$AA@ 100074c8     usc:inst.obj
 0001:000064d0       ??_C@_05EPIABINO@IFMOV?$AA@ 100074d0     usc:inst.obj
 0001:000064d8       ??_C@_05CAOAIINM@ILIMM?$AA@ 100074d8     usc:inst.obj
 0001:000064e0       ??_C@_04JCGHICBF@IMOV?$AA@ 100074e0     usc:inst.obj
 0001:000064e8       ??_C@_07DJMIGIHO@Invalid?$AA@ 100074e8     usc:inst.obj
 0001:000064f0       g_psInstDesc               100074f0     usc:inst.obj
 0001:00008278       ??_C@_0FB@NKAKPDLO@H?3?2WINCE600?2PLATFORM?2SMDKV210?2SR@ 10009278     usc:inst.obj
 0001:000082d0       ??_C@_0FE@FOCPFJGJ@H?3?2WINCE600?2PLATFORM?2SMDKV210?2SR@ 100092d0     usc:iselect.obj
 0001:00008328       ??_C@_0FD@DMCIEOJF@H?3?2WINCE600?2PLATFORM?2SMDKV210?2SR@ 10009328     usc:intcvt.obj
 0001:000083b8       ??_C@_0FD@HDGFJLBE@H?3?2WINCE600?2PLATFORM?2SMDKV210?2SR@ 100093b8     usc:uspbin.obj
 0001:0000840c       ??_C@_0CI@HIPBGDKP@Failed?5to?5alloc?5space?5for?5USP?5PC@ 1000940c     usc:uspbin.obj
 0001:00008438       ??_C@_0FE@CPALOMJF@H?3?2WINCE600?2PLATFORM?2SMDKV210?2SR@ 10009438     usc:regpack.obj
 0001:00008490       ??_C@_0FF@HCLANLCA@H?3?2WINCE600?2PLATFORM?2SMDKV210?2SR@ 10009490     usc:finalise.obj
 0001:000084e8       ??_C@_0FF@KLGIOFA@H?3?2WINCE600?2PLATFORM?2SMDKV210?2SR@ 100094e8     usc:regalloc.obj
 0001:00008540       ??_C@_0FG@GBEEPKBO@H?3?2WINCE600?2PLATFORM?2SMDKV210?2SR@ 10009540     usc:iregalloc.obj
 0001:00008598       ??_C@_0CA@JOBGIMJA@Can?8t?5assign?5internal?5registers?$AA@ 10009598     usc:iregalloc.obj
 0001:000085b8       ??_C@_0FG@PAPFCNHD@H?3?2WINCE600?2PLATFORM?2SMDKV210?2SR@ 100095b8     usc:pregalloc.obj
 0001:00008610       ??_C@_04GHFGAMGM@BEEF?$AA@ 10009610     usc:efo.obj
 0001:00008618       ??_C@_04CAPGHGLM@AEEF?$AA@ 10009618     usc:efo.obj
 0001:00008620       ??_C@_04BMCBJMBE@AFBE?$AA@ 10009620     usc:efo.obj
 0001:00008628       ??_C@_04CFLJGADJ@AEBF?$AA@ 10009628     usc:efo.obj
 0001:00008630       ??_C@_03MIIOGCGK@FBC?$AA@  10009630     usc:efo.obj
 0001:00008634       ??_C@_03MKMINMDD@FAC?$AA@  10009634     usc:efo.obj
 0001:00008638       ??_C@_03NKDLMNIE@EBC?$AA@  10009638     usc:efo.obj
 0001:0000863c       ??_C@_03NIHNHDNN@EAC?$AA@  1000963c     usc:efo.obj
 0001:00008640       ??_C@_04GDNLHANO@BECF?$AA@ 10009640     usc:efo.obj
 0001:00008648       ??_C@_04CEHLAKAO@AECF?$AA@ 10009648     usc:efo.obj
 0001:00008650       ??_C@_03EFKKELGE@BAC?$AA@  10009650     usc:efo.obj
 0001:00008654       ??_C@_03FFFJFKND@ABC?$AA@  10009654     usc:efo.obj
 0001:00008658       ??_C@_02MJNHLAAE@EG?$AA@   10009658     usc:efo.obj
 0001:0000865c       ??_C@_03BGNCNGMO@A?9C?$AA@ 1000965c     usc:efo.obj
 0001:00008660       ??_C@_03EGHHJCA@B?9C?$AA@  10009660     usc:efo.obj
 0001:00008664       ??_C@_02MLJBAOFN@FG?$AA@   10009664     usc:efo.obj
 0001:00008668       ??_C@_03PNNMIEJN@E?9G?$AA@ 10009668     usc:efo.obj
 0001:0000866c       ??_C@_02KKLCNNNM@AC?$AA@   1000966c     usc:efo.obj
 0001:00008670       ??_C@_03OPGJCLHD@F?9G?$AA@ 10009670     usc:efo.obj
 0001:00008674       ??_C@_02KIPEGDIF@BC?$AA@   10009674     usc:efo.obj
 0001:00008678       ??_C@_03HAJFIBDK@BEA?$AA@  10009678     usc:efo.obj
 0001:0000867c       ??_C@_03HCNDDPGD@BFA?$AA@  1000967c     usc:efo.obj
 0001:00008680       ??_C@_03EJANHNBH@AEB?$AA@  10009680     usc:efo.obj
 0001:00008684       ??_C@_03ELELMDEO@AFB?$AA@  10009684     usc:efo.obj
 0001:00008688       ??_C@_02IPBDCKJM@?9G?$AA@  10009688     usc:efo.obj
 0001:0000868c       ??_C@_02OLHPOPJI@?9C?$AA@  1000968c     usc:efo.obj
 0001:00008690       ??_C@_01BBODEMC@G?$AA@     10009690     usc:efo.obj
 0001:00008694       ??_C@_03JNKHJILP@_EF?$AA@  10009694     usc:efo.obj
 0001:00008698       ??_C@_02NJEJINBK@?9A?$AA@  10009698     usc:efo.obj
 0001:0000869c       ??_C@_03MIGDBDOF@F1E?$AA@  1000969c     usc:efo.obj
 0001:000086a0       ??_C@_02PCGENONJ@?9B?$AA@  100096a0     usc:efo.obj
 0001:000086a4       ??_C@_03PBPLOPMI@E1F?$AA@  100096a4     usc:efo.obj
 0001:000086a8       ??_C@_02LNCFEIBO@?9E?$AA@  100096a8     usc:efo.obj
 0001:000086ac       ??_C@_03CDGNEBLG@B1A?$AA@  100096ac     usc:efo.obj
 0001:000086b0       ??_C@_02JGAIBLNN@?9F?$AA@  100096b0     usc:efo.obj
 0001:000086b4       ??_C@_03BKPFLNJL@A1B?$AA@  100096b4     usc:efo.obj
 0001:000086b8       ??_C@_03MBGGECJM@EAB?$AA@  100096b8     usc:efo.obj
 0001:000086bc       ??_C@_02NAMMIBEF@EF?$AA@   100096bc     usc:efo.obj
 0001:000086c0       ??_C@_03CNGBLIBD@AEF?$AA@  100096c0     usc:efo.obj
 0001:000086c4       ??_C@_02LDKJOMJN@AB?$AA@   100096c4     usc:efo.obj
 0001:000086c8       ??_C@_03BDPAOMOC@BAE?$AA@  100096c8     usc:efo.obj
 0001:000086cc       ??_C@_02NFIDJHMA@BF?$AA@   100096cc     usc:efo.obj
 0001:000086d0       ??_C@_03DINNLPCB@BAF?$AA@  100096d0     usc:efo.obj
 0001:000086d4       ??_C@_02POKOMEAD@BE?$AA@   100096d4     usc:efo.obj
 0001:000086d8       ??_C@_03DADPNFF@ABE?$AA@   100096d8     usc:efo.obj
 0001:000086dc       ??_C@_02NHMFCJJJ@AF?$AA@   100096dc     usc:efo.obj
 0001:000086e0       ??_C@_03CICOKOJG@ABF?$AA@  100096e0     usc:efo.obj
 0001:000086e4       ??_C@_02PMOIHKFK@AE?$AA@   100096e4     usc:efo.obj
 0001:000086e8       ??_C@_03KGJCAALM@BF_?$AA@  100096e8     usc:efo.obj
 0001:000086ec       ??_C@_03KENELOOF@BE_?$AA@  100096ec     usc:efo.obj
 0001:000086f0       ??_C@_03LECHKPFC@AF_?$AA@  100096f0     usc:efo.obj
 0001:000086f4       ??_C@_03LGGBBBAL@AE_?$AA@  100096f4     usc:efo.obj
 0001:000086f8       ??_C@_03COPJDPDH@FB_?$AA@  100096f8     usc:efo.obj
 0001:000086fc       ??_C@_01FHEEJDEE@A?$AA@    100096fc     usc:efo.obj
 0001:00008700       ??_C@_03DMEMJANJ@EB_?$AA@  10009700     usc:efo.obj
 0001:00008704       ??_C@_01DDCIFGEA@E?$AA@    10009704     usc:efo.obj
 0001:00008708       ??_C@_03CMLPIBGO@FA_?$AA@  10009708     usc:efo.obj
 0001:0000870c       ??_C@_01BIAFAFID@F?$AA@    1000970c     usc:efo.obj
 0001:00008710       ??_C@_01HMGJMAIH@B?$AA@    10009710     usc:efo.obj
 0001:00008714       ??_C@_03DOAKCOIA@EA_?$AA@  10009714     usc:efo.obj
 0001:000092d8       ??_C@_0FA@MHHBKHDK@H?3?2WINCE600?2PLATFORM?2SMDKV210?2SR@ 1000a2d8     usc:efo.obj
 0001:00009328       ??_C@_0FD@EEIBDBKF@H?3?2WINCE600?2PLATFORM?2SMDKV210?2SR@ 1000a328     usc:f16opt.obj
 0001:00009380       ??_C@_0FA@FKCBCJHN@H?3?2WINCE600?2PLATFORM?2SMDKV210?2SR@ 1000a380     usc:ssa.obj
 0001:00009400       ??_C@_0FG@KGIOKKN@H?3?2WINCE600?2PLATFORM?2SMDKV210?2SR@ 1000a400     usc:icvt_core.obj
 0001:00009458       ??_C@_0CK@IIKBJMGF@Texture?5dimensionality?5must?5be?51@ 1000a458     usc:icvt_core.obj
 0001:00009488       ??_C@_0EG@PONEANLB@Destination?5modifiers?5on?5texture@ 1000a488     usc:icvt_core.obj
 0001:000094d0       ??_C@_0DF@BEHGFGAJ@Pixelflex?5only?5supports?5texture?5@ 1000a4d0     usc:icvt_core.obj
 0001:00009508       ??_C@_0CI@BNIJLCI@?$HLIF?1BREAK?1CALL?$HNP?5with?5invalid?5sw@ 1000a508     usc:icvt_core.obj
 0001:00009530       ??_C@_0DI@IPLDEMFP@if?5source?5argument?5must?5be?5eithe@ 1000a530     usc:icvt_core.obj
 0001:00009568       ??_C@_0CM@FBJPAGGL@if?5source?5argument?5must?5be?5a?5boo@ 1000a568     usc:icvt_core.obj
 0001:00009594       ??_C@_0BF@MFMPPLG@No?5loop?5terminator?4?6?$AA@ 1000a594     usc:icvt_core.obj
 0001:000095ac       ??_C@_0O@MNLANCOH@MAIN?5FUNCTION?$AA@ 1000a5ac     usc:icvt_core.obj
 0001:000095bc       ??_C@_0BB@FLLMPGAP@SECONDARY?5UPDATE?$AA@ 1000a5bc     usc:icvt_core.obj
 0001:00009658       ??_C@_0FD@POCKMCBN@H?3?2WINCE600?2PLATFORM?2SMDKV210?2SR@ 1000a658     usc:layout.obj
 0001:000096ac       ??_C@_0CG@HHEEPOEO@Error?5generating?5subroutine?5USSE@ 1000a6ac     usc:layout.obj
 0001:000096d4       ??_C@_0CA@BIADDCMB@Error?5generating?5main?5USSE?5code?$AA@ 1000a6d4     usc:layout.obj
 0001:000096f4       ??_C@_0CF@PJEBCOKN@Error?5generating?5SA?9update?5USSE?5@ 1000a6f4     usc:layout.obj
 0001:00009728       ??_C@_0FA@FOOJDFFF@H?3?2WINCE600?2PLATFORM?2SMDKV210?2SR@ 1000a728     usc:asm.obj
 0001:00009778       ??_C@_0FF@LDNNACEB@H?3?2WINCE600?2PLATFORM?2SMDKV210?2SR@ 1000a778     usc:icvt_f32.obj
 0001:000097e0       ??_C@_0FF@EGHPMGHG@H?3?2WINCE600?2PLATFORM?2SMDKV210?2SR@ 1000a7e0     usc:icvt_f16.obj
 0001:00009838       ??_C@_0FF@DDNJAIBJ@H?3?2WINCE600?2PLATFORM?2SMDKV210?2SR@ 1000a838     usc:icvt_c10.obj
 0001:00009890       ??_C@_0FF@ECILLAJE@H?3?2WINCE600?2PLATFORM?2SMDKV210?2SR@ 1000a890     usc:icvt_i32.obj
 0001:000098e8       ??_C@_0FE@EIFHPDKJ@H?3?2WINCE600?2PLATFORM?2SMDKV210?2SR@ 1000a8e8     usc:precovr.obj
 0001:0000993c       ??_C@_0BK@FGDIKLKK@Invalid?5program?5structure?$AA@ 1000a93c     usc:precovr.obj
 0001:00009958       ??_C@_06CMDGOKBM@SGX545?$AA@ 1000a958     useasm:utils.obj
 0001:00009960       ??_C@_06HKGMENJK@SGX543?$AA@ 1000a960     useasm:utils.obj
 0001:00009968       ??_C@_06EIFKCPBI@SGX541?$AA@ 1000a968     useasm:utils.obj
 0001:00009970       ??_C@_06FBEBBOFJ@SGX540?$AA@ 1000a970     useasm:utils.obj
 0001:00009978       ??_C@_06CJHJPMJJ@SGX535?$AA@ 1000a978     useasm:utils.obj
 0001:00009980       ??_C@_06ENBFDJJN@SGX531?$AA@ 1000a980     useasm:utils.obj
 0001:00009988       ??_C@_06FEAOAINM@SGX530?$AA@ 1000a988     useasm:utils.obj
 0001:00009990       ??_C@_06FFMMGCOL@SGX520?$AA@ 1000a990     useasm:utils.obj
 0001:00009c38       ??_C@_05NCHGGDHJ@sprvv?$AA@ 1000ac38     useasm:usetab.obj
 0001:00009c40       ??_C@_06HFBPFKMP@idxscw?$AA@ 1000ac40     useasm:usetab.obj
 0001:00009c48       ??_C@_06IGIKOIK@idxscr?$AA@ 1000ac48     useasm:usetab.obj
 0001:00009c50       ??_C@_0L@JLOMIJPI@vpckc10c10?$AA@ 1000ac50     useasm:usetab.obj
 0001:00009c5c       ??_C@_0M@ECFENLNA@vpckfc10f32?$AA@ 1000ac5c     useasm:usetab.obj
 0001:00009c68       ??_C@_0L@PKGINOEM@vpckc10f16?$AA@ 1000ac68     useasm:usetab.obj
 0001:00009c74       ??_C@_0L@PONMFEDE@vpckf32c10?$AA@ 1000ac74     useasm:usetab.obj
 0001:00009c80       ??_C@_0L@PILABCOK@vpckf32f32?$AA@ 1000ac80     useasm:usetab.obj
 0001:00009c8c       ??_C@_0L@JPFIADIA@vpckf32f16?$AA@ 1000ac8c     useasm:usetab.obj
 0001:00009c98       ??_C@_0L@PIJPKECN@vpckf32s16?$AA@ 1000ac98     useasm:usetab.obj
 0001:00009ca4       ??_C@_0L@NNPEPLPB@vpckf32u16?$AA@ 1000aca4     useasm:usetab.obj
 0001:00009cb0       ??_C@_09PGEODABJ@vpckf32o8?$AA@ 1000acb0     useasm:usetab.obj
 0001:00009cbc       ??_C@_09ODHCGKAN@vpckf32s8?$AA@ 1000acbc     useasm:usetab.obj
 0001:00009cc8       ??_C@_08OHIHMNPI@vpckf2u8?$AA@ 1000acc8     useasm:usetab.obj
 0001:00009cd4       ??_C@_0L@EGJEFDPP@vpckf16c10?$AA@ 1000acd4     useasm:usetab.obj
 0001:00009ce0       ??_C@_0L@EAPIBFCB@vpckf16f32?$AA@ 1000ace0     useasm:usetab.obj
 0001:00009cec       ??_C@_0L@CHBAAEEL@vpckf16f16?$AA@ 1000acec     useasm:usetab.obj
 0001:00009cf8       ??_C@_0L@EANHKDOG@vpckf16s16?$AA@ 1000acf8     useasm:usetab.obj
 0001:00009d04       ??_C@_0L@GFLMPMDK@vpckf16u16?$AA@ 1000ad04     useasm:usetab.obj
 0001:00009d10       ??_C@_09DOMPECO@vpckf16o8?$AA@ 1000ad10     useasm:usetab.obj
 0001:00009d1c       ??_C@_09BGNAKODK@vpckf16s8?$AA@ 1000ad1c     useasm:usetab.obj
 0001:00009d28       ??_C@_09BCFNNCII@vpckf16u8?$AA@ 1000ad28     useasm:usetab.obj
 0001:00009d34       ??_C@_0M@MABDAOCA@vpcks16sf32?$AA@ 1000ad34     useasm:usetab.obj
 0001:00009d40       ??_C@_0L@BCPGLHCC@vpcks16f16?$AA@ 1000ad40     useasm:usetab.obj
 0001:00009d4c       ??_C@_0L@HFDBBAIP@vpcks16s16?$AA@ 1000ad4c     useasm:usetab.obj
 0001:00009d58       ??_C@_0L@FAFKEPFD@vpcks16u16?$AA@ 1000ad58     useasm:usetab.obj
 0001:00009d64       ??_C@_09FAPHGHAG@vpcks16o8?$AA@ 1000ad64     useasm:usetab.obj
 0001:00009d70       ??_C@_09EFMLDNBC@vpcks16s8?$AA@ 1000ad70     useasm:usetab.obj
 0001:00009d7c       ??_C@_09EBEGEBKA@vpcks16u8?$AA@ 1000ad7c     useasm:usetab.obj
 0001:00009d88       ??_C@_0M@GHMAHKH@vpcku16sf32?$AA@ 1000ad88     useasm:usetab.obj
 0001:00009d94       ??_C@_0L@HBCGICBI@vpcku16f16?$AA@ 1000ad94     useasm:usetab.obj
 0001:00009da0       ??_C@_0L@BGOBCFLF@vpcku16s16?$AA@ 1000ada0     useasm:usetab.obj
 0001:00009dac       ??_C@_0L@DDIKHKGJ@vpcku16u16?$AA@ 1000adac     useasm:usetab.obj
 0001:00009db8       ??_C@_09IGKOIEBL@vpcku16o8?$AA@ 1000adb8     useasm:usetab.obj
 0001:00009dc4       ??_C@_09JDJCNOAP@vpcku16s8?$AA@ 1000adc4     useasm:usetab.obj
 0001:00009dd0       ??_C@_09JHBPKCLN@vpcku16u8?$AA@ 1000add0     useasm:usetab.obj
 0001:00009ddc       ??_C@_0L@GCHMNGAD@vpcko8sf32?$AA@ 1000addc     useasm:usetab.obj
 0001:00009de8       ??_C@_09BKFPOGAB@vpcko8f16?$AA@ 1000ade8     useasm:usetab.obj
 0001:00009df4       ??_C@_09HNJIEBKM@vpcko8s16?$AA@ 1000adf4     useasm:usetab.obj
 0001:00009e00       ??_C@_09FIPDBOHA@vpcko8u16?$AA@ 1000ae00     useasm:usetab.obj
 0001:00009e0c       ??_C@_08JEJLGJEL@vpcko8o8?$AA@ 1000ae0c     useasm:usetab.obj
 0001:00009e18       ??_C@_08IBKHDDFP@vpcko8s8?$AA@ 1000ae18     useasm:usetab.obj
 0001:00009e24       ??_C@_08IFCKEPON@vpcko8u8?$AA@ 1000ae24     useasm:usetab.obj
 0001:00009e30       ??_C@_0L@MCACCALJ@vpcks8sf32?$AA@ 1000ae30     useasm:usetab.obj
 0001:00009e3c       ??_C@_09GOELCEOB@vpcks8f16?$AA@ 1000ae3c     useasm:usetab.obj
 0001:00009e48       ??_C@_09JIMIDEM@vpcks8s16?$AA@ 1000ae48     useasm:usetab.obj
 0001:00009e54       ??_C@_09CMOHNMJA@vpcks8u16?$AA@ 1000ae54     useasm:usetab.obj
 0001:00009e60       ??_C@_08DBILBDMI@vpcks8o8?$AA@ 1000ae60     useasm:usetab.obj
 0001:00009e6c       ??_C@_08CELHEJNM@vpcks8s8?$AA@ 1000ae6c     useasm:usetab.obj
 0001:00009e78       ??_C@_08CADKDFGO@vpcks8u8?$AA@ 1000ae78     useasm:usetab.obj
 0001:00009e84       ??_C@_0L@KBNCBFID@vpcku8sf32?$AA@ 1000ae84     useasm:usetab.obj
 0001:00009e90       ??_C@_09LIBCMHPM@vpcku8f16?$AA@ 1000ae90     useasm:usetab.obj
 0001:00009e9c       ??_C@_09NPNFGAFB@vpcku8s16?$AA@ 1000ae9c     useasm:usetab.obj
 0001:00009ea8       ??_C@_09PKLODPIN@vpcku8u16?$AA@ 1000aea8     useasm:usetab.obj
 0001:00009eb4       ??_C@_08LOMLOGGI@vpcku8o8?$AA@ 1000aeb4     useasm:usetab.obj
 0001:00009ec0       ??_C@_08KLPHLMHM@vpcku8s8?$AA@ 1000aec0     useasm:usetab.obj
 0001:00009ecc       ??_C@_08KPHKMAMO@vpcku8u8?$AA@ 1000aecc     useasm:usetab.obj
 0001:00009ed8       ??_C@_04DGGKFKKC@vexp?$AA@ 1000aed8     useasm:usetab.obj
 0001:00009ee0       ??_C@_04FHIICEEL@vlog?$AA@ 1000aee0     useasm:usetab.obj
 0001:00009ee8       ??_C@_04OOOKOLCE@vrsq?$AA@ 1000aee8     useasm:usetab.obj
 0001:00009ef0       ??_C@_04OLNHHJBF@vrcp?$AA@ 1000aef0     useasm:usetab.obj
 0001:00009ef8       ??_C@_06BKGGAFJG@vf16dp?$AA@ 1000aef8     useasm:usetab.obj
 0001:00009f00       ??_C@_07JOHMCFEH@vf16max?$AA@ 1000af00     useasm:usetab.obj
 0001:00009f08       ??_C@_07IMPHMBCI@vf16min?$AA@ 1000af08     useasm:usetab.obj
 0001:00009f10       ??_C@_07OFMNCMJC@vf16dsy?$AA@ 1000af10     useasm:usetab.obj
 0001:00009f18       ??_C@_07PMNGBNND@vf16dsx?$AA@ 1000af18     useasm:usetab.obj
 0001:00009f20       ??_C@_07POCLHEPF@vf16frc?$AA@ 1000af20     useasm:usetab.obj
 0001:00009f28       ??_C@_07DEBGAFEJ@vf16add?$AA@ 1000af28     useasm:usetab.obj
 0001:00009f30       ??_C@_07KLPNPJLO@vf16mul?$AA@ 1000af30     useasm:usetab.obj
 0001:00009f38       ??_C@_07HIALHIBK@vf16mad?$AA@ 1000af38     useasm:usetab.obj
 0001:00009f40       ??_C@_03PAAOMFKJ@vdp?$AA@  1000af40     useasm:usetab.obj
 0001:00009f44       ??_C@_04FDEBGJGP@vdsy?$AA@ 1000af44     useasm:usetab.obj
 0001:00009f4c       ??_C@_04EKFKFICO@vdsx?$AA@ 1000af4c     useasm:usetab.obj
 0001:00009f54       ??_C@_04CIPAGALK@vmax?$AA@ 1000af54     useasm:usetab.obj
 0001:00009f5c       ??_C@_04DKHLIENF@vmin?$AA@ 1000af5c     useasm:usetab.obj
 0001:00009f64       ??_C@_04EIKHDBAI@vfrc?$AA@ 1000af64     useasm:usetab.obj
 0001:00009f6c       ??_C@_04ICJKEALE@vadd?$AA@ 1000af6c     useasm:usetab.obj
 0001:00009f74       ??_C@_04BNHBLMED@vmul?$AA@ 1000af74     useasm:usetab.obj
 0001:00009f7c       ??_C@_04MOIHDNOH@vmad?$AA@ 1000af7c     useasm:usetab.obj
 0001:00009f84       ??_C@_07PJIFHDOJ@vmovcu8?$AA@ 1000af84     useasm:usetab.obj
 0001:00009f8c       ??_C@_05IPANMIKP@vmovc?$AA@ 1000af8c     useasm:usetab.obj
 0001:00009f94       ??_C@_04LMONGADO@vmov?$AA@ 1000af94     useasm:usetab.obj
 0001:00009f9c       ??_C@_05HKPHADDM@vmov4?$AA@ 1000af9c     useasm:usetab.obj
 0001:00009fa4       ??_C@_05DFLGJFPL@vmov3?$AA@ 1000afa4     useasm:usetab.obj
 0001:00009fac       ??_C@_05LKKHNEHN@vssq4?$AA@ 1000afac     useasm:usetab.obj
 0001:00009fb4       ??_C@_05PFOGECLK@vssq3?$AA@ 1000afb4     useasm:usetab.obj
 0001:00009fbc       ??_C@_05IBKMJGII@vsub4?$AA@ 1000afbc     useasm:usetab.obj
 0001:00009fc4       ??_C@_05MOONAAEP@vsub3?$AA@ 1000afc4     useasm:usetab.obj
 0001:00009fcc       ??_C@_05HHKEBOCC@vadd4?$AA@ 1000afcc     useasm:usetab.obj
 0001:00009fd4       ??_C@_05DIOFIIOF@vadd3?$AA@ 1000afd4     useasm:usetab.obj
 0001:00009fdc       ??_C@_05FEOCJCGB@vmul4?$AA@ 1000afdc     useasm:usetab.obj
 0001:00009fe4       ??_C@_05BLKDAEKG@vmul3?$AA@ 1000afe4     useasm:usetab.obj
 0001:00009fec       ??_C@_05IFIKADBB@vmad4?$AA@ 1000afec     useasm:usetab.obj
 0001:00009ff4       ??_C@_05MKMLJFNG@vmad3?$AA@ 1000aff4     useasm:usetab.obj
 0001:00009ffc       ??_C@_04BENAOGHO@vdp4?$AA@ 1000affc     useasm:usetab.obj
 0001:0000a004       ??_C@_04FLJBHALJ@vdp3?$AA@ 1000b004     useasm:usetab.obj
 0001:0000a00c       ??_C@_0N@JGJIGCK@emitvcbstate?$AA@ 1000b00c     useasm:usetab.obj
 0001:0000a01c       ??_C@_0O@IBKGEAGF@emitvcbvertex?$AA@ 1000b01c     useasm:usetab.obj
 0001:0000a02c       ??_C@_0N@JECFFMDK@emitmtestate?$AA@ 1000b02c     useasm:usetab.obj
 0001:0000a03c       ??_C@_0O@JMIMBMNL@emitmtevertex?$AA@ 1000b03c     useasm:usetab.obj
 0001:0000a04c       ??_C@_03PENBPHC@cfi?$AA@   1000b04c     useasm:usetab.obj
 0001:0000a050       ??_C@_02POBAIDHK@ci?$AA@   1000b050     useasm:usetab.obj
 0001:0000a054       ??_C@_02HJIIJPLF@cf?$AA@   1000b054     useasm:usetab.obj
 0001:0000a058       ??_C@_05PACJMPIO@moest?$AA@ 1000b058     useasm:usetab.obj
 0001:0000a060       ??_C@_06FOOALFNH@fnrm16?$AA@ 1000b060     useasm:usetab.obj
 0001:0000a068       ??_C@_06DJAIKELN@fnrm32?$AA@ 1000b068     useasm:usetab.obj
 0001:0000a070       ??_C@_06KNGBBCNH@sablnd?$AA@ 1000b070     useasm:usetab.obj
 0001:0000a078       ??_C@_06DPIIDNJL@fpsub8?$AA@ 1000b078     useasm:usetab.obj
 0001:0000a080       ??_C@_06MJIALFDB@fpadd8?$AA@ 1000b080     useasm:usetab.obj
 0001:0000a088       ??_C@_06OKMGDJHC@fpmul8?$AA@ 1000b088     useasm:usetab.obj
 0001:0000a090       ??_C@_06BELDBAKP@isubu8?$AA@ 1000b090     useasm:usetab.obj
 0001:0000a098       ??_C@_06CCEGFCNB@iaddu8?$AA@ 1000b098     useasm:usetab.obj
 0001:0000a0a0       ??_C@_04HIHJCIAG@fpma?$AA@ 1000b0a0     useasm:usetab.obj
 0001:0000a0a8       ??_C@_06BODAOOPP@movmsk?$AA@ 1000b0a8     useasm:usetab.obj
 0001:0000a0b0       ??_C@_04CFJGHAMN@movc?$AA@ 1000b0b0     useasm:usetab.obj
 0001:0000a0b8       ??_C@_07MKEAMJFF@padding?$AA@ 1000b0b8     useasm:usetab.obj
 0001:0000a0c0       ??_C@_07BANDBPIA@iaddu32?$AA@ 1000b0c0     useasm:usetab.obj
 0001:0000a0c8       ??_C@_06DBFEDEDN@imov16?$AA@ 1000b0c8     useasm:usetab.obj
 0001:0000a0d0       ??_C@_06MNLAAEHH@imulu8?$AA@ 1000b0d0     useasm:usetab.obj
 0001:0000a0d8       ??_C@_05KNHGNCD@imul8?$AA@ 1000b0d8     useasm:usetab.obj
 0001:0000a0e0       ??_C@_05NPJJGJMK@isub8?$AA@ 1000b0e0     useasm:usetab.obj
 0001:0000a0e8       ??_C@_05CJJBOBGA@iadd8?$AA@ 1000b0e8     useasm:usetab.obj
 0001:0000a0f0       ??_C@_06KMLOELCJ@iadd32?$AA@ 1000b0f0     useasm:usetab.obj
 0001:0000a0f8       ??_C@_07EIGBPOGB@imulu16?$AA@ 1000b0f8     useasm:usetab.obj
 0001:0000a100       ??_C@_07MALAKHJD@isubu16?$AA@ 1000b100     useasm:usetab.obj
 0001:0000a108       ??_C@_07HHDLAOOK@iaddu16?$AA@ 1000b108     useasm:usetab.obj
 0001:0000a110       ??_C@_06CEKAAMOF@imul16?$AA@ 1000b110     useasm:usetab.obj
 0001:0000a118       ??_C@_06PNKDBIDN@isub16?$AA@ 1000b118     useasm:usetab.obj
 0001:0000a120       ??_C@_06MLFGFKED@iadd16?$AA@ 1000b120     useasm:usetab.obj
 0001:0000a128       ??_C@_05OJCDMDMI@asop2?$AA@ 1000b128     useasm:usetab.obj
 0001:0000a130       ??_C@_04BNKIMGJI@lrp2?$AA@ 1000b130     useasm:usetab.obj
 0001:0000a138       ??_C@_04DGIFJFFL@lrp1?$AA@ 1000b138     useasm:usetab.obj
 0001:0000a140       ??_C@_04JEDFNLGM@alrp?$AA@ 1000b140     useasm:usetab.obj
 0001:0000a148       ??_C@_05BLLJMLJF@arsop?$AA@ 1000b148     useasm:usetab.obj
 0001:0000a150       ??_C@_04IILBKMIG@asop?$AA@ 1000b150     useasm:usetab.obj
 0001:0000a158       ??_C@_04OBPEPKPD@asub?$AA@ 1000b158     useasm:usetab.obj
 0001:0000a160       ??_C@_04FAFKALCG@aadd?$AA@ 1000b160     useasm:usetab.obj
 0001:0000a168       ??_C@_07NOKJPFJG@aintrp2?$AA@ 1000b168     useasm:usetab.obj
 0001:0000a170       ??_C@_07PFIEKGFF@aintrp1?$AA@ 1000b170     useasm:usetab.obj
 0001:0000a178       ??_C@_04HDJKLMOD@phas?$AA@ 1000b178     useasm:usetab.obj
 0001:0000a180       ??_C@_04IPMEAKK@setm?$AA@  1000b180     useasm:usetab.obj
 0001:0000a188       ??_C@_03EEOHENCN@wop?$AA@  1000b188     useasm:usetab.obj
 0001:0000a18c       ??_C@_06CNLPFHCD@depthf?$AA@ 1000b18c     useasm:usetab.obj
 0001:0000a194       ??_C@_05LMCKLHKJ@atst8?$AA@ 1000b194     useasm:usetab.obj
 0001:0000a19c       ??_C@_05FFPFIJHE@ptoff?$AA@ 1000b19c     useasm:usetab.obj
 0001:0000a1a4       ??_C@_06GIPMBBEA@pcoeff?$AA@ 1000b1a4     useasm:usetab.obj
 0001:0000a1ac       ??_C@_03OJMAPEGJ@str?$AA@  1000b1ac     useasm:usetab.obj
 0001:0000a1b0       ??_C@_03PNJMBANA@ldr?$AA@  1000b1b0     useasm:usetab.obj
 0001:0000a1b4       ??_C@_07KLENHKKM@fsubflr?$AA@ 1000b1b4     useasm:usetab.obj
 0001:0000a1bc       ??_C@_07EOGFDLKI@release?$AA@ 1000b1bc     useasm:usetab.obj
 0001:0000a1c4       ??_C@_04MKMCLCOO@lock?$AA@ 1000b1c4     useasm:usetab.obj
 0001:0000a1cc       ??_C@_06OPKGODIN@fddpc4?$AA@ 1000b1cc     useasm:usetab.obj
 0001:0000a1d4       ??_C@_06KAOHHFEK@fddpc3?$AA@ 1000b1d4     useasm:usetab.obj
 0001:0000a1dc       ??_C@_05FCEHFDPG@fddpc?$AA@ 1000b1dc     useasm:usetab.obj
 0001:0000a1e4       ??_C@_05KHLNJIGF@fddp4?$AA@ 1000b1e4     useasm:usetab.obj
 0001:0000a1ec       ??_C@_05OIPMAOKC@fddp3?$AA@ 1000b1ec     useasm:usetab.obj
 0001:0000a1f4       ??_C@_04PLAKPAFB@fddp?$AA@ 1000b1f4     useasm:usetab.obj
 0001:0000a1fc       ??_C@_05GGKGEFIE@fdpc4?$AA@ 1000b1fc     useasm:usetab.obj
 0001:0000a204       ??_C@_05CJOHNDED@fdpc3?$AA@ 1000b204     useasm:usetab.obj
 0001:0000a20c       ??_C@_04IBMKLKGP@fdpc?$AA@ 1000b20c     useasm:usetab.obj
 0001:0000a214       ??_C@_04HEDAHBPM@fdp4?$AA@ 1000b214     useasm:usetab.obj
 0001:0000a21c       ??_C@_04DLHBOHDL@fdp3?$AA@ 1000b21c     useasm:usetab.obj
 0001:0000a224       ??_C@_05HEIOGBDD@setfc?$AA@ 1000b224     useasm:usetab.obj
 0001:0000a22c       ??_C@_03DKPPLHHB@imo?$AA@  1000b22c     useasm:usetab.obj
 0001:0000a230       ??_C@_04OHNFNFAF@smbo?$AA@ 1000b230     useasm:usetab.obj
 0001:0000a238       ??_C@_04PKDBBMEC@smso?$AA@ 1000b238     useasm:usetab.obj
 0001:0000a240       ??_C@_03PKDHGMJG@smr?$AA@  1000b240     useasm:usetab.obj
 0001:0000a244       ??_C@_04HFADBHGK@smia?$AA@ 1000b244     useasm:usetab.obj
 0001:0000a24c       ??_C@_06EOEAAGLO@u16tnz?$AA@ 1000b24c     useasm:usetab.obj
 0001:0000a254       ??_C@_05NKPLKFJF@u16tz?$AA@ 1000b254     useasm:usetab.obj
 0001:0000a25c       ??_C@_04FMGLMKJC@ftnz?$AA@ 1000b25c     useasm:usetab.obj
 0001:0000a264       ??_C@_03EGNONJMM@ftz?$AA@  1000b264     useasm:usetab.obj
 0001:0000a268       ??_C@_03GJPGFFDI@nop?$AA@  1000b268     useasm:usetab.obj
 0001:0000a26c       ??_C@_03FGBGECCC@dma?$AA@  1000b26c     useasm:usetab.obj
 0001:0000a270       ??_C@_03ODCMFNNH@sms?$AA@  1000b270     useasm:usetab.obj
 0001:0000a274       ??_C@_03BJDMMCMD@ams?$AA@  1000b274     useasm:usetab.obj
 0001:0000a278       ??_C@_03DHGNGCAI@smm?$AA@  1000b278     useasm:usetab.obj
 0001:0000a27c       ??_C@_03MNHNPNBM@amm?$AA@  1000b27c     useasm:usetab.obj
 0001:0000a280       ??_C@_03JEAJBGIL@sda?$AA@  1000b280     useasm:usetab.obj
 0001:0000a284       ??_C@_03DILMFJIH@sdm?$AA@  1000b284     useasm:usetab.obj
 0001:0000a288       ??_C@_07KLCMLLPD@setpneq?$AA@ 1000b288     useasm:usetab.obj
 0001:0000a290       ??_C@_07DCGPGNGK@setplte?$AA@ 1000b290     useasm:usetab.obj
 0001:0000a298       ??_C@_06IKNJBMPL@setplt?$AA@ 1000b298     useasm:usetab.obj
 0001:0000a2a0       ??_C@_06PIHPNDDB@setpeq?$AA@ 1000b2a0     useasm:usetab.obj
 0001:0000a2a8       ??_C@_07OFGOOKGL@setpgte?$AA@ 1000b2a8     useasm:usetab.obj
 0001:0000a2b0       ??_C@_06IGIMPDBK@setpgt?$AA@ 1000b2b0     useasm:usetab.obj
 0001:0000a2b8       ??_C@_04FDNECGOD@fsub?$AA@ 1000b2b8     useasm:usetab.obj
 0001:0000a2c0       ??_C@_04DGLGBLMD@fssq?$AA@ 1000b2c0     useasm:usetab.obj
 0001:0000a2c8       ??_C@_04OCHKNHDG@fadd?$AA@ 1000b2c8     useasm:usetab.obj
 0001:0000a2d0       ??_C@_04HNJBCLMB@fmul?$AA@ 1000b2d0     useasm:usetab.obj
 0001:0000a2d8       ??_C@_04NMANPHLM@fmov?$AA@ 1000b2d8     useasm:usetab.obj
 0001:0000a2e0       ??_C@_03CNBJFNFA@mov?$AA@  1000b2e0     useasm:usetab.obj
 0001:0000a2e4       ??_C@_07OLONFCKE@emitpds?$AA@ 1000b2e4     useasm:usetab.obj
 0001:0000a2ec       ??_C@_0O@LEENHJNO@emitprimitive?$AA@ 1000b2ec     useasm:usetab.obj
 0001:0000a2fc       ??_C@_0L@FAAMFGJF@emitvertex?$AA@ 1000b2fc     useasm:usetab.obj
 0001:0000a308       ??_C@_09BIBIIHIO@emitstate?$AA@ 1000b308     useasm:usetab.obj
 0001:0000a314       ??_C@_0L@ODEMBHIP@emitpixel2?$AA@ 1000b314     useasm:usetab.obj
 0001:0000a320       ??_C@_0L@MIGBEEEM@emitpixel1?$AA@ 1000b320     useasm:usetab.obj
 0001:0000a32c       ??_C@_03FECKBHBL@wdf?$AA@  1000b32c     useasm:usetab.obj
 0001:0000a330       ??_C@_03OEOMDHLH@idf?$AA@  1000b330     useasm:usetab.obj
 0001:0000a334       ??_C@_0L@JODEDCHK@bexception?$AA@ 1000b334     useasm:usetab.obj
 0001:0000a340       ??_C@_04PMKEFCPM@lapc?$AA@ 1000b340     useasm:usetab.obj
 0001:0000a348       ??_C@_02FGOECCNH@br?$AA@   1000b348     useasm:usetab.obj
 0001:0000a34c       ??_C@_02DHALGDEF@ba?$AA@   1000b34c     useasm:usetab.obj
 0001:0000a350       ??_C@_04GAAFJDCP@eldq?$AA@ 1000b350     useasm:usetab.obj
 0001:0000a358       ??_C@_04FHLAHFDL@eldd?$AA@ 1000b358     useasm:usetab.obj
 0001:0000a360       ??_C@_04GCOCNAN@sttq?$AA@  1000b360     useasm:usetab.obj
 0001:0000a368       ??_C@_04DBJLMLBJ@sttd?$AA@ 1000b368     useasm:usetab.obj
 0001:0000a370       ??_C@_04FAHEIKIL@sttw?$AA@ 1000b370     useasm:usetab.obj
 0001:0000a378       ??_C@_04GHMBGMJP@sttb?$AA@ 1000b378     useasm:usetab.obj
 0001:0000a380       ??_C@_04LEIHHKMB@ldtq?$AA@ 1000b380     useasm:usetab.obj
 0001:0000a388       ??_C@_04IDDCJMNF@ldtd?$AA@ 1000b388     useasm:usetab.obj
 0001:0000a390       ??_C@_04OCNNNNEH@ldtw?$AA@ 1000b390     useasm:usetab.obj
 0001:0000a398       ??_C@_04NFGIDLFD@ldtb?$AA@ 1000b398     useasm:usetab.obj
 0001:0000a3a0       ??_C@_04BEBLNPMF@stlq?$AA@ 1000b3a0     useasm:usetab.obj
 0001:0000a3a8       ??_C@_04CDKODJNB@stld?$AA@ 1000b3a8     useasm:usetab.obj
 0001:0000a3b0       ??_C@_04ECEBHIED@stlw?$AA@ 1000b3b0     useasm:usetab.obj
 0001:0000a3b8       ??_C@_04HFPEJOFH@stlb?$AA@ 1000b3b8     useasm:usetab.obj
 0001:0000a3c0       ??_C@_04KGLCIIAJ@ldlq?$AA@ 1000b3c0     useasm:usetab.obj
 0001:0000a3c8       ??_C@_04JBAHGOBN@ldld?$AA@ 1000b3c8     useasm:usetab.obj
 0001:0000a3d0       ??_C@_04PAOICPIP@ldlw?$AA@ 1000b3d0     useasm:usetab.obj
 0001:0000a3d8       ??_C@_04MHFNMJJL@ldlb?$AA@ 1000b3d8     useasm:usetab.obj
 0001:0000a3e0       ??_C@_04BMMDEMJG@staq?$AA@ 1000b3e0     useasm:usetab.obj
 0001:0000a3e8       ??_C@_04CLHGKKIC@stad?$AA@ 1000b3e8     useasm:usetab.obj
 0001:0000a3f0       ??_C@_04EKJJOLBA@staw?$AA@ 1000b3f0     useasm:usetab.obj
 0001:0000a3f8       ??_C@_04HNCMANAE@stab?$AA@ 1000b3f8     useasm:usetab.obj
 0001:0000a400       ??_C@_04KOGKBLFK@ldaq?$AA@ 1000b400     useasm:usetab.obj
 0001:0000a408       ??_C@_04JJNPPNEO@ldad?$AA@ 1000b408     useasm:usetab.obj
 0001:0000a410       ??_C@_04PIDALMNM@ldaw?$AA@ 1000b410     useasm:usetab.obj
 0001:0000a418       ??_C@_04MPIFFKMI@ldab?$AA@ 1000b418     useasm:usetab.obj
 0001:0000a420       ??_C@_09KIDJGAAM@smp3dgrad?$AA@ 1000b420     useasm:usetab.obj
 0001:0000a42c       ??_C@_09OEOGLLI@smp2dgrad?$AA@ 1000b42c     useasm:usetab.obj
 0001:0000a438       ??_C@_09DPKGHBCF@smp1dgrad?$AA@ 1000b438     useasm:usetab.obj
 0001:0000a444       ??_C@_0N@IMLLGHGO@smp3dreplace?$AA@ 1000b444     useasm:usetab.obj
 0001:0000a454       ??_C@_0N@GDHJAMFA@smp2dreplace?$AA@ 1000b454     useasm:usetab.obj
 0001:0000a464       ??_C@_0N@IIEOLHFD@smp1dreplace?$AA@ 1000b464     useasm:usetab.obj
 0001:0000a474       ??_C@_09OCECLLHE@smp3dbias?$AA@ 1000b474     useasm:usetab.obj
 0001:0000a480       ??_C@_09EEDFLAMA@smp2dbias?$AA@ 1000b480     useasm:usetab.obj
 0001:0000a48c       ??_C@_09HFNNKKFN@smp1dbias?$AA@ 1000b48c     useasm:usetab.obj
 0001:0000a498       ??_C@_05OOKKMHDJ@smp3d?$AA@ 1000b498     useasm:usetab.obj
 0001:0000a4a0       ??_C@_05OPGIKNAO@smp2d?$AA@ 1000b4a0     useasm:usetab.obj
 0001:0000a4a8       ??_C@_05ONCOBDFH@smp1d?$AA@ 1000b4a8     useasm:usetab.obj
 0001:0000a4b0       ??_C@_06GGGOMLOL@ssum16?$AA@ 1000b4b0     useasm:usetab.obj
 0001:0000a4b8       ??_C@_05COGELEAH@firhh?$AA@ 1000b4b8     useasm:usetab.obj
 0001:0000a4c0       ??_C@_04JDNAGPBH@firh?$AA@ 1000b4c0     useasm:usetab.obj
 0001:0000a4c8       ??_C@_05FCKLBLAM@bilin?$AA@ 1000b4c8     useasm:usetab.obj
 0001:0000a4d0       ??_C@_05DINMDKHN@firvh?$AA@ 1000b4d0     useasm:usetab.obj
 0001:0000a4d8       ??_C@_04EHJBFAMI@firv?$AA@ 1000b4d8     useasm:usetab.obj
 0001:0000a4e0       ??_C@_07DLAPIEBJ@adifsum?$AA@ 1000b4e0     useasm:usetab.obj
 0001:0000a4e8       ??_C@_04FNGKAKMF@adif?$AA@ 1000b4e8     useasm:usetab.obj
 0001:0000a4f0       ??_C@_04CHNIFDFF@idiv?$AA@ 1000b4f0     useasm:usetab.obj
 0001:0000a4f8       ??_C@_05EIKDCMOM@ima32?$AA@ 1000b4f8     useasm:usetab.obj
 0001:0000a500       ??_C@_04DFCMAMPF@imae?$AA@ 1000b500     useasm:usetab.obj
 0001:0000a508       ??_C@_05CPELDNIG@ima16?$AA@ 1000b508     useasm:usetab.obj
 0001:0000a510       ??_C@_04DKDJCPOM@ima8?$AA@ 1000b510     useasm:usetab.obj
 0001:0000a518       ??_C@_0L@DAOCLPMG@u16dot4off?$AA@ 1000b518     useasm:usetab.obj
 0001:0000a524       ??_C@_0L@ICMCGDNG@u16dot3off?$AA@ 1000b524     useasm:usetab.obj
 0001:0000a530       ??_C@_09GIAJOEKF@u8dot4off?$AA@ 1000b530     useasm:usetab.obj
 0001:0000a53c       ??_C@_09NKCJDILF@u8dot3off?$AA@ 1000b53c     useasm:usetab.obj
 0001:0000a548       ??_C@_07EFHPPAJH@u16dot4?$AA@ 1000b548     useasm:usetab.obj
 0001:0000a550       ??_C@_07KDOGGFA@u16dot3?$AA@ 1000b550     useasm:usetab.obj
 0001:0000a558       ??_C@_06NDMPFPGO@u8dot4?$AA@ 1000b558     useasm:usetab.obj
 0001:0000a560       ??_C@_06JMIOMJKJ@u8dot3?$AA@ 1000b560     useasm:usetab.obj
 0001:0000a568       ??_C@_04EEHAHIMI@sop3?$AA@ 1000b568     useasm:usetab.obj
 0001:0000a570       ??_C@_06GEKMOMGC@sop2wm?$AA@ 1000b570     useasm:usetab.obj
 0001:0000a578       ??_C@_04FNGLEJIJ@sop2?$AA@ 1000b578     useasm:usetab.obj
 0001:0000a580       ??_C@_03HBHPADEG@rlp?$AA@  1000b580     useasm:usetab.obj
 0001:0000a584       ??_C@_03JFEOOAEC@rol?$AA@  1000b584     useasm:usetab.obj
 0001:0000a588       ??_C@_03BGJPHNPI@asr?$AA@  1000b588     useasm:usetab.obj
 0001:0000a58c       ??_C@_03PMPMKOHN@shr?$AA@  1000b58c     useasm:usetab.obj
 0001:0000a590       ??_C@_03CILNJBKC@shl?$AA@  1000b590     useasm:usetab.obj
 0001:0000a594       ??_C@_03COLCDPPJ@xor?$AA@  1000b594     useasm:usetab.obj
 0001:0000a598       ??_C@_02FODMLBIE@or?$AA@   1000b598     useasm:usetab.obj
 0001:0000a59c       ??_C@_03BOPJPIAM@and?$AA@  1000b59c     useasm:usetab.obj
 0001:0000a5a0       ??_C@_0M@CDGCCNBB@unpckc10c10?$AA@ 1000b5a0     useasm:usetab.obj
 0001:0000a5ac       ??_C@_09KNIBBCKD@unpcku8u8?$AA@ 1000b5ac     useasm:usetab.obj
 0001:0000a5b8       ??_C@_0M@MLPMEEHP@unpcks16c10?$AA@ 1000b5b8     useasm:usetab.obj
 0001:0000a5c4       ??_C@_0L@GDPGIBDB@unpcks16o8?$AA@ 1000b5c4     useasm:usetab.obj
 0001:0000a5d0       ??_C@_0L@HGMKNLCF@unpcks16s8?$AA@ 1000b5d0     useasm:usetab.obj
 0001:0000a5dc       ??_C@_0L@HCEHKHJH@unpcks16u8?$AA@ 1000b5dc     useasm:usetab.obj
 0001:0000a5e8       ??_C@_0M@MNLPLEGG@unpcks16s16?$AA@ 1000b5e8     useasm:usetab.obj
 0001:0000a5f4       ??_C@_0M@OINEOLLK@unpcks16u16?$AA@ 1000b5f4     useasm:usetab.obj
 0001:0000a600       ??_C@_0M@KKHIBDML@unpcks16f16?$AA@ 1000b600     useasm:usetab.obj
 0001:0000a60c       ??_C@_0M@KICMHBEF@unpcku16c10?$AA@ 1000b60c     useasm:usetab.obj
 0001:0000a618       ??_C@_0L@LFKPGCCM@unpcku16o8?$AA@ 1000b618     useasm:usetab.obj
 0001:0000a624       ??_C@_0L@KAJDDIDI@unpcku16s8?$AA@ 1000b624     useasm:usetab.obj
 0001:0000a630       ??_C@_0L@KEBOEEIK@unpcku16u8?$AA@ 1000b630     useasm:usetab.obj
 0001:0000a63c       ??_C@_0M@KOGPIBFM@unpcku16s16?$AA@ 1000b63c     useasm:usetab.obj
 0001:0000a648       ??_C@_0M@ILAENOIA@unpcku16u16?$AA@ 1000b648     useasm:usetab.obj
 0001:0000a654       ??_C@_0M@MJKICGPB@unpcku16f16?$AA@ 1000b654     useasm:usetab.obj
 0001:0000a660       ??_C@_0M@POBKPHBG@unpckf16c10?$AA@ 1000b660     useasm:usetab.obj
 0001:0000a66c       ??_C@_0L@DAONBCBJ@unpckf16o8?$AA@ 1000b66c     useasm:usetab.obj
 0001:0000a678       ??_C@_0L@CFNBEIAN@unpckf16s8?$AA@ 1000b678     useasm:usetab.obj
 0001:0000a684       ??_C@_0L@CBFMDELP@unpckf16u8?$AA@ 1000b684     useasm:usetab.obj
 0001:0000a690       ??_C@_0M@PIFJAHAP@unpckf16s16?$AA@ 1000b690     useasm:usetab.obj
 0001:0000a69c       ??_C@_0M@NNDCFIND@unpckf16u16?$AA@ 1000b69c     useasm:usetab.obj
 0001:0000a6a8       ??_C@_0M@JPJOKAKC@unpckf16f16?$AA@ 1000b6a8     useasm:usetab.obj
 0001:0000a6b4       ??_C@_0M@EGFCPANN@unpckf32c10?$AA@ 1000b6b4     useasm:usetab.obj
 0001:0000a6c0       ??_C@_0L@MFEPNGCO@unpckf32o8?$AA@ 1000b6c0     useasm:usetab.obj
 0001:0000a6cc       ??_C@_0L@NAHDIMDK@unpckf32s8?$AA@ 1000b6cc     useasm:usetab.obj
 0001:0000a6d8       ??_C@_0L@NEPOPAII@unpckf32u8?$AA@ 1000b6d8     useasm:usetab.obj
 0001:0000a6e4       ??_C@_0M@EABBAAME@unpckf32s16?$AA@ 1000b6e4     useasm:usetab.obj
 0001:0000a6f0       ??_C@_0M@GFHKFPBI@unpckf32u16?$AA@ 1000b6f0     useasm:usetab.obj
 0001:0000a6fc       ??_C@_0M@CHNGKHGJ@unpckf32f16?$AA@ 1000b6fc     useasm:usetab.obj
 0001:0000a708       ??_C@_0M@EADOLGAD@unpckf32f32?$AA@ 1000b708     useasm:usetab.obj
 0001:0000a714       ??_C@_09DDFDIML@pckc10s16?$AA@ 1000b714     useasm:usetab.obj
 0001:0000a720       ??_C@_09CGFOGHBH@pckc10u16?$AA@ 1000b720     useasm:usetab.obj
 0001:0000a72c       ??_C@_09GEPCJPGG@pckc10f16?$AA@ 1000b72c     useasm:usetab.obj
 0001:0000a738       ??_C@_09DBKIOAM@pckc10f32?$AA@ 1000b738     useasm:usetab.obj
 0001:0000a744       ??_C@_08IDEMMIKL@pcko8s16?$AA@ 1000b744     useasm:usetab.obj
 0001:0000a750       ??_C@_08KGCHJHHH@pcko8u16?$AA@ 1000b750     useasm:usetab.obj
 0001:0000a75c       ??_C@_08OEILGPAG@pcko8f16?$AA@ 1000b75c     useasm:usetab.obj
 0001:0000a768       ??_C@_08IDGDHOGM@pcko8f32?$AA@ 1000b768     useasm:usetab.obj
 0001:0000a774       ??_C@_08PHFIAKEL@pcks8s16?$AA@ 1000b774     useasm:usetab.obj
 0001:0000a780       ??_C@_08NCDDFFJH@pcks8u16?$AA@ 1000b780     useasm:usetab.obj
 0001:0000a78c       ??_C@_08JAJPKNOG@pcks8f16?$AA@ 1000b78c     useasm:usetab.obj
 0001:0000a798       ??_C@_08PHHHLMIM@pcks8f32?$AA@ 1000b798     useasm:usetab.obj
 0001:0000a7a4       ??_C@_08CBABOJFG@pcku8s16?$AA@ 1000b7a4     useasm:usetab.obj
 0001:0000a7b0       ??_C@_08EGKLGIK@pcku8u16?$AA@ 1000b7b0     useasm:usetab.obj
 0001:0000a7bc       ??_C@_08EGMGEOPL@pcku8f16?$AA@ 1000b7bc     useasm:usetab.obj
 0001:0000a7c8       ??_C@_08CBCOFPJB@pcku8f32?$AA@ 1000b7c8     useasm:usetab.obj
 0001:0000a7d4       ??_C@_09OLKLFBKF@pcks16s16?$AA@ 1000b7d4     useasm:usetab.obj
 0001:0000a7e0       ??_C@_09MOMAAOHJ@pcks16u16?$AA@ 1000b7e0     useasm:usetab.obj
 0001:0000a7ec       ??_C@_09IMGMPGAI@pcks16f16?$AA@ 1000b7ec     useasm:usetab.obj
 0001:0000a7f8       ??_C@_09OLIEOHGC@pcks16f32?$AA@ 1000b7f8     useasm:usetab.obj
 0001:0000a804       ??_C@_09IIHLGEJP@pcku16s16?$AA@ 1000b804     useasm:usetab.obj
 0001:0000a810       ??_C@_09KNBADLED@pcku16u16?$AA@ 1000b810     useasm:usetab.obj
 0001:0000a81c       ??_C@_09OPLMMDDC@pcku16f16?$AA@ 1000b81c     useasm:usetab.obj
 0001:0000a828       ??_C@_09IIFENCFI@pcku16f32?$AA@ 1000b828     useasm:usetab.obj
 0001:0000a834       ??_C@_09NOENOCMM@pckf16s16?$AA@ 1000b834     useasm:usetab.obj
 0001:0000a840       ??_C@_09PLCGLNBA@pckf16u16?$AA@ 1000b840     useasm:usetab.obj
 0001:0000a84c       ??_C@_09LJIKEFGB@pckf16f16?$AA@ 1000b84c     useasm:usetab.obj
 0001:0000a858       ??_C@_09NOGCFEAL@pckf16f32?$AA@ 1000b858     useasm:usetab.obj
 0001:0000a864       ??_C@_03HMHMOHCI@efo?$AA@  1000b864     useasm:usetab.obj
 0001:0000a868       ??_C@_07BJAGEKCG@fmaxmin?$AA@ 1000b868     useasm:usetab.obj
 0001:0000a870       ??_C@_07IHOEOAG@fminmax?$AA@ 1000b870     useasm:usetab.obj
 0001:0000a878       ??_C@_06ICDMGFKB@fmad16?$AA@ 1000b878     useasm:usetab.obj
 0001:0000a880       ??_C@_04DDKBPOON@fdsy?$AA@ 1000b880     useasm:usetab.obj
 0001:0000a888       ??_C@_04CKLKMPKM@fdsx?$AA@ 1000b888     useasm:usetab.obj
 0001:0000a890       ??_C@_04EIBAPHDI@fmax?$AA@ 1000b890     useasm:usetab.obj
 0001:0000a898       ??_C@_04FKJLBDFH@fmin?$AA@ 1000b898     useasm:usetab.obj
 0001:0000a8a0       ??_C@_03KABHJCDG@fdp?$AA@  1000b8a0     useasm:usetab.obj
 0001:0000a8a4       ??_C@_04EBKFHEMK@fcos?$AA@ 1000b8a4     useasm:usetab.obj
 0001:0000a8ac       ??_C@_04OKFNDDPL@fsin?$AA@ 1000b8ac     useasm:usetab.obj
 0001:0000a8b4       ??_C@_05OBEHOPDB@fsqrt?$AA@ 1000b8b4     useasm:usetab.obj
 0001:0000a8bc       ??_C@_04FGIKMNCA@fexp?$AA@ 1000b8bc     useasm:usetab.obj
 0001:0000a8c4       ??_C@_04DHGILDMJ@flog?$AA@ 1000b8c4     useasm:usetab.obj
 0001:0000a8cc       ??_C@_04IOAKHMKG@frsq?$AA@ 1000b8cc     useasm:usetab.obj
 0001:0000a8d4       ??_C@_04ILDHOOJH@frcp?$AA@ 1000b8d4     useasm:usetab.obj
 0001:0000a8dc       ??_C@_04CIEHKGIK@ffrc?$AA@ 1000b8dc     useasm:usetab.obj
 0001:0000a8e4       ??_C@_04MMLCCJDO@fmsa?$AA@ 1000b8e4     useasm:usetab.obj
 0001:0000a8ec       ??_C@_04DDLIGMHP@fadm?$AA@ 1000b8ec     useasm:usetab.obj
 0001:0000a8f4       ??_C@_04KOGHKKGF@fmad?$AA@ 1000b8f4     useasm:usetab.obj
 0001:0000a8fc       ??_C@_0BC@EOODDAGN@filter?5coefficent?$AA@ 1000b8fc     useasm:usetab.obj
 0001:0000a910       ??_C@_0BE@FBIDIDIB@8?9bit?5source?5select?$AA@ 1000b910     useasm:usetab.obj
 0001:0000a924       ??_C@_07FAJBBDOC@swizzle?$AA@ 1000b924     useasm:usetab.obj
 0001:0000a92c       ??_C@_0N@KBLPGIGB@address?5mode?$AA@ 1000b92c     useasm:usetab.obj
 0001:0000a93c       ??_C@_09DBIHEPNC@clipplane?$AA@ 1000b93c     useasm:usetab.obj
 0001:0000a948       ??_C@_09OKBKKDGM@predicate?$AA@ 1000b948     useasm:usetab.obj
 0001:0000a954       ??_C@_05IDCCNNGI@label?$AA@ 1000b954     useasm:usetab.obj
 0001:0000a95c       ??_C@_03HDFKMEON@drc?$AA@  1000b95c     useasm:usetab.obj
 0001:0000a960       ??_C@_04OHHBHOGB@link?$AA@ 1000b960     useasm:usetab.obj
 0001:0000a968       ??_C@_09MBGEJPJA@immediate?$AA@ 1000b968     useasm:usetab.obj
 0001:0000a974       ??_C@_08LEPPLCNF@internal?$AA@ 1000b974     useasm:usetab.obj
 0001:0000a980       ??_C@_08KFDOCAEB@constant?$AA@ 1000b980     useasm:usetab.obj
 0001:0000a98c       ??_C@_06FJKEMHGD@global?$AA@ 1000b98c     useasm:usetab.obj
 0001:0000a994       ??_C@_05FKHKFDID@index?$AA@ 1000b994     useasm:usetab.obj
 0001:0000a99c       ??_C@_0BE@EDPEAKOB@secondary?5attribute?$AA@ 1000b99c     useasm:usetab.obj
 0001:0000a9b0       ??_C@_0BC@FEBGALFK@primary?5attribute?$AA@ 1000b9b0     useasm:usetab.obj
 0001:0000a9c4       ??_C@_06DKIGHACF@output?$AA@ 1000b9c4     useasm:usetab.obj
 0001:0000a9cc       ??_C@_09CAHPDAG@temporary?$AA@ 1000b9cc     useasm:usetab.obj
 0001:0000a9d8       pszTypeToString            1000b9d8     useasm:usetab.obj
 0001:0000aa28       g_pfHardwareConstants      1000ba28     useasm:usetab.obj
 0001:0000ab08       g_asUseInstDesc            1000bb08     useasm:usetab.obj
 0001:0000bbd8       ??_C@_0EL@CEJMDIFD@Branch?5destination?5is?5out?5of?5ran@ 1000cbd8     useasm:useasm.obj
 0001:0000bc28       ??_C@_0EM@IGAKCAGC@Branch?5destination?5is?5out?5of?5ran@ 1000cc28     useasm:useasm.obj
 0001:0000bc78       ??_C@_0JC@CGJAIGHK@The?5destination?5label?5for?5a?5bran@ 1000cc78     useasm:useasm.obj
 0001:0000bd0c       ??_C@_0DK@NIFCHDCD@A?5swizzle?5is?5invalid?5for?5argumen@ 1000cd0c     useasm:useasm.obj
 0001:0000bd48       ??_C@_0EC@FENPMIAM@The?5modifiers?5?4flt32?0?5?4flt16?0?5?4c@ 1000cd48     useasm:useasm.obj
 0001:0000bd8c       ??_C@_0DE@EJENDBGB@?4u8?5is?5invalid?5for?5argument?5?$CFd?5f@ 1000cd8c     useasm:useasm.obj
 0001:0000bdc0       ??_C@_0DF@KNCENLBB@?4c10?5is?5invalid?5for?5argument?5?$CFd?5@ 1000cdc0     useasm:useasm.obj
 0001:0000bdf8       ??_C@_0DH@LCLAOIMP@?4flt16?5is?5invalid?5for?5argument?5?$CF@ 1000cdf8     useasm:useasm.obj
 0001:0000be30       ??_C@_0DH@IAOLGEKP@?4flt32?5is?5invalid?5for?5argument?5?$CF@ 1000ce30     useasm:useasm.obj
 0001:0000be68       ??_C@_0EC@LIBCAICE@Disable?5writeback?5is?5invalid?5for@ 1000ce68     useasm:useasm.obj
 0001:0000beac       ??_C@_0DG@MICEFMNE@?4comp?5is?5invalid?5for?5argument?5?$CFd@ 1000ceac     useasm:useasm.obj
 0001:0000bee4       ??_C@_0DH@BJDJAOJN@?4alpha?5is?5invalid?5for?5argument?5?$CF@ 1000cee4     useasm:useasm.obj
 0001:0000bf1c       ??_C@_0DG@NIHNAGBL@?4high?5is?5invalid?5for?5argument?5?$CFd@ 1000cf1c     useasm:useasm.obj
 0001:0000bf54       ??_C@_0DF@HFACOLNL@?4low?5is?5invalid?5for?5argument?5?$CFd?5@ 1000cf54     useasm:useasm.obj
 0001:0000bf8c       ??_C@_0DI@BMAPILCJ@?4invert?5is?5invalid?5for?5argument?5@ 1000cf8c     useasm:useasm.obj
 0001:0000bfc4       ??_C@_0DK@PJAHFLKI@A?5bytemask?5is?5invalid?5for?5argume@ 1000cfc4     useasm:useasm.obj
 0001:0000c000       ??_C@_0EC@IJJBJBBP@A?5component?5select?5is?5invalid?5fo@ 1000d000     useasm:useasm.obj
 0001:0000c044       ??_C@_0DE@NBGIMLFH@?4abs?5is?5invalid?5for?5argument?5?$CFd?5@ 1000d044     useasm:useasm.obj
 0001:0000c078       ??_C@_0DE@MPDILDBH@?4neg?5is?5invalid?5for?5argument?5?$CFd?5@ 1000d078     useasm:useasm.obj
 0001:0000c0ac       ??_C@_0CG@HDBABLGF@?4minp?5is?5invalid?5for?5this?5instru@ 1000d0ac     useasm:useasm.obj
 0001:0000c0d4       ??_C@_0CG@JNEGBJAJ@?4irsd?5is?5invalid?5for?5this?5instru@ 1000d0d4     useasm:useasm.obj
 0001:0000c0fc       ??_C@_0CH@MOFKMNFF@?4pwait?5is?5invalid?5for?5this?5instr@ 1000d0fc     useasm:useasm.obj
 0001:0000c124       ??_C@_0CI@FJKAAMII@?4noread?5is?5invalid?5for?5this?5inst@ 1000d124     useasm:useasm.obj
 0001:0000c14c       ??_C@_0CM@BKAEHGEJ@?4dm_nomatch?5is?5invalid?5for?5this?5@ 1000d14c     useasm:useasm.obj
 0001:0000c178       ??_C@_0CI@LAPAEMDG@?4global?5is?5invalid?5for?5this?5inst@ 1000d178     useasm:useasm.obj
 0001:0000c1a0       ??_C@_0CI@JBBFIBPL@?4gpiext?5is?5invalid?5for?5this?5inst@ 1000d1a0     useasm:useasm.obj
 0001:0000c1c8       ??_C@_0CK@DEEAJLON@?4bypassl1?5is?5invalid?5for?5this?5in@ 1000d1c8     useasm:useasm.obj
 0001:0000c1f4       ??_C@_0CF@EHCJCPGO@?4cut?5is?5invalid?5for?5this?5instruc@ 1000d1f4     useasm:useasm.obj
 0001:0000c21c       ??_C@_0CL@OGDOHFNH@?4threepart?5is?5invalid?5for?5this?5i@ 1000d21c     useasm:useasm.obj
 0001:0000c248       ??_C@_0CJ@FCBBHHDD@?4twopart?5is?5invalid?5for?5this?5ins@ 1000d248     useasm:useasm.obj
 0001:0000c274       ??_C@_0CJ@GOGNFJGL@?4trigger?5is?5invalid?5for?5this?5ins@ 1000d274     useasm:useasm.obj
 0001:0000c2a0       ??_C@_0CJ@GIKGIFLP@?4syncend?5is?5invalid?5for?5this?5ins@ 1000d2a0     useasm:useasm.obj
 0001:0000c2cc       ??_C@_0CG@IHPDGLHB@?4sinf?5is?5invalid?5for?5this?5instru@ 1000d2cc     useasm:useasm.obj
 0001:0000c2f4       ??_C@_0CF@NKHJPKHH@?4rsd?5is?5invalid?5for?5this?5instruc@ 1000d2f4     useasm:useasm.obj
 0001:0000c31c       ??_C@_0CI@NKNMDDOG@?4pcff16?5is?5invalid?5for?5this?5inst@ 1000d31c     useasm:useasm.obj
 0001:0000c344       ??_C@_0CF@CNBHLDDL@?4pcf?5is?5invalid?5for?5this?5instruc@ 1000d344     useasm:useasm.obj
 0001:0000c36c       ??_C@_0CG@KBDEHIIG@?4incs?5is?5invalid?5for?5this?5instru@ 1000d36c     useasm:useasm.obj
 0001:0000c394       ??_C@_0CF@HDBKEIDN@?4tog?5is?5invalid?5for?5this?5instruc@ 1000d394     useasm:useasm.obj
 0001:0000c3bc       ??_C@_0CF@CPPKEJPF@?4c10?5is?5invalid?5for?5this?5instruc@ 1000d3bc     useasm:useasm.obj
 0001:0000c3e4       ??_C@_0CH@JJCJAFEG@?4tpres?5is?5invalid?5for?5this?5instr@ 1000d3e4     useasm:useasm.obj
 0001:0000c40c       ??_C@_0CF@KOMKFHLA@?4i10?5is?5invalid?5for?5this?5instruc@ 1000d40c     useasm:useasm.obj
 0001:0000c434       ??_C@_0CF@KACIFBOK@?4flt?5is?5invalid?5for?5this?5instruc@ 1000d434     useasm:useasm.obj
 0001:0000c45c       ??_C@_0CF@KDIDNMAN@?4i32?5is?5invalid?5for?5this?5instruc@ 1000d45c     useasm:useasm.obj
 0001:0000c484       ??_C@_0CF@HFMHLBAE@?4i16?5is?5invalid?5for?5this?5instruc@ 1000d484     useasm:useasm.obj
 0001:0000c4ac       ??_C@_0CF@GBAIFKNL@?4sat?5is?5invalid?5for?5this?5instruc@ 1000d4ac     useasm:useasm.obj
 0001:0000c4d4       ??_C@_0DE@KONNOGII@pre?9?1post?9increment?5is?5invalid?5f@ 1000d4d4     useasm:useasm.obj
 0001:0000c508       ??_C@_0CH@MJONMLMP@?4scale?5is?5invalid?5for?5this?5instr@ 1000d508     useasm:useasm.obj
 0001:0000c530       ??_C@_0CH@BGLMLOBA@?4taske?5is?5invalid?5for?5this?5instr@ 1000d530     useasm:useasm.obj
 0001:0000c558       ??_C@_0CH@OIAHEBAH@?4tasks?5is?5invalid?5for?5this?5instr@ 1000d558     useasm:useasm.obj
 0001:0000c580       ??_C@_0CI@JKBHNFPL@?4fcfill?5is?5invalid?5for?5this?5inst@ 1000d580     useasm:useasm.obj
 0001:0000c5a8       ??_C@_0CJ@POAKEGNN@?4bpcache?5is?5invalid?5for?5this?5ins@ 1000d5a8     useasm:useasm.obj
 0001:0000c5d4       ??_C@_0CK@NHGHHGDI@?4onceonly?5is?5invalid?5for?5this?5in@ 1000d5d4     useasm:useasm.obj
 0001:0000c600       ??_C@_0CH@OGBNJBLO@?4freep?5is?5invalid?5for?5this?5instr@ 1000d600     useasm:useasm.obj
 0001:0000c628       ??_C@_0CH@NCCAPODE@?4fetch?5is?5invalid?5for?5this?5instr@ 1000d628     useasm:useasm.obj
 0001:0000c650       ??_C@_0CL@BFLFDPDE@testenable?5is?5invalid?5for?5this?5i@ 1000d650     useasm:useasm.obj
 0001:0000c67c       ??_C@_0CM@GBLJGDF@rangeneable?5is?5invalid?5for?5this?5@ 1000d67c     useasm:useasm.obj
 0001:0000c6a8       ??_C@_0CO@LDDPCEIK@postincrement?5is?5invalid?5for?5thi@ 1000d6a8     useasm:useasm.obj
 0001:0000c6d8       ??_C@_0CN@ILKEEOL@preincrement?5is?5invalid?5for?5this@ 1000d6d8     useasm:useasm.obj
 0001:0000c708       ??_C@_0CH@PGFJCIMI@?4flt16?5is?5invalid?5for?5this?5instr@ 1000d708     useasm:useasm.obj
 0001:0000c730       ??_C@_0DD@MCGMIGNN@This?5instruction?5can?8t?5be?5part?5o@ 1000d730     useasm:useasm.obj
 0001:0000c764       ??_C@_0CJ@OKDELEHB@?4renable?5is?5invalid?5for?5this?5ins@ 1000d764     useasm:useasm.obj
 0001:0000c790       ??_C@_0CF@FIFBOHH@?4abs?5is?5invalid?5for?5this?5instruc@ 1000d790     useasm:useasm.obj
 0001:0000c7b8       ??_C@_0CF@KMGKJBBN@?4mon?5is?5invalid?5for?5this?5instruc@ 1000d7b8     useasm:useasm.obj
 0001:0000c7e0       ??_C@_0CG@HGFIGOGH@?4mask?5is?5invalid?5for?5this?5instru@ 1000d7e0     useasm:useasm.obj
 0001:0000c808       ??_C@_0CJ@BJIFKGIO@?4partial?5is?5invalid?5for?5this?5ins@ 1000d808     useasm:useasm.obj
 0001:0000c834       ??_C@_0CK@IEFIOMMP@?4savelink?5is?5invalid?5for?5this?5in@ 1000d834     useasm:useasm.obj
 0001:0000c860       ??_C@_0CH@EIPKEMIK@?4synce?5is?5invalid?5for?5this?5instr@ 1000d860     useasm:useasm.obj
 0001:0000c888       ??_C@_0CF@KFDDBKGG@?4end?5is?5invalid?5for?5this?5instruc@ 1000d888     useasm:useasm.obj
 0001:0000c8b0       ??_C@_0CM@ONJAAFFM@A?5predicate?5is?5invalid?5for?5this?5@ 1000d8b0     useasm:useasm.obj
 0001:0000c8dc       ??_C@_0CO@HKFMBEAO@A?5repeat?5mask?5is?5invalid?5for?5thi@ 1000d8dc     useasm:useasm.obj
 0001:0000c90c       ??_C@_0CI@BKLOOKDP@?4repeat?5is?5invalid?5for?5this?5inst@ 1000d90c     useasm:useasm.obj
 0001:0000c934       ??_C@_0CJ@JOPLONOF@?4nosched?5is?5invalid?5for?5this?5ins@ 1000d934     useasm:useasm.obj
 0001:0000c960       ??_C@_0CH@LGEBLDJN@?4syncs?5is?5invalid?5for?5this?5instr@ 1000d960     useasm:useasm.obj
 0001:0000c988       ??_C@_0CE@LNKCCLIM@?4i8?5is?5invalid?5for?5this?5instruct@ 1000d988     useasm:useasm.obj
 0001:0000c9ac       ??_C@_0CJ@MMEFPBHM@?4skipinv?5is?5invalid?5for?5this?5ins@ 1000d9ac     useasm:useasm.obj
 0001:0000c9d8       ??_C@_0DP@KIFGKPIF@Offset?5into?5indexed?5register?5ban@ 1000d9d8     useasm:useasm.obj
 0001:0000ca18       ??_C@_0CC@LJGIDMA@Register?5type?5?$CFs?5is?5not?5indexabl@ 1000da18     useasm:useasm.obj
 0001:0000ca3c       ??_C@_0BO@NAKOKMPE@?$CFs?5is?5not?5a?5valid?5destination?$AA@ 1000da3c     useasm:useasm.obj
 0001:0000ca5c       ??_C@_0CK@FBILJLCJ@Destination?5must?5be?5a?5modifiable@ 1000da5c     useasm:useasm.obj
 0001:0000ca88       ??_C@_0CK@JGFFOFI@Invalid?5internal?5register?5specif@ 1000da88     useasm:useasm.obj
 0001:0000cab4       ??_C@_0CO@LBPJMKJE@Invalid?5fp?5internal?5register?5spe@ 1000dab4     useasm:useasm.obj
 0001:0000cae4       ??_C@_0CI@BLCMIAIL@Invalid?5global?5register?5specifie@ 1000dae4     useasm:useasm.obj
 0001:0000cb0c       ??_C@_0CH@OHEKEBML@Invalid?5index?5mask?5specified?5?$CIwa@ 1000db0c     useasm:useasm.obj
 0001:0000cb34       ??_C@_0DG@PBPNOJGF@Invalid?5secondary?5attribute?5regi@ 1000db34     useasm:useasm.obj
 0001:0000cb6c       ??_C@_0DB@FPFAHPGJ@Destination?5type?5is?5invalid?5for?5@ 1000db6c     useasm:useasm.obj
 0001:0000cba0       ??_C@_0DE@LFLBECCD@Invalid?5primary?5attribute?5regist@ 1000dba0     useasm:useasm.obj
 0001:0000cbd4       ??_C@_0CI@JCGMLMHK@Invalid?5output?5register?5specifie@ 1000dbd4     useasm:useasm.obj
 0001:0000cbfc       ??_C@_0CL@BINLLFEH@Invalid?5temporary?5register?5speci@ 1000dbfc     useasm:useasm.obj
 0001:0000cc28       ??_C@_0CP@DIKNGJCD@Source?50?5type?5can?8t?5be?5?$CFs?5for?5th@ 1000dc28     useasm:useasm.obj
 0001:0000cc58       ??_C@_0BK@EAPIEFOL@Source?50?5type?5can?8t?5be?5?$CFs?$AA@ 1000dc58     useasm:useasm.obj
 0001:0000cc74       ??_C@_0BK@DOBHJKGK@Source?50?5can?8t?5be?5indexed?$AA@ 1000dc74     useasm:useasm.obj
 0001:0000cc90       ??_C@_0DG@NFHFDDMG@?$CFs?5immediate?5value?5is?5too?5small?5@ 1000dc90     useasm:useasm.obj
 0001:0000ccc8       ??_C@_0DF@HLDFHJJG@?$CFs?5immediate?5value?5is?5too?5large?5@ 1000dcc8     useasm:useasm.obj
 0001:0000cd00       ??_C@_0DI@KIGIDHNA@Indexed?5sources?5are?5not?5availabl@ 1000dd00     useasm:useasm.obj
 0001:0000cd38       ??_C@_0BK@JHBKMFLD@Source?51?5type?5can?8t?5be?5?$CFs?$AA@ 1000dd38     useasm:useasm.obj
 0001:0000cd54       ??_C@_0DL@PKMEEOIP@Source?51?5immediate?5value?5is?5too?5@ 1000dd54     useasm:useasm.obj
 0001:0000cd90       ??_C@_08IPCCDMEN@Source?51?$AA@ 1000dd90     useasm:useasm.obj
 0001:0000cd9c       ??_C@_0CK@INEOLDIC@Invalid?5constant?5register?5specif@ 1000dd9c     useasm:useasm.obj
 0001:0000cdc8       ??_C@_0HF@OJAOJKHK@Sequence?5number?5?$CIg?$CFd?$CJ?0?5edge?5mask@ 1000ddc8     useasm:useasm.obj
 0001:0000ce40       ??_C@_0DK@LCPGEMNK@Task?5queue?5data?5?$CIg?$CFd?5to?5g?$CFd?$CJ?5can@ 1000de40     useasm:useasm.obj
 0001:0000ce7c       ??_C@_0CP@JHOJPLGE@Source?51?5type?5can?8t?5be?5?$CFs?5for?5th@ 1000de7c     useasm:useasm.obj
 0001:0000ceac       ??_C@_0BK@DEEMEDBK@Source?52?5type?5can?8t?5be?5?$CFs?$AA@ 1000deac     useasm:useasm.obj
 0001:0000cec8       ??_C@_0DL@EAJBEKJI@Source?52?5immediate?5value?5is?5too?5@ 1000dec8     useasm:useasm.obj
 0001:0000cf04       ??_C@_08KEAPGPIO@Source?52?$AA@ 1000df04     useasm:useasm.obj
 0001:0000cf10       ??_C@_0CP@LNFFELOM@Source?52?5type?5can?8t?5be?5?$CFs?5for?5th@ 1000df10     useasm:useasm.obj
 0001:0000cf40       ??_C@_0CM@IBHBOODC@Invalid?5predicate?5type?5for?5this?5@ 1000df40     useasm:useasm.obj
 0001:0000cf6c       ??_C@_0DN@GHBJDHKE@The?5third?5argument?5to?5dot3?1dot4?5@ 1000df6c     useasm:useasm.obj
 0001:0000cfac       ??_C@_0DH@BBGJEJBC@No?5flags?5are?5valid?5for?5the?5third@ 1000dfac     useasm:useasm.obj
 0001:0000cfe8       ??_C@_0EE@JPJEDBPB@The?5third?5argument?5to?5dot3?1dot4?5@ 1000dfe8     useasm:useasm.obj
 0001:0000d02c       ??_C@_0DP@MPNPCIOH@The?5second?5argument?5to?5dot3?1dot4@ 1000e02c     useasm:useasm.obj
 0001:0000d06c       ??_C@_0DI@NLNHCCFG@No?5flags?5are?5valid?5for?5the?5secon@ 1000e06c     useasm:useasm.obj
 0001:0000d0a8       ??_C@_0EF@EFCBABKE@The?5second?5argument?5to?5dot3?1dot4@ 1000e0a8     useasm:useasm.obj
 0001:0000d0f0       ??_C@_0DJ@JGDEEONP@Invalid?5integer?5source?5for?5the?5t@ 1000e0f0     useasm:useasm.obj
 0001:0000d130       ??_C@_0EE@ELFDABMP@Only?5the?5complement?5flag?5is?5vali@ 1000e130     useasm:useasm.obj
 0001:0000d178       ??_C@_0EC@DANPAEGJ@The?5third?5argument?5to?5aintrp1?5mu@ 1000e178     useasm:useasm.obj
 0001:0000d1bc       ??_C@_0DK@OPCNMALF@Invalid?5integer?5source?5for?5the?5s@ 1000e1bc     useasm:useasm.obj
 0001:0000d1f8       ??_C@_0DG@NPKDEALG@No?5flags?5are?5valid?5for?5the?5secon@ 1000e1f8     useasm:useasm.obj
 0001:0000d230       ??_C@_0ED@NIBLILEL@The?5second?5argument?5to?5aintrp1?5m@ 1000e230     useasm:useasm.obj
 0001:0000d274       ??_C@_0CM@NAFINKIH@The?5fifth?5argument?5to?5aadd?1asub?5@ 1000e274     useasm:useasm.obj
 0001:0000d2a0       ??_C@_0DH@LBMFOABC@No?5flags?5are?5valid?5for?5the?5fifth@ 1000e2a0     useasm:useasm.obj
 0001:0000d2d8       ??_C@_0EE@NHDHBHPH@The?5fifth?5argument?5to?5aadd?1asub?5@ 1000e2d8     useasm:useasm.obj
 0001:0000d320       ??_C@_0EH@BNLGGDIJ@Only?5the?5complement?5flag?5is?5vali@ 1000e320     useasm:useasm.obj
 0001:0000d368       ??_C@_0EF@BHNJGLAO@The?5fourth?5argument?5to?5aadd?1asub@ 1000e368     useasm:useasm.obj
 0001:0000d3b0       ??_C@_0CM@LAIDNOIF@The?5third?5argument?5to?5aadd?1asub?5@ 1000e3b0     useasm:useasm.obj
 0001:0000d3e0       ??_C@_0EG@KPNPAEGJ@Only?5the?5complement?5flag?5is?5vali@ 1000e3e0     useasm:useasm.obj
 0001:0000d428       ??_C@_0EE@HCICJMII@The?5third?5argument?5to?5aadd?1asub?5@ 1000e428     useasm:useasm.obj
 0001:0000d470       ??_C@_0FM@FCNEOKCI@Invalid?5choice?5for?5the?5second?5ar@ 1000e470     useasm:useasm.obj
 0001:0000d4d0       ??_C@_0EH@COHNMHNB@Only?5the?5complement?5flag?5is?5vali@ 1000e4d0     useasm:useasm.obj
 0001:0000d518       ??_C@_0EF@KIDHKMNN@The?5second?5argument?5to?5aadd?1asub@ 1000e518     useasm:useasm.obj
 0001:0000d560       ??_C@_0DO@NPGGCMGL@The?5first?5argument?5to?5aadd?1asub?5@ 1000e560     useasm:useasm.obj
 0001:0000d5a0       ??_C@_0CN@JFFLIFPF@An?5integer?5source?5selection?5is?5n@ 1000e5a0     useasm:useasm.obj
 0001:0000d5d0       ??_C@_0DH@DLDDAMMA@No?5flags?5are?5valid?5for?5the?5first@ 1000e5d0     useasm:useasm.obj
 0001:0000d608       ??_C@_0EE@BEBPNCHP@The?5first?5argument?5to?5aadd?1asub?5@ 1000e608     useasm:useasm.obj
 0001:0000d64c       ??_C@_0CN@IACABJMC@Coissued?5instruction?5with?5no?5alp@ 1000e64c     useasm:useasm.obj
 0001:0000d67c       ??_C@_0BP@IIAMCHDC@Integer?5dot4?5can?8t?5be?5coissued?$AA@ 1000e67c     useasm:useasm.obj
 0001:0000d69c       ??_C@_0DF@OBCJJOLL@Maximum?5repeat?5count?5on?5an?5integ@ 1000e69c     useasm:useasm.obj
 0001:0000d6d8       ??_C@_0EN@JPNNFBOP@Only?5?4bytemask1111?5is?5supported?5@ 1000e6d8     useasm:useasm.obj
 0001:0000d728       ??_C@_0FG@MFNCNONI@Only?5?4bytemask1111?5is?5supported?5@ 1000e728     useasm:useasm.obj
 0001:0000d780       ??_C@_0DM@GCKABEIE@Conditional?5code?5update?5isn?8t?5av@ 1000e780     useasm:useasm.obj
 0001:0000d7c0       ??_C@_0EP@POLKDPLI@For?5a?5test?5instruction?5with?5a?5re@ 1000e7c0     useasm:useasm.obj
 0001:0000d810       ??_C@_0EC@NOAGCNPB@A?5repeated?5dotproduct?5with?5test?5@ 1000e810     useasm:useasm.obj
 0001:0000d854       ??_C@_0DO@IKLPLKIL@A?5repeated?5test?5instruction?5isn?8@ 1000e854     useasm:useasm.obj
 0001:0000d894       ??_C@_0DE@KBHBIIMG@The?5maximum?5repeat?5count?5for?5thi@ 1000e894     useasm:useasm.obj
 0001:0000d8c8       ??_C@_0DB@JAOCBPNH@A?5repeat?5count?5is?5not?5valid?5for?5@ 1000e8c8     useasm:useasm.obj
 0001:0000d8fc       ??_C@_0DA@INBPMMOK@A?5repeat?5mask?5is?5not?5valid?5for?5t@ 1000e8fc     useasm:useasm.obj
 0001:0000d930       ??_C@_0HE@BDIBHBCH@For?5?$CFs?5with?5test?5the?5type?5of?5sou@ 1000e930     useasm:useasm.obj
 0001:0000d9a4       ??_C@_0CM@MLIIJFEL@The?5maximum?5predicate?5register?5n@ 1000e9a4     useasm:useasm.obj
 0001:0000d9d0       ??_C@_0CG@GNGAJDLD@Predicate?5registers?5are?5not?5inde@ 1000e9d0     useasm:useasm.obj
 0001:0000d9f8       ??_C@_0EL@MGFIGPBH@The?5second?5destination?5for?5a?5tes@ 1000e9f8     useasm:useasm.obj
 0001:0000da44       ??_C@_0DM@JKJAHMJO@No?5flags?5are?5valid?5for?5the?5predi@ 1000ea44     useasm:useasm.obj
 0001:0000da80       ??_C@_0BH@CFEGILC@Unknown?5test?5mask?5type?$AA@ 1000ea80     useasm:useasm.obj
 0001:0000da98       ??_C@_0BP@LBJMFOHM@Unknown?5channel?5combine?5option?$AA@ 1000ea98     useasm:useasm.obj
 0001:0000dab8       ??_C@_0CO@KFAIKBA@?4cperchan?5isn?8t?5supported?5on?5thi@ 1000eab8     useasm:useasm.obj
 0001:0000dae8       ??_C@_0DL@CIAFLBE@Partial?5modifier?5is?5only?5availab@ 1000eae8     useasm:useasm.obj
 0001:0000db28       ??_C@_0EP@HBANCFBC@Saturation?5modifier?5is?5only?5avai@ 1000eb28     useasm:useasm.obj
 0001:0000db78       ??_C@_0FG@HDDPHDFM@Only?5?40?5is?5a?5valid?5component?5sel@ 1000eb78     useasm:useasm.obj
 0001:0000dbd0       ??_C@_0FM@BHACNAEE@Only?5?40?5and?5?42?5are?5valid?5compone@ 1000ebd0     useasm:useasm.obj
 0001:0000dc2c       ??_C@_0CL@ONLJAILI@The?5maximum?5number?5of?5a?5drc?5regi@ 1000ec2c     useasm:useasm.obj
 0001:0000dc58       ??_C@_0DJ@KMKOLKOO@No?5flags?5are?5valid?5for?5a?5depende@ 1000ec58     useasm:useasm.obj
 0001:0000dc98       ??_C@_0EE@BEFGELHF@A?5dependent?5read?5counter?5registe@ 1000ec98     useasm:useasm.obj
 0001:0000dce0       ??_C@_0FI@PNECLJK@The?5last?5argument?5to?5a?5normalise@ 1000ece0     useasm:useasm.obj
 0001:0000dd38       ??_C@_0CF@LANAPEBC@Invalid?5choice?5for?5argument?5?$CFd?5t@ 1000ed38     useasm:useasm.obj
 0001:0000dd60       ??_C@_0CK@DBEGJBPP@Integer?5source?5selectors?5aren?8t?5@ 1000ed60     useasm:useasm.obj
 0001:0000dd8c       ??_C@_0CJ@GGNGAINM@No?5flags?5are?5valid?5for?5argument?5@ 1000ed8c     useasm:useasm.obj
 0001:0000ddb8       ??_C@_0DH@CDAHKKKK@Argument?5?$CFd?5to?5?$CFs?5should?5be?5an?5i@ 1000edb8     useasm:useasm.obj
 0001:0000ddf0       ??_C@_0CB@FIJFOLFN@Invalid?5swizzle?5component?5select@ 1000edf0     useasm:useasm.obj
 0001:0000de14       ??_C@_0CB@LDONDCDD@No?5flags?5are?5valid?5for?5a?5swizzle@ 1000ee14     useasm:useasm.obj
 0001:0000de38       ??_C@_0CM@FIPFFMDN@A?5swizzle?5can?8t?5be?5accessed?5in?5i@ 1000ee38     useasm:useasm.obj
 0001:0000de64       ??_C@_0DN@HIOOPOOE@The?5third?5argument?5to?5a?5fnrm16?5i@ 1000ee64     useasm:useasm.obj
 0001:0000dea8       ??_C@_0FJ@MPJBDJBG@The?5destination?5for?5a?5normalise?5@ 1000eea8     useasm:useasm.obj
 0001:0000df04       ??_C@_0CE@CEEDGDDA@fnrm32?5isn?8t?5supported?5on?5this?5c@ 1000ef04     useasm:useasm.obj
 0001:0000df28       ??_C@_0DH@NJHBIBLI@The?5normalise?5instruction?5isn?8t?5@ 1000ef28     useasm:useasm.obj
 0001:0000df60       ??_C@_0BG@BCKONFFM@sop2?5must?5be?5coissued?$AA@ 1000ef60     useasm:useasm.obj
 0001:0000df78       ??_C@_0EP@OFCLCBOD@Invalid?5choice?5for?5the?5fifth?5arg@ 1000ef78     useasm:useasm.obj
 0001:0000dfc8       ??_C@_0DC@FMNAGAJ@No?5flags?5are?5valid?5for?5the?5fifth@ 1000efc8     useasm:useasm.obj
 0001:0000e000       ??_C@_0FK@HNEAMMLH@Invalid?5choice?5for?5the?5fourth?5ar@ 1000f000     useasm:useasm.obj
 0001:0000e05c       ??_C@_0DE@HFBEDGPO@No?5flags?5are?5valid?5for?5the?5fourt@ 1000f05c     useasm:useasm.obj
 0001:0000e090       ??_C@_0EC@PPEKPMIP@The?5fourth?5argument?5to?5asop2?5sho@ 1000f090     useasm:useasm.obj
 0001:0000e0d8       ??_C@_0FO@OLALHECM@Invalid?5choice?5for?5the?5third?5arg@ 1000f0d8     useasm:useasm.obj
 0001:0000e138       ??_C@_0DE@CMCBMCHC@Only?5?4comp?5is?5valid?5for?5the?5thir@ 1000f138     useasm:useasm.obj
 0001:0000e170       ??_C@_0EB@OGKIIKPK@The?5third?5argument?5to?5asop2?5shou@ 1000f170     useasm:useasm.obj
 0001:0000e1b8       ??_C@_0GB@FOOKGLAG@Invalid?5choice?5for?5the?5second?5ar@ 1000f1b8     useasm:useasm.obj
 0001:0000e21c       ??_C@_0DF@BKFNFPMB@Only?5?4comp?5is?5valid?5for?5the?5seco@ 1000f21c     useasm:useasm.obj
 0001:0000e258       ??_C@_0EC@JKPDJLLN@The?5second?5argument?5to?5asop2?5sho@ 1000f258     useasm:useasm.obj
 0001:0000e29c       ??_C@_0DD@KLICCPHA@No?5flags?5are?5valid?5for?5the?5first@ 1000f29c     useasm:useasm.obj
 0001:0000e2d0       ??_C@_0EB@BIMJBGCB@The?5first?5argument?5to?5asop2?5shou@ 1000f2d0     useasm:useasm.obj
 0001:0000e314       ??_C@_0CB@PNFMFKCL@sop2?5must?5be?5coissued?5with?5asop2@ 1000f314     useasm:useasm.obj
 0001:0000e338       ??_C@_0FJ@BADDHEFO@Invalid?5choice?5for?5the?5seventh?5a@ 1000f338     useasm:useasm.obj
 0001:0000e394       ??_C@_0DE@KEDJMMFI@No?5flags?5are?5valid?5for?5the?5seven@ 1000f394     useasm:useasm.obj
 0001:0000e3c8       ??_C@_0EC@HGMCGKBA@The?5seventh?5argument?5to?5sop2?5sho@ 1000f3c8     useasm:useasm.obj
 0001:0000e410       ??_C@_0HE@GKGLGGOL@Invalid?5choice?5for?5the?5sixth?5arg@ 1000f410     useasm:useasm.obj
 0001:0000e484       ??_C@_0DM@OGJGMIAI@Only?5the?5?4comp?5flag?5is?5valid?5for@ 1000f484     useasm:useasm.obj
 0001:0000e4c0       ??_C@_0EA@JBHMMHBL@The?5sixth?5argument?5to?5sop2?5shoul@ 1000f4c0     useasm:useasm.obj
 0001:0000e500       ??_C@_0HG@HJBDHCLG@Invalid?5choice?5for?5the?5fifth?5arg@ 1000f500     useasm:useasm.obj
 0001:0000e578       ??_C@_0DM@OEOABLFP@Only?5the?5?4comp?5flag?5is?5valid?5for@ 1000f578     useasm:useasm.obj
 0001:0000e5b8       ??_C@_0EA@PEDOBCNH@The?5fifth?5argument?5to?5sop2?5shoul@ 1000f5b8     useasm:useasm.obj
 0001:0000e5f8       ??_C@_0FB@HBOJEBLF@Invalid?5choices?5for?5the?5fourth?5a@ 1000f5f8     useasm:useasm.obj
 0001:0000e64c       ??_C@_0DD@GDJINGEN@No?5flags?5are?5valid?5for?5the?5fourt@ 1000f64c     useasm:useasm.obj
 0001:0000e680       ??_C@_0EB@JLEKLKIL@The?5fourth?5argument?5to?5sop2?5shou@ 1000f680     useasm:useasm.obj
 0001:0000e6c4       ??_C@_0DF@CEJLKMBG@Only?5nearest?5rounding?5is?5support@ 1000f6c4     useasm:useasm.obj
 0001:0000e6fc       ??_C@_0CM@OHMDJNLO@An?5integer?5source?5selector?5can?8t@ 1000f6fc     useasm:useasm.obj
 0001:0000e728       ??_C@_0DC@PDLMCMGO@No?5flags?5are?5valid?5for?5an?5intege@ 1000f728     useasm:useasm.obj
 0001:0000e760       ??_C@_0EP@KFBPJKBI@The?5fourth?5argument?5to?5a?5pack?5in@ 1000f760     useasm:useasm.obj
 0001:0000e7b0       ??_C@_0FK@IMCFLHOE@Invalid?5bytemask?5specified?5?$CIlega@ 1000f7b0     useasm:useasm.obj
 0001:0000e80c       ??_C@_0DM@CMGEAEEG@Invalid?5bytemask?5specified?5?$CIlega@ 1000f80c     useasm:useasm.obj
 0001:0000e848       ??_C@_0DD@DLOGHDFD@The?5renable?5flag?5isn?8t?5supported@ 1000f848     useasm:useasm.obj
 0001:0000e880       ??_C@_0EO@CDMEKOCM@The?5renable?5flag?5is?5only?5valid?5w@ 1000f880     useasm:useasm.obj
 0001:0000e8d0       ??_C@_0FI@FHLKJJEN@The?5scale?5flag?5is?5only?5valid?5whe@ 1000f8d0     useasm:useasm.obj
 0001:0000e928       ??_C@_0CD@DJDKIHIP@The?5maximum?5predicate?5number?5is?5@ 1000f928     useasm:useasm.obj
 0001:0000e94c       ??_C@_0CF@LNBFBGED@Predicate?5registers?5can?8t?5be?5ind@ 1000f94c     useasm:useasm.obj
 0001:0000e974       ??_C@_0DF@HMHEIKHA@No?5flags?5are?5valid?5for?5the?5predi@ 1000f974     useasm:useasm.obj
 0001:0000e9ac       ??_C@_0CP@OJDGHEAF@The?5second?5argument?5to?5rlp?5must?5@ 1000f9ac     useasm:useasm.obj
 0001:0000e9e0       ??_C@_0IC@LCJCDNFN@An?5immediate?5source?5argument?5to?5@ 1000f9e0     useasm:useasm.obj
 0001:0000ea64       ??_C@_0DB@JHGOCNIO@imul8?1imulu8?5is?5only?5valid?5with?5@ 1000fa64     useasm:useasm.obj
 0001:0000ea98       ??_C@_0DC@NCLFMCHI@fpadd8?1fpsub8?5is?5only?5valid?5with@ 1000fa98     useasm:useasm.obj
 0001:0000eacc       ??_C@_0DA@KAKEJMDJ@A?5mask?5is?5not?5valid?5on?5a?5dotprod@ 1000facc     useasm:useasm.obj
 0001:0000eafc       ??_C@_0DC@PDHCBKCD@A?5repeat?5is?5not?5valid?5on?5a?5dotpr@ 1000fafc     useasm:useasm.obj
 0001:0000eb30       ??_C@_0EI@JILLLJML@This?5instruction?5isn?8t?5available@ 1000fb30     useasm:useasm.obj
 0001:0000eb78       ??_C@_0CE@PCBCMLOI@The?5maximum?5clip?5plane?5number?5is@ 1000fb78     useasm:useasm.obj
 0001:0000eb9c       ??_C@_0CH@BBGNDHF@A?5clip?5plane?5argument?5is?5not?5ind@ 1000fb9c     useasm:useasm.obj
 0001:0000ebc4       ??_C@_0CM@KGNDPEIK@No?5flags?5are?5valid?5for?5a?5clippla@ 1000fbc4     useasm:useasm.obj
 0001:0000ebf0       ??_C@_0EL@OICFHNIF@The?5second?5argument?5to?5a?5fdpc?5in@ 1000fbf0     useasm:useasm.obj
 0001:0000ec3c       ??_C@_0DI@HLMNAEHK@Only?5i0?5and?5i1?5may?5be?5destinatio@ 1000fc3c     useasm:useasm.obj
 0001:0000ec74       ??_C@_0CF@KCFJPPBJ@Internal?5registers?5are?5not?5index@ 1000fc74     useasm:useasm.obj
 0001:0000ec9c       ??_C@_0DF@KGNOHAA@No?5flags?5are?5valid?5for?5an?5intern@ 1000fc9c     useasm:useasm.obj
 0001:0000ecd8       ??_C@_0FC@GFPCKLPP@The?5second?5argument?5to?5a?5fddp?5in@ 1000fcd8     useasm:useasm.obj
 0001:0000ed30       ??_C@_0EL@NPBIKIOJ@The?5fourth?5argument?5to?5a?5fdpc?5in@ 1000fd30     useasm:useasm.obj
 0001:0000ed80       ??_C@_0EL@DBBJIGNF@The?5third?5argument?5to?5a?5fddpc?5in@ 1000fd80     useasm:useasm.obj
 0001:0000edd0       ??_C@_0FD@HOIBEICL@The?5second?5argument?5to?5a?5fddpc?5i@ 1000fdd0     useasm:useasm.obj
 0001:0000ee24       ??_C@_0DG@EDCHLIHP@Only?5?4tz?0?5?4t?$CBz?0?5?4tn?5or?5?4tp?$HMz?5are@ 1000fe24     useasm:useasm.obj
 0001:0000ee60       ??_C@_0EG@LBAJMGGK@A?5movc?5instruction?5must?5specify?5@ 1000fe60     useasm:useasm.obj
 0001:0000eea8       ??_C@_0GA@OJMMLLIA@On?5this?5processor?5MOVC?5on?5C10?5fo@ 1000fea8     useasm:useasm.obj
 0001:0000ef08       ??_C@_0DP@CLFDAIAM@A?5movc?5instruction?5must?5include?5@ 1000ff08     useasm:useasm.obj
 0001:0000ef48       ??_C@_0FL@OJDHBDDM@The?5instruction?5is?5affected?5by?5B@ 1000ff48     useasm:useasm.obj
 0001:0000efa8       ??_C@_0IC@ONGMFPGB@The?5instruction?5is?5affected?5by?5B@ 1000ffa8     useasm:useasm.obj
 0001:0000f02c       ??_C@_0DP@GHIBIMHL@The?5maximum?5repeat?5count?5for?5an?5@ 1001002c     useasm:useasm.obj
 0001:0000f070       ??_C@_0EC@JJHLNPNF@The?5seventh?5argument?5to?5sop2wm?5i@ 10010070     useasm:useasm.obj
 0001:0000f0b4       ??_C@_0DG@GBFNJGMB@No?5flags?5are?5valid?5for?5the?5seven@ 100100b4     useasm:useasm.obj
 0001:0000f0f0       ??_C@_0EE@EGJILBFH@The?5seventh?5argument?5to?5sop2wm?5s@ 100100f0     useasm:useasm.obj
 0001:0000f138       ??_C@_0EA@HOMFHCNO@The?5sixth?5argument?5to?5sop2wm?5is?5@ 10010138     useasm:useasm.obj
 0001:0000f178       ??_C@_0DE@FDGMDKAF@No?5flags?5are?5valid?5for?5the?5sixth@ 10010178     useasm:useasm.obj
 0001:0000f1b0       ??_C@_0EC@NALFAHH@The?5sixth?5argument?5to?5sop2wm?5sho@ 100101b0     useasm:useasm.obj
 0001:0000f1f4       ??_C@_0DP@BGLACGDG@The?5fifth?5argument?5to?5sop2wm?5is?5@ 100101f4     useasm:useasm.obj
 0001:0000f234       ??_C@_0DM@MLIHGKIL@Only?5?4comp?5is?5a?5valid?5flag?5for?5t@ 10010234     useasm:useasm.obj
 0001:0000f270       ??_C@_0EC@JMPNILCM@The?5fifth?5argument?5to?5sop2wm?5sho@ 10010270     useasm:useasm.obj
 0001:0000f2b8       ??_C@_0EA@NCGPJLOA@The?5fourth?5argument?5to?5sop2wm?5is@ 100102b8     useasm:useasm.obj
 0001:0000f2f8       ??_C@_0DN@NLJCHBJL@Only?5?4comp?5is?5a?5valid?5flag?5for?5t@ 100102f8     useasm:useasm.obj
 0001:0000f338       ??_C@_0ED@FCPONNNK@The?5fourth?5argument?5to?5sop2wm?5sh@ 10010338     useasm:useasm.obj
 0001:0000f380       ??_C@_0EN@MDJOPIF@Invalid?5choice?5for?5the?5third?5arg@ 10010380     useasm:useasm.obj
 0001:0000f3d0       ??_C@_0DC@DCENAPP@No?5flags?5are?5valid?5for?5the?5third@ 100103d0     useasm:useasm.obj
 0001:0000f404       ??_C@_0DO@EELLDBBD@The?5third?5argument?5to?5asop?5must?5@ 10010404     useasm:useasm.obj
 0001:0000f448       ??_C@_0HF@CBIPLOPP@Invalid?5choice?5for?5the?5second?5ar@ 10010448     useasm:useasm.obj
 0001:0000f4c0       ??_C@_0DL@GPHBDAAM@Only?5?4comp?5is?5a?5valid?5flag?5for?5t@ 100104c0     useasm:useasm.obj
 0001:0000f4fc       ??_C@_0DP@KOIBPLMG@The?5second?5argument?5to?5asop?5must@ 100104fc     useasm:useasm.obj
 0001:0000f540       ??_C@_0HE@JFMMNFAC@Invalid?5choice?5for?5the?5first?5arg@ 10010540     useasm:useasm.obj
 0001:0000f5b4       ??_C@_0DK@OKDCCLBL@Only?5?4comp?5is?5a?5valid?5flag?5for?5t@ 100105b4     useasm:useasm.obj
 0001:0000f5f0       ??_C@_0DO@EOKHKJGH@The?5first?5argument?5to?5asop?5must?5@ 100105f0     useasm:useasm.obj
 0001:0000f630       ??_C@_0CA@LJJNKDND@lrp1?5must?5be?5coissued?5with?5asop?$AA@ 10010630     useasm:useasm.obj
 0001:0000f650       ??_C@_0BH@DOCDFOCO@lrp1?5must?5be?5coisssued?$AA@ 10010650     useasm:useasm.obj
 0001:0000f668       ??_C@_0BG@CHKAJNEL@lrp1?5must?5be?5coissued?$AA@ 10010668     useasm:useasm.obj
 0001:0000f680       ??_C@_0EO@FKMJCGBG@Invalid?5choice?5for?5the?5seventh?5a@ 10010680     useasm:useasm.obj
 0001:0000f6d0       ??_C@_0DE@MPNHBAIK@No?5flags?5are?5valid?5for?5the?5seven@ 100106d0     useasm:useasm.obj
 0001:0000f708       ??_C@_0EB@NCENCBNO@The?5seventh?5argument?5to?5lrp1?5mus@ 10010708     useasm:useasm.obj
 0001:0000f750       ??_C@_0EN@NGJPOHKM@Invalid?5choice?5for?5the?5sixth?5arg@ 10010750     useasm:useasm.obj
 0001:0000f7a0       ??_C@_0DM@INHIBENK@Only?5the?5?4comp?5flag?5is?5valid?5for@ 100107a0     useasm:useasm.obj
 0001:0000f7dc       ??_C@_0DP@NEMNCNNA@The?5sixth?5argument?5to?5lrp1?5must?5@ 100107dc     useasm:useasm.obj
 0001:0000f820       ??_C@_0FA@BCOHELNN@Invalid?5choice?5for?5the?5fifth?5arg@ 10010820     useasm:useasm.obj
 0001:0000f870       ??_C@_0CM@KDAMEKKC@An?5integer?5source?5selector?5is?5no@ 10010870     useasm:useasm.obj
 0001:0000f89c       ??_C@_0DM@IPAOMHIN@Only?5the?5?4comp?5flag?5is?5valid?5for@ 1001089c     useasm:useasm.obj
 0001:0000f8d8       ??_C@_0DP@CGMBCHII@The?5fifth?5argument?5to?5lrp1?5must?5@ 100108d8     useasm:useasm.obj
 0001:0000f918       ??_C@_0BG@IEPGBLOC@lrp2?5must?5be?5coissued?$AA@ 10010918     useasm:useasm.obj
 0001:0000f930       ??_C@_0EJ@KJLKFMN@Only?5zero?0?5one?5and?5s2a?5are?5valid@ 10010930     useasm:useasm.obj
 0001:0000f97c       ??_C@_0DE@FDNIJKHO@Only?5?4comp?5is?5valid?5for?5the?5seco@ 1001097c     useasm:useasm.obj
 0001:0000f9b0       ??_C@_0DP@GCMJDOBH@The?5second?5argument?5to?5alrp?5must@ 100109b0     useasm:useasm.obj
 0001:0000f9f0       ??_C@_0EI@POLJNHOP@Only?5zero?0?5one?5and?5s1a?5are?5valid@ 100109f0     useasm:useasm.obj
 0001:0000fa38       ??_C@_0DD@LEOOHHIE@Only?5?4comp?5is?5valid?5for?5the?5firs@ 10010a38     useasm:useasm.obj
 0001:0000fa6c       ??_C@_0DO@ICOPGMLG@The?5first?5argument?5to?5alrp?5must?5@ 10010a6c     useasm:useasm.obj
 0001:0000faac       ??_C@_0CA@BBLPFF@lrp2?5must?5be?5coissued?5with?5alrp?$AA@ 10010aac     useasm:useasm.obj
 0001:0000fad0       ??_C@_0FD@JFBMKMNH@Invalid?5choice?5for?5the?5seventh?5a@ 10010ad0     useasm:useasm.obj
 0001:0000fb28       ??_C@_0EN@GMGJLELO@If?5the?5seventh?5argument?5to?5lrp2?5@ 10010b28     useasm:useasm.obj
 0001:0000fb78       ??_C@_0FB@FJHLFMAN@If?5the?5seventh?5argument?5to?5lrp2?5@ 10010b78     useasm:useasm.obj
 0001:0000fbd0       ??_C@_0EP@GBKEKGGN@If?5the?5seventh?5argument?5to?5lrp2?5@ 10010bd0     useasm:useasm.obj
 0001:0000fc20       ??_C@_0EK@MPPLIHCI@If?5the?5seventh?5argument?5to?5lrp2?5@ 10010c20     useasm:useasm.obj
 0001:0000fc6c       ??_C@_0DN@BJBDMCPE@Only?5the?5?4comp?5flag?5is?5valid?5for@ 10010c6c     useasm:useasm.obj
 0001:0000fcb0       ??_C@_0EA@MACNPBPH@The?5eighth?5argument?5to?5lrp2?5must@ 10010cb0     useasm:useasm.obj
 0001:0000fcf0       ??_C@_0DO@GLBNDEGP@Only?5the?5?4comp?5flag?5is?5valid?5for@ 10010cf0     useasm:useasm.obj
 0001:0000fd30       ??_C@_0EB@JPKFCBLJ@The?5seventh?5argument?5to?5lrp2?5mus@ 10010d30     useasm:useasm.obj
 0001:0000fd78       ??_C@_0HH@IBAGBKNH@Invalid?5choice?5for?5the?5sixth?5arg@ 10010d78     useasm:useasm.obj
 0001:0000fdf0       ??_C@_0DM@KGFFEHBJ@Only?5the?5?4comp?5flag?5is?5valid?5for@ 10010df0     useasm:useasm.obj
 0001:0000fe2c       ??_C@_0DP@JJCFCNLH@The?5sixth?5argument?5to?5lrp2?5must?5@ 10010e2c     useasm:useasm.obj
 0001:0000fe70       ??_C@_0HI@KGJMFIGE@Invalid?5choice?5for?5the?5fifth?5arg@ 10010e70     useasm:useasm.obj
 0001:0000fee8       ??_C@_0DM@PNPLCKBO@Only?5the?5?4comp?5flag?5is?5valid?5for@ 10010ee8     useasm:useasm.obj
 0001:0000ff24       ??_C@_0DP@JFIMNECE@The?5fifth?5argument?5to?5sop3?5must?5@ 10010f24     useasm:useasm.obj
 0001:0000ff68       ??_C@_0EP@LFLPCFJM@Invalid?5choice?5for?5the?5second?5ar@ 10010f68     useasm:useasm.obj
 0001:0000ffb8       ??_C@_0DE@GEPIHLDC@No?5flags?5are?5valid?5for?5the?5secon@ 10010fb8     useasm:useasm.obj
 0001:0000fff0       ??_C@_0EA@CILJPHKB@The?5second?5argument?5to?5arsop?5mus@ 10010ff0     useasm:useasm.obj
 0001:00010030       ??_C@_0FO@BGCOGJJP@Invalid?5choice?5for?5the?5first?5arg@ 10011030     useasm:useasm.obj
 0001:00010090       ??_C@_0DE@LFEIHKHD@Only?5?4comp?5is?5valid?5for?5the?5firs@ 10011090     useasm:useasm.obj
 0001:000100c4       ??_C@_0DP@IJIIECIN@The?5first?5argument?5to?5arsop?5must@ 100110c4     useasm:useasm.obj
 0001:00010108       ??_C@_0EK@DIJKPKNM@SOP3?5with?5ARSOP?5and?5a?5complement@ 10011108     useasm:useasm.obj
 0001:00010158       ??_C@_0EO@BNBKMGBP@Invalid?5choice?5for?5the?5second?5ar@ 10011158     useasm:useasm.obj
 0001:000101a8       ??_C@_0DD@KDAMLAMK@No?5flags?5are?5valid?5for?5the?5secon@ 100111a8     useasm:useasm.obj
 0001:000101e0       ??_C@_0FN@ONPCNNEO@Invalid?5choice?5for?5the?5first?5arg@ 100111e0     useasm:useasm.obj
 0001:00010240       ??_C@_0DD@KIGKAAGO@Only?5?4comp?5is?5valid?5for?5the?5firs@ 10011240     useasm:useasm.obj
 0001:00010278       ??_C@_0FE@LNCOBNA@Invalid?5choice?5for?5the?5first?5arg@ 10011278     useasm:useasm.obj
 0001:000102d0       ??_C@_0FE@JJEFPIJ@Invalid?5choice?5for?5the?5first?5arg@ 100112d0     useasm:useasm.obj
 0001:00010328       ??_C@_0ED@PGOFNOAD@sop3?5with?5a?5negate?5destination?5m@ 10011328     useasm:useasm.obj
 0001:0001036c       ??_C@_0CE@OHCGBBLC@sop3?5without?5a?5coissued?5instruct@ 1001136c     useasm:useasm.obj
 0001:00010390       ??_C@_0BG@MFEMFFAE@sop3?5must?5be?5coissued?$AA@ 10011390     useasm:useasm.obj
 0001:000103a8       ??_C@_0EL@GLFHPIPJ@Invalid?5choice?5for?5eighth?5argume@ 100113a8     useasm:useasm.obj
 0001:000103f8       ??_C@_0EA@DOIIACDM@The?5eighth?5argument?5to?5sop3?5must@ 100113f8     useasm:useasm.obj
 0001:00010438       ??_C@_0EP@LLOJFENH@Invalid?5choice?5for?5the?5seventh?5a@ 10011438     useasm:useasm.obj
 0001:00010488       ??_C@_0DE@LNCCPNBJ@No?5flags?5are?5valid?5for?5the?5seven@ 10011488     useasm:useasm.obj
 0001:000104c0       ??_C@_0EB@GBAANCHC@The?5seventh?5argument?5to?5sop3?5mus@ 100114c0     useasm:useasm.obj
 0001:00010508       ??_C@_0HE@NOFOGDCI@Invalid?5choice?5for?5the?5sixth?5arg@ 10011508     useasm:useasm.obj
 0001:0001057c       ??_C@_0DK@GPFHLHKL@Only?5?4comp?5is?5a?5valid?5flag?5for?5t@ 1001157c     useasm:useasm.obj
 0001:000105b8       ??_C@_0DP@GHIANOHM@The?5sixth?5argument?5to?5sop3?5must?5@ 100115b8     useasm:useasm.obj
 0001:000105f8       ??_C@_0HE@OENIBECC@Invalid?5choice?5for?5the?5fifth?5arg@ 100115f8     useasm:useasm.obj
 0001:0001066c       ??_C@_0DK@GNCBGEPM@Only?5?4comp?5is?5a?5valid?5flag?5for?5t@ 1001166c     useasm:useasm.obj
 0001:000106a8       ??_C@_0BH@NMPINIEC@sop3?5can?8t?5be?5repeated?$AA@ 100116a8     useasm:useasm.obj
 0001:000106c0       ??_C@_0DK@OMANMEPM@Only?5s2a?5is?5a?5valid?5choice?5for?5t@ 100116c0     useasm:useasm.obj
 0001:000106fc       ??_C@_0DK@DPJMNKAL@Only?5?4comp?5is?5a?5valid?5flag?5for?5t@ 100116fc     useasm:useasm.obj
 0001:00010738       ??_C@_0DP@BFGILNHD@The?5tenth?5argument?5to?5ima8?5must?5@ 10011738     useasm:useasm.obj
 0001:00010778       ??_C@_0DL@FMNMANPN@Only?5s1a?5is?5a?5valid?5choice?5for?5t@ 10011778     useasm:useasm.obj
 0001:000107b4       ??_C@_0DL@PMLPCLJP@Only?5?4comp?5is?5a?5valid?5flag?5for?5t@ 100117b4     useasm:useasm.obj
 0001:000107f0       ??_C@_0EA@OKAGHCFL@The?5nineth?5argument?5to?5ima8?5must@ 100117f0     useasm:useasm.obj
 0001:00010830       ??_C@_0ED@FKCOCDED@Only?5s0a?5and?5s1a?5are?5valid?5choic@ 10011830     useasm:useasm.obj
 0001:00010874       ??_C@_0DL@HABGHCJK@Only?5?4comp?5is?5a?5valid?5flag?5for?5t@ 10011874     useasm:useasm.obj
 0001:000108b0       ??_C@_0EA@EABBPNKK@The?5eighth?5argument?5to?5ima8?5must@ 100118b0     useasm:useasm.obj
 0001:000108f0       ??_C@_0ED@FDKGPKDC@Only?5s2?5and?5s2a?5are?5valid?5choice@ 100118f0     useasm:useasm.obj
 0001:00010934       ??_C@_0DM@LBKALADI@Only?5?4comp?5is?5a?5valid?5flag?5for?5t@ 10011934     useasm:useasm.obj
 0001:00010970       ??_C@_0EB@BPJJCNOE@The?5seventh?5argument?5to?5ima8?5mus@ 10011970     useasm:useasm.obj
 0001:000109b8       ??_C@_0EB@CLJBDDPJ@Only?5s1?5and?5s1a?5are?5valid?5choice@ 100119b8     useasm:useasm.obj
 0001:000109fc       ??_C@_0DK@BBBOOAIP@Only?5?4comp?5is?5a?5valid?5flag?5for?5t@ 100119fc     useasm:useasm.obj
 0001:00010a38       ??_C@_0DP@BJBJCBOK@The?5sixth?5argument?5to?5ima8?5must?5@ 10011a38     useasm:useasm.obj
 0001:00010a78       ??_C@_0EK@KADHKBHD@Only?5s0?0?5s1?0?5s0a?5and?5s1a?5are?5val@ 10011a78     useasm:useasm.obj
 0001:00010ac4       ??_C@_0DK@BDGIDDNI@Only?5?4comp?5is?5a?5valid?5flag?5for?5t@ 10011ac4     useasm:useasm.obj
 0001:00010b00       ??_C@_0DP@OLBFCLLC@The?5fifth?5argument?5to?5ima8?5must?5@ 10011b00     useasm:useasm.obj
 0001:00010b40       ??_C@_0EK@HCFFGHCH@Third?5argument?5to?5ima16?5is?58?9bit@ 10011b40     useasm:useasm.obj
 0001:00010b90       ??_C@_0EL@EFNHNPFP@Second?5argument?5to?5ima16?5is?58?9bi@ 10011b90     useasm:useasm.obj
 0001:00010bdc       ??_C@_0DD@DHKGKKGN@No?5flags?5are?5valid?5for?5the?5sixth@ 10011bdc     useasm:useasm.obj
 0001:00010c10       ??_C@_0CM@KFKJJGEN@The?5sixth?5argument?5to?5ima16?5isn?8@ 10011c10     useasm:useasm.obj
 0001:00010c3c       ??_C@_0DC@FLFMKFFD@The?5sixth?5argument?5to?5ima16?5must@ 10011c3c     useasm:useasm.obj
 0001:00010c70       ??_C@_0EN@LDKLHMAN@Invalid?5source?5data?5format?5for?5i@ 10011c70     useasm:useasm.obj
 0001:00010cc0       ??_C@_0DD@MCKLBIOJ@No?5flags?5are?5valid?5for?5the?5fifth@ 10011cc0     useasm:useasm.obj
 0001:00010cf4       ??_C@_0CM@LHIIENBO@The?5fifth?5argument?5to?5ima16?5isn?8@ 10011cf4     useasm:useasm.obj
 0001:00010d20       ??_C@_0DC@CIEPCOAH@The?5fifth?5argument?5to?5ima16?5must@ 10011d20     useasm:useasm.obj
 0001:00010d54       ??_C@_0DJ@KMFCNFLN@Only?5one?5of?5?4s?5and?5?4u?5can?5be?5spe@ 10011d54     useasm:useasm.obj
 0001:00010d90       ??_C@_0DN@LMMEBOND@The?5maximum?5destination?5shift?5fo@ 10011d90     useasm:useasm.obj
 0001:00010dd0       ??_C@_0EA@BEAJFKLN@The?5maximum?5register?5number?5for?5@ 10011dd0     useasm:useasm.obj
 0001:00010e10       ??_C@_0CL@DOOAPBOB@The?5eighth?5source?5to?5imae?5can?8t?5@ 10011e10     useasm:useasm.obj
 0001:00010e3c       ??_C@_0DB@PKHIFEJJ@No?5flags?5are?5valid?5for?5the?5eight@ 10011e3c     useasm:useasm.obj
 0001:00010e70       ??_C@_0EI@OMIBHEJN@The?5eighth?5source?5to?5imae?5should@ 10011e70     useasm:useasm.obj
 0001:00010eb8       ??_C@_0EH@DLKGLNI@Only?5cie?5or?5nothing?5are?5valid?5ch@ 10011eb8     useasm:useasm.obj
 0001:00010f00       ??_C@_0DE@MMHOIJCE@No?5flags?5are?5valid?5for?5the?5seven@ 10011f00     useasm:useasm.obj
 0001:00010f34       ??_C@_0CN@IKCGDAFI@The?5seventh?5argument?5to?5imae?5isn@ 10011f34     useasm:useasm.obj
 0001:00010f64       ??_C@_0DE@IAOPODPF@The?5seventh?5argument?5to?5imae?5mus@ 10011f64     useasm:useasm.obj
 0001:00010f98       ??_C@_0EF@JBDPGDKG@Only?5coe?5or?5nothing?5are?5valid?5ch@ 10011f98     useasm:useasm.obj
 0001:00010fe0       ??_C@_0DC@GPPMJACC@No?5flags?5are?5valid?5for?5the?5sixth@ 10011fe0     useasm:useasm.obj
 0001:00011014       ??_C@_0CL@CDIKAGGM@The?5sixth?5argument?5to?5imae?5isn?8t@ 10012014     useasm:useasm.obj
 0001:00011040       ??_C@_0DC@HDJGOJKK@The?5sixth?5argument?5to?5imae?5must?5@ 10012040     useasm:useasm.obj
 0001:00011074       ??_C@_0DD@DNBAOKIA@?4low?5and?5?4high?5are?5meaningless?5f@ 10012074     useasm:useasm.obj
 0001:000110a8       ??_C@_0EG@PNOIEBGC@One?5of?5?4low?5or?5?4high?5should?5be?5s@ 100120a8     useasm:useasm.obj
 0001:000110f0       ??_C@_0EH@DLDLJEEK@One?5of?5?4low?5or?5?4high?5should?5be?5s@ 100120f0     useasm:useasm.obj
 0001:00011138       ??_C@_0EG@HGBJOGAP@One?5of?5?4low?5or?5?4high?5should?5be?5s@ 10012138     useasm:useasm.obj
 0001:00011180       ??_C@_0BN@MCMCHHHO@Invalid?5data?5format?5for?5imae?$AA@ 10012180     useasm:useasm.obj
 0001:000111a0       ??_C@_0DC@GNIKEDHF@No?5flags?5are?5valid?5for?5the?5fifth@ 100121a0     useasm:useasm.obj
 0001:000111d4       ??_C@_0CL@LFLIAFDF@The?5fifth?5argument?5to?5imae?5isn?8t@ 100121d4     useasm:useasm.obj
 0001:00011200       ??_C@_0DB@NOAIOELF@The?5fifth?5argument?5to?5imae?5must?5@ 10012200     useasm:useasm.obj
 0001:00011234       ??_C@_0DM@EHOELKCO@The?5maximum?5destination?5shift?5fo@ 10012234     useasm:useasm.obj
 0001:00011270       ??_C@_0DE@JCLFGKBG@Maximum?5repeat?5count?5on?5an?5integ@ 10012270     useasm:useasm.obj
 0001:000112a8       ??_C@_0EG@JFIEFIAN@Only?5u8?5or?5s8?5are?5valid?5as?5a?5cho@ 100122a8     useasm:useasm.obj
 0001:000112f0       ??_C@_0DF@BFAJNMNE@No?5flags?5are?5valid?5for?5the?5ninet@ 100122f0     useasm:useasm.obj
 0001:00011328       ??_C@_0EB@EPNJCIMP@The?5nineth?5argument?5to?5ssum16?5mu@ 10012328     useasm:useasm.obj
 0001:00011370       ??_C@_0EM@CDDPPEDE@Only?5iadd?5or?5nothing?5is?5valid?5as@ 10012370     useasm:useasm.obj
 0001:000113bc       ??_C@_0DF@HKMJENGI@No?5flags?5are?5valid?5for?5the?5eight@ 100123bc     useasm:useasm.obj
 0001:000113f8       ??_C@_0EB@IFMJPNMK@The?5eighth?5argument?5to?5ssum16?5mu@ 100123f8     useasm:useasm.obj
 0001:00011440       ??_C@_0ED@OAGGGGIH@Only?5i0?5or?5r1?5valid?5as?5a?5choice?5@ 10012440     useasm:useasm.obj
 0001:00011484       ??_C@_0CF@BGFEHLBP@An?5internal?5register?5isn?8t?5index@ 10012484     useasm:useasm.obj
 0001:000114ac       ??_C@_0DG@GDJPLBEI@No?5flags?5are?5valid?5for?5the?5seven@ 100124ac     useasm:useasm.obj
 0001:000114e8       ??_C@_0EC@BEPCBJIN@The?5seventh?5argument?5to?5ssum16?5m@ 100124e8     useasm:useasm.obj
 0001:00011530       ??_C@_0EL@BECKFGPA@Only?5iadd?5or?5nothing?5is?5valid?5as@ 10012530     useasm:useasm.obj
 0001:0001157c       ??_C@_0DE@FBKOBNIM@No?5flags?5are?5valid?5for?5the?5sixth@ 1001257c     useasm:useasm.obj
 0001:000115b0       ??_C@_0EA@PDEMLEIG@The?5sixth?5argument?5to?5ssum16?5mus@ 100125b0     useasm:useasm.obj
 0001:000115f0       ??_C@_0EL@HFHGKGHC@Only?5idst?5or?5nothing?5is?5valid?5as@ 100125f0     useasm:useasm.obj
 0001:0001163c       ??_C@_0CL@KCGNBGBH@An?5integer?5source?5selector?5isn?8t@ 1001263c     useasm:useasm.obj
 0001:00011668       ??_C@_0DE@LLIOFHAH@No?5flags?5are?5valid?5for?5the?5fifth@ 10012668     useasm:useasm.obj
 0001:000116a0       ??_C@_0EA@JGAOGBEK@The?5fifth?5argument?5to?5ssum16?5mus@ 100126a0     useasm:useasm.obj
 0001:000116e0       ??_C@_0DE@IJOOAFAA@Maximum?5repeat?5count?5on?5an?5SSUM1@ 100126e0     useasm:useasm.obj
 0001:00011714       ??_C@_0CJ@EGABLJED@ssum16?5isn?8t?5available?5on?5this?5p@ 10012714     useasm:useasm.obj
 0001:00011740       ??_C@_0EL@LEHINHKP@Only?5scale?5or?5nothing?5is?5valid?5a@ 10012740     useasm:useasm.obj
 0001:0001178c       ??_C@_0DD@MBMDINHI@No?5flags?5are?5valid?5for?5the?5eight@ 1001278c     useasm:useasm.obj
 0001:000117c0       ??_C@_0DP@DNLIJOFH@The?5eighth?5argument?5to?5firv?5must@ 100127c0     useasm:useasm.obj
 0001:00011800       ??_C@_0EL@PLEHJOGF@Only?5iadd?5or?5nothing?5is?5valid?5as@ 10012800     useasm:useasm.obj
 0001:0001184c       ??_C@_0DE@LOMDNFBJ@No?5flags?5are?5valid?5for?5the?5seven@ 1001284c     useasm:useasm.obj
 0001:00011880       ??_C@_0EA@LAOANIGO@The?5seventh?5argument?5to?5firv?5mus@ 10012880     useasm:useasm.obj
 0001:000118c0       ??_C@_0EM@PPMBHMLB@Only?5?$CLsrc2?42?5or?5nothing?5is?5valid@ 100128c0     useasm:useasm.obj
 0001:0001190c       ??_C@_0DC@BNEBMMBP@No?5flags?5are?5valid?5for?5the?5sixth@ 1001290c     useasm:useasm.obj
 0001:00011940       ??_C@_0DO@IGFJMJCL@The?5sixth?5argument?5to?5firv?5must?5@ 10012940     useasm:useasm.obj
 0001:00011980       ??_C@_0CL@MDHBFNJL@The?5fifth?5argument?5to?5firv?5isn?8t@ 10012980     useasm:useasm.obj
 0001:000119ac       ??_C@_0DC@BPDHBPEI@No?5flags?5are?5valid?5for?5the?5fifth@ 100129ac     useasm:useasm.obj
 0001:000119e0       ??_C@_0DP@LCJNOCNN@The?5fifth?5argument?5to?5firv?5must?5@ 100129e0     useasm:useasm.obj
 0001:00011a20       ??_C@_0HP@FKECLPEM@The?5register?5bank?5for?5firv?5sourc@ 10012a20     useasm:useasm.obj
 0001:00011aa0       ??_C@_0EG@NEGMNEOD@The?5register?5banks?5for?5source?50?5@ 10012aa0     useasm:useasm.obj
 0001:00011ae8       ??_C@_0CD@BDBMNPHP@Maximum?5repeat?5count?5on?5firv?5is?5@ 10012ae8     useasm:useasm.obj
 0001:00011b10       ??_C@_0EK@MMLIIHNN@Only?5scale?5or?5nothing?5is?5valid?5a@ 10012b10     useasm:useasm.obj
 0001:00011b60       ??_C@_0EJ@NGJACPPH@Only?5iadd?5or?5nothing?5is?5valid?5as@ 10012b60     useasm:useasm.obj
 0001:00011bac       ??_C@_0DO@OIFDNPHI@The?5fifth?5argument?5to?5firv?5must?5@ 10012bac     useasm:useasm.obj
 0001:00011bf0       ??_C@_0EN@EIOOMBFD@Only?5?$CLsrc2?42?5or?5nothing?5is?5valid@ 10012bf0     useasm:useasm.obj
 0001:00011c40       ??_C@_0DP@FGKELBIB@The?5fourth?5argument?5to?5firv?5must@ 10012c40     useasm:useasm.obj
 0001:00011c80       ??_C@_0EE@EGNLBLOB@The?5register?5bank?5for?5firvh?5sour@ 10012c80     useasm:useasm.obj
 0001:00011cc4       ??_C@_0CE@HBKLLEAA@Maximum?5repeat?5count?5on?5firvh?5is@ 10012cc4     useasm:useasm.obj
 0001:00011ce8       ??_C@_0CI@CFGKFHCM@firvh?5isn?8t?5available?5on?5this?5pr@ 10012ce8     useasm:useasm.obj
 0001:00011d10       ??_C@_0EA@CNFLJPLE@The?5nineth?5argument?5to?5bilin?5mus@ 10012d10     useasm:useasm.obj
 0001:00011d50       ??_C@_0DE@OJKKKHIL@No?5flags?5are?5valid?5for?5the?5ninet@ 10012d50     useasm:useasm.obj
 0001:00011d84       ??_C@_0CN@DJDNLEIC@The?5nineth?5argument?5to?5bilin?5isn@ 10012d84     useasm:useasm.obj
 0001:00011db4       ??_C@_0DH@HFBBMNAM@The?5nineth?5argument?5to?5bilin?5mus@ 10012db4     useasm:useasm.obj
 0001:00011df0       ??_C@_0EA@OPFHNAEG@The?5eighth?5argument?5to?5bilin?5mus@ 10012df0     useasm:useasm.obj
 0001:00011e30       ??_C@_0DE@JJEMPKFN@No?5flags?5are?5valid?5for?5the?5eight@ 10012e30     useasm:useasm.obj
 0001:00011e64       ??_C@_0CN@MBAHDJDB@The?5eighth?5argument?5to?5bilin?5isn@ 10012e64     useasm:useasm.obj
 0001:00011e98       ??_C@_0EJ@BIMEJMPB@The?5eighth?5argument?5to?5bilin?5mus@ 10012e98     useasm:useasm.obj
 0001:00011ee8       ??_C@_0EB@LANPAAAI@The?5seventh?5argument?5to?5bilin?5mu@ 10012ee8     useasm:useasm.obj
 0001:00011f2c       ??_C@_0DF@KDIGKLML@No?5flags?5are?5valid?5for?5the?5seven@ 10012f2c     useasm:useasm.obj
 0001:00011f64       ??_C@_0CO@HELDAPEL@The?5seventh?5argument?5to?5bilin?5is@ 10012f64     useasm:useasm.obj
 0001:00011f98       ??_C@_0EF@CJMNJFOI@The?5seventh?5argument?5to?5bilin?5mu@ 10012f98     useasm:useasm.obj
 0001:00011fe0       ??_C@_0EG@CPMAHDPO@The?5sixth?5argument?5to?5bilin?5must@ 10012fe0     useasm:useasm.obj
 0001:00012028       ??_C@_0DD@EKEGIMOH@No?5flags?5are?5valid?5for?5the?5sixth@ 10013028     useasm:useasm.obj
 0001:0001205c       ??_C@_0CM@FFKOFHMI@The?5sixth?5argument?5to?5bilin?5isn?8@ 1001305c     useasm:useasm.obj
 0001:00012088       ??_C@_0EA@HDMMDEFM@The?5sixth?5argument?5to?5bilin?5must@ 10013088     useasm:useasm.obj
 0001:000120c8       ??_C@_0EA@BGIOOBJA@The?5fifth?5argument?5to?5bilin?5must@ 100130c8     useasm:useasm.obj
 0001:00012108       ??_C@_0DD@LPELDOGD@No?5flags?5are?5valid?5for?5the?5fifth@ 10013108     useasm:useasm.obj
 0001:0001213c       ??_C@_0CM@EHIPIMJL@The?5fifth?5argument?5to?5bilin?5isn?8@ 1001313c     useasm:useasm.obj
 0001:00012168       ??_C@_0EB@ILBDCOKI@The?5fifth?5argument?5to?5bilin?5must@ 10013168     useasm:useasm.obj
 0001:000121ac       ??_C@_0CE@PONMLKAD@Maximum?5repeat?5count?5on?5bilin?5is@ 100131ac     useasm:useasm.obj
 0001:000121d0       ??_C@_0DE@JHKIEKPM@The?5range?5of?5the?5nineth?5argument@ 100131d0     useasm:useasm.obj
 0001:00012204       ??_C@_0DH@KHNFKIAG@The?5nineth?5argument?5to?5firh?5must@ 10013204     useasm:useasm.obj
 0001:0001223c       ??_C@_0DF@JCFPNCKH@The?5range?5of?5the?5eighth?5argument@ 1001323c     useasm:useasm.obj
 0001:00012274       ??_C@_0DH@BGJCEECP@The?5eighth?5argument?5to?5firh?5must@ 10013274     useasm:useasm.obj
 0001:000122ac       ??_C@_0CI@HEOOLMFP@The?5maximum?5filter?5coefficent?5se@ 100132ac     useasm:useasm.obj
 0001:000122d4       ??_C@_0DC@CJJPPKOA@No?5flags?5are?5valid?5for?5a?5filter?5@ 100132d4     useasm:useasm.obj
 0001:00012308       ??_C@_0CI@BPHBGDKA@Filter?5coefficent?5sets?5aren?8t?5in@ 10013308     useasm:useasm.obj
 0001:00012330       ??_C@_0DN@NIIJMAFI@The?5seventh?5argument?5to?5firh?5mus@ 10013330     useasm:useasm.obj
 0001:00012370       ??_C@_0CK@MCCCMAME@No?5flags?5are?5valid?5for?5an?5immedi@ 10013370     useasm:useasm.obj
 0001:0001239c       ??_C@_0CE@BOJPMEGF@An?5immediate?5value?5is?5not?5indexa@ 1001339c     useasm:useasm.obj
 0001:000123c0       ??_C@_0DK@HBKJDJHH@The?5sixth?5argument?5to?5firh?5must?5@ 100133c0     useasm:useasm.obj
 0001:000123fc       ??_C@_0DC@MLHGCAJH@No?5flags?5are?5valid?5for?5the?5fifth@ 100133fc     useasm:useasm.obj
 0001:00012430       ??_C@_0CL@PEPPBDAK@The?5fifth?5argument?5to?5firh?5isn?8t@ 10013430     useasm:useasm.obj
 0001:0001245c       ??_C@_0DN@JOJEKONN@The?5fifth?5argument?5to?5firh?5must?5@ 1001345c     useasm:useasm.obj
 0001:000124a0       ??_C@_0HP@FIJDICNA@The?5register?5bank?5for?5firh?5sourc@ 100134a0     useasm:useasm.obj
 0001:00012520       ??_C@_0EG@FDFDPJHP@The?5register?5banks?5for?5source?50?5@ 10013520     useasm:useasm.obj
 0001:00012568       ??_C@_0CD@HKCNPMGG@Maximum?5repeat?5count?5on?5firh?5is?5@ 10013568     useasm:useasm.obj
 0001:0001258c       ??_C@_0DP@DKFIGMEP@The?5destination?5argument?5to?5firh@ 1001358c     useasm:useasm.obj
 0001:000125cc       ??_C@_0DF@BDOGECIG@The?5range?5of?5the?5nineth?5argument@ 100135cc     useasm:useasm.obj
 0001:00012604       ??_C@_0DI@PJONGPDL@The?5nineth?5argument?5to?5firhh?5mus@ 10013604     useasm:useasm.obj
 0001:0001263c       ??_C@_0DG@KGIDPMLA@The?5range?5of?5the?5eighth?5argument@ 1001363c     useasm:useasm.obj
 0001:00012674       ??_C@_0DI@LLOOLALL@The?5eighth?5argument?5to?5firhh?5mus@ 10013674     useasm:useasm.obj
 0001:000126ac       ??_C@_0DO@EEFEJEHK@The?5seventh?5argument?5to?5firhh?5mu@ 100136ac     useasm:useasm.obj
 0001:000126ec       ??_C@_0DL@OHNCDOMJ@The?5sixth?5argument?5to?5firhh?5must@ 100136ec     useasm:useasm.obj
 0001:00012728       ??_C@_0DD@MDIEJBGI@No?5flags?5are?5valid?5for?5the?5fifth@ 10013728     useasm:useasm.obj
 0001:0001275c       ??_C@_0CM@DLIOMDAE@The?5fifth?5argument?5to?5firhh?5isn?8@ 1001375c     useasm:useasm.obj
 0001:00012788       ??_C@_0DO@NGNIOBOG@The?5fifth?5argument?5to?5firhh?5must@ 10013788     useasm:useasm.obj
 0001:000127c8       ??_C@_0IA@FCFJDLLG@The?5register?5bank?5for?5firhh?5sour@ 100137c8     useasm:useasm.obj
 0001:00012848       ??_C@_0EH@HPAOOKCK@The?5register?5banks?5for?5source?50?5@ 10013848     useasm:useasm.obj
 0001:00012890       ??_C@_0CE@BFKJCNOD@Maximum?5repeat?5count?5on?5firhh?5is@ 10013890     useasm:useasm.obj
 0001:000128b4       ??_C@_0CI@CPDCNICP@firhh?5isn?8t?5available?5on?5this?5pr@ 100138b4     useasm:useasm.obj
 0001:000128dc       ??_C@_0DC@OJMFLOPA@A?5repeat?5count?5isn?8t?5supported?5o@ 100138dc     useasm:useasm.obj
 0001:00012910       ??_C@_0DJ@PFEOBFIJ@Valid?5values?5for?5argument?5?$CFd?5to?5@ 10013910     useasm:useasm.obj
 0001:0001294c       ??_C@_0DK@PJMBECMK@On?5this?5core?5SMP?5result?5format?5c@ 1001394c     useasm:useasm.obj
 0001:00012988       ??_C@_0FI@CPMJEANO@The?5fourth?5argument?5to?5a?5sampler@ 10013988     useasm:useasm.obj
 0001:000129e0       ??_C@_0FD@LADDBKEH@The?5destination?5for?5a?5SMP?5must?5b@ 100139e0     useasm:useasm.obj
 0001:00012a34       ??_C@_0CM@KHPAMMAK@The?5destination?5for?5an?5SMP?5can?8t@ 10013a34     useasm:useasm.obj
 0001:00012a60       ??_C@_0DC@EEBJMIBO@A?5?$CFs?5instruction?5can?8t?5be?5predic@ 10013a60     useasm:useasm.obj
 0001:00012a94       ??_C@_0DC@DNHACGFH@?4fcfill?5and?5?4bypassl1?5can?8t?5be?5s@ 10013a94     useasm:useasm.obj
 0001:00012ac8       ??_C@_0DD@BEGMGHDH@?4bpcache?5and?5?4bypassl1?5can?8t?5be?5@ 10013ac8     useasm:useasm.obj
 0001:00012afc       ??_C@_0DB@JCFACDNN@?4bpcache?5and?5?4fcfill?5can?8t?5be?5sp@ 10013afc     useasm:useasm.obj
 0001:00012b30       ??_C@_0FD@KGBKPKPH@The?5last?5argument?5to?5a?5load?5inst@ 10013b30     useasm:useasm.obj
 0001:00012b84       ??_C@_0CL@NHIEGIGG@The?5destination?5for?5an?5LD?5can?8t?5@ 10013b84     useasm:useasm.obj
 0001:00012bb0       ??_C@_0FD@DHDGKGAN@The?5destination?5for?5an?5LD?5must?5b@ 10013bb0     useasm:useasm.obj
 0001:00012c04       ??_C@_0DD@ECJPHDDF@A?5load?1store?5can?8t?5be?5both?5pre?9?5@ 10013c04     useasm:useasm.obj
 0001:00012c38       ??_C@_0FC@LJJNHLCE@?$CFs?5can?8t?5be?5used?5with?5non?9pre?1po@ 10013c38     useasm:useasm.obj
 0001:00012c90       ??_C@_0EN@GCEEDLLB@Pre?1post?9increment?5can?8t?5be?5spec@ 10013c90     useasm:useasm.obj
 0001:00012ce0       ??_C@_0ED@IMFMHAAP@Source?51?5can?8t?5be?5immediate?5for?5@ 10013ce0     useasm:useasm.obj
 0001:00012d24       ??_C@_0CA@BFMOGGHL@?$CFs?5isn?8t?5supported?5on?5this?5core?$AA@ 10013d24     useasm:useasm.obj
 0001:00012d44       ??_C@_0CJ@NLADGPEP@The?5argument?5to?5a?5branch?5must?5be@ 10013d44     useasm:useasm.obj
 0001:00012d70       ??_C@_0DD@COOIGJEM@Pn?5isn?8t?5a?5valid?5predicate?5for?5b@ 10013d70     useasm:useasm.obj
 0001:00012da4       ??_C@_0DI@LKENEFMD@Only?5drc0?5can?5be?5used?5with?5PBE?5d@ 10013da4     useasm:useasm.obj
 0001:00012ddc       ??_C@_0BL@DDAKDDCD@Invalid?5data?5path?5selector?$AA@ 10013ddc     useasm:useasm.obj
 0001:00012df8       ??_C@_0CM@EIBHGDCN@No?5flags?5are?5valid?5for?5a?5data?5pa@ 10013df8     useasm:useasm.obj
 0001:00012e24       ??_C@_0CG@LCIGPPNF@A?5data?5path?5selector?5is?5not?5inde@ 10013e24     useasm:useasm.obj
 0001:00012e4c       ??_C@_0DI@IKADLPJL@The?5second?5argument?5to?5idf?5must?5@ 10013e4c     useasm:useasm.obj
 0001:00012e84       ??_C@_0CG@BCCKICBA@The?5maximum?5drc?5register?5number?5@ 10013e84     useasm:useasm.obj
 0001:00012eac       ??_C@_0CG@NKPGJMIA@No?5flags?5are?5valid?5for?5a?5drc?5reg@ 10013eac     useasm:useasm.obj
 0001:00012ed4       ??_C@_0CA@BNCKADBN@A?5drc?5register?5is?5not?5indexable?$AA@ 10013ed4     useasm:useasm.obj
 0001:00012ef4       ??_C@_0DB@EIJIPLBA@The?5first?5argument?5to?5idf?5must?5b@ 10013ef4     useasm:useasm.obj
 0001:00012f28       ??_C@_0CL@HOIKEHND@The?5argument?5to?5wdf?5must?5be?5a?5dr@ 10013f28     useasm:useasm.obj
 0001:00012f54       ??_C@_0DI@ECFOFJCH@The?5last?5argument?5to?5an?5emit?5mus@ 10013f54     useasm:useasm.obj
 0001:00012f90       ??_C@_0EE@FPKMHEIB@The?5maximum?5immediate?5value?5for?5@ 10013f90     useasm:useasm.obj
 0001:00012fd4       ??_C@_0DJ@EENABCEN@The?5first?5argument?5to?5an?5emit?5mu@ 10013fd4     useasm:useasm.obj
 0001:00013010       ??_C@_0CF@OIPADGLP@?$CFs?5isn?8t?5supported?5on?5this?5proce@ 10014010     useasm:useasm.obj
 0001:00013038       ??_C@_0CL@BLKOKIML@No?5flags?5are?5valid?5for?5argument?5@ 10014038     useasm:useasm.obj
 0001:00013068       ??_C@_0FK@GPIOMEID@Argument?5?$CFd?5to?5smoa?5is?5not?5a?5leg@ 10014068     useasm:useasm.obj
 0001:000130c4       ??_C@_0CM@OICCJGCF@Argument?5?$CFd?5to?5smoa?5must?5be?5an?5a@ 100140c4     useasm:useasm.obj
 0001:000130f0       ??_C@_0CL@BPCDNEHJ@No?5flags?5are?5valid?5for?5argument?5@ 100140f0     useasm:useasm.obj
 0001:0001311c       ??_C@_0CF@KHLJFLDD@Argument?5?$CFd?5to?5smoa?5can?8t?5be?5ind@ 1001411c     useasm:useasm.obj
 0001:00013148       ??_C@_0EB@LMPOCDMD@Argument?5?$CFd?5to?5smoa?5is?5out?5of?5ra@ 10014148     useasm:useasm.obj
 0001:0001318c       ??_C@_0CP@JENPMIGB@Argument?5?$CFd?5to?5smoa?5must?5be?5an?5i@ 1001418c     useasm:useasm.obj
 0001:000131c0       ??_C@_0EI@CHCGIOOA@Loading?5the?5MOE?5state?5from?5regis@ 100141c0     useasm:useasm.obj
 0001:00013208       ??_C@_0DA@OPFKEKGA@Argument?5?$CFd?5to?5smlsi?5should?5be?5a@ 10014208     useasm:useasm.obj
 0001:00013238       ??_C@_0EG@BJPEDDED@Argument?5?$CFd?5to?5smlsi?5is?5out?5of?5r@ 10014238     useasm:useasm.obj
 0001:00013280       ??_C@_0DA@FCAKILOF@Argument?5?$CFd?5to?5smlsi?5must?5be?5an?5@ 10014280     useasm:useasm.obj
 0001:000132b0       ??_C@_0CM@LFIFLNIO@No?5flags?5are?5valid?5for?5argument?5@ 100142b0     useasm:useasm.obj
 0001:000132dc       ??_C@_0CG@PJFPKLPN@Argument?5?$CFd?5to?5smlsi?5can?8t?5be?5in@ 100142dc     useasm:useasm.obj
 0001:00013304       ??_C@_0DP@NNLBIBNI@Argument?5?$CFd?5to?5smlsi?5is?5out?5of?5r@ 10014304     useasm:useasm.obj
 0001:00013344       ??_C@_0CL@MJEEEJFH@Argument?5?$CFd?5to?5smlsi?5isn?8t?5a?5val@ 10014344     useasm:useasm.obj
 0001:00013370       ??_C@_0DM@BDMFEIMC@Argument?5?$CFd?5uses?5component?5selec@ 10014370     useasm:useasm.obj
 0001:000133ac       ??_C@_0DN@CBDPLAND@Argument?5?$CFd?5to?5smlsi?5must?5be?5an?5@ 100143ac     useasm:useasm.obj
 0001:000133f0       ??_C@_0EH@PIBJEHLO@Loading?5the?5MOE?5state?5from?5regis@ 100143f0     useasm:useasm.obj
 0001:00013438       ??_C@_0CD@DAICKOIL@Argument?5?$CFd?5to?5?$CFs?5can?8t?5be?5index@ 10014438     useasm:useasm.obj
 0001:0001345c       ??_C@_0DL@DAGJDBAJ@Argument?5?$CFd?5to?5?$CFs?5is?5out?5of?5rang@ 1001445c     useasm:useasm.obj
 0001:00013498       ??_C@_0DN@OPLIFLFN@Argument?5?$CFd?5to?5imo?5is?5out?5of?5ran@ 10014498     useasm:useasm.obj
 0001:000134d8       ??_C@_0DH@LBKJPHME@Argument?5?$CFd?5to?5smr?1smbo?1imo?5must@ 100144d8     useasm:useasm.obj
 0001:00013510       ??_C@_0EC@LGDHIHKO@Loading?5the?5MOE?5state?5from?5regis@ 10014510     useasm:useasm.obj
 0001:00013554       ??_C@_0CM@PAFKAACO@No?5flags?5are?5valid?5for?5argument?5@ 10014554     useasm:useasm.obj
 0001:00013580       ??_C@_0CG@JIFDPGCJ@Argument?5?$CFd?5to?5setfc?5can?8t?5be?5in@ 10014580     useasm:useasm.obj
 0001:000135a8       ??_C@_0DA@FIKLGADO@Argument?5?$CFd?5to?5setfc?5is?5must?5be?5@ 100145a8     useasm:useasm.obj
 0001:000135d8       ??_C@_0DA@PNIDFAOJ@Argument?5?$CFd?5to?5setfc?5must?5be?5an?5@ 100145d8     useasm:useasm.obj
 0001:00013608       ??_C@_0DC@IGFMAGID@Only?5?$CFd?5mutex?$CIes?$CJ?5are?5supported?5@ 10014608     useasm:useasm.obj
 0001:0001363c       ??_C@_0CE@FKFABDHJ@An?5immediate?5value?5can?8t?5be?5inde@ 1001463c     useasm:useasm.obj
 0001:00013660       ??_C@_0CK@FKJKMHCB@No?5flags?5are?5valid?5for?5the?5argum@ 10014660     useasm:useasm.obj
 0001:0001368c       ??_C@_0CI@GKLFIIMC@The?5argument?5to?5?$CFs?5must?5be?5an?5im@ 1001468c     useasm:useasm.obj
 0001:000136b8       ??_C@_0EI@IMBJAMEN@The?5maximum?5immediate?5value?5for?5@ 100146b8     useasm:useasm.obj
 0001:00013700       ??_C@_0DB@KGKPELKC@The?5third?5argument?5to?5ldr?5must?5b@ 10014700     useasm:useasm.obj
 0001:00013738       ??_C@_0EP@HFAIINHO@The?5destination?5for?5ldr?5must?5be?5@ 10014738     useasm:useasm.obj
 0001:00013788       ??_C@_0CJ@PBDIHBBP@The?5destination?5for?5ldr?5can?8t?5be@ 10014788     useasm:useasm.obj
 0001:000137b4       ??_C@_0DP@EOJFCBDD@The?5seventh?5argument?5to?5atst8?5mu@ 100147b4     useasm:useasm.obj
 0001:000137f4       ??_C@_0DC@GPFGCALA@An?5integer?5source?5selector?5value@ 100147f4     useasm:useasm.obj
 0001:00013828       ??_C@_0DM@KLBODCDM@The?5sixth?5argument?5to?5atst8?5must@ 10014828     useasm:useasm.obj
 0001:00013868       ??_C@_0EF@HHNKPNHB@No?5flags?5except?5disable?5writebac@ 10014868     useasm:useasm.obj
 0001:000138b0       ??_C@_0CG@EAILMAJF@A?5predicate?5register?5is?5not?5inde@ 100148b0     useasm:useasm.obj
 0001:000138d8       ??_C@_0DP@IJEBNLPN@The?5destination?5argument?5to?5atst@ 100148d8     useasm:useasm.obj
 0001:00013918       ??_C@_0DJ@CANNFGLC@The?5fifth?5argument?5to?5depthf?5mus@ 10014918     useasm:useasm.obj
 0001:00013954       ??_C@_0DO@JJIFGFHO@The?5fourth?5argument?5to?5depthf?5mu@ 10014954     useasm:useasm.obj
 0001:00013994       ??_C@_0DG@DJLDOPBE@The?5maximum?5monitor?5supported?5on@ 10014994     useasm:useasm.obj
 0001:000139cc       ??_C@_0CM@EANNIMNI@Monitors?5aren?8t?5supported?5on?5thi@ 100149cc     useasm:useasm.obj
 0001:000139f8       ??_C@_0DA@NGKNOLIJ@The?5argument?5to?5setm?5must?5be?5an?5@ 100149f8     useasm:useasm.obj
 0001:00013a28       ??_C@_0CK@FLEIDBJB@The?5maximum?5immediate?5value?5for?5@ 10014a28     useasm:useasm.obj
 0001:00013a54       ??_C@_0CP@KDAJINNH@The?5argument?5to?5wop?5must?5be?5an?5i@ 10014a54     useasm:useasm.obj
 0001:00013a84       ??_C@_0BE@CMNIOOMH@Unknown?5instruction?$AA@ 10014a84     useasm:useasm.obj
 0001:00013a98       ??_C@_0BN@FNBEMNH@?$CFs?5should?5have?5been?5coissued?$AA@ 10014a98     useasm:useasm.obj
 0001:00013ab8       ??_C@_0CC@NGMENPIE@?8?$CFs?8?5?3?5syntax?5error?$DL?5parse?5error@ 10014ab8     glsl_parser:parser.obj
 0001:00013adc       ??_C@_0CA@HKJBOAOI@Unexpected?5end?5of?5source?5found?6?$AA@ 10014adc     glsl_parser:parser.obj
 0001:00013afc       ??_C@_05IFHLPLPC@using?$AA@ 10014afc     glsl_parser:lex.obj
 0001:00013b04       ??_C@_09KPMGAFNI@namespace?$AA@ 10014b04     glsl_parser:lex.obj
 0001:00013b10       ??_C@_04HJDBPPOC@cast?$AA@ 10014b10     glsl_parser:lex.obj
 0001:00013b18       ??_C@_06FPFOALMG@sizeof?$AA@ 10014b18     glsl_parser:lex.obj
 0001:00013b20       ??_C@_0BE@HDPBANEK@sampler2DRectShadow?$AA@ 10014b20     glsl_parser:lex.obj
 0001:00013b34       ??_C@_0O@FCABDPDE@sampler3DRect?$AA@ 10014b34     glsl_parser:lex.obj
 0001:00013b44       ??_C@_0O@PEHGDEIA@sampler2DRect?$AA@ 10014b44     glsl_parser:lex.obj
 0001:00013b54       ??_C@_0BA@JPCOHDB@sampler2DShadow?$AA@ 10014b54     glsl_parser:lex.obj
 0001:00013b64       ??_C@_0BA@DAHPNLPE@sampler1DShadow?$AA@ 10014b64     glsl_parser:lex.obj
 0001:00013b74       ??_C@_09LAHPNHHH@sampler3D?$AA@ 10014b74     glsl_parser:lex.obj
 0001:00013b80       ??_C@_09LDPLADBJ@sampler1D?$AA@ 10014b80     glsl_parser:lex.obj
 0001:00013b8c       ??_C@_05BLEBCGML@fvec4?$AA@ 10014b8c     glsl_parser:lex.obj
 0001:00013b94       ??_C@_05FEAALAAM@fvec3?$AA@ 10014b94     glsl_parser:lex.obj
 0001:00013b9c       ??_C@_05ENBLIBEN@fvec2?$AA@ 10014b9c     glsl_parser:lex.obj
 0001:00013ba4       ??_C@_05FGIJIHMA@dvec4?$AA@ 10014ba4     glsl_parser:lex.obj
 0001:00013bac       ??_C@_05BJMIBBAH@dvec3?$AA@ 10014bac     glsl_parser:lex.obj
 0001:00013bb4       ??_C@_05NDCAEG@dvec2?$AA@  10014bb4     glsl_parser:lex.obj
 0001:00013bbc       ??_C@_05CBELEHLL@hvec4?$AA@ 10014bbc     glsl_parser:lex.obj
 0001:00013bc4       ??_C@_05GOAKNBHM@hvec3?$AA@ 10014bc4     glsl_parser:lex.obj
 0001:00013bcc       ??_C@_05HHBBOADN@hvec2?$AA@ 10014bcc     glsl_parser:lex.obj
 0001:00013bd4       ??_C@_05DFJCHPDH@input?$AA@ 10014bd4     glsl_parser:lex.obj
 0001:00013bdc       ??_C@_06GJJMFEHD@superp?$AA@ 10014bdc     glsl_parser:lex.obj
 0001:00013be4       ??_C@_08CLLOMHGD@unsigned?$AA@ 10014be4     glsl_parser:lex.obj
 0001:00013bf0       ??_C@_05OFLEIIDM@fixed?$AA@ 10014bf0     glsl_parser:lex.obj
 0001:00013bf8       ??_C@_04GBGPFKGN@half?$AA@ 10014bf8     glsl_parser:lex.obj
 0001:00013c00       ??_C@_06BNJCAIGJ@double?$AA@ 10014c00     glsl_parser:lex.obj
 0001:00013c08       ??_C@_05BFKKPKCG@short?$AA@ 10014c08     glsl_parser:lex.obj
 0001:00013c10       ??_C@_04GOKPGOLB@long?$AA@ 10014c10     glsl_parser:lex.obj
 0001:00013c18       ??_C@_04FMBJNPFB@flat?$AA@ 10014c18     glsl_parser:lex.obj
 0001:00013c20       ??_C@_09NFKLEKPH@interface?$AA@ 10014c20     glsl_parser:lex.obj
 0001:00013c2c       ??_C@_08OIBPHJGN@external?$AA@ 10014c2c     glsl_parser:lex.obj
 0001:00013c38       ??_C@_06PAMNHHEG@extern?$AA@ 10014c38     glsl_parser:lex.obj
 0001:00013c40       ??_C@_06GGHJAEBN@static?$AA@ 10014c40     glsl_parser:lex.obj
 0001:00013c48       ??_C@_06EOMAMIIF@public?$AA@ 10014c48     glsl_parser:lex.obj
 0001:00013c50       ??_C@_08PABEKFH@volatile?$AA@ 10014c50     glsl_parser:lex.obj
 0001:00013c5c       ??_C@_08OIGDDPGB@noinline?$AA@ 10014c5c     glsl_parser:lex.obj
 0001:00013c68       ??_C@_06OGMBMJA@inline?$AA@ 10014c68     glsl_parser:lex.obj
 0001:00013c70       ??_C@_07DLHCIBDH@default?$AA@ 10014c70     glsl_parser:lex.obj
 0001:00013c78       ??_C@_06DOPOGBGP@switch?$AA@ 10014c78     glsl_parser:lex.obj
 0001:00013c80       ??_C@_04MABHPDAO@goto?$AA@ 10014c80     glsl_parser:lex.obj
 0001:00013c88       ??_C@_06DAGLPGKC@packed?$AA@ 10014c88     glsl_parser:lex.obj
 0001:00013c90       ??_C@_04IIAJELJL@this?$AA@ 10014c90     glsl_parser:lex.obj
 0001:00013c98       ??_C@_08FJNLKCPH@template?$AA@ 10014c98     glsl_parser:lex.obj
 0001:00013ca4       ??_C@_07FIDIHKEG@typedef?$AA@ 10014ca4     glsl_parser:lex.obj
 0001:00013cac       ??_C@_04DBJPMPLO@enum?$AA@ 10014cac     glsl_parser:lex.obj
 0001:00013cb4       ??_C@_05MNALHJLP@union?$AA@ 10014cb4     glsl_parser:lex.obj
 0001:00013cbc       ??_C@_05ENKANFLO@class?$AA@ 10014cbc     glsl_parser:lex.obj
 0001:00013cc4       ??_C@_03NLMFHDGG@asm?$AA@  10014cc4     glsl_parser:lex.obj
 0001:00013cc8       ??_C@_0BB@LEFHFFO@samplerStreamIMG?$AA@ 10014cc8     glsl_parser:lex.obj
 0001:00013cdc       ??_C@_0M@JKFFOHJO@samplerCube?$AA@ 10014cdc     glsl_parser:lex.obj
 0001:00013ce8       ??_C@_09LBLNLNEA@sampler2D?$AA@ 10014ce8     glsl_parser:lex.obj
 0001:00013cf4       ??_C@_04DDDHBIAD@mat4?$AA@ 10014cf4     glsl_parser:lex.obj
 0001:00013cfc       ??_C@_04HMHGIOME@mat3?$AA@ 10014cfc     glsl_parser:lex.obj
 0001:00013d04       ??_C@_04GFGNLPIF@mat2?$AA@ 10014d04     glsl_parser:lex.obj
 0001:00013d0c       ??_C@_06LNOFJDNM@return?$AA@ 10014d0c     glsl_parser:lex.obj
 0001:00013d14       ??_C@_07FGAIHHOI@discard?$AA@ 10014d14     glsl_parser:lex.obj
 0001:00013d1c       ??_C@_05OODBEKIG@while?$AA@ 10014d1c     glsl_parser:lex.obj
 0001:00013d24       ??_C@_03JOHEBPFF@for?$AA@  10014d24     glsl_parser:lex.obj
 0001:00013d28       ??_C@_02KNAFDCHJ@do?$AA@   10014d28     glsl_parser:lex.obj
 0001:00013d2c       ??_C@_08DLICDMBN@continue?$AA@ 10014d2c     glsl_parser:lex.obj
 0001:00013d38       ??_C@_05ELPHFHOI@break?$AA@ 10014d38     glsl_parser:lex.obj
 0001:00013fe4       ??_C@_0CO@FIFCCL@Reached?5end?5of?5GLSL?5source?5insid@ 10014fe4     glsl_parser:lex.obj
 0001:00014014       ??_C@_0CP@BAHGCENG@?$CFd?3?$CFd?$CFd?5?8?$CFc?8?5is?5an?5invalid?5chara@ 10015014     glsl_parser:lex.obj
 0001:00014044       ??_C@_0CJ@PKMNFKJG@?$CFd?3?$CFd?3?$CFd?5invalid?5number?5literal?5@ 10015044     glsl_parser:lex.obj
 0001:00014070       ??_C@_0CB@CLPPICJH@?$CFd?3?$CFd?3?$CFd?5reserved?5keyword?5?8?$CFs?8?4?6@ 10015070     glsl_parser:lex.obj
 0001:00014590       UFRegATableGetMaxComponent 10015590 f   ic2uf.obj
 0001:00014b04       GetStructAllocInfo         10015b04 f   ic2uf.obj
 0001:000189a8       DestroyUniFlexCode         100199a8 f   ic2uf.obj
 0001:000195c8       GenerateUniPatchInput      1001a5c8 f   ic2uf.obj
 0001:00019888       GetSupportedExtensions     1001a888 f   ic2uf.obj
 0001:0001d368       GenerateUniFlexInput       1001e368 f   ic2uf.obj
 0001:0001d5d8       GLSLFreeCompiledUniflexProgram 1001e5d8 f   glsl2uf.obj
 0001:0001d7d4       GLSLCompileToUniflex       1001e7d4 f   glsl2uf.obj
 0001:0001d970       GLSLDisplayMetrics         1001e970 f   glsl2uf.obj
 0001:0001e254       GenerateBindingSymbolList  1001f254 f   bindingsym.obj
 0001:0001e39c       DestroyBindingSymbolList   1001f39c f   bindingsym.obj
 0001:0001e454       InitSymbolTableManager     1001f454 f   glsl_parser:symtab.obj
 0001:0001e474       DestroySymbolTableManager  1001f474 f   glsl_parser:symtab.obj
 0001:0001e59c       RemoveSymbolTableFromManager 1001f59c f   glsl_parser:symtab.obj
 0001:0001e5dc       CreateSymTable             1001f5dc f   glsl_parser:symtab.obj
 0001:0001e6d0       DestroySymTable            1001f6d0 f   glsl_parser:symtab.obj
 0001:0001e824       FindSymbol                 1001f824 f   glsl_parser:symtab.obj
 0001:0001e8a4       GetSymbolDatafn            1001f8a4 f   glsl_parser:symtab.obj
 0001:0001ea94       AddSymbol                  1001fa94 f   glsl_parser:symtab.obj
 0001:0001eac8       RemoveSymbol               1001fac8 f   glsl_parser:symtab.obj
 0001:0001eb14       GetSymbolNamefn            1001fb14 f   glsl_parser:symtab.obj
 0001:0001eb3c       IncreaseScopeLevel         1001fb3c f   glsl_parser:symtab.obj
 0001:0001ebc4       DecreaseScopeLevel         1001fbc4 f   glsl_parser:symtab.obj
 0001:0001ec5c       GetScopeLevel              1001fc5c f   glsl_parser:symtab.obj
 0001:0001ec64       GetSymbolScopeLevelfn      1001fc64 f   glsl_parser:symtab.obj
 0001:0001ec98       ResetGetNextSymbolCounter  1001fc98 f   glsl_parser:symtab.obj
 0001:0001eca8       GetNextSymbol              1001fca8 f   glsl_parser:symtab.obj
 0001:0001ed3c       ICAddTemporary             1001fd3c f   glsl_core:icgen.obj
 0001:0001ee9c       ICAddBoolPredicate         1001fe9c f   glsl_core:icgen.obj
 0001:0001efe0       ICInitICOperand            1001ffe0 f   glsl_core:icgen.obj
 0001:0001f018       ICInitOperandInfo          10020018 f   glsl_core:icgen.obj
 0001:0001f130       ICAddOperandOffset         10020130 f   glsl_core:icgen.obj
 0001:0001f178       ICFreeOperandOffsetList    10020178 f   glsl_core:icgen.obj
 0001:0001f324       ICRemoveInstruction        10020324 f   glsl_core:icgen.obj
 0001:0001f348       ICRemoveInstructionRange   10020348 f   glsl_core:icgen.obj
 0001:0001f3e8       ICGetSymbolInformation     100203e8 f   glsl_core:icgen.obj
 0001:0001f550       ICGetSymbolTypeSpecifier   10020550 f   glsl_core:icgen.obj
 0001:0001f568       ICGetSymbolPrecision       10020568 f   glsl_core:icgen.obj
 0001:0001f580       GetIndexedType             10020580 f   glsl_core:icgen.obj
 0001:0001f6fc       IsSymbolIntConstant        100206fc f   glsl_core:icgen.obj
 0001:0001f798       IsSymbolLValue             10020798 f   glsl_core:icgen.obj
 0001:0001f988       CloneICodeInstructions     10020988 f   glsl_core:icgen.obj
 0001:0001faf8       ICAddICInstruction0        10020af8 f   glsl_core:icgen.obj
 0001:0001fb4c       ICAddICInstruction1        10020b4c f   glsl_core:icgen.obj
 0001:0001fbb0       ICAddICInstruction1a       10020bb0 f   glsl_core:icgen.obj
 0001:0001fc34       ICAddICInstruction2        10020c34 f   glsl_core:icgen.obj
 0001:0001fca8       ICAddICInstruction2a       10020ca8 f   glsl_core:icgen.obj
 0001:0001fd3c       ICAddICInstruction2b       10020d3c f   glsl_core:icgen.obj
 0001:0001fde8       ICAddICInstruction2c       10020de8 f   glsl_core:icgen.obj
 0001:0001fe7c       ICAddICInstruction3        10020e7c f   glsl_core:icgen.obj
 0001:0001ff00       ICAddICInstruction3a       10020f00 f   glsl_core:icgen.obj
 0001:0001ffa4       ICAddICInstruction3b       10020fa4 f   glsl_core:icgen.obj
 0001:00020060       ICAddICInstruction3c       10021060 f   glsl_core:icgen.obj
 0001:0002011c       ICAddICInstruction3d       1002111c f   glsl_core:icgen.obj
 0001:000201f0       ICAddICInstruction3e       100211f0 f   glsl_core:icgen.obj
 0001:000202ac       ICAddICInstruction4        100212ac f   glsl_core:icgen.obj
 0001:00020340       ICAddICInstruction         10021340 f   glsl_core:icgen.obj
 0001:000203e8       ICAddICInstructiona        100213e8 f   glsl_core:icgen.obj
 0001:000204b0       ICIsSymbolScalar           100214b0 f   glsl_core:icgen.obj
 0001:000206d0       ICAddICInstructionIFP      100216d0 f   glsl_core:icgen.obj
 0001:000208b4       ICCombineTwoConstantSwizzles 100218b4 f   glsl_core:icgen.obj
 0001:00020940       ICAdjustOperandLastOffset  10021940 f   glsl_core:icgen.obj
 0001:000217a8       ICProcessNodeOperand       100227a8 f   glsl_core:icgen.obj
 0001:00024868       ICTraverseAST              10025868 f   glsl_core:icgen.obj
 0001:00024a50       ASTValidateNodeCreationFn  10025a50 f   glsl_core:common.obj
 0001:00024a70       ASTCreateNewNodeFn         10025a70 f   glsl_core:common.obj
 0001:00024ad0       ASTAddNodeChildFn          10025ad0 f   glsl_core:common.obj
 0001:00024c48       AddIdentifierDataToTable   10025c48 f   glsl_core:common.obj
 0001:00024d50       AddSwizzleData             10025d50 f   glsl_core:common.obj
 0001:00024d84       AddMemberSelectionData     10025d84 f   glsl_core:common.obj
 0001:00024db8       AddIdentifierDatafn        10025db8 f   glsl_core:common.obj
 0001:00024ddc       AddParameterDatafn         10025ddc f   glsl_core:common.obj
 0001:00024ee0       AddResultDatafn            10025ee0 f   glsl_core:common.obj
 0001:00024f04       AddFunctionCallData        10025f04 f   glsl_core:common.obj
 0001:00024f98       AddFunctionDefinitionData  10025f98 f   glsl_core:common.obj
 0001:0002530c       AddStructureDefinition     1002630c f   glsl_core:common.obj
 0001:000257b0       GetSymbolTableDatafn       100267b0 f   glsl_core:common.obj
 0001:0002581c       GetSymbolInfofn            1002681c f   glsl_core:common.obj
 0001:00025c44       AddBuiltInIdentifier       10026c44 f   glsl_core:common.obj
 0001:00025d44       AddBoolConstant            10026d44 f   glsl_core:common.obj
 0001:00025e50       AddIntConstant             10026e50 f   glsl_core:common.obj
 0001:00025f90       AddFloatConstant           10026f90 f   glsl_core:common.obj
 0001:00026130       AddFloatVecConstant        10027130 f   glsl_core:common.obj
 0001:000261f0       SetErrorLog                100271f0 f   glsl_core:error.obj
 0001:0002620c       FreeErrorLogMessages       1002720c f   glsl_core:error.obj
 0001:00026510       LogProgramError            10027510 f   glsl_core:error.obj
 0001:00026544       LogProgramWarning          10027544 f   glsl_core:error.obj
 0001:00026578       LogProgramNodeError        10027578 f   glsl_core:error.obj
 0001:000265c0       LogProgramNodeWarning      100275c0 f   glsl_core:error.obj
 0001:00026608       LogProgramParseTreeError   10027608 f   glsl_core:error.obj
 0001:00026650       LogProgramTokenError       10027650 f   glsl_core:error.obj
 0001:00026688       LogProgramTokenWarning     10027688 f   glsl_core:error.obj
 0001:000266c0       LogProgramParserError      100276c0 f   glsl_core:error.obj
 0001:00026898       GLSLFreeBuiltInState       10027898 f   glsl_core:glsl.obj
 0001:000268f4       GLSLInitCompiler           100278f4 f   glsl_core:glsl.obj
 0001:00026a18       GLSLShutDownCompiler       10027a18 f   glsl_core:glsl.obj
 0001:00026a84       GLSLGenerateInfoLog        10027a84 f   glsl_core:glsl.obj
 0001:00026bac       GLSLFreeInfoLog            10027bac f   glsl_core:glsl.obj
 0001:00026bc8       GLSLCompileToIntermediateCode 10027bc8 f   glsl_core:glsl.obj
 0001:00026e68       GLSLFreeIntermediateCode   10027e68 f   glsl_core:glsl.obj
 0001:0002893c       ICFindBuiltInVariables     1002993c f   glsl_core:icbuiltin.obj
 0001:0002ae9c       ICProcessBuiltInFunctionCall 1002be9c f   glsl_core:icbuiltin.obj
 0001:0002bd8c       ICUnrollLoopFOR            1002cd8c f   glsl_core:icunroll.obj
 0001:0002d588       ASTBIAddBuiltInData        1002e588 f   glsl_core:astbuiltin.obj
 0001:0002f73c       ASTBIResetBuiltInData      1003073c f   glsl_core:astbuiltin.obj
 0001:00032380       PPPreProcessTokenList      10033380 f   glsl_core:prepro.obj
 0001:0003298c       PPDestroyPreProcessorData  1003398c f   glsl_core:prepro.obj
 0001:000357ec       CheckGLSLTreeCompleteness  100367ec f   glsl_core:glsltree.obj
 0001:0003592c       DestroyGLSLTreeContext     1003692c f   glsl_core:glsltree.obj
 0001:0003bba0       CreateGLSLTreeContext      1003cba0 f   glsl_core:glsltree.obj
 0001:0003bd54       GenerateICodeProgram       1003cd54 f   glsl_core:icode.obj
 0001:0003bf5c       DestroyICodeProgram        1003cf5c f   glsl_core:icode.obj
 0001:0003cab4       ICEmulateBIFNtan           1003dab4 f   glsl_core:icemul.obj
 0001:0003d510       ICEmulateBIFNArcTrigs      1003e510 f   glsl_core:icemul.obj
 0001:0003d820       ICEmulateBIFNpow           1003e820 f   glsl_core:icemul.obj
 0001:0003d96c       ICEmulateBIFNfract         1003e96c f   glsl_core:icemul.obj
 0001:0003da80       ICEmulateBIFNmod           1003ea80 f   glsl_core:icemul.obj
 0001:0003e348       ICEmulateBIFNshadowFunc    1003f348 f   glsl_core:icemul.obj
 0001:0003e730       ICEmulateBIFNnoise1        1003f730 f   glsl_core:icemul.obj
 0001:0003e848       ICEmulateBIFNnoise2        1003f848 f   glsl_core:icemul.obj
 0001:0003eb28       ICEmulateBIFNnoise3        1003fb28 f   glsl_core:icemul.obj
 0001:0003eec4       ICEmulateBIFNnoise4        1003fec4 f   glsl_core:icemul.obj
 0001:0003f2f0       ICAddArcSinCos2FunctionBody 100402f0 f   glsl_core:icemul.obj
 0001:0003fc9c       ICAddArcTanFunctionBody    10040c9c f   glsl_core:icemul.obj
 0001:00040638       ICAddArcTan2FunctionBody   10041638 f   glsl_core:icemul.obj
 0001:00040e8c       ICAddNoise1DFunctionBody   10041e8c f   glsl_core:icemul.obj
 0001:00041578       ICAddNoise2DFunctionBody   10042578 f   glsl_core:icemul.obj
 0001:00041fa4       ICAddNoise3DFunctionBody   10042fa4 f   glsl_core:icemul.obj
 0001:000434f8       ICAddNoise4DFunctionBody   100444f8 f   glsl_core:icemul.obj
 0001:000456f8       ICEmulateTextureProj       100466f8 f   glsl_core:icemul.obj
 0001:00045ac4       ASTSemCreateHashedFunctionName 10046ac4 f   glsl_core:semantic.obj
 0001:00045cc8       ASTSemGetSizeInfo          10046cc8 f   glsl_core:semantic.obj
 0001:00048ef4       ASTSemCheckTypeSpecifiersMatch 10049ef4 f   glsl_core:semantic.obj
 0001:000491f8       ASTSemGetArraySize         1004a1f8 f   glsl_core:semantic.obj
 0001:000498c8       ASTUpdateConditionalIdentifierUsage 1004a8c8 f   glsl_core:semantic.obj
 0001:0004a044       ASTSemAddIdentifierToSymbolTable 1004b044 f   glsl_core:semantic.obj
 0001:0004b000       ASTSemCheckTypesAndCalculateResult 1004c000 f   glsl_core:semantic.obj
 0001:0004c790       EmulateBuiltInFunction     1004d790 f   glsl_core:glslfns.obj
 0001:0004ea10       SGXBS_CreateBinaryProgram  1004fa10 f   glsl_binshader:esbinshader.obj
 0001:0004ebf8       PVRUniFlexInitInst         1004fbf8 f   usc:usc_utils.obj
 0001:0004ec1c       UscAbort                   1004fc1c f   usc:usc.obj
 0001:0004ec44       UscAlloc                   1004fc44 f   usc:usc.obj
 0001:0004eca8       _UscFree                   1004fca8 f   usc:usc.obj
 0001:0004ecf0       GetNextRegister            1004fcf0 f   usc:usc.obj
 0001:0004ee34       SetBlockSwitch             1004fe34 f   usc:usc.obj
 0001:0004ef9c       SetBlockUnconditional      1004ff9c f   usc:usc.obj
 0001:0004f0bc       RedirectEdgesFromPredecessors 100500bc f   usc:usc.obj
 0001:0004f1e0       RedirectEdge               100501e0 f   usc:usc.obj
 0001:0004f250       AllocateBlock              10050250 f   usc:usc.obj
 0001:0004f3a0       FreeBlock                  100503a0 f   usc:usc.obj
 0001:0004f590       IsCall                     10050590 f   usc:usc.obj
 0001:0004f62c       DoDataflow                 1005062c f   usc:usc.obj
 0001:0004f7fc       DoOnCfgBasicBlocks         100507fc f   usc:usc.obj
 0001:0004f8a4       DoOnAllBasicBlocks         100508a4 f   usc:usc.obj
 0001:0004f984       DebugPrintSF               10050984 f   usc:usc.obj
 0001:0004f9cc       InlineFunction             100509cc f   usc:usc.obj
 0001:0004fd34       PVRUniFlexDestroyContext   10050d34 f   usc:usc.obj
 0001:0004fd48       AppendInst                 10050d48 f   usc:usc.obj
 0001:0004fddc       RemoveInst                 10050ddc f   usc:usc.obj
 0001:0004fe38       MaskToSwiz                 10050e38 f   usc:usc.obj
 0001:0004fe70       CompOpToTest               10050e70 f   usc:usc.obj
 0001:0004fefc       GetPredicate               10050efc f   usc:usc.obj
 0001:0004ff94       AllocFunction              10050f94 f   usc:usc.obj
 0001:0005003c       FreeFunction               1005103c f   usc:usc.obj
 0001:00050208       InitialiseIndexableTemps   10051208 f   usc:usc.obj
 0001:0005023c       InitState                  1005123c f   usc:usc.obj
 0001:00050494       ReleaseState               10051494 f   usc:usc.obj
 0001:00050afc       PVRUniFlexCreateContext    10051afc f   usc:usc.obj
 0001:00050b68       PVRUniFlexDestroyUspBin    10051b68 f   usc:usc.obj
 0001:00050b6c       GetNextRegisterCount       10051b6c f   usc:usc.obj
 0001:00050b90       SetBlockConditional        10051b90 f   usc:usc.obj
 0001:00050d08       MergeBasicBlocks           10051d08 f   usc:usc.obj
 0001:00050fb0       MergeAllBasicBlocks        10051fb0 f   usc:usc.obj
 0001:00050fe0       FinaliseIntermediateCode   10051fe0 f   usc:usc.obj
 0001:00051118       InsertInstBefore           10052118 f   usc:usc.obj
 0001:00051478       ConvertSwitchBP            10052478 f   usc:usc.obj
 0001:00052afc       CompileIntermediate        10053afc f   usc:usc.obj
 0001:00052ec8       PVRUniFlexCompileToUspBin  10053ec8 f   usc:usc.obj
 0001:0005300c       ResizeArray                1005400c f   usc:data.obj
 0001:0005312c       ClearArray                 1005412c f   usc:data.obj
 0001:000531d8       FreeArray                  100541d8 f   usc:data.obj
 0001:00053218       NewArray                   10054218 f   usc:data.obj
 0001:00053470       ArrayGet                   10054470 f   usc:data.obj
 0001:00053570       ArraySet                   10054570 f   usc:data.obj
 0001:000535c0       ClearVector                100545c0 f   usc:data.obj
 0001:00053630       FreeVector                 10054630 f   usc:data.obj
 0001:0005366c       InitVector                 1005466c f   usc:data.obj
 0001:000536a4       NewVector                  100546a4 f   usc:data.obj
 0001:000536d0       VectorGet                  100546d0 f   usc:data.obj
 0001:00053818       ArrayElemOp                10054818 f   usc:data.obj
 0001:00053c3c       VectorOp                   10054c3c f   usc:data.obj
 0001:00053cf4       VectorCopy                 10054cf4 f   usc:data.obj
 0001:00053e10       VectorSet                  10054e10 f   usc:data.obj
 0001:00053f14       VectorGetRange             10054f14 f   usc:data.obj
 0001:00054198       VectorSetRange             10055198 f   usc:data.obj
 0001:0005425c       VectorOrRange              1005525c f   usc:data.obj
 0001:00054314       VectorAndRange             10055314 f   usc:data.obj
 0001:000543d8       NewGraph                   100553d8 f   usc:data.obj
 0001:00054408       ClearGraph                 10055408 f   usc:data.obj
 0001:00054444       FreeGraph                  10055444 f   usc:data.obj
 0001:00054480       GraphGet                   10055480 f   usc:data.obj
 0001:00054510       GraphSet                   10055510 f   usc:data.obj
 0001:00054614       GraphColRef                10055614 f   usc:data.obj
 0001:00054650       GraphDupCol                10055650 f   usc:data.obj
 0001:00054734       GraphClearCol              10055734 f   usc:data.obj
 0001:0005476c       GraphOrCol                 1005576c f   usc:data.obj
 0001:00054878       GraphCopy                  10055878 f   usc:data.obj
 0001:00054a18       InsertSort                 10055a18 f   usc:data.obj
 0001:00054b5c       InitialiseAdjacencyList    10055b5c f   usc:data.obj
 0001:00054b70       DeleteAdjacencyList        10055b70 f   usc:data.obj
 0001:00054ba0       DeleteAdjacencyListIndirect 10055ba0 f   usc:data.obj
 0001:00054bf4       ReplaceInAdjacencyList     10055bf4 f   usc:data.obj
 0001:00054c8c       RemoveFromAdjacencyList    10055c8c f   usc:data.obj
 0001:00054d94       AddToAdjacencyList         10055d94 f   usc:data.obj
 0001:00054e00       CloneAdjacencyList         10055e00 f   usc:data.obj
 0001:00054e98       ClearRegLiveSet            10055e98 f   usc:dce.obj
 0001:00054ee8       InitRegLiveSet             10055ee8 f   usc:dce.obj
 0001:00054f50       FreeRegLiveSet             10055f50 f   usc:dce.obj
 0001:00054f9c       AllocRegLiveSet            10055f9c f   usc:dce.obj
 0001:00055d7c       GetLiveChansInArgument     10056d7c f   usc:dce.obj
 0001:00055d98       GetChansUsedFromResult     10056d98 f   usc:dce.obj
 0001:00055e78       GetLiveChansInArg          10056e78 f   usc:dce.obj
 0001:00055f70       GetRegisterLiveMask        10056f70 f   usc:dce.obj
 0001:000560b0       SetRegisterLiveMask        100570b0 f   usc:dce.obj
 0001:00056474       IncreaseRegisterLiveMask   10057474 f   usc:dce.obj
 0001:000571b8       DeadCodeSplitBlock         100581b8 f   usc:dce.obj
 0001:00057274       DeadCodeEliminationBP      10058274 f   usc:dce.obj
 0001:000577d0       DoSALiveness               100587d0 f   usc:dce.obj
 0001:000578d0       DeadCodeElimination        100588d0 f   usc:dce.obj
 0001:00057b98       InitRegUseDef              10058b98 f   usc:dce.obj
 0001:00057c0c       ClearRegUseDef             10058c0c f   usc:dce.obj
 0001:00057c68       InitUseDef                 10058c68 f   usc:dce.obj
 0001:00057c80       ClearUseDef                10058c80 f   usc:dce.obj
 0001:00057ca0       GetRegUseDef               10058ca0 f   usc:dce.obj
 0001:00057d9c       IncreaseRegUseDef          10058d9c f   usc:dce.obj
 0001:00057f00       ReduceRegUseDef            10058f00 f   usc:dce.obj
 0001:00058088       InstUseSubset              10059088 f   usc:dce.obj
 0001:000583c8       InstUse                    100593c8 f   usc:dce.obj
 0001:000583d0       InstDef                    100593d0 f   usc:dce.obj
 0001:000585bc       ComputeInstUseDef          100595bc f   usc:dce.obj
 0001:0005861c       DisjointUseDef             1005961c f   usc:dce.obj
 0001:000589bc       RegUseInst                 100599bc f   usc:dce.obj
 0001:00058a4c       RegUseBlock                10059a4c f   usc:dce.obj
 0001:00058c00       InstUseDefined             10059c00 f   usc:dce.obj
 0001:00058ca8       InstDefReferenced          10059ca8 f   usc:dce.obj
 0001:00058d8c       CanHaveSourceModifier      10059d8c f   usc:inst.obj
 0001:00058ddc       GetUSPPerSampleTemporaryCount 10059ddc f   usc:inst.obj
 0001:00058e10       GetRegisterGroupCount      10059e10 f   usc:inst.obj
 0001:00058e44       GetRegisterGroupDetails    10059e44 f   usc:inst.obj
 0001:00058f58       IsArgInRegisterGroup       10059f58 f   usc:inst.obj
 0001:00058fd4       HasC10FmtControl           10059fd4 f   usc:inst.obj
 0001:00059024       RequiresGradients          1005a024 f   usc:inst.obj
 0001:00059058       GetMaxRepeatCountInst      1005a058 f   usc:inst.obj
 0001:00059080       CanRepeatInst              1005a080 f   usc:inst.obj
 0001:00059150       HasF16F32SelectInst        1005a150 f   usc:inst.obj
 0001:000591a0       WroteAllLiveChannels       1005a1a0 f   usc:inst.obj
 0001:000591d8       CanUseDest                 1005a1d8 f   usc:inst.obj
 0001:00059264       CanUseSrc                  1005a264 f   usc:inst.obj
 0001:000594f0       GetChannelsWrittenInRegister 1005a4f0 f   usc:inst.obj
 0001:0005959c       GetChannelsWrittenInArg    1005a59c f   usc:inst.obj
 0001:00059704       FreeInst                   1005a704 f   usc:inst.obj
 0001:00059764       InitInstArg                1005a764 f   usc:inst.obj
 0001:00059a60       SetOpcode                  1005aa60 f   usc:inst.obj
 0001:00059b9c       AllocateInst               1005ab9c f   usc:inst.obj
 0001:00059c6c       CopyInst                   1005ac6c f   usc:inst.obj
 0001:00059fb8       FormMove                   1005afb8 f   usc:inst.obj
 0001:0005a048       IsMove                     1005b048 f   usc:inst.obj
 0001:0005a294       GetDestMaskIdx             1005b294 f   usc:inst.obj
 0001:0005a2b8       GetDestMask                1005b2b8 f   usc:inst.obj
 0001:0005a2ec       ConvertRegister            1005b2ec f   usc:inst.obj
 0001:0005a36c       SameRegister               1005b36c f   usc:inst.obj
 0001:0005a3b4       EqualArgsIgnoreNegate      1005b3b4 f   usc:inst.obj
 0001:0005a478       EqualArgs                  1005b478 f   usc:inst.obj
 0001:0005a480       IsDeschedBeforeInst        1005b480 f   usc:inst.obj
 0001:0005a4ac       IsDeschedAfterInst         1005b4ac f   usc:inst.obj
 0001:0005a4f0       IsDeschedulingPoint        1005b4f0 f   usc:inst.obj
 0001:0005a530       CanUseSource0              1005b530 f   usc:inst.obj
 0001:0005a69c       EqualInstructionModes      1005b69c f   usc:inst.obj
 0001:0005cb90       OverwritesIndex            1005db90 f   usc:iselect.obj
 0001:0005cbb0       CanUseArgInRegisterGroup   1005dbb0 f   usc:iselect.obj
 0001:0005d90c       GlobalDefaultUpdateBlock   1005e90c f   usc:iselect.obj
 0001:0005e018       DoGlobalMoveReplace        1005f018 f   usc:iselect.obj
 0001:0006118c       FlattenProgramConditionals 1006218c f   usc:iselect.obj
 0001:000624a0       ConvertPredicatedMovesToMovcBP 100634a0 f   usc:iselect.obj
 0001:00062f90       FixInvalidSourceBanksBP    10063f90 f   usc:iselect.obj
 0001:00063da8       SimplifyArithmetic         10064da8 f   usc:iselect.obj
 0001:000642a0       EliminateGlobalMove        100652a0 f   usc:iselect.obj
 0001:00064358       EliminateMovesBP           10065358 f   usc:iselect.obj
 0001:00064960       EliminateMovesAndFuncs     10065960 f   usc:iselect.obj
 0001:000649e0       MergeIdenticalInstructionsBP 100659e0 f   usc:iselect.obj
 0001:000657ac       ExtractConstantCalculations 100667ac f   usc:iselect.obj
 0001:000658c0       OptimiseUSPSamplesBP       100668c0 f   usc:iselect.obj
 0001:0006597c       RemoveUnnecessarySaturationsBP 1006697c f   usc:iselect.obj
 0001:00065bec       GenerateNonEfoInstructionsBP 10066bec f   usc:iselect.obj
 0001:0006dea8       IntegerOptimize            1006eea8 f   usc:intcvt.obj
 0001:0006e1c4       GetHWOperandsUsedForArg    1006f1c4 f   usc:uspbin.obj
 0001:00070534       CreateUspBinOutput         10071534 f   usc:uspbin.obj
 0001:00070730       DestroyUspBinOutput        10071730 f   usc:uspbin.obj
 0001:00070d78       InsertAlternateResults     10071d78 f   usc:uspbin.obj
 0001:00071038       IsInstReferingShaderResult 10072038 f   usc:uspbin.obj
 0001:00071274       CalcDoms                   10072274 f   usc:domcalc.obj
 0001:00071560       Dominates                  10072560 f   usc:domcalc.obj
 0001:00071598       PostDominated              10072598 f   usc:domcalc.obj
 0001:00071638       ComputeLoopNestingTree     10072638 f   usc:domcalc.obj
 0001:00071718       IsLoopHeader               10072718 f   usc:domcalc.obj
 0001:00071768       LoopDepth                  10072768 f   usc:domcalc.obj
 0001:0007194c       PackCalculatedSecondaryAttributes 1007294c f   usc:regpack.obj
 0001:00071f5c       GetHardwareConstantValueu  10072f5c f   usc:regpack.obj
 0001:00071f88       GetHardwareConstantValue   10072f88 f   usc:regpack.obj
 0001:00071f98       IsStaticC10Value           10072f98 f   usc:regpack.obj
 0001:00072160       AddNewCalculatedSecAttrs   10073160 f   usc:regpack.obj
 0001:000721a4       AddNewInRegisterConstant   100731a4 f   usc:regpack.obj
 0001:00072228       AddStaticSecAttrRange      10073228 f   usc:regpack.obj
 0001:00072374       AddStaticSecAttr           10073374 f   usc:regpack.obj
 0001:00072394       ReplaceHardwareConstBySecAttr 10073394 f   usc:regpack.obj
 0001:00073764       SetC10RGBAConstant         10074764 f   usc:regpack.obj
 0001:000737d8       IsC10RGBAConstant          100747d8 f   usc:regpack.obj
 0001:00073c5c       PackPrimaryAttributeRegisters 10074c5c f   usc:regpack.obj
 0001:00074374       PackConstantRegisters      10075374 f   usc:regpack.obj
 0001:00075094       ReorderInstructionsBP      10076094 f   usc:reorder.obj
 0001:00075290       SplitFeedback              10076290 f   usc:reorder.obj
 0001:00075a24       PeepholeOptimizeBlock      10076a24 f   usc:reorder.obj
 0001:00075a68       SupportNoSched             10076a68 f   usc:finalise.obj
 0001:00075aa4       UpdateIRegsLive            10076aa4 f   usc:finalise.obj
 0001:00078d80       FinaliseShader             10079d80 f   usc:finalise.obj
 0001:00079608       GetIRegsWrittenMask        1007a608 f   usc:regalloc.obj
 0001:00079650       GetIRegsReadMask           1007a650 f   usc:regalloc.obj
 0001:000796cc       UpdateIRegs                1007a6cc f   usc:regalloc.obj
 0001:00079e68       NodeActivity               1007ae68 f   usc:regalloc.obj
 0001:00079f80       InitRegInterval            1007af80 f   usc:regalloc.obj
 0001:00079fbc       DeleteRegInterval          1007afbc f   usc:regalloc.obj
 0001:00079fe8       FreeRegIntervalList        1007afe8 f   usc:regalloc.obj
 0001:0007a064       EarlierThan                1007b064 f   usc:regalloc.obj
 0001:0007a074       IntervalLive               1007b074 f   usc:regalloc.obj
 0001:0007a0bc       IntervalLength             1007b0bc f   usc:regalloc.obj
 0001:0007a0c4       ProcListFindPos            1007b0c4 f   usc:regalloc.obj
 0001:0007a188       RegIntvlFindWith           1007b188 f   usc:regalloc.obj
 0001:0007a2c8       ProcListFindStart          1007b2c8 f   usc:regalloc.obj
 0001:0007a2f0       ProcListCons               1007b2f0 f   usc:regalloc.obj
 0001:0007a300       RegIntvlDrop               1007b300 f   usc:regalloc.obj
 0001:0007a338       ProcListAdd                1007b338 f   usc:regalloc.obj
 0001:0007a3c0       ProcListRemove             1007b3c0 f   usc:regalloc.obj
 0001:0007fcc8       AssignRegisters            10080cc8 f   usc:regalloc.obj
 0001:0007fda4       MergeIntervals             10080da4 f   usc:regalloc.obj
 0001:000811a8       CalcInstSrcChans           100821a8 f   usc:iregalloc.obj
 0001:000875b0       AssignRegistersC10         100885b0 f   usc:iregalloc.obj
 0001:000884f4       AssignPredicateRegisters   100894f4 f   usc:pregalloc.obj
 0001:000899a4       SetupSyncStartInformation  1008a9a4 f   usc:pregalloc.obj
 0001:0008b578       SetupEfoUsage              1008c578 f   usc:efo.obj
 0001:00093c18       GenerateEfoInstructionsBP  10094c18 f   usc:efo.obj
 0001:00097144       EliminateF16MovesBP        10098144 f   usc:f16opt.obj
 0001:000978e8       CombineFMad16Swizzle       100988e8 f   usc:f16opt.obj
 0001:000978f8       SubstituteFMad16Swizzle    100988f8 f   usc:f16opt.obj
 0001:00098210       AssignIndexRegistersBP     10099210 f   usc:indexreg.obj
 0001:00099568       ValueNumbering             1009a568 f   usc:ssa.obj
 0001:00099b00       LoadConstantNoHWReg        1009ab00 f   usc:icvt_core.obj
 0001:00099cf0       LoadConstant               1009acf0 f   usc:icvt_core.obj
 0001:00099e14       NewVecArrayData            1009ae14 f   usc:icvt_core.obj
 0001:00099e64       LoadStoreIndexableTemp     1009ae64 f   usc:icvt_core.obj
 0001:0009a18c       AddNewInternalIntermediateArray 1009b18c f   usc:icvt_core.obj
 0001:0009a23c       LoadIndexableTempFromIntermediateArray 1009b23c f   usc:icvt_core.obj
 0001:0009a3a0       StoreIndexableTemp         1009b3a0 f   usc:icvt_core.obj
 0001:0009a760       ReduceAngleBetweenNegPieToPie 1009b760 f   usc:icvt_core.obj
 0001:0009b244       LabelToInst                1009c244 f   usc:icvt_core.obj
 0001:0009b278       IsInputInstFlowControl     1009c278 f   usc:icvt_core.obj
 0001:0009c20c       GetPredicateInst           1009d20c f   usc:icvt_core.obj
 0001:0009c270       GetRegisterFormat          1009d270 f   usc:icvt_core.obj
 0001:0009c42c       ConvertSamplerInstructionCore 1009d42c f   usc:icvt_core.obj
 0001:0009cefc       ConvertSincosCore          1009defc f   usc:icvt_core.obj
 0001:0009d3ec       ConvertSincos2Core         1009e3ec f   usc:icvt_core.obj
 0001:0009ef44       ConvertVertexInputInstructionCore 1009ff44 f   usc:icvt_core.obj
 0001:000a03d0       ConvertToIntermediate      100a13d0 f   usc:icvt_core.obj
 0001:000a1204       NewDGraphState             100a2204 f   usc:dgraph.obj
 0001:000a13fc       FreeDGraphState            100a23fc f   usc:dgraph.obj
 0001:000a159c       AddNewInstToDGraph         100a259c f   usc:dgraph.obj
 0001:000a1664       GetNextAvailable           100a2664 f   usc:dgraph.obj
 0001:000a1730       AddDependency              100a2730 f   usc:dgraph.obj
 0001:000a1ae0       RemoveDependency           100a2ae0 f   usc:dgraph.obj
 0001:000a1ba4       SplitInstructions          100a2ba4 f   usc:dgraph.obj
 0001:000a1f50       MergeInstructions          100a2f50 f   usc:dgraph.obj
 0001:000a22cc       RemoveInstruction          100a32cc f   usc:dgraph.obj
 0001:000a2478       ComputeClosedDependencyGraph 100a3478 f   usc:dgraph.obj
 0001:000a2688       UpdateClosedDependencyGraph 100a3688 f   usc:dgraph.obj
 0001:000a2a44       ComputeDependencyGraph     100a3a44 f   usc:dgraph.obj
 0001:000a2f68       AddClosedDependency        100a3f68 f   usc:dgraph.obj
 0001:000a2fd4       TypeUsesFormatControl      100a3fd4 f   usc:groupinst.obj
 0001:000a3b50       MoeArgToInstArg            100a4b50 f   usc:groupinst.obj
 0001:000a3e7c       IsValidSwapInst            100a4e7c f   usc:groupinst.obj
 0001:000a7d64       GroupInstructionsProgram   100a8d64 f   usc:groupinst.obj
 0001:000a7f98       IsIllegalInstructionPair   100a8f98 f   usc:layout.obj
 0001:000a8018       IsSyncEndDest              100a9018 f   usc:layout.obj
 0001:000a8100       NoSchedLabelCB             100a9100 f   usc:layout.obj
 0001:000a811c       CommonBranchCB             100a911c f   usc:layout.obj
 0001:000a8704       LayoutProgram              100a9704 f   usc:layout.obj
 0001:000a89b8       CanSetEndFlag              100a99b8 f   usc:layout.obj
 0001:000a8a74       PointActionsHwCB           100a9a74 f   usc:layout.obj
 0001:000aa554       EncodeInst                 100ab554 f   usc:asm.obj
 0001:000aa5a8       EncodeJump                 100ab5a8 f   usc:asm.obj
 0001:000aa6cc       PackPSOutputNum            100ab6cc f   usc:icvt_f32.obj
 0001:000aa774       GenerateDestModF32         100ab774 f   usc:icvt_f32.obj
 0001:000aa988       LoadIteratedValue          100ab988 f   usc:icvt_f32.obj
 0001:000aac18       ApplySourceModF32          100abc18 f   usc:icvt_f32.obj
 0001:000aae3c       DestChanOverlapsSrc        100abe3c f   usc:icvt_f32.obj
 0001:000abbb4       ConvertAddressValue        100acbb4 f   usc:icvt_f32.obj
 0001:000ac1ac       GetDestinationF32          100ad1ac f   usc:icvt_f32.obj
 0001:000ac2f8       GetSourceF32               100ad2f8 f   usc:icvt_f32.obj
 0001:000acd48       ConvertBitwiseInstructionF32 100add48 f   usc:icvt_f32.obj
 0001:000adb3c       CreateComparisonFloat      100aeb3c f   usc:icvt_f32.obj
 0001:000adc18       ConvertSetpInstructionNonC10 100aec18 f   usc:icvt_f32.obj
 0001:000ae930       GetGradientsF32            100af930 f   usc:icvt_f32.obj
 0001:000aea0c       GetLODAdjustmentF32        100afa0c f   usc:icvt_f32.obj
 0001:000aeab4       GetSampleCoordinatesF32    100afab4 f   usc:icvt_f32.obj
 0001:000b0a18       ConvertTexkillInstructionFloat 100b1a18 f   usc:icvt_f32.obj
 0001:000b18ac       ConvertMovaInstructionFloat 100b28ac f   usc:icvt_f32.obj
 0001:000b1afc       ConvertInstToIntermediateF32 100b2afc f   usc:icvt_f32.obj
 0001:000b2a00       GetSingleSourceF16         100b3a00 f   usc:icvt_f16.obj
 0001:000b2a2c       GetSingleSourceConvertToF32 100b3a2c f   usc:icvt_f16.obj
 0001:000b3cd8       GetGradientsF16            100b4cd8 f   usc:icvt_f16.obj
 0001:000b3e2c       GetLODAdjustmentF16        100b4e2c f   usc:icvt_f16.obj
 0001:000b4e84       EmitNormaliseF16           100b5e84 f   usc:icvt_f16.obj
 0001:000b5004       ConvertNormaliseF16        100b6004 f   usc:icvt_f16.obj
 0001:000b5ed4       GetSampleCoordinatesF16    100b6ed4 f   usc:icvt_f16.obj
 0001:000b667c       ConvertInstToIntermediateF16 100b767c f   usc:icvt_f16.obj
 0001:000b841c       CanOverrideSwiz            100b941c f   usc:icvt_c10.obj
 0001:000b8b20       GetSourceC10               100b9b20 f   usc:icvt_c10.obj
 0001:000b941c       CheckDuplicateChannel      100ba41c f   usc:icvt_c10.obj
 0001:000bd6d8       CreateComparisonC10        100be6d8 f   usc:icvt_c10.obj
 0001:000be174       GetGradientsC10            100bf174 f   usc:icvt_c10.obj
 0001:000be290       GetLODAdjustmentC10        100bf290 f   usc:icvt_c10.obj
 0001:000be384       GetSampleCoordinatesC10    100bf384 f   usc:icvt_c10.obj
 0001:000bed04       ConvertInstToIntermediateC10 100bfd04 f   usc:icvt_c10.obj
 0001:000bef98       LoadImmediate              100bff98 f   usc:icvt_i32.obj
 0001:000bfb4c       ConvertF32ConversionInstructionInt32 100c0b4c f   usc:icvt_i32.obj
 0001:000c04a8       IntegerNegate              100c14a8 f   usc:icvt_i32.obj
 0001:000c1e2c       GenerateIntegerArithmetic  100c2e2c f   usc:icvt_i32.obj
 0001:000c1fd0       CreateComparisonInt32      100c2fd0 f   usc:icvt_i32.obj
 0001:000c2ca0       ConvertInstToIntermediateInt32 100c3ca0 f   usc:icvt_i32.obj
 0001:000c31e0       SwizzleMask                100c41e0 f   usc:precovr.obj
 0001:000c469c       SkipInstBlock              100c569c f   usc:precovr.obj
 0001:000c4774       ConvertOperationsToInteger 100c5774 f   usc:precovr.obj
 0001:000c4f9c       OverrideFloat16Precisions  100c5f9c f   usc:precovr.obj
 0001:000c5518       GetFeatureEntry            100c6518 f   useasm:utils.obj
 0001:000c5580       GetBugEntry                100c6580 f   useasm:utils.obj
 0001:000c55e8       FixBRN21697                100c65e8 f   useasm:utils.obj
 0001:000c5604       FixBRN21713                100c6604 f   useasm:utils.obj
 0001:000c5620       FixBRN23062                100c6620 f   useasm:utils.obj
 0001:000c563c       FixBRN23164                100c663c f   useasm:utils.obj
 0001:000c5658       FixBRN23461                100c6658 f   useasm:utils.obj
 0001:000c5674       FixBRN23960                100c6674 f   useasm:utils.obj
 0001:000c5690       FixBRN24895                100c6690 f   useasm:utils.obj
 0001:000c56ac       FixBRN25355                100c66ac f   useasm:utils.obj
 0001:000c56c8       FixBRN25060                100c66c8 f   useasm:utils.obj
 0001:000c56e4       FixBRN25580                100c66e4 f   useasm:utils.obj
 0001:000c5700       FixBRN25582                100c6700 f   useasm:utils.obj
 0001:000c571c       FixBRN26570                100c671c f   useasm:utils.obj
 0001:000c5738       FixBRN26681                100c6738 f   useasm:utils.obj
 0001:000c5754       IsEnhancedNoSched          100c6754 f   useasm:utils.obj
 0001:000c5770       IsHighPrecisionFIR         100c6770 f   useasm:utils.obj
 0001:000c578c       IsLoadMOEStateFromRegisters 100c678c f   useasm:utils.obj
 0001:000c57a8       IsPerInstMoeIncrements     100c67a8 f   useasm:utils.obj
 0001:000c57c4       HasNewEfoOptions           100c67c4 f   useasm:utils.obj
 0001:000c57e0       HasPackMultipleRoundModes  100c67e0 f   useasm:utils.obj
 0001:000c57fc       HasNoInstructionPairing    100c67fc f   useasm:utils.obj
 0001:000c5818       NumberOfMutexesSupported   100c6818 f   useasm:utils.obj
 0001:000c5828       NumberOfMonitorsSupported  100c6828 f   useasm:utils.obj
 0001:000c5838       NumberOfProgramCounterBits 100c6838 f   useasm:utils.obj
 0001:000c5848       SupportsFmad16Swizzles     100c6848 f   useasm:utils.obj
 0001:000c5864       SupportsFnormalise         100c6864 f   useasm:utils.obj
 0001:000c5880       SupportsIndexTwoBanks      100c6880 f   useasm:utils.obj
 0001:000c589c       OpcodeArgumentCount        100c689c f   useasm:usetab.obj
 0001:000c58b4       OpcodeName                 100c68b4 f   useasm:usetab.obj
 0001:000c66dc       FloatToCstIndex            100c76dc f   useasm:useasm.obj
 0001:000d6014       UseAssembleInstruction     100d7014 f   useasm:useasm.obj
 0001:000d6bbc       PVRSRVAllocUserModeMem     100d7bbc f   srvclum:SRVCLUM.dll
 0001:000d6bcc       PVRSRVReallocUserModeMem   100d7bcc f   srvclum:SRVCLUM.dll
 0001:000d6bdc       PVRSRVFreeUserModeMem      100d7bdc f   srvclum:SRVCLUM.dll
 0001:000d6bec       PVRSRVCallocUserModeMem    100d7bec f   srvclum:SRVCLUM.dll
 0001:000d6bfc       PVRSRVSetLocale            100d7bfc f   srvclum:SRVCLUM.dll
 0001:000d6c0c       DllMain                    100d7c0c f   corelib0:dllmain.obj
 0001:000d6d28       _DllMainCRTStartup         100d7d28 f   corelib0:pegdmain.obj
 0001:000d6d58       __GSHandlerCheckCommon     100d7d58 f   corelib0:gshandler.obj
 0001:000d6d94       __GSHandlerCheck           100d7d94 f   corelib0:gshandler.obj
 0001:000d6db8       __security_init_cookie     100d7db8 f   corelib0:seccinit.obj
 0001:000d6e14       __security_check_cookie    100d7e14 f   corelib0:armsecgs.obj
 0001:000d6e28       __gsfailure                100d7e28 f   corelib0:armsecgs.obj
 0001:000d6f34       _cexit                     100d7f34 f   corelib0:cexit.obj
 0001:000d6f50       _initterm                  100d7f50 f   corelib0:crt0dat.obj
 0001:000d6f84       _cinit                     100d7f84 f   corelib0:crt0dat.obj
 0001:000d6fb8       memcpy                     100d7fb8 f   corelib1:COREDLL.dll
 0001:000d6fc8       memset                     100d7fc8 f   corelib1:COREDLL.dll
 0001:000d6fd8       fflush                     100d7fd8 f   corelib1:COREDLL.dll
 0001:000d6fe8       strcpy                     100d7fe8 f   corelib1:COREDLL.dll
 0001:000d6ff8       strlen                     100d7ff8 f   corelib1:COREDLL.dll
 0001:000d7008       sprintf                    100d8008 f   corelib1:COREDLL.dll
 0001:000d7018       strncpy                    100d8018 f   corelib1:COREDLL.dll
 0001:000d7028       strcmp                     100d8028 f   corelib1:COREDLL.dll
 0001:000d7038       _vsnprintf                 100d8038 f   corelib1:COREDLL.dll
 0001:000d7048       vsprintf                   100d8048 f   corelib1:COREDLL.dll
 0001:000d7058       strcat                     100d8058 f   corelib1:COREDLL.dll
 0001:000d7068       printf                     100d8068 f   corelib1:COREDLL.dll
 0001:000d7078       strncmp                    100d8078 f   corelib1:COREDLL.dll
 0001:000d7088       strtol                     100d8088 f   corelib1:COREDLL.dll
 0001:000d7098       strstr                     100d8098 f   corelib1:COREDLL.dll
 0001:000d70a8       strtod                     100d80a8 f   corelib1:COREDLL.dll
 0001:000d70b8       longjmp                    100d80b8 f   corelib1:COREDLL.dll
 0001:000d70c8       setjmp                     100d80c8 f   corelib1:COREDLL.dll
 0001:000d70d8       memmove                    100d80d8 f   corelib1:COREDLL.dll
 0001:000d70e8       memcmp                     100d80e8 f   corelib1:COREDLL.dll
 0001:000d70f8       _XcptFilter                100d80f8 f   corelib1:COREDLL.dll
 0001:000d7108       __C_specific_handler       100d8108 f   corelib1:COREDLL.dll
 0001:000d7118       __security_gen_cookie2     100d8118 f   corelib1:COREDLL.dll
 0001:000d7128       __report_gsfailure         100d8128 f   corelib1:COREDLL.dll
 0001:000d7138       free                       100d8138 f   corelib1:COREDLL.dll
 0001:000d7148       DebugCreateHeapfn          100d8148 f   glsl_parser:memmgr.obj
 0001:000d71cc       DebugAllocHeapItemfn       100d81cc f   glsl_parser:memmgr.obj
 0001:000d7210       DebugFreeHeapItemfn        100d8210 f   glsl_parser:memmgr.obj
 0001:000d7220       DebugDestroyHeapfn         100d8220 f   glsl_parser:memmgr.obj
 0001:000d7278       CreateLanguageContext      100d8278 f   glsl_parser:parser.obj
 0001:000d72ec       DestroyLanguageContext     100d82ec f   glsl_parser:parser.obj
 0001:000d77d8       DestroyParseTree           100d87d8 f   glsl_parser:parser.obj
 0001:000d7884       DestroyParseContext        100d8884 f   glsl_parser:parser.obj
 0001:000d7db4       CreateParseContext         100d8db4 f   glsl_parser:parser.obj
 0001:000d7f74       ParseTreeValidateBranchFn  100d8f74 f   glsl_parser:parsetools.obj
 0001:000d7f9c       GetRuleSize                100d8f9c f   glsl_parser:syntax.obj
 0001:000d7fa8       StopBackTrackingEnabled    100d8fa8 f   glsl_parser:syntax.obj
 0001:000d81d4       CreateSyntaxTable          100d91d4 f   glsl_parser:syntax.obj
 0001:000d878c       DestroySyntaxTable         100d978c f   glsl_parser:syntax.obj
 0001:000d87b8       GetSyntaxSymbolLRSymbolName 100d97b8 f   glsl_parser:syntax.obj
 0001:000d87c8       LexDestroyTokenList        100d97c8 f   glsl_parser:lex.obj
 0001:000d9404       LexCreateTokenList         100da404 f   glsl_parser:lex.obj
 0001:000d9570       DisableThreadLibraryCalls  100da570 f   coredll:COREDLL.dll
 0001:000d9580       TerminateProcess           100da580 f   coredll:COREDLL.dll
 0001:000d9628       __IMPORT_DESCRIPTOR_SRVCLUM 100da628     srvclum:SRVCLUM.dll
 0001:000d963c       __IMPORT_DESCRIPTOR_COREDLL 100da63c     corelib1:COREDLL.dll
 0001:000d9650       __NULL_IMPORT_DESCRIPTOR   100da650     srvclum:SRVCLUM.dll
 0002:00000000       __imp___ges                100db000     corelib1:COREDLL.dll
 0002:00000004       __imp_DisableThreadLibraryCalls 100db004     coredll:COREDLL.dll
 0002:00000008       __imp_memcpy               100db008     corelib1:COREDLL.dll
 0002:0000000c       __imp___rt_udiv            100db00c     corelib1:COREDLL.dll
 0002:00000010       __imp_memset               100db010     corelib1:COREDLL.dll
 0002:00000014       __imp_fflush               100db014     corelib1:COREDLL.dll
 0002:00000018       __imp_strcpy               100db018     corelib1:COREDLL.dll
 0002:0000001c       __imp_strlen               100db01c     corelib1:COREDLL.dll
 0002:00000020       __imp___itos               100db020     corelib1:COREDLL.dll
 0002:00000024       __imp_sprintf              100db024     corelib1:COREDLL.dll
 0002:00000028       __imp_strncpy              100db028     corelib1:COREDLL.dll
 0002:0000002c       __imp_strcmp               100db02c     corelib1:COREDLL.dll
 0002:00000030       __imp___stod               100db030     corelib1:COREDLL.dll
 0002:00000034       __imp__vsnprintf           100db034     corelib1:COREDLL.dll
 0002:00000038       __imp_vsprintf             100db038     corelib1:COREDLL.dll
 0002:0000003c       __imp_strcat               100db03c     corelib1:COREDLL.dll
 0002:00000040       __imp___rt_sdiv            100db040     corelib1:COREDLL.dll
 0002:00000044       __imp_printf               100db044     corelib1:COREDLL.dll
 0002:00000048       __imp_strncmp              100db048     corelib1:COREDLL.dll
 0002:0000004c       __imp_strtol               100db04c     corelib1:COREDLL.dll
 0002:00000050       __imp_strstr               100db050     corelib1:COREDLL.dll
 0002:00000054       __imp_strtod               100db054     corelib1:COREDLL.dll
 0002:00000058       __imp___dtos               100db058     corelib1:COREDLL.dll
 0002:0000005c       __imp___adds               100db05c     corelib1:COREDLL.dll
 0002:00000060       __imp_tan                  100db060     corelib1:COREDLL.dll
 0002:00000064       __imp___nes                100db064     corelib1:COREDLL.dll
 0002:00000068       __imp___stoi               100db068     corelib1:COREDLL.dll
 0002:0000006c       __imp___muls               100db06c     corelib1:COREDLL.dll
 0002:00000070       __imp___negs               100db070     corelib1:COREDLL.dll
 0002:00000074       __imp___divs               100db074     corelib1:COREDLL.dll
 0002:00000078       __imp___subs               100db078     corelib1:COREDLL.dll
 0002:0000007c       __imp_TerminateProcess     100db07c     coredll:COREDLL.dll
 0002:00000080       __imp___les                100db080     corelib1:COREDLL.dll
 0002:00000084       __imp___gts                100db084     corelib1:COREDLL.dll
 0002:00000088       __imp___lts                100db088     corelib1:COREDLL.dll
 0002:0000008c       __imp_sin                  100db08c     corelib1:COREDLL.dll
 0002:00000090       __imp_cos                  100db090     corelib1:COREDLL.dll
 0002:00000094       __imp_asin                 100db094     corelib1:COREDLL.dll
 0002:00000098       __imp_acos                 100db098     corelib1:COREDLL.dll
 0002:0000009c       __imp_atan2                100db09c     corelib1:COREDLL.dll
 0002:000000a0       __imp_atan                 100db0a0     corelib1:COREDLL.dll
 0002:000000a4       __imp_exp                  100db0a4     corelib1:COREDLL.dll
 0002:000000a8       __imp_pow                  100db0a8     corelib1:COREDLL.dll
 0002:000000ac       __imp_log                  100db0ac     corelib1:COREDLL.dll
 0002:000000b0       __imp___divd               100db0b0     corelib1:COREDLL.dll
 0002:000000b4       __imp_fabs                 100db0b4     corelib1:COREDLL.dll
 0002:000000b8       __imp_ceil                 100db0b8     corelib1:COREDLL.dll
 0002:000000bc       __imp_floor                100db0bc     corelib1:COREDLL.dll
 0002:000000c0       __imp_sqrt                 100db0c0     corelib1:COREDLL.dll
 0002:000000c4       __imp___eqs                100db0c4     corelib1:COREDLL.dll
 0002:000000c8       __imp_longjmp              100db0c8     corelib1:COREDLL.dll
 0002:000000cc       __imp_setjmp               100db0cc     corelib1:COREDLL.dll
 0002:000000d0       __imp_memmove              100db0d0     corelib1:COREDLL.dll
 0002:000000d4       __imp_memcmp               100db0d4     corelib1:COREDLL.dll
 0002:000000d8       __imp___utos               100db0d8     corelib1:COREDLL.dll
 0002:000000dc       __imp__XcptFilter          100db0dc     corelib1:COREDLL.dll
 0002:000000e0       __imp___C_specific_handler 100db0e0     corelib1:COREDLL.dll
 0002:000000e4       __imp___security_gen_cookie2 100db0e4     corelib1:COREDLL.dll
 0002:000000e8       __imp___report_gsfailure   100db0e8     corelib1:COREDLL.dll
 0002:000000ec       __imp_free                 100db0ec     corelib1:COREDLL.dll
 0002:000000f0       \177COREDLL_NULL_THUNK_DATA 100db0f0     corelib1:COREDLL.dll
 0002:000000f4       __imp_PVRSRVSetLocale      100db0f4     srvclum:SRVCLUM.dll
 0002:000000f8       __imp_PVRSRVCallocUserModeMem 100db0f8     srvclum:SRVCLUM.dll
 0002:000000fc       __imp_PVRSRVFreeUserModeMem 100db0fc     srvclum:SRVCLUM.dll
 0002:00000100       __imp_PVRSRVReallocUserModeMem 100db100     srvclum:SRVCLUM.dll
 0002:00000104       __imp_PVRSRVAllocUserModeMem 100db104     srvclum:SRVCLUM.dll
 0002:00000108       \177SRVCLUM_NULL_THUNK_DATA 100db108     srvclum:SRVCLUM.dll
 0002:0000010c       __security_cookie          100db10c     corelib0:seccinit.obj
 0002:00000110       __security_cookie_complement 100db110     corelib0:seccinit.obj
 0002:00000114       _exitflag                  100db114     corelib0:cexit.obj
 0002:00000118       __onexitend                100db118     <common>
 0002:0000011c       __onexitbegin              100db11c     <common>
 0002:00000120       _pRawDllMain               100db120     <common>

 entry point at        0001:000d6d28

 Static symbols

 0001:000140c0       IC2UF_GetDestMask          100150c0 f   ic2uf.obj
 0001:000141d0       ConvertToUFDestination     100151d0 f   ic2uf.obj
 0001:00014230       ConvertToUFSource          10015230 f   ic2uf.obj
 0001:00014314       ConvertToUFPredicate       10015314 f   ic2uf.obj
 0001:00014350       AddHWSymbolToList          10015350 f   ic2uf.obj
 0001:0001441c       CreateInstruction          1001541c f   ic2uf.obj
 0001:00014494       UFRegATableAssignRegisters 10015494 f   ic2uf.obj
 0001:0001459c       GetTemporary               1001559c f   ic2uf.obj
 0001:00014610       GetIntConst                10015610 f   ic2uf.obj
 0001:0001468c       AddMOVAToUFCode            1001568c f   ic2uf.obj
 0001:00014704       BuildStructBaseMembers     10015704 f   ic2uf.obj
 0001:00014878       BuildStructAllocInfo       10015878 f   ic2uf.obj
 0001:00014b64       AssignSamplerTexUnit       10015b64 f   ic2uf.obj
 0001:00014c58       ConvertPrecisionToUFRegFormat 10015c58 f   ic2uf.obj
 0001:00014cf4       UpdateOperandUFSwiz        10015cf4 f   ic2uf.obj
 0001:00014e70       ApplyMoreSwiz              10015e70 f   ic2uf.obj
 0001:00014ed8       ChooseMatrixColumn         10015ed8 f   ic2uf.obj
 0001:00014fcc       ChooseMatrixComponent      10015fcc f   ic2uf.obj
 0001:0001513c       ChooseVectorComponent      1001613c f   ic2uf.obj
 0001:000151c4       ChooseStructMember         100161c4 f   ic2uf.obj
 0001:00015254       AddAluToUFCode             10016254 f   ic2uf.obj
 0001:000152f4       AddIFCToUFCode             100162f4 f   ic2uf.obj
 0001:0001537c       AddUpRelativeOffsetToUFCode 1001637c f   ic2uf.obj
 0001:000154dc       ProcessOperandOffsets      100164dc f   ic2uf.obj
 0001:000158e8       GetHWSymbolEntry           100168e8 f   ic2uf.obj
 0001:00015bc4       AddSimpleALUToUFCode       10016bc4 f   ic2uf.obj
 0001:00015d30       AddComparisonToUFCode      10016d30 f   ic2uf.obj
 0001:00015f3c       AddIFComparisonToUFCode    10016f3c f   ic2uf.obj
 0001:00015fd8       AddVectorSALLToUFCode      10016fd8 f   ic2uf.obj
 0001:0001614c       AddNOTToUFCode             1001714c f   ic2uf.obj
 0001:000161e0       ProcessICInstIFNOT         100171e0 f   ic2uf.obj
 0001:00016268       ProcessICInstLOOP          10017268 f   ic2uf.obj
 0001:000162c8       AddDirectTextureLookupToUFCode 100172c8 f   ic2uf.obj
 0001:0001641c       UpdateInterferenceGraph    1001741c f   ic2uf.obj
 0001:000164b0       GetChannelsLiveInSource    100174b0 f   ic2uf.obj
 0001:00016720       GetFunctionNestingLevel    10017720 f   ic2uf.obj
 0001:000167f0       GenerateInterferenceGraph  100177f0 f   ic2uf.obj
 0001:00016c68       AssignTempRegisters        10017c68 f   ic2uf.obj
 0001:00017088       GenerateFrontFacingData    10018088 f   ic2uf.obj
 0001:000171a4       AddDataConversionMOV       100181a4 f   ic2uf.obj
 0001:0001752c       ProcessICInstMUL           1001852c f   ic2uf.obj
 0001:000179f8       ProcessICInstDIV           100189f8 f   ic2uf.obj
 0001:00017acc       ProcessICInstLABEL         10018acc f   ic2uf.obj
 0001:00017b8c       ProcessICInstCALL          10018b8c f   ic2uf.obj
 0001:00017c54       ProcessICInstSANY          10018c54 f   ic2uf.obj
 0001:00017d4c       ProcessICInstSGN           10018d4c f   ic2uf.obj
 0001:00017eb0       ProcessICInstDOT           10018eb0 f   ic2uf.obj
 0001:00017f90       ProcessICInstCROSS         10018f90 f   ic2uf.obj
 0001:000180a0       ProcessICInstNRM3          100190a0 f   ic2uf.obj
 0001:000181ac       ProcessICInstMOD           100191ac f   ic2uf.obj
 0001:00018340       ProcessVPInstTEXLDP        10019340 f   ic2uf.obj
 0001:000184b4       ProcessFPInstTEXLDP        100194b4 f   ic2uf.obj
 0001:000185bc       ProcessICInstTEXLDD        100195bc f   ic2uf.obj
 0001:000186f8       CreateUniFlexContext       100196f8 f   ic2uf.obj
 0001:00018a74       PrepareUFCodeOutput        10019a74 f   ic2uf.obj
 0001:00018b70       ReassignVSOutputRegisters  10019b70 f   ic2uf.obj
 0001:00018cc4       DoesTypeContainBigArrays   10019cc4 f   ic2uf.obj
 0001:00018dc8       FindEmptyRectSpace         10019dc8 f   ic2uf.obj
 0001:000192ec       AllocateAllVaryings        1001a2ec f   ic2uf.obj
 0001:00019894       GetTypeAllocInfo           1001a894 f   ic2uf.obj
 0001:00019a60       AssignHWSymbolRegisters    1001aa60 f   ic2uf.obj
 0001:00019bd8       AllocateHWSymbolRegisters  1001abd8 f   ic2uf.obj
 0001:00019eb4       ProcessICOperand           1001aeb4 f   ic2uf.obj
 0001:00019fac       AllocateAllUFRegisters     1001afac f   ic2uf.obj
 0001:0001a31c       InitICUFOperand            1001b31c f   ic2uf.obj
 0001:0001a368       IC2UF_GetPredicate         1001b368 f   ic2uf.obj
 0001:0001a3cc       GetFixedConst              1001b3cc f   ic2uf.obj
 0001:0001a438       AddArrayComparison         1001b438 f   ic2uf.obj
 0001:0001a80c       AddPredicatedWholeTypeComparision 1001b80c f   ic2uf.obj
 0001:0001ace4       GenerateColorOutput        1001bce4 f   ic2uf.obj
 0001:0001aeb0       GenerateZOutput            1001beb0 f   ic2uf.obj
 0001:0001af7c       GenerateFaceSelection      1001bf7c f   ic2uf.obj
 0001:0001b0c8       GenerateFragCoordAdjust    1001c0c8 f   ic2uf.obj
 0001:0001b340       AddArrayMOV                1001c340 f   ic2uf.obj
 0001:0001b6b8       ProcessICInstMOV           1001c6b8 f   ic2uf.obj
 0001:0001bc8c       AddWholeTypeComparision    1001cc8c f   ic2uf.obj
 0001:0001be98       ProcessICInstEXP           1001ce98 f   ic2uf.obj
 0001:0001bf58       ProcessICInstLOG           1001cf58 f   ic2uf.obj
 0001:0001c014       ProcessICInstSINCOS        1001d014 f   ic2uf.obj
 0001:0001c25c       ProcessICInstTAN           1001d25c f   ic2uf.obj
 0001:0001c508       GenerateUniFlexInstructions 1001d508 f   ic2uf.obj
 0001:0001d27c       PostGenerateUniFlexCode    1001e27c f   ic2uf.obj
 0001:0001d634       GLSLGenerateUniflexProgram 1001e634 f   glsl2uf.obj
 0001:0001d974       CopyConstantData           1001e974 f   bindingsym.obj
 0001:0001da64       ProcessBindingSymbolEntry  1001ea64 f   bindingsym.obj
 0001:0001dc50       AddBindingSymbol           1001ec50 f   bindingsym.obj
 0001:0001dd40       RecursivelyAddStructMembers 1001ed40 f   bindingsym.obj
 0001:0001e044       ProcessHWSymbolEntry       1001f044 f   bindingsym.obj
 0001:0001e49c       AttachSymbolTableToContext 1001f49c f   glsl_parser:symtab.obj
 0001:0001e738       FindSymbolInTable          1001f738 f   glsl_parser:symtab.obj
 0001:0001e840       GetSymbolTableEntry        1001f840 f   glsl_parser:symtab.obj
 0001:0001e8c4       AddSymbolToTable           1001f8c4 f   glsl_parser:symtab.obj
 0001:0001f050       ICSetupICOperand           10020050 f   glsl_core:icgen.obj
 0001:0001f1b0       UnhookInstructions         100201b0 f   glsl_core:icgen.obj
 0001:0001f224       InsertInstructionsAfter    10020224 f   glsl_core:icgen.obj
 0001:0001f298       FreeICInstruction          10020298 f   glsl_core:icgen.obj
 0001:0001f384       ICGetNewInstruction        10020384 f   glsl_core:icgen.obj
 0001:0001f4fc       ICGetSymbolFullType        100204fc f   glsl_core:icgen.obj
 0001:0001f844       IsSymbolBoolConstant       10020844 f   glsl_core:icgen.obj
 0001:0001f8e0       ValidateICInstruction      100208e0 f   glsl_core:icgen.obj
 0001:00020548       IsSimpleConditionCheck     10021548 f   glsl_core:icgen.obj
 0001:0002061c       ICAddICInstruction3aWithPred 1002161c f   glsl_core:icgen.obj
 0001:00020764       GenerateCodeForPredicateXOR 10021764 f   glsl_core:icgen.obj
 0001:00020950       ReplaceInlinedInstOperand  10021950 f   glsl_core:icgen.obj
 0001:00020b74       ProcessNodeFUNCTIONDEFINITION 10021b74 f   glsl_core:icgen.obj
 0001:00020c88       GetTypeNumElements         10021c88 f   glsl_core:icgen.obj
 0001:00020d5c       IsFunctionToBeInlined      10021d5c f   glsl_core:icgen.obj
 0001:00020f14       ProcessNodeSHADER          10021f14 f   glsl_core:icgen.obj
 0001:0002122c       EvaluateNodeARRAYSPECIFIER 1002222c f   glsl_core:icgen.obj
 0001:00021360       EvaluateNodeFIELDSELECTION 10022360 f   glsl_core:icgen.obj
 0001:0002148c       PostEvaluateFunctionCall   1002248c f   glsl_core:icgen.obj
 0001:00021578       PostEvaluateNode           10022578 f   glsl_core:icgen.obj
 0001:000216dc       IsNodeDirectOperand        100226dc f   glsl_core:icgen.obj
 0001:00021884       ProcessNodeBasicOp         10022884 f   glsl_core:icgen.obj
 0001:000219b0       ProcessNodePreIncDec       100229b0 f   glsl_core:icgen.obj
 0001:00021aec       InsertPostfixCode          10022aec f   glsl_core:icgen.obj
 0001:00021c80       ProcessNodeComparisonOp    10022c80 f   glsl_core:icgen.obj
 0001:00021dac       GenerateOptimisedConditionCode 10022dac f   glsl_core:icgen.obj
 0001:00021ed8       GenerateSetPredicateCode   10022ed8 f   glsl_core:icgen.obj
 0001:000223d8       ICTraverseCondition        100233d8 f   glsl_core:icgen.obj
 0001:00022490       ProcessNodeQUESTION        10023490 f   glsl_core:icgen.obj
 0001:00022664       ProcessNodeLogicalOR       10023664 f   glsl_core:icgen.obj
 0001:000227ac       ProcessNodeLogicalXOR      100237ac f   glsl_core:icgen.obj
 0001:00022868       ProcessNodeLogicalAND      10023868 f   glsl_core:icgen.obj
 0001:000229b0       ProcessNodeNOT             100239b0 f   glsl_core:icgen.obj
 0001:00022ab0       ProcessConstructorForBasicType 10023ab0 f   glsl_core:icgen.obj
 0001:000231d0       ProcessArrayConstructor    100241d0 f   glsl_core:icgen.obj
 0001:000232d4       ICProcessSturctureConstructor 100242d4 f   glsl_core:icgen.obj
 0001:0002343c       ICProcessInlinedFunctionCall 1002443c f   glsl_core:icgen.obj
 0001:000238a0       ICProcessUserDefinedFunctionCall 100248a0 f   glsl_core:icgen.obj
 0001:00023bd4       ProcessNodeFUNCTIONCALL    10024bd4 f   glsl_core:icgen.obj
 0001:00023e04       ProcessNodeRETURN          10024e04 f   glsl_core:icgen.obj
 0001:00023ebc       ProcessNode                10024ebc f   glsl_core:icgen.obj
 0001:000241d8       ProcessNodeFOR             100251d8 f   glsl_core:icgen.obj
 0001:0002443c       ProcessNodeWHILE           1002543c f   glsl_core:icgen.obj
 0001:000245cc       ProcessNodeDO              100255cc f   glsl_core:icgen.obj
 0001:0002471c       ProcessNodeIF              1002571c f   glsl_core:icgen.obj
 0001:00024b44       FreeConstantData           10025b44 f   glsl_core:common.obj
 0001:00024b54       AddGenericData             10025b54 f   glsl_core:common.obj
 0001:00024c20       FreeIdentifierData         10025c20 f   glsl_core:common.obj
 0001:00024f48       FreeFunctionDefinitionData 10025f48 f   glsl_core:common.obj
 0001:00025144       FreeStructureDefinitionData 10026144 f   glsl_core:common.obj
 0001:00025198       AddStructureDefinitionData 10026198 f   glsl_core:common.obj
 0001:0002624c       LogErrorMessageBuffer      1002724c f   glsl_core:error.obj
 0001:0002639c       LogErrorMessage            1002739c f   glsl_core:error.obj
 0001:000263fc       FindNearestForwardToken    100273fc f   glsl_core:error.obj
 0001:00026438       FindNearestPreviousToken   10027438 f   glsl_core:error.obj
 0001:00026474       FindNearestToken           10027474 f   glsl_core:error.obj
 0001:000266f8       UniFlexAlloc               100276f8 f   glsl_core:glsl.obj
 0001:000266fc       UniFlexFree                100276fc f   glsl_core:glsl.obj
 0001:00026708       UniFlexPrint               10027708 f   glsl_core:glsl.obj
 0001:0002675c       GLSLAddBuiltInState        1002775c f   glsl_core:glsl.obj
 0001:00026eb0       ICProcessBIFNradians       10027eb0 f   glsl_core:icbuiltin.obj
 0001:00026f94       ICProcessBIFNdegrees       10027f94 f   glsl_core:icbuiltin.obj
 0001:00027078       ICProcessBIFNsin           10028078 f   glsl_core:icbuiltin.obj
 0001:000270f0       ICProcessBIFNcos           100280f0 f   glsl_core:icbuiltin.obj
 0001:00027168       ICProcessBIFNtan           10028168 f   glsl_core:icbuiltin.obj
 0001:00027208       ICProcessBIFNasin          10028208 f   glsl_core:icbuiltin.obj
 0001:000272b0       ICProcessBIFNacos          100282b0 f   glsl_core:icbuiltin.obj
 0001:00027358       ICProcessBIFNatan          10028358 f   glsl_core:icbuiltin.obj
 0001:00027424       ICProcessBIFNpow           10028424 f   glsl_core:icbuiltin.obj
 0001:000274e8       ICProcessBIFNexp           100284e8 f   glsl_core:icbuiltin.obj
 0001:00027560       ICProcessBIFNlog           10028560 f   glsl_core:icbuiltin.obj
 0001:000275d8       ICProcessBIFNexp2          100285d8 f   glsl_core:icbuiltin.obj
 0001:00027650       ICProcessBIFNlog2          10028650 f   glsl_core:icbuiltin.obj
 0001:000276c8       ICProcessBIFNsqrt          100286c8 f   glsl_core:icbuiltin.obj
 0001:000277d4       ICProcessBIFNinversesqrt   100287d4 f   glsl_core:icbuiltin.obj
 0001:0002784c       ICProcessBIFNabs           1002884c f   glsl_core:icbuiltin.obj
 0001:000278c4       ICProcessBIFNsign          100288c4 f   glsl_core:icbuiltin.obj
 0001:0002793c       ICProcessBIFNfloor         1002893c f   glsl_core:icbuiltin.obj
 0001:000279b4       ICProcessBIFNceil          100289b4 f   glsl_core:icbuiltin.obj
 0001:00027a2c       ICProcessBIFNfract         10028a2c f   glsl_core:icbuiltin.obj
 0001:00027acc       ICProcessBIFNmod           10028acc f   glsl_core:icbuiltin.obj
 0001:00027b90       ICProcessBIFNmin           10028b90 f   glsl_core:icbuiltin.obj
 0001:00027c2c       ICProcessBIFNmax           10028c2c f   glsl_core:icbuiltin.obj
 0001:00027cc8       ICProcessBIFNclamp         10028cc8 f   glsl_core:icbuiltin.obj
 0001:00027e28       ICProcessBIFNmix           10028e28 f   glsl_core:icbuiltin.obj
 0001:00027ed0       ICProcessBIFNstep          10028ed0 f   glsl_core:icbuiltin.obj
 0001:00027ff8       ICProcessBIFNsmoothstep    10028ff8 f   glsl_core:icbuiltin.obj
 0001:000283a0       ICProcessBIFNlength        100293a0 f   glsl_core:icbuiltin.obj
 0001:000284b8       ICProcessBIFNdistance      100294b8 f   glsl_core:icbuiltin.obj
 0001:0002866c       ICProcessBIFNdot           1002966c f   glsl_core:icbuiltin.obj
 0001:00028708       ICProcessBIFNcross         10029708 f   glsl_core:icbuiltin.obj
 0001:000287a4       ICProcessBIFNnormalize     100297a4 f   glsl_core:icbuiltin.obj
 0001:00028988       ICProcessBIFNftransform    10029988 f   glsl_core:icbuiltin.obj
 0001:00028a0c       ICProcessBIFNfaceforward   10029a0c f   glsl_core:icbuiltin.obj
 0001:00028c3c       ICProcessBIFNreflect       10029c3c f   glsl_core:icbuiltin.obj
 0001:00028e60       ICProcessBIFNrefract       10029e60 f   glsl_core:icbuiltin.obj
 0001:000292bc       ICProcessBIFNmatrixCompMult 1002a2bc f   glsl_core:icbuiltin.obj
 0001:000293f4       ICProcessBIFNtranspose     1002a3f4 f   glsl_core:icbuiltin.obj
 0001:00029554       ICProcessBIFNouterProduct  1002a554 f   glsl_core:icbuiltin.obj
 0001:000296fc       ICProcessBIFNlessThan      1002a6fc f   glsl_core:icbuiltin.obj
 0001:00029798       ICProcessBIFNlessThanEqual 1002a798 f   glsl_core:icbuiltin.obj
 0001:00029834       ICProcessBIFNgreaterThan   1002a834 f   glsl_core:icbuiltin.obj
 0001:000298d0       ICProcessBIFNgreaterThanEqual 1002a8d0 f   glsl_core:icbuiltin.obj
 0001:0002996c       ICProcessBIFNequal         1002a96c f   glsl_core:icbuiltin.obj
 0001:00029a08       ICProcessBIFNnotEqual      1002aa08 f   glsl_core:icbuiltin.obj
 0001:00029aa4       ICProcessBIFNany           1002aaa4 f   glsl_core:icbuiltin.obj
 0001:00029b1c       ICProcessBIFNall           1002ab1c f   glsl_core:icbuiltin.obj
 0001:00029b94       ICProcessBIFNnot           1002ab94 f   glsl_core:icbuiltin.obj
 0001:00029c0c       ICProcessBIFNtexture1D     1002ac0c f   glsl_core:icbuiltin.obj
 0001:00029d48       ICProcessBIFNtexture1DProj 1002ad48 f   glsl_core:icbuiltin.obj
 0001:00029e18       ICProcessBIFNtexture1DLod  1002ae18 f   glsl_core:icbuiltin.obj
 0001:00029ec0       ICProcessBIFNtexture1DProjLod 1002aec0 f   glsl_core:icbuiltin.obj
 0001:00029ee4       ICProcessBIFNtexture2D     1002aee4 f   glsl_core:icbuiltin.obj
 0001:0002a020       ICProcessBIFNtexture2DProj 1002b020 f   glsl_core:icbuiltin.obj
 0001:0002a0f0       ICProcessBIFNtexture2DLod  1002b0f0 f   glsl_core:icbuiltin.obj
 0001:0002a198       ICProcessBIFNtexture2DProjLod 1002b198 f   glsl_core:icbuiltin.obj
 0001:0002a1bc       ICProcessBIFNtexture3D     1002b1bc f   glsl_core:icbuiltin.obj
 0001:0002a2f8       ICProcessBIFNtexture3DProj 1002b2f8 f   glsl_core:icbuiltin.obj
 0001:0002a3c8       ICProcessBIFNtexture3DLod  1002b3c8 f   glsl_core:icbuiltin.obj
 0001:0002a470       ICProcessBIFNtexture3DProjLod 1002b470 f   glsl_core:icbuiltin.obj
 0001:0002a494       ICProcessBIFNtextureCube   1002b494 f   glsl_core:icbuiltin.obj
 0001:0002a5d0       ICProcessBIFNtextureCubeLod 1002b5d0 f   glsl_core:icbuiltin.obj
 0001:0002a678       ICProcessBIFNshadow1D      1002b678 f   glsl_core:icbuiltin.obj
 0001:0002a694       ICProcessBIFNshadow2D      1002b694 f   glsl_core:icbuiltin.obj
 0001:0002a6b0       ICProcessBIFNshadow1DProj  1002b6b0 f   glsl_core:icbuiltin.obj
 0001:0002a6cc       ICProcessBIFNshadow2DProj  1002b6cc f   glsl_core:icbuiltin.obj
 0001:0002a6e8       ICProcessBIFNshadow1DLod   1002b6e8 f   glsl_core:icbuiltin.obj
 0001:0002a704       ICProcessBIFNshadow2DLod   1002b704 f   glsl_core:icbuiltin.obj
 0001:0002a720       ICProcessBIFNshadow1DProjLod 1002b720 f   glsl_core:icbuiltin.obj
 0001:0002a73c       ICProcessBIFNshadow2DProjLod 1002b73c f   glsl_core:icbuiltin.obj
 0001:0002a758       ICProcessBIFNtextureStream 1002b758 f   glsl_core:icbuiltin.obj
 0001:0002a7f4       ICProcessBIFNtextureStreamProj 1002b7f4 f   glsl_core:icbuiltin.obj
 0001:0002a890       ICProcessBIFNdFdx          1002b890 f   glsl_core:icbuiltin.obj
 0001:0002a908       ICProcessBIFNdFdy          1002b908 f   glsl_core:icbuiltin.obj
 0001:0002a980       ICProcessBIFNfwidth        1002b980 f   glsl_core:icbuiltin.obj
 0001:0002ab10       ICProcessBIFNnoise1        1002bb10 f   glsl_core:icbuiltin.obj
 0001:0002ab14       ICProcessBIFNnoise2        1002bb14 f   glsl_core:icbuiltin.obj
 0001:0002ab18       ICProcessBIFNnoise3        1002bb18 f   glsl_core:icbuiltin.obj
 0001:0002ab1c       ICProcessBIFNnoise4        1002bb1c f   glsl_core:icbuiltin.obj
 0001:0002ab20       ICProcessBIFNtexture1DProjGrad 1002bb20 f   glsl_core:icbuiltin.obj
 0001:0002ab44       ICProcessBIFNtexture1DGrad 1002bb44 f   glsl_core:icbuiltin.obj
 0001:0002abec       ICProcessBIFNtexture2DProjGrad 1002bbec f   glsl_core:icbuiltin.obj
 0001:0002ac10       ICProcessBIFNtexture2DGrad 1002bc10 f   glsl_core:icbuiltin.obj
 0001:0002acb8       ICProcessBIFNtexture3DProjGrad 1002bcb8 f   glsl_core:icbuiltin.obj
 0001:0002acdc       ICProcessBIFNtexture3DGrad 1002bcdc f   glsl_core:icbuiltin.obj
 0001:0002ad84       ICProcessBIFNtextureCubeGrad 1002bd84 f   glsl_core:icbuiltin.obj
 0001:0002ae2c       ICProcessBIFNshadow1DProjGrad 1002be2c f   glsl_core:icbuiltin.obj
 0001:0002ae48       ICProcessBIFNshadow1DGrad  1002be48 f   glsl_core:icbuiltin.obj
 0001:0002ae64       ICProcessBIFNshadow2DProjGrad 1002be64 f   glsl_core:icbuiltin.obj
 0001:0002ae80       ICProcessBIFNshadow2DGrad  1002be80 f   glsl_core:icbuiltin.obj
 0001:0002af38       FindWrittenToLineForSymbolID 1002bf38 f   glsl_core:icunroll.obj
 0001:0002afc4       ExamineLoopUpdateCode      1002bfc4 f   glsl_core:icunroll.obj
 0001:0002b2cc       ExamineLoopBodyCode        1002c2cc f   glsl_core:icunroll.obj
 0001:0002b644       ExamineLoopConditionCode   1002c644 f   glsl_core:icunroll.obj
 0001:0002b738       RewriteLoopCode            1002c738 f   glsl_core:icunroll.obj
 0001:0002bae4       EvaluateCondition          1002cae4 f   glsl_core:icunroll.obj
 0001:0002bbac       UnrollLoopFORCode          1002cbac f   glsl_core:icunroll.obj
 0001:0002c024       ASTBICheckForUseOfState    1002d024 f   glsl_core:astbuiltin.obj
 0001:0002c094       ASTBIAddConstructor        1002d094 f   glsl_core:astbuiltin.obj
 0001:0002c270       ASTBIAddFunction1          1002d270 f   glsl_core:astbuiltin.obj
 0001:0002c6ac       ASTBIAddFunction2          1002d6ac f   glsl_core:astbuiltin.obj
 0001:0002cafc       ASTBIAddFunction3          1002dafc f   glsl_core:astbuiltin.obj
 0001:0002cf50       ASTBIAddFunction4          1002df50 f   glsl_core:astbuiltin.obj
 0001:0002d3b8       ASTBIAddGLState            1002e3b8 f   glsl_core:astbuiltin.obj
 0001:0002d494       ASTAddGLStructureMember    1002e494 f   glsl_core:astbuiltin.obj
 0001:0002f860       PPFreeDefineMacro          10030860 f   glsl_core:prepro.obj
 0001:0002f8e8       PPGetNextDirectiveTokenEntry 100308e8 f   glsl_core:prepro.obj
 0001:0002f980       PPCreateTokenLinkedList    10030980 f   glsl_core:prepro.obj
 0001:0002fa84       PPInsertTokensIntoLinkedList 10030a84 f   glsl_core:prepro.obj
 0001:0002fae4       PPCheckForMacroReplacement 10030ae4 f   glsl_core:prepro.obj
 0001:000301c0       PPAddChildNode             100311c0 f   glsl_core:prepro.obj
 0001:00030254       PPAddParentNode            10031254 f   glsl_core:prepro.obj
 0001:00030324       PPCleanUpBranches          10031324 f   glsl_core:prepro.obj
 0001:00030368       PPFreeExpressionTree       10031368 f   glsl_core:prepro.obj
 0001:000303c8       PPCreateExpressionTree     100313c8 f   glsl_core:prepro.obj
 0001:0003060c       PPCalculateResultOfExpressionTree 1003160c f   glsl_core:prepro.obj
 0001:00030a10       PPProcessIf                10031a10 f   glsl_core:prepro.obj
 0001:00030b70       PPProcessElif              10031b70 f   glsl_core:prepro.obj
 0001:00030ccc       PPProcessIfdef             10031ccc f   glsl_core:prepro.obj
 0001:00030e1c       PPProcessLine              10031e1c f   glsl_core:prepro.obj
 0001:00030f40       PPProcessPragma            10031f40 f   glsl_core:prepro.obj
 0001:000311c8       ProcessDefineMacro         100321c8 f   glsl_core:prepro.obj
 0001:0003171c       ProcessUndef               1003271c f   glsl_core:prepro.obj
 0001:0003187c       PPProcessVersion           1003287c f   glsl_core:prepro.obj
 0001:00031a30       PPIsExtensionSupported     10032a30 f   glsl_core:prepro.obj
 0001:00031aa4       PPProcessExtension         10032aa4 f   glsl_core:prepro.obj
 0001:00031d0c       PPProcessDirective         10032d0c f   glsl_core:prepro.obj
 0001:000321fc       PPSetDefaultDefine         100331fc f   glsl_core:prepro.obj
 0001:000329a8       ASTCheckFeatureVersion     100339a8 f   glsl_core:glsltree.obj
 0001:00032a98       GetRule                    10033a98 f   glsl_core:glsltree.obj
 0001:00032b10       ASTCreateSwizzleNode       10033b10 f   glsl_core:glsltree.obj
 0001:00032d74       ASTCreateIDENTIFIERNode    10033d74 f   glsl_core:glsltree.obj
 0001:00032eb0       ASTCreateFLOATCONSTANTNode 10033eb0 f   glsl_core:glsltree.obj
 0001:00032ff0       ASTCreateINTCONSTANTNode   10033ff0 f   glsl_core:glsltree.obj
 0001:000330d4       ASTCreateBOOLCONSTANTNode  100340d4 f   glsl_core:glsltree.obj
 0001:000331e0       ASTAddFunctionState        100341e0 f   glsl_core:glsltree.obj
 0001:000332ec       ASTCreateFunctionNode      100342ec f   glsl_core:glsltree.obj
 0001:000339e4       ASTProcessConstructorIdentifier 100349e4 f   glsl_core:glsltree.obj
 0001:00033bb8       ASTProcessFunctionIdentifier 10034bb8 f   glsl_core:glsltree.obj
 0001:00033d00       ASTRegisterFunctionCall    10034d00 f   glsl_core:glsltree.obj
 0001:00033e4c       ASTFindFunction            10034e4c f   glsl_core:glsltree.obj
 0001:00034258       ASTProcessFieldSelection   10035258 f   glsl_core:glsltree.obj
 0001:00034530       ASTProcessUnaryOperator    10035530 f   glsl_core:glsltree.obj
 0001:00034630       ASTProcessAssignmentOperator 10035630 f   glsl_core:glsltree.obj
 0001:000347a8       ASTProcessAssignmentExpression 100357a8 f   glsl_core:glsltree.obj
 0001:00034984       ASTProcessExpression       10035984 f   glsl_core:glsltree.obj
 0001:00034b48       ASTProcessExpressionStatement 10035b48 f   glsl_core:glsltree.obj
 0001:00034bd0       ASTProcessTypeQualifier    10035bd0 f   glsl_core:glsltree.obj
 0001:00034ce4       ASTProcessPrecisionQualifier 10035ce4 f   glsl_core:glsltree.obj
 0001:00034dfc       ASTUpdateInvariantStatus   10035dfc f   glsl_core:glsltree.obj
 0001:00034ed0       ASTProcessParameterQualifier 10035ed0 f   glsl_core:glsltree.obj
 0001:00034f94       FreePrecisionModifierData  10035f94 f   glsl_core:glsltree.obj
 0001:00034fac       GetCurrentPrecision        10035fac f   glsl_core:glsltree.obj
 0001:000350ec       ModifyDefaultPrecision     100360ec f   glsl_core:glsltree.obj
 0001:00035248       ASTProcessJumpStatement    10036248 f   glsl_core:glsltree.obj
 0001:00035448       ASTProcessStatementNoNewScope 10036448 f   glsl_core:glsltree.obj
 0001:00035510       DestroyAbstractSyntaxTree  10036510 f   glsl_core:glsltree.obj
 0001:00035568       CheckWhichFunctionsCalled  10036568 f   glsl_core:glsltree.obj
 0001:0003568c       ReOrderTopLevelNodes       1003668c f   glsl_core:glsltree.obj
 0001:00035950       ASTDecreaseScope           10036950 f   glsl_core:glsltree.obj
 0001:000359a0       ASTProcessFunctionCallHeaderWithParameters 100369a0 f   glsl_core:glsltree.obj
 0001:00035b80       ASTProcessFunctionCallGeneric 10036b80 f   glsl_core:glsltree.obj
 0001:00035ce0       ASTProcessFunctionCall     10036ce0 f   glsl_core:glsltree.obj
 0001:000360a4       ASTProcessPrimaryExpression 100370a4 f   glsl_core:glsltree.obj
 0001:0003623c       ASTProcessPostFixExpressionLR 1003723c f   glsl_core:glsltree.obj
 0001:00036580       ASTProcessPostFixExpression 10037580 f   glsl_core:glsltree.obj
 0001:000366c4       ASTProcessUnaryExpression  100376c4 f   glsl_core:glsltree.obj
 0001:000368f0       ASTProcessMultiplicativeExpressionLR 100378f0 f   glsl_core:glsltree.obj
 0001:00036ac8       ASTProcessMultiplicativeExpression 10037ac8 f   glsl_core:glsltree.obj
 0001:00036b84       ASTProcessAdditiveExpressionLR 10037b84 f   glsl_core:glsltree.obj
 0001:00036d4c       ASTProcessAdditiveExpression 10037d4c f   glsl_core:glsltree.obj
 0001:00036e08       ASTProcessShiftExpressionLR 10037e08 f   glsl_core:glsltree.obj
 0001:00036ff4       ASTProcessShiftExpression  10037ff4 f   glsl_core:glsltree.obj
 0001:000370b0       ASTProcessRelationalExpressionLR 100380b0 f   glsl_core:glsltree.obj
 0001:000372a0       ASTProcessRelationalExpression 100382a0 f   glsl_core:glsltree.obj
 0001:0003735c       ASTProcessEqualityExpressionLR 1003835c f   glsl_core:glsltree.obj
 0001:00037524       ASTProcessEqualityExpression 10038524 f   glsl_core:glsltree.obj
 0001:000375d8       ASTProcessAndExpressionLR  100385d8 f   glsl_core:glsltree.obj
 0001:000377ac       ASTProcessAndExpression    100387ac f   glsl_core:glsltree.obj
 0001:00037868       ASTProcessExclusiveOrExpressionLR 10038868 f   glsl_core:glsltree.obj
 0001:00037a3c       ASTProcessExclusiveOrExpression 10038a3c f   glsl_core:glsltree.obj
 0001:00037af4       ASTProcessInclusiveOrExpressionLR 10038af4 f   glsl_core:glsltree.obj
 0001:00037cc8       ASTProcessInclusiveOrExpression 10038cc8 f   glsl_core:glsltree.obj
 0001:00037d84       ASTProcessLogicalAndExpressionLR 10038d84 f   glsl_core:glsltree.obj
 0001:00037f38       ASTProcessLogicalAndExpression 10038f38 f   glsl_core:glsltree.obj
 0001:00037ff4       ASTProcessLogicalXorExpressionLR 10038ff4 f   glsl_core:glsltree.obj
 0001:000381a8       ASTProcessLogicalXorExpression 100391a8 f   glsl_core:glsltree.obj
 0001:00038264       ASTProcessLogicalOrExpressionLR 10039264 f   glsl_core:glsltree.obj
 0001:00038418       ASTProcessLogicalOrExpression 10039418 f   glsl_core:glsltree.obj
 0001:000384d4       ASTProcessQuestionExpression 100394d4 f   glsl_core:glsltree.obj
 0001:00038678       ASTProcessConditionalExpression 10039678 f   glsl_core:glsltree.obj
 0001:00038760       ASTProcessTypeSpecifier    10039760 f   glsl_core:glsltree.obj
 0001:000389b4       ASTProcessFullySpecifiedType 100399b4 f   glsl_core:glsltree.obj
 0001:00038ab4       ASTProcessParameterTypeSpecifier 10039ab4 f   glsl_core:glsltree.obj
 0001:00038b74       ASTProcessFunctionHeader   10039b74 f   glsl_core:glsltree.obj
 0001:00038cbc       ASTProcessCompoundStatement 10039cbc f   glsl_core:glsltree.obj
 0001:00038d7c       ASTProcessSelectionStatement 10039d7c f   glsl_core:glsltree.obj
 0001:00038f7c       ASTProcessArraySpecifier   10039f7c f   glsl_core:glsltree.obj
 0001:0003910c       ASTProcessArraySpecifierOpt 1003a10c f   glsl_core:glsltree.obj
 0001:00039184       ASTProcessStructDeclaratorList 1003a184 f   glsl_core:glsltree.obj
 0001:0003945c       ASTProcessStructDeclarationList 1003a45c f   glsl_core:glsltree.obj
 0001:00039578       ASTProcessStructSpecifier  1003a578 f   glsl_core:glsltree.obj
 0001:00039708       ASTProcessTypeSpecifierNoPrec 1003a708 f   glsl_core:glsltree.obj
 0001:00039ac4       ASTGenerateDeclarationChildNode 1003aac4 f   glsl_core:glsltree.obj
 0001:00039e70       ASTProcessSingleDeclaration 1003ae70 f   glsl_core:glsltree.obj
 0001:00039ff4       ASTProcessParameterDeclarator 1003aff4 f   glsl_core:glsltree.obj
 0001:0003a1b8       ASTProcessParameterDeclaration 1003b1b8 f   glsl_core:glsltree.obj
 0001:0003a50c       ASTProcessFunctionDeclarator 1003b50c f   glsl_core:glsltree.obj
 0001:0003a678       ASTProcessInitDeclaratorList 1003b678 f   glsl_core:glsltree.obj
 0001:0003a908       ASTProcessDeclaration      1003b908 f   glsl_core:glsltree.obj
 0001:0003ab5c       ASTProcessCondition        1003bb5c f   glsl_core:glsltree.obj
 0001:0003ad14       ASTProcessForInitStatement 1003bd14 f   glsl_core:glsltree.obj
 0001:0003ae10       ASTProcessIterationStatement 1003be10 f   glsl_core:glsltree.obj
 0001:0003b318       ASTProcessSimpleStatement  1003c318 f   glsl_core:glsltree.obj
 0001:0003b48c       ASTProcessStatement        1003c48c f   glsl_core:glsltree.obj
 0001:0003b548       ASTProcessStatementList    1003c548 f   glsl_core:glsltree.obj
 0001:0003b658       ASTProcessCompoundStatementNoNewScope 1003c658 f   glsl_core:glsltree.obj
 0001:0003b748       ASTProcessFunctionDefinition 1003c748 f   glsl_core:glsltree.obj
 0001:0003b8b4       ASTProcessExternalDeclaration 1003c8b4 f   glsl_core:glsltree.obj
 0001:0003ba8c       ASTProcessTranslationUnit  1003ca8c f   glsl_core:glsltree.obj
 0001:0003bff8       ICInitOperandInfoWithSwiz  1003cff8 f   glsl_core:icemul.obj
 0001:0003c054       ICApplyOperandMoreSwiz     1003d054 f   glsl_core:icemul.obj
 0001:0003c0ac       _MUL                       1003d0ac f   glsl_core:icemul.obj
 0001:0003c178       _ADD                       1003d178 f   glsl_core:icemul.obj
 0001:0003c244       _SUB                       1003d244 f   glsl_core:icemul.obj
 0001:0003c310       _MOV                       1003d310 f   glsl_core:icemul.obj
 0001:0003c3a8       _RCP                       1003d3a8 f   glsl_core:icemul.obj
 0001:0003c440       _MAD                       1003d440 f   glsl_core:icemul.obj
 0001:0003c614       _FLR                       1003d614 f   glsl_core:icemul.obj
 0001:0003c6ac       _FRC                       1003d6ac f   glsl_core:icemul.obj
 0001:0003c7dc       _DOT                       1003d7dc f   glsl_core:icemul.obj
 0001:0003c8a8       _LABEL                     1003d8a8 f   glsl_core:icemul.obj
 0001:0003c8e8       _TEXLD                     1003d8e8 f   glsl_core:icemul.obj
 0001:0003c9b4       _MIX                       1003d9b4 f   glsl_core:icemul.obj
 0001:0003cc24       ICAddFunctionDefinitionToSymTab 1003dc24 f   glsl_core:icemul.obj
 0001:0003d060       ICAddArcCos2FunctionDefinition 1003e060 f   glsl_core:icemul.obj
 0001:0003d144       ICAddArcSin2FunctionDefinition 1003e144 f   glsl_core:icemul.obj
 0001:0003d228       ICAddArcTanFunctionDefinition 1003e228 f   glsl_core:icemul.obj
 0001:0003d30c       ICAddArcTan2FunctionDefinition 1003e30c f   glsl_core:icemul.obj
 0001:0003d3f8       ICAddNoiseFunctionDefinition 1003e3f8 f   glsl_core:icemul.obj
 0001:0003dc0c       ICAddDepthCompare          1003ec0c f   glsl_core:icemul.obj
 0001:0003e1fc       GetDepthTextureDescID      1003f1fc f   glsl_core:icemul.obj
 0001:00040cd0       ICInitNoiseFuncRegisters   10041cd0 f   glsl_core:icemul.obj
 0001:00045910       ASTSemRemoveChildNode      10046910 f   glsl_core:semantic.obj
 0001:00045a1c       ASTSemGetResultName        10046a1c f   glsl_core:semantic.obj
 0001:00045c14       ASTCheckNodeNumChildren    10046c14 f   glsl_core:semantic.obj
 0001:00045d9c       ASTSemGetIdentifierData    10046d9c f   glsl_core:semantic.obj
 0001:00045eb8       ASTSemConvertMatrix        10046eb8 f   glsl_core:semantic.obj
 0001:00045fa4       ASTSemConvertTypes         10046fa4 f   glsl_core:semantic.obj
 0001:000465dc       ASTSemReduceConstantConstructor 100475dc f   glsl_core:semantic.obj
 0001:00046a08       ASTSemInsertConstructor    10047a08 f   glsl_core:semantic.obj
 0001:00046ed4       ASTSemReduceConstantArraySpecifier 10047ed4 f   glsl_core:semantic.obj
 0001:00047150       ASTSemReduceConstantFieldSelection 10048150 f   glsl_core:semantic.obj
 0001:00047534       ASTSemReduceConstantMatrixMath 10048534 f   glsl_core:semantic.obj
 0001:000476b4       ASTSemReduceConstantMaths  100486b4 f   glsl_core:semantic.obj
 0001:00048ccc       ASTSemReduceConstantExpression 10049ccc f   glsl_core:semantic.obj
 0001:00048e50       ASTSemReportLValueError    10049e50 f   glsl_core:semantic.obj
 0001:00048f3c       ASTSemReduceConstantBuiltInFunction 10049f3c f   glsl_core:semantic.obj
 0001:00049290       ASTSemCheckAndUpdateArraySizes 1004a290 f   glsl_core:semantic.obj
 0001:00049558       ASTWarnUnitialisedData     1004a558 f   glsl_core:semantic.obj
 0001:00049648       ASTUpdateBuiltInsReferenced 1004a648 f   glsl_core:semantic.obj
 0001:00049808       ASTUpdateParamIdentifierUsage 1004a808 f   glsl_core:semantic.obj
 0001:0004994c       ASTUpdateReadIdentifierUsage 1004a94c f   glsl_core:semantic.obj
 0001:00049a1c       ASTUpdateIdentifierUsage   1004aa1c f   glsl_core:semantic.obj
 0001:00049b14       ASTSemCheckAssignment      1004ab14 f   glsl_core:semantic.obj
 0001:00049cb8       ASTSemCheckForReplacementWithConstantData 1004acb8 f   glsl_core:semantic.obj
 0001:00049ddc       ASTSemGetResultPrecision   1004addc f   glsl_core:semantic.obj
 0001:0004a494       ASTSemCheckFunctionCallParameters 1004b494 f   glsl_core:semantic.obj
 0001:0004e22c       SGXBS_ComputeHash          1004f22c f   glsl_binshader:esbinshader.obj
 0001:0004e304       GetNumOfBytesForWritingBindings 1004f304 f   glsl_binshader:esbinshader.obj
 0001:0004e350       WriteU8                    1004f350 f   glsl_binshader:esbinshader.obj
 0001:0004e398       WriteU16                   1004f398 f   glsl_binshader:esbinshader.obj
 0001:0004e3fc       WriteU32                   1004f3fc f   glsl_binshader:esbinshader.obj
 0001:0004e474       PackSymbolBindings         1004f474 f   glsl_binshader:esbinshader.obj
 0001:0004e5e0       PackUniflexProgram         1004f5e0 f   glsl_binshader:esbinshader.obj
 0001:0004e7f0       PackUserBindings           1004f7f0 f   glsl_binshader:esbinshader.obj
 0001:0004e8a4       PackProgramBinary          1004f8a4 f   glsl_binshader:esbinshader.obj
 0001:0004ed04       RemoveFromPredecessors     1004fd04 f   usc:usc.obj
 0001:0004eda4       AddAsPredecessor           1004fda4 f   usc:usc.obj
 0001:0004f348       FreeInsts                  10050348 f   usc:usc.obj
 0001:0004f5b4       FillPredecessorArraysBP    100505b4 f   usc:usc.obj
 0001:0004f8fc       DebugPrintSortRecursive    100508fc f   usc:usc.obj
 0001:000501bc       IntegerOptimizeBP          100511bc f   usc:usc.obj
 0001:000505fc       GenerateSwitchTest         100515fc f   usc:usc.obj
 0001:00050744       CmpArraySetupData          10051744 f   usc:usc.obj
 0001:00050790       SetupLoadStoreArray        10051790 f   usc:usc.obj
 0001:00050ad0       EliminateNewMovesBP        10051ad0 f   usc:usc.obj
 0001:000511c0       AddFixForBRN21752BP        100521c0 f   usc:usc.obj
 0001:000515cc       EmitLdStRegIndex           100525cc f   usc:usc.obj
 0001:00051788       EmitLdStRegMove            10052788 f   usc:usc.obj
 0001:00051bac       ExpandRegLdStInst          10052bac f   usc:usc.obj
 0001:00052020       GetLocalAddressingMemoryOffset 10053020 f   usc:usc.obj
 0001:000521a4       ExpandLoadStoreInst        100531a4 f   usc:usc.obj
 0001:000529e4       ExpandMemLoadStoreBP       100539e4 f   usc:usc.obj
 0001:00052a58       ExpandLoadStoreBP          10053a58 f   usc:usc.obj
 0001:00053080       NewChunk                   10054080 f   usc:data.obj
 0001:00053250       ArrayChunkGet              10054250 f   usc:data.obj
 0001:000533b0       BaseArrayGet               100543b0 f   usc:data.obj
 0001:0005348c       BaseArraySet               1005448c f   usc:data.obj
 0001:00053798       CalcVecOp                  10054798 f   usc:data.obj
 0001:00053854       VectorOpWorker             10054854 f   usc:data.obj
 0001:000540f4       VectorGetElement           100550f4 f   usc:data.obj
 0001:00054fb8       CopyRegLiveSet             10055fb8 f   usc:dce.obj
 0001:00055028       GetSourcesUsedFromPack     10056028 f   usc:dce.obj
 0001:00055120       RemapC10Channels           10056120 f   usc:dce.obj
 0001:00055174       GetLiveChansInSOP2Argument 10056174 f   usc:dce.obj
 0001:000552e0       GetLiveChansInLRP1Argument 100562e0 f   usc:dce.obj
 0001:000553fc       GetLiveChansInSOP3Argument 100563fc f   usc:dce.obj
 0001:000555b8       GetLiveChansInFPMAArgument 100565b8 f   usc:dce.obj
 0001:000556f4       GetLiveChansInSOPWMArgument 100566f4 f   usc:dce.obj
 0001:000557bc       GetLiveChansInArgumentPreVec 100567bc f   usc:dce.obj
 0001:00055ebc       MergeLivesets              10056ebc f   usc:dce.obj
 0001:00056298       ChangeRegisterLiveMask     10057298 f   usc:dce.obj
 0001:000564a8       IncreaseIndexedRegisterLiveMask 100574a8 f   usc:dce.obj
 0001:000565d4       GetTestChans               100575d4 f   usc:dce.obj
 0001:0005666c       SwapPackSources            1005766c f   usc:dce.obj
 0001:000568b0       ReduceInstDestMask         100578b0 f   usc:dce.obj
 0001:00056a24       HandleEFODest              10057a24 f   usc:dce.obj
 0001:00056bbc       IncreaseLiveMaskForRead    10057bbc f   usc:dce.obj
 0001:00056c88       ComputeLivenessForInst     10057c88 f   usc:dce.obj
 0001:000573a4       LivenessDF                 100583a4 f   usc:dce.obj
 0001:000576c0       DoLiveness                 100586c0 f   usc:dce.obj
 0001:00058744       InstRegUse                 10059744 f   usc:dce.obj
 0001:000588c0       InstRegDef                 100598c0 f   usc:dce.obj
 0001:000595c4       DeinitInst                 1005a5c4 f   usc:inst.obj
 0001:000597a4       InitInst                   1005a7a4 f   usc:inst.obj
 0001:0005a564       EqualEfo                   1005b564 f   usc:inst.obj
 0001:0005aab4       FindMSAPart                1005bab4 f   usc:iselect.obj
 0001:0005ac04       FindMulX2                  1005bc04 f   usc:iselect.obj
 0001:0005acf8       FindAdd                    1005bcf8 f   usc:iselect.obj
 0001:0005ae0c       TermsCancelOut             1005be0c f   usc:iselect.obj
 0001:0005b044       DoF32Test                  1005c044 f   usc:iselect.obj
 0001:0005b1a4       CombineMovcTest            1005c1a4 f   usc:iselect.obj
 0001:0005b640       MergeIdenticalTest         1005c640 f   usc:iselect.obj
 0001:0005b71c       InvertTest                 1005c71c f   usc:iselect.obj
 0001:0005b874       FoldConstantTest           1005c874 f   usc:iselect.obj
 0001:0005bb0c       FoldTESTMASK_MOVC          1005cb0c f   usc:iselect.obj
 0001:0005bd08       FoldTESTMASK_TEST          1005cd08 f   usc:iselect.obj
 0001:0005bea4       UNPCKF32U8ToUNPCKF32O8     1005cea4 f   usc:iselect.obj
 0001:0005c03c       FoldMINOrMAX_UNPCKF32U8    1005d03c f   usc:iselect.obj
 0001:0005c1a0       FoldMOVC_MUL               1005d1a0 f   usc:iselect.obj
 0001:0005c388       FoldMUL16_ADD16            1005d388 f   usc:iselect.obj
 0001:0005c5a0       FoldADD_ADDorMUL_ADM       1005d5a0 f   usc:iselect.obj
 0001:0005c764       FoldMUL_ADDOrMUL           1005d764 f   usc:iselect.obj
 0001:0005c9b4       FoldADD_ADD                1005d9b4 f   usc:iselect.obj
 0001:0005cb40       HasSourceModifier          1005db40 f   usc:iselect.obj
 0001:0005cbe0       CanCombineRegistersBackwards 1005dbe0 f   usc:iselect.obj
 0001:0005cf0c       CombineRegistersBackwards  1005df0c f   usc:iselect.obj
 0001:0005d1d4       ReplaceSmpArgument         1005e1d4 f   usc:iselect.obj
 0001:0005d710       EliminatePredicateMove     1005e710 f   usc:iselect.obj
 0001:0005d9a0       ElimGlobMovDomTree         1005e9a0 f   usc:iselect.obj
 0001:0005e134       NegateTest                 1005f134 f   usc:iselect.obj
 0001:0005e190       ReplaceConstantArg         1005f190 f   usc:iselect.obj
 0001:0005e1f8       ExtractConstantCalculationsInst 1005f1f8 f   usc:iselect.obj
 0001:0005efb0       SetChansReadFromMain       1005ffb0 f   usc:iselect.obj
 0001:0005f084       AssignInternOrSARegsToTempRegs 10060084 f   usc:iselect.obj
 0001:0005f6a4       FinalizeExtractionInsts    100606a4 f   usc:iselect.obj
 0001:0005f7e0       Extract40BitInstsToSAUpdate 100607e0 f   usc:iselect.obj
 0001:00060730       AddSAOutputsBP             10061730 f   usc:iselect.obj
 0001:00060848       ReplaceF32ByF16Source      10061848 f   usc:iselect.obj
 0001:00060a70       CombineF32PacksBlock       10061a70 f   usc:iselect.obj
 0001:00060d98       MovePredicateInsts         10061d98 f   usc:iselect.obj
 0001:00060e38       CanFlatten                 10061e38 f   usc:iselect.obj
 0001:00060fa0       FlattenConditional         10061fa0 f   usc:iselect.obj
 0001:00061110       FlattenConditionalsDomTree 10062110 f   usc:iselect.obj
 0001:00061224       OptimiseUSPSampleDestFmt   10062224 f   usc:iselect.obj
 0001:00061f18       IsSaturatedSample          10062f18 f   usc:iselect.obj
 0001:00061fbc       IsSaturatedArgument        10062fbc f   usc:iselect.obj
 0001:00062130       UpdateSaturatedResult      10063130 f   usc:iselect.obj
 0001:00062224       TryRemoveSaturate          10063224 f   usc:iselect.obj
 0001:00062390       TrySimplifyTest            10063390 f   usc:iselect.obj
 0001:00062844       FixInvalidSourceBanks_GetCReg 10063844 f   usc:iselect.obj
 0001:00062904       AddMoveForInvalidSourceBank 10063904 f   usc:iselect.obj
 0001:000629fc       FixInvalidSourceBanksInst  100639fc f   usc:iselect.obj
 0001:0006301c       FoldSeperateTest           1006401c f   usc:iselect.obj
 0001:0006342c       OptimizeInstructionSequence 1006442c f   usc:iselect.obj
 0001:00063618       SimplifyArithmeticInst     10064618 f   usc:iselect.obj
 0001:00063bac       SimplifyInst               10064bac f   usc:iselect.obj
 0001:00063cdc       ChangeTestForSourceMod     10064cdc f   usc:iselect.obj
 0001:00063f4c       GlobalReplaceArguments     10064f4c f   usc:iselect.obj
 0001:00065084       ExtractConstantCalculationsBP 10066084 f   usc:iselect.obj
 0001:00065e20       IsAlphaMultiply            10066e20 f   usc:intcvt.obj
 0001:00065ec0       IsSOPWMMultiply            10066ec0 f   usc:intcvt.obj
 0001:00065f4c       IsSOPWMMove                10066f4c f   usc:intcvt.obj
 0001:00065fac       CombineDifferentSrcFmtPacks 10066fac f   usc:intcvt.obj
 0001:000661ec       SwapArgsInSrcSel           100671ec f   usc:intcvt.obj
 0001:00066290       SelectAlphaInSrcSel        10067290 f   usc:intcvt.obj
 0001:00066304       CombineSopwmsMatchingArgsIntoSop2 10067304 f   usc:intcvt.obj
 0001:000664b4       CombineSopwmsWithSpareArgIntoSop2 100674b4 f   usc:intcvt.obj
 0001:000665b8       CombineSopwms              100675b8 f   usc:intcvt.obj
 0001:0006695c       RemoveRedundantConversion  1006795c f   usc:intcvt.obj
 0001:00066b20       CombineSOPWMMulSOPWMDouble 10067b20 f   usc:intcvt.obj
 0001:00066c54       SOPWMToMove                10067c54 f   usc:intcvt.obj
 0001:00066d00       DropRedundantMinMax        10067d00 f   usc:intcvt.obj
 0001:00066ef4       GlobalReplaceIntegerMoveArguments 10067ef4 f   usc:intcvt.obj
 0001:00067014       FormatConvert_MergeSets    10068014 f   usc:intcvt.obj
 0001:00067150       FormatConvert_ApplyUpdates 10068150 f   usc:intcvt.obj
 0001:0006732c       AddRegisterToConversionSet 1006832c f   usc:intcvt.obj
 0001:00067584       FormatConvert_DeleteRegisterSet 10068584 f   usc:intcvt.obj
 0001:00067618       FormatConvert_CheckRegisterOverwrite 10068618 f   usc:intcvt.obj
 0001:00067770       ConvertRegisterFormatC10ToU8_Inst 10068770 f   usc:intcvt.obj
 0001:00067d68       CheckIntegerComponentMoveBanks 10068d68 f   usc:intcvt.obj
 0001:00067f48       CheckIntegerComponentMoveFormat_ComplexOp 10068f48 f   usc:intcvt.obj
 0001:0006806c       CheckIntegerComponentMoveFormat_PCK 1006906c f   usc:intcvt.obj
 0001:000682b4       CheckIntegerComponentMoveFormat_TEST 100692b4 f   usc:intcvt.obj
 0001:00068494       CheckIntegerComponentMoveFormat_INTARITH 10069494 f   usc:intcvt.obj
 0001:000685e4       CheckIntegerComponentMoveFormat 100695e4 f   usc:intcvt.obj
 0001:00068778       GlobalIntegerComponentMoveUpdateBlock 10069778 f   usc:intcvt.obj
 0001:00068834       GlobalReplaceIntegerComponentMoveArguments 10069834 f   usc:intcvt.obj
 0001:000689a0       CanEliminateIntegerComponentMoveForward 100699a0 f   usc:intcvt.obj
 0001:00068bd0       EliminateIntegerComponentMoveForward 10069bd0 f   usc:intcvt.obj
 0001:00068f90       CanEliminateIntegerMoveBackward 10069f90 f   usc:intcvt.obj
 0001:000690bc       EliminateIntegerMoveBackward 1006a0bc f   usc:intcvt.obj
 0001:0006921c       SubstituteAlphaSwizzle     1006a21c f   usc:intcvt.obj
 0001:000693d4       CanEliminateAlphaSwizzle   1006a3d4 f   usc:intcvt.obj
 0001:000695dc       EliminateAlphaSwizzle      1006a5dc f   usc:intcvt.obj
 0001:000697e0       EliminateIntegerMoves      1006a7e0 f   usc:intcvt.obj
 0001:0006a00c       CombineMulMulToSOP3        1006b00c f   usc:intcvt.obj
 0001:0006a2a4       CombineAddMovToSOP3        1006b2a4 f   usc:intcvt.obj
 0001:0006a4d0       CombineMulMovToLRP1        1006b4d0 f   usc:intcvt.obj
 0001:0006a738       CombineMOVSOPWM            1006b738 f   usc:intcvt.obj
 0001:0006a8e0       ConvertPackToMove          1006b8e0 f   usc:intcvt.obj
 0001:0006a9d8       CombineMULMOVToSOP2        1006b9d8 f   usc:intcvt.obj
 0001:0006abd4       CombineMOVMOVToSOP2        1006bbd4 f   usc:intcvt.obj
 0001:0006ad9c       CombinePacksToU8C10        1006bd9c f   usc:intcvt.obj
 0001:0006b000       CombineSharedDestInstructions 1006c000 f   usc:intcvt.obj
 0001:0006bb80       AddAlphaSwizzleC10Constant 1006cb80 f   usc:intcvt.obj
 0001:0006bc70       CombineIntMulAdd           1006cc70 f   usc:intcvt.obj
 0001:0006c1c8       FoldC10Combine             1006d1c8 f   usc:intcvt.obj
 0001:0006c4a0       ConvertUnpacksToO8         1006d4a0 f   usc:intcvt.obj
 0001:0006c648       IsSOP2DoubleMove           1006d648 f   usc:intcvt.obj
 0001:0006c700       CombineSOPWMSOP2Move       1006d700 f   usc:intcvt.obj
 0001:0006c998       CombineSOP2MoveSOPWMMultiply 1006d998 f   usc:intcvt.obj
 0001:0006cba4       CheckForScale              1006dba4 f   usc:intcvt.obj
 0001:0006cfac       CheckIntegerMaxMin         1006dfac f   usc:intcvt.obj
 0001:0006d0a4       ConvertMinMaxToFormatConvert 1006e0a4 f   usc:intcvt.obj
 0001:0006d218       FoldDestFormatConversion   1006e218 f   usc:intcvt.obj
 0001:0006d324       OptimizeDependentIntegerInstructions 1006e324 f   usc:intcvt.obj
 0001:0006d4e0       CouldBeEqualRegister       1006e4e0 f   usc:intcvt.obj
 0001:0006d580       FindOtherInstruction       1006e580 f   usc:intcvt.obj
 0001:0006d780       NormaliseIntegerInstructions 1006e780 f   usc:intcvt.obj
 0001:0006e0a0       PCShaderSkip4              1006f0a0 f   usc:uspbin.obj
 0001:0006e0b0       PCShaderSkip2              1006f0b0 f   usc:uspbin.obj
 0001:0006e0c0       PCShaderSkip1              1006f0c0 f   usc:uspbin.obj
 0001:0006e0d0       PCShaderSkipN              1006f0d0 f   usc:uspbin.obj
 0001:0006e0e0       PCShaderWrite4             1006f0e0 f   usc:uspbin.obj
 0001:0006e11c       PCShaderWrite2             1006f11c f   usc:uspbin.obj
 0001:0006e148       PCShaderWrite1             1006f148 f   usc:uspbin.obj
 0001:0006e164       PCShaderWriteN             1006f164 f   usc:uspbin.obj
 0001:0006e18c       UseAssemblerGetLabelAddress 1006f18c f   usc:uspbin.obj
 0001:0006e194       UseAssemblerError          1006f194 f   usc:uspbin.obj
 0001:0006e268       GetShaderAltResultRegs     1006f268 f   usc:uspbin.obj
 0001:0006e358       BuildPCProgDescHdr         1006f358 f   usc:uspbin.obj
 0001:0006eb04       BuildPCProgDescPSInputList 1006fb04 f   usc:uspbin.obj
 0001:0006ed04       AddC10ConstantEntry        1006fd04 f   usc:uspbin.obj
 0001:0006ed8c       BuildPCProgDescConstListForMemoryMappedConsts 1006fd8c f   usc:uspbin.obj
 0001:0006f0a8       BuildPCProgDescConstList   100700a8 f   usc:uspbin.obj
 0001:0006f338       EncodeInstsBP              10070338 f   usc:uspbin.obj
 0001:0006f390       BuildPCProgDesc            10070390 f   usc:uspbin.obj
 0001:0006f624       SetupPCInstDesc            10070624 f   usc:uspbin.obj
 0001:0006f6d8       BuildHWCodeBlock           100706d8 f   usc:uspbin.obj
 0001:0006f948       BuildPCLabelCB             10070948 f   usc:uspbin.obj
 0001:0006f98c       BuildPCBranchCB            1007098c f   usc:uspbin.obj
 0001:0006fa78       BuildSampleBlock           10070a78 f   usc:uspbin.obj
 0001:00070148       BuildPCDataForBasicBlockCB 10071148 f   usc:uspbin.obj
 0001:000703b8       PointActionsUspBinCB       100713b8 f   usc:uspbin.obj
 0001:00070474       AlignToEvenUspBinCB        10071474 f   usc:uspbin.obj
 0001:00070478       BuildPCShader              10071478 f   usc:uspbin.obj
 0001:00070748       InsertAltOutPutsAndRecordResultRefsBP 10071748 f   usc:uspbin.obj
 0001:00071078       GetBestOfAnyAncestor       10072078 f   usc:domcalc.obj
 0001:000710dc       DoDfs                      100720dc f   usc:domcalc.obj
 0001:00071198       AddToParent                10072198 f   usc:domcalc.obj
 0001:000715d0       MarkInLoop                 100725d0 f   usc:domcalc.obj
 0001:000717a4       IsSecAttrsUsedInRegisterGroupBP 100727a4 f   usc:regpack.obj
 0001:0007188c       RemapSecAttrsBP            1007288c f   usc:regpack.obj
 0001:00072088       IsStaticConst              10073088 f   usc:regpack.obj
 0001:00072400       RemapPrimaryAttributesBP   10073400 f   usc:regpack.obj
 0001:00072550       MoveTextureLoad            10073550 f   usc:regpack.obj
 0001:000726bc       IsLastCoordUsed            100736bc f   usc:regpack.obj
 0001:0007293c       PackPrimaryAttributes      1007393c f   usc:regpack.obj
 0001:000730cc       GetRangeCheck              100740cc f   usc:regpack.obj
 0001:000731fc       FindRange                  100741fc f   usc:regpack.obj
 0001:00073294       ApplyConstantRemapping     10074294 f   usc:regpack.obj
 0001:000734d0       SwapRedAndBlueChans        100744d0 f   usc:regpack.obj
 0001:000735cc       GenerateMemoryLoad         100745cc f   usc:regpack.obj
 0001:0007382c       PackPARegsBP               1007482c f   usc:regpack.obj
 0001:00073e04       SearchConstBufsBP          10074e04 f   usc:regpack.obj
 0001:00073fcc       ReplaceConstsBP            10074fcc f   usc:regpack.obj
 0001:00074b6c       MakeDummyFetch             10075b6c f   usc:reorder.obj
 0001:00074ccc       FindFetch                  10075ccc f   usc:reorder.obj
 0001:00075110       AreInternalRegsAndPredicatesLiveAtFB 10076110 f   usc:reorder.obj
 0001:0007587c       PeepholeOptimizer          1007687c f   usc:reorder.obj
 0001:00075adc       SetNoSchedFlagForBasicBlockNoPairs 10076adc f   usc:finalise.obj
 0001:00075bc4       SetNoSchedFlagForBasicBlock 10076bc4 f   usc:finalise.obj
 0001:00075f9c       CopySkipinvState           10076f9c f   usc:finalise.obj
 0001:00075fec       MergeSkipinvState          10076fec f   usc:finalise.obj
 0001:00076108       SetSkipInvalidFlagForInst  10077108 f   usc:finalise.obj
 0001:00076878       SetSkipInvalidDF           10077878 f   usc:finalise.obj
 0001:00076b44       DoSkipInvalid              10077b44 f   usc:finalise.obj
 0001:00076c8c       DetermineNonAnisoTextureStagesBP 10077c8c f   usc:finalise.obj
 0001:00076cd8       SetSkipInvAllInstsBP       10077cd8 f   usc:finalise.obj
 0001:00076d2c       SetupSkipInvalidFlag       10077d2c f   usc:finalise.obj
 0001:00076ed4       CheckForFetch              10077ed4 f   usc:finalise.obj
 0001:000772d8       ExpandLoadForRangeCheck    100782d8 f   usc:finalise.obj
 0001:00077694       RegisterUsedInRange        10078694 f   usc:finalise.obj
 0001:00077774       OptimizeAddressCalc        10078774 f   usc:finalise.obj
 0001:00077a84       OptimizeAddressCalc_RangeCheck 10078a84 f   usc:finalise.obj
 0001:00077d78       OptimizeAddressCalc_545    10078d78 f   usc:finalise.obj
 0001:00078058       PostFetchOptimizationBlock 10079058 f   usc:finalise.obj
 0001:000781d8       GenerateFetchInstructionsBP 100791d8 f   usc:finalise.obj
 0001:00078270       GetWaitInstIdx             10079270 f   usc:finalise.obj
 0001:00078504       CheckInsertWaits           10079504 f   usc:finalise.obj
 0001:000785a0       InsertWaitsBP              100795a0 f   usc:finalise.obj
 0001:00078980       SetSyncStartBeforeInst     10079980 f   usc:finalise.obj
 0001:00078a0c       SetSyncStartBP             10079a0c f   usc:finalise.obj
 0001:00078a70       NoSchedAlignToEvenCB       10079a70 f   usc:finalise.obj
 0001:00078aa4       NoSchedBranchCB            10079aa4 f   usc:finalise.obj
 0001:00078ae0       FinaliseIndexableTempsBP   10079ae0 f   usc:finalise.obj
 0001:00078c2c       RemoveNoEmitInstructionsBP 10079c2c f   usc:finalise.obj
 0001:00078c80       AddFixForBRN25804ForBlock  10079c80 f   usc:finalise.obj
 0001:00078d30       IsTESTMASKUsedInBlock      10079d30 f   usc:finalise.obj
 0001:00079138       DoOnAllFuncGroupBasicBlocks 1007a138 f   usc:regalloc.obj
 0001:000791c8       NodeToRegister             1007a1c8 f   usc:regalloc.obj
 0001:00079238       RegisterToNode             1007a238 f   usc:regalloc.obj
 0001:00079294       ArgumentToNode             1007a294 f   usc:regalloc.obj
 0001:00079300       MakeGroup                  1007a300 f   usc:regalloc.obj
 0001:000793a0       AddToGroup                 1007a3a0 f   usc:regalloc.obj
 0001:00079570       RemoveFromGroup            1007a570 f   usc:regalloc.obj
 0001:00079710       AdjustBaseAddress          1007a710 f   usc:regalloc.obj
 0001:00079854       GroupArrayRegs             1007a854 f   usc:regalloc.obj
 0001:00079a1c       FormFetchGroup             1007aa1c f   usc:regalloc.obj
 0001:00079cac       SetupSpillAreaBP           1007acac f   usc:regalloc.obj
 0001:00079dfc       RegIsNode                  1007adfc f   usc:regalloc.obj
 0001:0007a40c       FreeRAGColState            1007b40c f   usc:regalloc.obj
 0001:0007a5cc       AllocateRAGColState        1007b5cc f   usc:regalloc.obj
 0001:0007a7f4       ResetRAGColState           1007b7f4 f   usc:regalloc.obj
 0001:0007ac40       InsertSpill                1007bc40 f   usc:regalloc.obj
 0001:0007b030       AddRegToInstGroup          1007c030 f   usc:regalloc.obj
 0001:0007b294       RegisterGrouping           1007c294 f   usc:regalloc.obj
 0001:0007b5dc       FormOptRegGroupBP          1007c5dc f   usc:regalloc.obj
 0001:0007b6b0       AddEdge                    1007c6b0 f   usc:regalloc.obj
 0001:0007b760       InsertNode                 1007c760 f   usc:regalloc.obj
 0001:0007b8a4       RemoveFromGraph            1007c8a4 f   usc:regalloc.obj
 0001:0007b9ec       SimplifyGraph              1007c9ec f   usc:regalloc.obj
 0001:0007ba80       UpdateInterferenceGraph    1007ca80 f   usc:regalloc.obj
 0001:0007bb94       ReplaceRegisterInstsBP     1007cb94 f   usc:regalloc.obj
 0001:0007bd38       CoalesceRegister           1007cd38 f   usc:regalloc.obj
 0001:0007bf74       IsValidGroup               1007cf74 f   usc:regalloc.obj
 0001:0007c134       SetupConsecutiveRegisterSets 1007d134 f   usc:regalloc.obj
 0001:0007c3b4       AddTempNodesForRegisterSetsBP 1007d3b4 f   usc:regalloc.obj
 0001:0007c518       UpdateInterferenceGraphForArgument 1007d518 f   usc:regalloc.obj
 0001:0007c6a4       MakeInterfereWithAllOutputRegs 1007d6a4 f   usc:regalloc.obj
 0001:0007c724       ConstructInterferenceGraphForImmTemps 1007d724 f   usc:regalloc.obj
 0001:0007c7dc       IndexedArgumentToNodeRange 1007d7dc f   usc:regalloc.obj
 0001:0007c860       FlagC10NodesInst           1007d860 f   usc:regalloc.obj
 0001:0007c9f4       FlagC10NodesBP             1007d9f4 f   usc:regalloc.obj
 0001:0007ca28       UpdateInterferenceGraphForDestNode 1007da28 f   usc:regalloc.obj
 0001:0007cbbc       ConstructInterferenceGraphForInst 1007dbbc f   usc:regalloc.obj
 0001:0007cf9c       ConstructInterferenceGraphForBlock 1007df9c f   usc:regalloc.obj
 0001:0007d3dc       CanNodeUseColour           1007e3dc f   usc:regalloc.obj
 0001:0007d554       ColourNodeRange            1007e554 f   usc:regalloc.obj
 0001:0007d670       ColourNode                 1007e670 f   usc:regalloc.obj
 0001:0007db74       AddToSpillList             1007eb74 f   usc:regalloc.obj
 0001:0007dd10       SpillRegistersForInst      1007ed10 f   usc:regalloc.obj
 0001:0007df6c       SpillRegistersBP           1007ef6c f   usc:regalloc.obj
 0001:0007e034       SpillPlainNodes            1007f034 f   usc:regalloc.obj
 0001:0007e254       PrepRegStateBP             1007f254 f   usc:regalloc.obj
 0001:0007e3e0       SortRegsByDegree           1007f3e0 f   usc:regalloc.obj
 0001:0007e548       AssignColours              1007f548 f   usc:regalloc.obj
 0001:0007e9bc       RenameReg                  1007f9bc f   usc:regalloc.obj
 0001:0007ea8c       DropInst                   1007fa8c f   usc:regalloc.obj
 0001:0007eb00       RenameRegistersBP          1007fb00 f   usc:regalloc.obj
 0001:0007ec50       CoalesceGroups             1007fc50 f   usc:regalloc.obj
 0001:0007ed90       CanCoalesceGroups          1007fd90 f   usc:regalloc.obj
 0001:0007f1b4       ExtendLiveRangeForEquivalent 100801b4 f   usc:regalloc.obj
 0001:0007f2fc       MergeCRegMovesBP           100802fc f   usc:regalloc.obj
 0001:0007f498       CoalesceRegistersForMOVsBP 10080498 f   usc:regalloc.obj
 0001:0007f6e4       ConvertMOVToPCKBP          100806e4 f   usc:regalloc.obj
 0001:0007f7c8       AssignRegistersOffLineFuncGroup 100807c8 f   usc:regalloc.obj
 0001:0007fe3c       InitIRegState              10080e3c f   usc:iregalloc.obj
 0001:0007ffa0       AllocIRegState             10080fa0 f   usc:iregalloc.obj
 0001:000800d8       SetHwReg                   100810d8 f   usc:iregalloc.obj
 0001:00080134       IRegIsNode                 10081134 f   usc:iregalloc.obj
 0001:00080180       PLRemoveIntvl              10081180 f   usc:iregalloc.obj
 0001:000801d0       RegIntvlPush               100811d0 f   usc:iregalloc.obj
 0001:000802c8       SpillOrder                 100812c8 f   usc:iregalloc.obj
 0001:000803b0       FindColour                 100813b0 f   usc:iregalloc.obj
 0001:0008053c       CloseActiveInterval        1008153c f   usc:iregalloc.obj
 0001:00080620       ComputeIRegColours         10081620 f   usc:iregalloc.obj
 0001:0008074c       GetSaveRegs                1008174c f   usc:iregalloc.obj
 0001:000807f4       MergeC10IntervalList       100817f4 f   usc:iregalloc.obj
 0001:000808d8       ProcOpenIntervals          100818d8 f   usc:iregalloc.obj
 0001:00080a10       CalcIntervalBlock          10081a10 f   usc:iregalloc.obj
 0001:00080ba8       CalcIntervalDst            10081ba8 f   usc:iregalloc.obj
 0001:00081038       CalcIntervalSrc            10082038 f   usc:iregalloc.obj
 0001:000811ec       IRegIntervalCB             100821ec f   usc:iregalloc.obj
 0001:000813b0       AllocSpillData             100823b0 f   usc:iregalloc.obj
 0001:00081494       OperandData                10082494 f   usc:iregalloc.obj
 0001:000815a0       GetChanUse                 100825a0 f   usc:iregalloc.obj
 0001:000815dc       FoldNodeReg                100825dc f   usc:iregalloc.obj
 0001:00081860       FoldNodeInst               10082860 f   usc:iregalloc.obj
 0001:00081a60       ExpandSaveC10FullPred      10082a60 f   usc:iregalloc.obj
 0001:00081d90       ExpandSaveC10ShortPred     10082d90 f   usc:iregalloc.obj
 0001:00081f64       ExpandSaveC10              10082f64 f   usc:iregalloc.obj
 0001:0008208c       ExpandRestoreC10           1008308c f   usc:iregalloc.obj
 0001:0008229c       MergeC10SaveComb           1008329c f   usc:iregalloc.obj
 0001:000823f8       SplitSop3                  100833f8 f   usc:iregalloc.obj
 0001:00082b80       SplitC10Inst               10083b80 f   usc:iregalloc.obj
 0001:00083360       MergeC10SavePair           10084360 f   usc:iregalloc.obj
 0001:000834e8       MergeC10SaveInst           100844e8 f   usc:iregalloc.obj
 0001:00083688       MergeC10SavePack           10084688 f   usc:iregalloc.obj
 0001:00083b80       MergeC10Save               10084b80 f   usc:iregalloc.obj
 0001:00083e40       FormSaveC10                10084e40 f   usc:iregalloc.obj
 0001:00083f8c       ExtractNodeSrc             10084f8c f   usc:iregalloc.obj
 0001:000842d8       ExtractInstSrc             100852d8 f   usc:iregalloc.obj
 0001:00084424       MergeC10Restore            10085424 f   usc:iregalloc.obj
 0001:000847c4       FormRestoreC10             100857c4 f   usc:iregalloc.obj
 0001:000848e8       SaveC10Interval            100858e8 f   usc:iregalloc.obj
 0001:00084a28       MarkInstSrc                10085a28 f   usc:iregalloc.obj
 0001:00084ac8       RestoreC10Interval         10085ac8 f   usc:iregalloc.obj
 0001:00084c6c       FindSpillIReg              10085c6c f   usc:iregalloc.obj
 0001:00084ddc       MarkC10Write               10085ddc f   usc:iregalloc.obj
 0001:00084ecc       SpillC10Reg                10085ecc f   usc:iregalloc.obj
 0001:00085690       RenameC10Reg               10086690 f   usc:iregalloc.obj
 0001:00085d80       SaveIRegisters             10086d80 f   usc:iregalloc.obj
 0001:00085f08       SetupInstIRegs             10086f08 f   usc:iregalloc.obj
 0001:00086088       RenameC10BP                10087088 f   usc:iregalloc.obj
 0001:00086950       RenameC10Registers         10087950 f   usc:iregalloc.obj
 0001:00086ad0       CanPeepholeSplit           10087ad0 f   usc:iregalloc.obj
 0001:00086d5c       PeepholeSplit              10087d5c f   usc:iregalloc.obj
 0001:00086f2c       FoldIRegInst               10087f2c f   usc:iregalloc.obj
 0001:00087088       PeepholeC10BP              10088088 f   usc:iregalloc.obj
 0001:00087358       AssignRegistersC10LScan    10088358 f   usc:iregalloc.obj
 0001:000875b4       FreeRegState               100885b4 f   usc:pregalloc.obj
 0001:00087698       UpdatePredicateInterferenceGraph 10088698 f   usc:pregalloc.obj
 0001:00087748       CheckPredicateRepeat       10088748 f   usc:pregalloc.obj
 0001:0008789c       ConstructPredicateInterferenceGraphBP 1008889c f   usc:pregalloc.obj
 0001:00087a58       InsertNode                 10088a58 f   usc:pregalloc.obj
 0001:00087b04       RemoveFromGraph            10088b04 f   usc:pregalloc.obj
 0001:00087bb0       SimplifyGraph              10088bb0 f   usc:pregalloc.obj
 0001:00087c50       RestorePredicate           10088c50 f   usc:pregalloc.obj
 0001:00087dc0       SaveInstResult             10088dc0 f   usc:pregalloc.obj
 0001:00087fe4       CanUseTestMaskSpillModeBP  10088fe4 f   usc:pregalloc.obj
 0001:00088074       SpillPredRegBP             10089074 f   usc:pregalloc.obj
 0001:00088240       RenamePredRegBP            10089240 f   usc:pregalloc.obj
 0001:0008834c       AllocRegState              1008934c f   usc:pregalloc.obj
 0001:000889bc       LocateSyncs                100899bc f   usc:pregalloc.obj
 0001:00088d44       GetFlagSetter              10089d44 f   usc:pregalloc.obj
 0001:00088ddc       DoRestructuring            10089ddc f   usc:pregalloc.obj
 0001:00089224       Restructure                1008a224 f   usc:pregalloc.obj
 0001:00089508       SetSyncEnd                 1008a508 f   usc:pregalloc.obj
 0001:0008958c       SetSyncStartEnd            1008a58c f   usc:pregalloc.obj
 0001:00089ad4       SetDependency              1008aad4 f   usc:efo.obj
 0001:00089b84       SetupIRegDests             1008ab84 f   usc:efo.obj
 0001:00089bd8       CheckEfoIReg               1008abd8 f   usc:efo.obj
 0001:00089cf4       GetArg                     1008acf4 f   usc:efo.obj
 0001:00089da0       SetupEfoStageData          1008ada0 f   usc:efo.obj
 0001:00089e48       CreateEfoInst              1008ae48 f   usc:efo.obj
 0001:00089ee8       CanUseEfoSrc               1008aee8 f   usc:efo.obj
 0001:00089fac       UpdateClosedEfoDependencyGraph 1008afac f   usc:efo.obj
 0001:0008a0fc       AddToEfoReaderList         1008b0fc f   usc:efo.obj
 0001:0008a150       ReplaceHardwareConstants   1008b150 f   usc:efo.obj
 0001:0008a204       MakeEfo_MulMad_SharedSrc   1008b204 f   usc:efo.obj
 0001:0008a510       MakeEfo_MulMad_Square      1008b510 f   usc:efo.obj
 0001:0008a7b8       MakeEfo_MulMad_IRegSrcs    1008b7b8 f   usc:efo.obj
 0001:0008aa8c       MakeEfo_MadMad_Lrp         1008ba8c f   usc:efo.obj
 0001:0008ae58       MakeEfo_EfoMad_Lrp_535     1008be58 f   usc:efo.obj
 0001:0008b1e4       MakeEfo_EfoMad_Lrp_545     1008c1e4 f   usc:efo.obj
 0001:0008ba98       IsInstDependentOnGroup     1008ca98 f   usc:efo.obj
 0001:0008bb28       IsGroupDependentOnInst     1008cb28 f   usc:efo.obj
 0001:0008bc0c       IsDescheduleBetweenGroupAndInsts 1008cc0c f   usc:efo.obj
 0001:0008bcd8       IsGroupDependentOnGroup    1008ccd8 f   usc:efo.obj
 0001:0008bdd0       CheckEfoGroupOrder         1008cdd0 f   usc:efo.obj
 0001:0008be7c       CheckEfoGroupDependency    1008ce7c f   usc:efo.obj
 0001:0008bfdc       WouldBeInterveningIRegWrite 1008cfdc f   usc:efo.obj
 0001:0008c090       IsInterveningIRegWriteForRead 1008d090 f   usc:efo.obj
 0001:0008c188       IsDescheduleBetweenGroups  1008d188 f   usc:efo.obj
 0001:0008c230       CountArgs                  1008d230 f   usc:efo.obj
 0001:0008c2f4       CheckEfoGroupDependencyForMad 1008d2f4 f   usc:efo.obj
 0001:0008c3d0       FindMadForEfoWriteBack     1008d3d0 f   usc:efo.obj
 0001:0008c61c       BuildExtraAddInst          1008d61c f   usc:efo.obj
 0001:0008c854       IsIRegDestOverwrite        1008d854 f   usc:efo.obj
 0001:0008c9d4       CheckSrcToIReg             1008d9d4 f   usc:efo.obj
 0001:0008cd04       AddIRegDependency          1008dd04 f   usc:efo.obj
 0001:0008cdfc       MergeEfoGroup              1008ddfc f   usc:efo.obj
 0001:0008d02c       IsInterveningGroup         1008e02c f   usc:efo.obj
 0001:0008d0f0       IsEfoOrDeschedDependent    1008e0f0 f   usc:efo.obj
 0001:0008d35c       CheckWriteAfterReadDependency 1008e35c f   usc:efo.obj
 0001:0008d3d0       CanReplaceIRegMove         1008e3d0 f   usc:efo.obj
 0001:0008db58       ReplaceIRegMove            1008eb58 f   usc:efo.obj
 0001:0008df68       CanWriteDestUsingEfo       1008ef68 f   usc:efo.obj
 0001:0008e1f4       AddDepsForWriteDestUsingEfo 1008f1f4 f   usc:efo.obj
 0001:0008e388       TryReorderPacks            1008f388 f   usc:efo.obj
 0001:0008e9bc       IsInterveningInst          1008f9bc f   usc:efo.obj
 0001:0008ea80       CreateNewEfoGroup          1008fa80 f   usc:efo.obj
 0001:0008eb14       AddToEfoWriterList         1008fb14 f   usc:efo.obj
 0001:0008eb90       TryCombineDependentInstructions 1008fb90 f   usc:efo.obj
 0001:0008f2c8       GenerateEfosFromDependentInstructions 100902c8 f   usc:efo.obj
 0001:0008f6a8       UnwindEfoToEfo             100906a8 f   usc:efo.obj
 0001:0008fac0       UnwindEfo                  10090ac0 f   usc:efo.obj
 0001:00090148       ConvertM0ToA0              10091148 f   usc:efo.obj
 0001:000902a4       SetupDeschedDependencyState 100912a4 f   usc:efo.obj
 0001:000903e0       SetupGroupDependencyGraph  100913e0 f   usc:efo.obj
 0001:00090604       OutputInstructionsInGroupOrder 10091604 f   usc:efo.obj
 0001:00090a98       ConvertSingleInstToEfo     10091a98 f   usc:efo.obj
 0001:00090d0c       CanConvertSingleInstToEfo  10091d0c f   usc:efo.obj
 0001:00090e74       WriteDestUsingNonEfo       10091e74 f   usc:efo.obj
 0001:00091340       CanReplaceSourceByIReg     10092340 f   usc:efo.obj
 0001:00091734       SetupEfoInstExtraIRegs     10092734 f   usc:efo.obj
 0001:000919f4       TryEfoCombineExtraIRegsMULMUL 100929f4 f   usc:efo.obj
 0001:00091e44       TryEfoCombineExtraIRegsMADMUL 10092e44 f   usc:efo.obj
 0001:00092420       TryEfoCombineExtraIRegsMADMAD 10093420 f   usc:efo.obj
 0001:0009298c       TryEfoCombineExtraIRegs    1009398c f   usc:efo.obj
 0001:00092b94       CheckEfoTemplate           10093b94 f   usc:efo.obj
 0001:00092f90       CheckEfoTemplateTable      10093f90 f   usc:efo.obj
 0001:00093014       CanCombineIntoEfo          10094014 f   usc:efo.obj
 0001:00093338       WriteDestUsingEfo          10094338 f   usc:efo.obj
 0001:00093628       TryEfoCombineWithEfo       10094628 f   usc:efo.obj
 0001:000938e8       TryEfoCombine              100948e8 f   usc:efo.obj
 0001:00093a64       CreateEfoInstructions      10094a64 f   usc:efo.obj
 0001:00094314       CanSubstituteF16RegisterSwizzle 10095314 f   usc:f16opt.obj
 0001:0009447c       CanSubstituteF16FormatConvert 1009547c f   usc:f16opt.obj
 0001:0009462c       CanCombineF16Registers     1009562c f   usc:f16opt.obj
 0001:0009490c       SubstituteF16Argument      1009590c f   usc:f16opt.obj
 0001:000951f8       CombineF16Registers        100961f8 f   usc:f16opt.obj
 0001:000954b0       F16SwizzleToComponent      100964b0 f   usc:f16opt.obj
 0001:00095510       MovePackToMUL16Source      10096510 f   usc:f16opt.obj
 0001:0009572c       OptimizeDependentF16Instructions 1009672c f   usc:f16opt.obj
 0001:00095f90       CompressF16Masks           10096f90 f   usc:f16opt.obj
 0001:000960d8       ExpandF16Masks             100970d8 f   usc:f16opt.obj
 0001:00096210       Float16Optimize            10097210 f   usc:f16opt.obj
 0001:000963c8       GlobalF16HalfPackUpdateBlock 100973c8 f   usc:f16opt.obj
 0001:00096490       GlobalF32F16PackReplaceArguments 10097490 f   usc:f16opt.obj
 0001:00096684       GlobalF32F16PackUpdateBlock 10097684 f   usc:f16opt.obj
 0001:00096724       GlobalF16HalfPackReplaceArguments 10097724 f   usc:f16opt.obj
 0001:00096a3c       GlobalF16FullPackUpdateBlock 10097a3c f   usc:f16opt.obj
 0001:00096aec       GlobalF16FullPackReplaceArguments 10097aec f   usc:f16opt.obj
 0001:00096d9c       PromoteFARITH16ToF32       10097d9c f   usc:f16opt.obj
 0001:000979c8       FixMultipleIndexRegConflict 100989c8 f   usc:indexreg.obj
 0001:00097be0       FixOffsetConflict          10098be0 f   usc:indexreg.obj
 0001:00097e28       AdjustIndexOffsets         10098e28 f   usc:indexreg.obj
 0001:0009806c       GetIndexRange              1009906c f   usc:indexreg.obj
 0001:0009842c       InitRegisterMap            1009942c f   usc:ssa.obj
 0001:00098488       GetSet                     10099488 f   usc:ssa.obj
 0001:000984bc       GetIntermediateReg         100994bc f   usc:ssa.obj
 0001:00098578       DisambiguateRegistersInst  10099578 f   usc:ssa.obj
 0001:000988ac       MergeRegisterMaps          100998ac f   usc:ssa.obj
 0001:000989e8       RemapBlockLiveOutForType   100999e8 f   usc:ssa.obj
 0001:00098a98       AddLiveRegistersToMap      10099a98 f   usc:ssa.obj
 0001:00098b84       RenameRegisterInst         10099b84 f   usc:ssa.obj
 0001:00098cd4       RenameRegistersBP          10099cd4 f   usc:ssa.obj
 0001:00098e94       DisambiguateTraversal      10099e94 f   usc:ssa.obj
 0001:0009931c       ReserveInExitMap           1009a31c f   usc:ssa.obj
 0001:0009935c       FixFinalReg                1009a35c f   usc:ssa.obj
 0001:000993c4       ApplyToFixedRegs           1009a3c4 f   usc:ssa.obj
 0001:000999b8       CheckForStaticConst        1009a9b8 f   usc:icvt_core.obj
 0001:00099a24       ConvertRelativeOffset      1009aa24 f   usc:icvt_core.obj
 0001:0009a3ec       EmitGradCalc               1009b3ec f   usc:icvt_core.obj
 0001:0009a9ec       GetInputConst              1009b9ec f   usc:icvt_core.obj
 0001:0009ab38       UFRegIsConst               1009bb38 f   usc:icvt_core.obj
 0001:0009ab90       UFConstComp                1009bb90 f   usc:icvt_core.obj
 0001:0009adf4       AddD3DLoopProlog           1009bdf4 f   usc:icvt_core.obj
 0001:0009afbc       AddD3DLoopEpilog           1009bfbc f   usc:icvt_core.obj
 0001:0009b2b8       ConvertSwitch              1009c2b8 f   usc:icvt_core.obj
 0001:0009b608       MakeDynamicWopInst         1009c608 f   usc:icvt_core.obj
 0001:0009b7f8       GotoNextOutPutBuff         1009c7f8 f   usc:icvt_core.obj
 0001:0009b9d0       ConvertEmitInstruction     1009c9d0 f   usc:icvt_core.obj
 0001:0009bbc8       AllocInputInst             1009cbc8 f   usc:icvt_core.obj
 0001:0009bc08       CopyInputInst              1009cc08 f   usc:icvt_core.obj
 0001:0009bc9c       RemapInputSwizzle          1009cc9c f   usc:icvt_core.obj
 0001:0009bd14       ExpandTRC                  1009cd14 f   usc:icvt_core.obj
 0001:0009be78       ExpandRNE                  1009ce78 f   usc:icvt_core.obj
 0001:0009bfc4       ExpandCEIL                 1009cfc4 f   usc:icvt_core.obj
 0001:0009c0e0       ExpandPOW                  1009d0e0 f   usc:icvt_core.obj
 0001:0009c278       ExpandRelativeIndex        1009d278 f   usc:icvt_core.obj
 0001:0009dab0       ConvertInstToIntermediate  1009eab0 f   usc:icvt_core.obj
 0001:0009dbf8       SearchBackwardsSetp        1009ebf8 f   usc:icvt_core.obj
 0001:0009dca4       DoFlowControlTest          1009eca4 f   usc:icvt_core.obj
 0001:0009e498       ConvertLoop                1009f498 f   usc:icvt_core.obj
 0001:0009e744       ConvertCall                1009f744 f   usc:icvt_core.obj
 0001:0009e9d8       ConvertConditional         1009f9d8 f   usc:icvt_core.obj
 0001:0009eba4       GetSourceConvertToU16      1009fba4 f   usc:icvt_core.obj
 0001:0009f1e0       DoConvert                  100a01e0 f   usc:icvt_core.obj
 0001:0009f5fc       ExpandMacro                100a05fc f   usc:icvt_core.obj
 0001:000a0324       BuildCFG                   100a1324 f   usc:icvt_core.obj
 0001:000a11c8       FreeIntList                100a21c8 f   usc:dgraph.obj
 0001:000a1680       AddToDepGraph              100a2680 f   usc:dgraph.obj
 0001:000a17fc       FindReaders                100a27fc f   usc:dgraph.obj
 0001:000a18d8       FindRegArrayReaders        100a28d8 f   usc:dgraph.obj
 0001:000a1a58       InsertInAvailableList      100a2a58 f   usc:dgraph.obj
 0001:000a275c       RecordWrite                100a375c f   usc:dgraph.obj
 0001:000a27f0       AddDestDependencies        100a37f0 f   usc:dgraph.obj
 0001:000a299c       RecordRead                 100a399c f   usc:dgraph.obj
 0001:000a3004       CheckArgSwizzleMode        100a4004 f   usc:groupinst.obj
 0001:000a30d4       CheckArg                   100a40d4 f   usc:groupinst.obj
 0001:000a3338       IsDoubleDotProduct         100a4338 f   usc:groupinst.obj
 0001:000a34a8       CouldUseBaseOffset         100a44a8 f   usc:groupinst.obj
 0001:000a35e0       GetArgumentFormatControlRequirements 100a45e0 f   usc:groupinst.obj
 0001:000a3674       GetFormatControlRequirements 100a4674 f   usc:groupinst.obj
 0001:000a3780       CheckFormatControl         100a4780 f   usc:groupinst.obj
 0001:000a3990       MoeToInst                  100a4990 f   usc:groupinst.obj
 0001:000a3a5c       EqualMoeData               100a4a5c f   usc:groupinst.obj
 0001:000a3aec       ResetMoeOpState            100a4aec f   usc:groupinst.obj
 0001:000a3bfc       RecalcInstRegs             100a4bfc f   usc:groupinst.obj
 0001:000a3f04       UpdateKillFlags            100a4f04 f   usc:groupinst.obj
 0001:000a3ff4       RemapIncrements            100a4ff4 f   usc:groupinst.obj
 0001:000a413c       CheckExistingMoeState      100a513c f   usc:groupinst.obj
 0001:000a42bc       SwitchToRepeatMask         100a52bc f   usc:groupinst.obj
 0001:000a45b8       CheckIncrements            100a55b8 f   usc:groupinst.obj
 0001:000a4718       SaveRegNumsBP              100a5718 f   usc:groupinst.obj
 0001:000a47bc       GetBaseOffsetRange         100a57bc f   usc:groupinst.obj
 0001:000a4ac4       CheckBaseOffset            100a5ac4 f   usc:groupinst.obj
 0001:000a4d3c       CheckPossibleSwizzle       100a5d3c f   usc:groupinst.obj
 0001:000a4e4c       EqualArgModes              100a5e4c f   usc:groupinst.obj
 0001:000a4ed4       GenerateDotProducts        100a5ed4 f   usc:groupinst.obj
 0001:000a570c       ExpandMacroInstruction     100a670c f   usc:groupinst.obj
 0001:000a598c       OptimizePFlagCalc          100a698c f   usc:groupinst.obj
 0001:000a5be4       GenerateDotProdBP          100a6be4 f   usc:groupinst.obj
 0001:000a5eb4       UpdateF16RegistersBP       100a6eb4 f   usc:groupinst.obj
 0001:000a5f94       SearchFormatControlBP      100a6f94 f   usc:groupinst.obj
 0001:000a6040       CheckBaseOffsetBasicBlock  100a7040 f   usc:groupinst.obj
 0001:000a60bc       CheckFormatControlBasicBlock 100a70bc f   usc:groupinst.obj
 0001:000a611c       GroupInstsDF               100a711c f   usc:groupinst.obj
 0001:000a6300       CheckFeaturesUsedBP        100a7300 f   usc:groupinst.obj
 0001:000a642c       DoMOEPass                  100a742c f   usc:groupinst.obj
 0001:000a6624       SMLSI_ProcessFuncEnd       100a7624 f   usc:groupinst.obj
 0001:000a673c       SMLSI_Merge                100a773c f   usc:groupinst.obj
 0001:000a6790       SMLSI_UpdateStateAfterCall 100a7790 f   usc:groupinst.obj
 0001:000a6798       SMLSI_SetDefault           100a7798 f   usc:groupinst.obj
 0001:000a679c       SMBO_SetDefault            100a779c f   usc:groupinst.obj
 0001:000a67bc       SMBO_Merge                 100a77bc f   usc:groupinst.obj
 0001:000a6800       SMBO_UpdateStateAfterCall  100a7800 f   usc:groupinst.obj
 0001:000a6830       SMBO_ProcessFuncEnd        100a7830 f   usc:groupinst.obj
 0001:000a6904       SETFC_SetDefault           100a7904 f   usc:groupinst.obj
 0001:000a691c       SETFC_Merge                100a791c f   usc:groupinst.obj
 0001:000a698c       SETFC_UpdateStateAfterCall 100a798c f   usc:groupinst.obj
 0001:000a69ac       InsertSetfc                100a79ac f   usc:groupinst.obj
 0001:000a6b68       CheckInstGroup             100a7b68 f   usc:groupinst.obj
 0001:000a705c       FindPotentialGroup         100a805c f   usc:groupinst.obj
 0001:000a7200       GroupInstructions          100a8200 f   usc:groupinst.obj
 0001:000a7934       GroupInstructionsBasicBlock 100a8934 f   usc:groupinst.obj
 0001:000a821c       LayoutCall                 100a921c f   usc:layout.obj
 0001:000a83c0       LayoutBlockBP              100a93c0 f   usc:layout.obj
 0001:000a8c34       EncodeEfoArith             100a9c34 f   usc:asm.obj
 0001:000a8dbc       EncodeEfo                  100a9dbc f   usc:asm.obj
 0001:000a9034       EncodeSOP2Modes            100aa034 f   usc:asm.obj
 0001:000a9194       EncodeLRP1Modes            100aa194 f   usc:asm.obj
 0001:000a9298       EncodeSOP3Modes            100aa298 f   usc:asm.obj
 0001:000a943c       EncodePred                 100aa43c f   usc:asm.obj
 0001:000a952c       CopySource                 100aa52c f   usc:asm.obj
 0001:000a9750       GetUseasmOpcodeForSmp      100aa750 f   usc:asm.obj
 0001:000a993c       ConvertInstructionToUseasm 100aa93c f   usc:asm.obj
 0001:000aafbc       CreateComparisonF32        100abfbc f   usc:icvt_f32.obj
 0001:000ab1fc       ConvertF16AddressValue     100ac1fc f   usc:icvt_f32.obj
 0001:000ab62c       ConvertC10AddressValue     100ac62c f   usc:icvt_f32.obj
 0001:000abfc4       GetVSOutputSource          100acfc4 f   usc:icvt_f32.obj
 0001:000ac878       ConvertDotProductInstructionF32 100ad878 f   usc:icvt_f32.obj
 0001:000ad1f4       ConvertVertexInputInstructionF32 100ae1f4 f   usc:icvt_f32.obj
 0001:000ad2d0       ConvertVectorInstructionF32 100ae2d0 f   usc:icvt_f32.obj
 0001:000adeac       ConvertComparisonInstructionF32 100aeeac f   usc:icvt_f32.obj
 0001:000ae83c       UnpackTexture              100af83c f   usc:icvt_f32.obj
 0001:000aed34       ConvertSamplerInstructionF32 100afd34 f   usc:icvt_f32.obj
 0001:000aee28       ConvertLitInstructionF32   100afe28 f   usc:icvt_f32.obj
 0001:000af8f8       ConvertNormaliseF32        100b08f8 f   usc:icvt_f32.obj
 0001:000afa9c       ConvertSincosF32           100b0a9c f   usc:icvt_f32.obj
 0001:000afc1c       ConvertSincos2F32          100b0c1c f   usc:icvt_f32.obj
 0001:000afe18       ConvertLogpInstructionF32  100b0e18 f   usc:icvt_f32.obj
 0001:000b04a0       ConvertExppInstructionF32  100b14a0 f   usc:icvt_f32.obj
 0001:000b0928       ConvertTexkillInstructionBit 100b1928 f   usc:icvt_f32.obj
 0001:000b0d88       ConvertIntegerDot34        100b1d88 f   usc:icvt_f32.obj
 0001:000b10a8       ConvertIntegerToF32        100b20a8 f   usc:icvt_f32.obj
 0001:000b143c       ConvertReformatInstructionF32 100b243c f   usc:icvt_f32.obj
 0001:000b1e38       GetIteratedValueF16        100b2e38 f   usc:icvt_f16.obj
 0001:000b20c8       ConvertDestinationF16      100b30c8 f   usc:icvt_f16.obj
 0001:000b219c       GetDestinationF16          100b319c f   usc:icvt_f16.obj
 0001:000b2294       GetF16StaticDoubleConst    100b3294 f   usc:icvt_f16.obj
 0001:000b23b4       GetF16StaticConstant       100b33b4 f   usc:icvt_f16.obj
 0001:000b24b8       DoF16UnalignedAccess       100b34b8 f   usc:icvt_f16.obj
 0001:000b259c       GetF16Source               100b359c f   usc:icvt_f16.obj
 0001:000b2cf8       GenerateDestModF16         100b3cf8 f   usc:icvt_f16.obj
 0001:000b3038       ConvertScalarInstructionF16 100b4038 f   usc:icvt_f16.obj
 0001:000b32c4       ConvertF32OnlyInstructionF16 100b42c4 f   usc:icvt_f16.obj
 0001:000b36b0       ConvertSincosF16           100b46b0 f   usc:icvt_f16.obj
 0001:000b3934       ConvertSincos2F16          100b4934 f   usc:icvt_f16.obj
 0001:000b3f40       UnpackTextureF16           100b4f40 f   usc:icvt_f16.obj
 0001:000b4090       ConvertSamplerInstructionF16 100b5090 f   usc:icvt_f16.obj
 0001:000b41c4       ConvertMoveInstructionF16  100b51c4 f   usc:icvt_f16.obj
 0001:000b462c       ConvertComparisonInstructionF16 100b562c f   usc:icvt_f16.obj
 0001:000b4c14       ConvertDotProductInstructionF16 100b5c14 f   usc:icvt_f16.obj
 0001:000b5400       GetDoubleSourceF16         100b6400 f   usc:icvt_f16.obj
 0001:000b5a00       ConvertMadInstructionF16   100b6a00 f   usc:icvt_f16.obj
 0001:000b63d8       ConvertDot4InstructionF16  100b73d8 f   usc:icvt_f16.obj
 0001:000b6960       ConvertDestinationC10      100b7960 f   usc:icvt_c10.obj
 0001:000b6a80       GetDestinationC10          100b7a80 f   usc:icvt_c10.obj
 0001:000b6c58       GenerateDestModC10         100b7c58 f   usc:icvt_c10.obj
 0001:000b7268       SwizzleC10                 100b8268 f   usc:icvt_c10.obj
 0001:000b7410       ApplySourceModC10          100b8410 f   usc:icvt_c10.obj
 0001:000b7744       GetIteratedValueC10        100b8744 f   usc:icvt_c10.obj
 0001:000b7a90       LoadVSInputC10             100b8a90 f   usc:icvt_c10.obj
 0001:000b7bd8       LoadVSOutputC10            100b8bd8 f   usc:icvt_c10.obj
 0001:000b7d1c       LoadHwConstC10             100b8d1c f   usc:icvt_c10.obj
 0001:000b808c       LoadBackfaceC10            100b908c f   usc:icvt_c10.obj
 0001:000b828c       GetC10OrU8StaticConstant   100b928c f   usc:icvt_c10.obj
 0001:000b844c       ExpandAlignedConstantAccess 100b944c f   usc:icvt_c10.obj
 0001:000b8628       ExpandUnalignedConstantAccess 100b9628 f   usc:icvt_c10.obj
 0001:000b8960       ConvertU8ArgToC10          100b9960 f   usc:icvt_c10.obj
 0001:000b8a40       ConvertC10ArgToU8          100b9a40 f   usc:icvt_c10.obj
 0001:000b9484       ConvertScalarInstructionC10 100ba484 f   usc:icvt_c10.obj
 0001:000b98e4       ConvertDotProductInstructionC10 100ba8e4 f   usc:icvt_c10.obj
 0001:000b9fd0       ConvertFloatOnlyInstructionC10 100bafd0 f   usc:icvt_c10.obj
 0001:000ba33c       ConvertLrpInstructionC10   100bb33c f   usc:icvt_c10.obj
 0001:000ba78c       ConvertMadInstructionC10   100bb78c f   usc:icvt_c10.obj
 0001:000bac58       ConvertVectorTwoArgInstructionC10 100bbc58 f   usc:icvt_c10.obj
 0001:000bb1d4       ConvertMovaInstructionC10  100bc1d4 f   usc:icvt_c10.obj
 0001:000bb490       LoadC10One                 100bc490 f   usc:icvt_c10.obj
 0001:000bb570       ConvertComparisonInstructionC10 100bc570 f   usc:icvt_c10.obj
 0001:000bbeb8       ConvertSamplerInstructionC10 100bceb8 f   usc:icvt_c10.obj
 0001:000bc1e8       ConvertMoveInstructionC10  100bd1e8 f   usc:icvt_c10.obj
 0001:000bcf34       ConvertSincosC10           100bdf34 f   usc:icvt_c10.obj
 0001:000bd244       ConvertSincos2C10          100be244 f   usc:icvt_c10.obj
 0001:000bdcc8       ConvertSetpInstructionC10  100becc8 f   usc:icvt_c10.obj
 0001:000bdf44       KillOneChannel             100bef44 f   usc:icvt_c10.obj
 0001:000be040       ConvertTexkillInstructionC10 100bf040 f   usc:icvt_c10.obj
 0001:000be89c       ConvertNormaliseC10        100bf89c f   usc:icvt_c10.obj
 0001:000bf034       Generate32bitIntegerMulNonNeg_Non545 100c0034 f   usc:icvt_i32.obj
 0001:000bf7b4       Generate32bitIntegerMul_Non545 100c07b4 f   usc:icvt_i32.obj
 0001:000c025c       GenerateOrTest             100c125c f   usc:icvt_i32.obj
 0001:000c0308       MoveTempToDestination      100c1308 f   usc:icvt_i32.obj
 0001:000c03cc       ConvertVertexInputInstructionI32 100c13cc f   usc:icvt_i32.obj
 0001:000c05f0       Generate32bitIntegerAdd_Non545 100c15f0 f   usc:icvt_i32.obj
 0001:000c0c5c       Generate32bitIntegerMad_Non545 100c1c5c f   usc:icvt_i32.obj
 0001:000c0d50       GenerateIntegerDividePostCheck_Non545 100c1d50 f   usc:icvt_i32.obj
 0001:000c18e0       GenerateIntegerDivide_Non545 100c28e0 f   usc:icvt_i32.obj
 0001:000c1f34       GenerateSignResult         100c2f34 f   usc:icvt_i32.obj
 0001:000c2298       ConvertComparisonInstructionInt32 100c3298 f   usc:icvt_i32.obj
 0001:000c241c       ConvertIntegerInstruction  100c341c f   usc:icvt_i32.obj
 0001:000c2dc0       GetSourceLiveChans         100c3dc0 f   usc:precovr.obj
 0001:000c3040       IsResultUsed               100c4040 f   usc:precovr.obj
 0001:000c3228       AddPackedRegister          100c4228 f   usc:precovr.obj
 0001:000c3338       IsSaturatedTemp            100c4338 f   usc:precovr.obj
 0001:000c3518       IsSaturatedSource          100c4518 f   usc:precovr.obj
 0001:000c3704       ConvertMoveInstruction     100c4704 f   usc:precovr.obj
 0001:000c3808       ConvertMulInstruction      100c4808 f   usc:precovr.obj
 0001:000c3a4c       IsStaticConstInRange       100c4a4c f   usc:precovr.obj
 0001:000c3b48       ConvertMinMaxInstruction   100c4b48 f   usc:precovr.obj
 0001:000c3cb0       ConvertAddInstruction      100c4cb0 f   usc:precovr.obj
 0001:000c3e54       ConvertInstructionToInteger 100c4e54 f   usc:precovr.obj
 0001:000c3fd8       ConvertDotProduct          100c4fd8 f   usc:precovr.obj
 0001:000c419c       AddPackToInteger           100c519c f   usc:precovr.obj
 0001:000c4234       FindPackedRegister         100c5234 f   usc:precovr.obj
 0001:000c4334       DoIntegerConversion        100c5334 f   usc:precovr.obj
 0001:000c49f4       ConvertInputInstF16ToF32   100c59f4 f   usc:precovr.obj
 0001:000c4af4       GetHwInstCountForF16Instruction 100c5af4 f   usc:precovr.obj
 0001:000c4c4c       CheckInstConversion        100c5c4c f   usc:precovr.obj
 0001:000c4dfc       ConvertRegisterPrecision   100c5dfc f   usc:precovr.obj
 0001:000c58c8       SetLabelAddress            100c68c8 f   useasm:useasm.obj
 0001:000c5a94       FixupLabelAddresses        100c6a94 f   useasm:useasm.obj
 0001:000c5be8       GetLabelAddress            100c6be8 f   useasm:useasm.obj
 0001:000c5d0c       CheckArgFlags              100c6d0c f   useasm:useasm.obj
 0001:000c5f98       CheckFlags                 100c6f98 f   useasm:useasm.obj
 0001:000c677c       EncodeIndex                100c777c f   useasm:useasm.obj
 0001:000c692c       EncodeDestBankAndNum       100c792c f   useasm:useasm.obj
 0001:000c6ca8       EncodeDest                 100c7ca8 f   useasm:useasm.obj
 0001:000c6cfc       GetSrc0EncodedBankAndNumber 100c7cfc f   useasm:useasm.obj
 0001:000c6f64       EncodeSrc0                 100c7f64 f   useasm:useasm.obj
 0001:000c6fbc       GetSrc1EncodedBankAndNumber 100c7fbc f   useasm:useasm.obj
 0001:000c74b4       EncodeSrc1                 100c84b4 f   useasm:useasm.obj
 0001:000c7528       GetSrc2EncodedBankAndNumber 100c8528 f   useasm:useasm.obj
 0001:000c79e4       EncodeSrc2                 100c89e4 f   useasm:useasm.obj
 0001:000c7a58       EncodePredicate            100c8a58 f   useasm:useasm.obj
 0001:000c7b40       AssembleDot34              100c8b40 f   useasm:useasm.obj
 0001:000c861c       EncodeTestInstruction_AluOp 100c961c f   useasm:useasm.obj
 0001:000c896c       EncodeTestInstruction_Repeat 100c996c f   useasm:useasm.obj
 0001:000c8b58       EncodeTestInstruction      100c9b58 f   useasm:useasm.obj
 0001:000c91ec       EncodeFloatInstruction     100ca1ec f   useasm:useasm.obj
 0001:000c9874       EncodeNormaliseInstruction 100ca874 f   useasm:useasm.obj
 0001:000c9e90       EncodeSOP2Instruction      100cae90 f   useasm:useasm.obj
 0001:000ca8bc       EncodePackInstruction      100cb8bc f   useasm:useasm.obj
 0001:000cb020       EncodeBitwiseInstruction   100cc020 f   useasm:useasm.obj
 0001:000cb50c       ExpandMacros               100cc50c f   useasm:useasm.obj
 0001:000cbf40       EncodeFDPCInstruction      100ccf40 f   useasm:useasm.obj
 0001:000cc218       EncodeFDDPInstruction      100cd218 f   useasm:useasm.obj
 0001:000cc560       EncodeFDDPCInstruction     100cd560 f   useasm:useasm.obj
 0001:000cc950       EncodeMovcInstruction      100cd950 f   useasm:useasm.obj
 0001:000cccb0       EncodeEfoInstruction       100cdcb0 f   useasm:useasm.obj
 0001:000ccfd8       EncodeSOPWMInstruction     100cdfd8 f   useasm:useasm.obj
 0001:000cd60c       EncodeLRP1Instruction      100ce60c f   useasm:useasm.obj
 0001:000cde18       EncodeLRP2Instruction      100cee18 f   useasm:useasm.obj
 0001:000ce6bc       EncodeSOP3Instruction      100cf6bc f   useasm:useasm.obj
 0001:000cf258       EncodeFPMAInstruction      100d0258 f   useasm:useasm.obj
 0001:000cf8fc       EncodeIMA16Instruction     100d08fc f   useasm:useasm.obj
 0001:000cfe54       EncodeIMAEInstruction      100d0e54 f   useasm:useasm.obj
 0001:000d049c       EncodeADIFInstruction      100d149c f   useasm:useasm.obj
 0001:000d0784       EncodeSSUM16Instruction    100d1784 f   useasm:useasm.obj
 0001:000d0d24       EncodeFIRVInstruction      100d1d24 f   useasm:useasm.obj
 0001:000d1234       EncodeFIRVHInstruction     100d2234 f   useasm:useasm.obj
 0001:000d15f4       EncodeBILINInstruction     100d25f4 f   useasm:useasm.obj
 0001:000d1b5c       EncodeFIRHInstruction      100d2b5c f   useasm:useasm.obj
 0001:000d210c       EncodeFIRHHInstruction     100d310c f   useasm:useasm.obj
 0001:000d270c       EncodeSMPInstruction       100d370c f   useasm:useasm.obj
 0001:000d2c78       EncodeLDSTCacheFlags       100d3c78 f   useasm:useasm.obj
 0001:000d2d40       EncodeLDSTInstruction      100d3d40 f   useasm:useasm.obj
 0001:000d33f0       EncodeBAInstruction        100d43f0 f   useasm:useasm.obj
 0001:000d357c       EncodeLAPCInstruction      100d457c f   useasm:useasm.obj
 0001:000d3638       EncodeBRInstruction        100d4638 f   useasm:useasm.obj
 0001:000d37c8       EncodeIDFInstruction       100d47c8 f   useasm:useasm.obj
 0001:000d39ac       EncodeWDFInstruction       100d49ac f   useasm:useasm.obj
 0001:000d3ab4       EncodeEmitInstruction      100d4ab4 f   useasm:useasm.obj
 0001:000d3f5c       EncodeSMOAInstruction      100d4f5c f   useasm:useasm.obj
 0001:000d427c       EncodeSMLSIInstruction     100d527c f   useasm:useasm.obj
 0001:000d4774       EncodeMOEInstruction       100d5774 f   useasm:useasm.obj
 0001:000d4a90       EncodeSETFCInstruction     100d5a90 f   useasm:useasm.obj
 0001:000d4bdc       EncodeMOVInstruction       100d5bdc f   useasm:useasm.obj
 0001:000d50c4       EncodeMutexInstruction     100d60c4 f   useasm:useasm.obj
 0001:000d521c       EncodeLDRSTRInstruction    100d621c f   useasm:useasm.obj
 0001:000d5608       EncodePTOFFPCOEFFInstruction 100d6608 f   useasm:useasm.obj
 0001:000d5784       EncodeATST8Instruction     100d6784 f   useasm:useasm.obj
 0001:000d5b24       EncodeDEPTHFInstruction    100d6b24 f   useasm:useasm.obj
 0001:000d5da8       EncodeSETMInstruction      100d6da8 f   useasm:useasm.obj
 0001:000d5f04       EncodeWOPInstruction       100d6f04 f   useasm:useasm.obj
 0001:000d6c2c       _DllMainCRTStartupHelper   100d7c2c f   corelib0:pegdmain.obj
 0001:000d6e6c       doexit                     100d7e6c f   corelib0:cexit.obj
 0001:000d7308       FindRule                   100d8308 f   glsl_parser:parser.obj
 0001:000d73b8       ParseTreeAddNextEntry      100d83b8 f   glsl_parser:parser.obj
 0001:000d750c       ParseTreeRemoveEntry       100d850c f   glsl_parser:parser.obj
 0001:000d75c4       ParseTreeFindNextUntriedEntry 100d85c4 f   glsl_parser:parser.obj
 0001:000d76b4       RemoveEmptyParseTreeBranches 100d86b4 f   glsl_parser:parser.obj
 0001:000d78ec       CreateParseTree            100d88ec f   glsl_parser:parser.obj
 0001:000d7fb4       SortSyntaxGrammar          100d8fb4 f   glsl_parser:syntax.obj
 0001:000d8804       LexCallocToken             100d9804 f   glsl_parser:lex.obj
 0001:000d888c       LexGeneratePreprocessorTokens 100d988c f   glsl_parser:lex.obj
 0001:000d9264       LexMatchKeywords           100da264 f   glsl_parser:lex.obj
